 RILGOBI

 Timestamp is 54004a12 (Fri Aug 29 17:38:26 2014)

 Preferred load address is 00100000

 Start         Length     Name                   Class
 0001:00000000 000a2fc8H .text                   CODE
 0001:000a2fc8 0000009cH .text$yc                CODE
 0001:000a3064 00000060H .text$yd                CODE
 0002:00000000 000bd554H .rdata                  DATA
 0002:000bd554 00000074H .rdata$debug            DATA
 0002:000bd5c8 000001bcH .rdata$r                DATA
 0002:000bd784 0000025cH .xdata                  DATA
 0002:000bd9e0 00000124H .xdata$x                DATA
 0002:000bdb04 0000008cH .idata$2                DATA
 0002:000bdb90 00000014H .idata$3                DATA
 0002:000bdba4 00000440H .idata$4                DATA
 0002:000bdfe4 00001076H .idata$6                DATA
 0002:000bf060 00000103H .edata                  DATA
 0003:00000000 00000440H .idata$5                DATA
 0003:00000440 00000004H .CRT$XCA                DATA
 0003:00000444 00000004H .CRT$XCAA               DATA
 0003:00000448 00000004H .CRT$XCC                DATA
 0003:0000044c 0000000cH .CRT$XCU                DATA
 0003:00000458 00000004H .CRT$XCZ                DATA
 0003:0000045c 00000004H .CRT$XIA                DATA
 0003:00000460 00000004H .CRT$XIZ                DATA
 0003:00000464 00000004H .CRT$XPA                DATA
 0003:00000468 00000004H .CRT$XPZ                DATA
 0003:0000046c 00000004H .CRT$XTA                DATA
 0003:00000470 00000004H .CRT$XTZ                DATA
 0003:00000478 00009870H .data                   DATA
 0003:00009ce8 0000038cH .bss                    DATA
 0004:00000000 00004778H .pdata                  DATA
 0005:00000000 000000a0H .rsrc$01                DATA
 0005:000000a0 000003f4H .rsrc$02                DATA

  Address         Publics by Value              Rva+Base       Lib:Object

 0000:00000000       ___safe_se_handler_count   00000000     <absolute>
 0000:00000000       ___safe_se_handler_table   00000000     <absolute>
 0001:00000008       ?QueueCmdWithTimeout@@YAHQAVCRilInstanceHandle@@KW4APIID@@PAXAAJKK@Z 00101008 f   atcmd.obj
 0001:00000530       ?QueueCmd@@YAHQAVCRilInstanceHandle@@KW4APIID@@PAXAAJK@Z 00101530 f   atcmd.obj
 0001:000005c4       ?CmdThreadProc@@YAKPAX@Z   001015c4 f   atcmd.obj
 0001:00000744       ?ReadThreadProc@@YAKPAX@Z  00101744 f   atcmd.obj
 0001:00000930       ?CommandThread@CRilHandle@@QAAKXZ 00101930 f   atcmd.obj
 0001:00000db8       ??0SYNCBLOCK_Implementation@@QAA@AAUCRITICAL_SECTION@@@Z 00101db8 f i atcmd.obj
 0001:00000df4       ??1SYNCBLOCK_Implementation@@QAA@XZ 00101df4 f i atcmd.obj
 0001:00000e10       ?GetID@CCommand@@QBAJXZ    00101e10 f i atcmd.obj
 0001:00000e3c       ?GetAPIID@CCommand@@QBA?AW4APIID@@XZ 00101e3c f i atcmd.obj
 0001:00000e68       ?GetCurrAPIID@CRilHandle@@QAAKXZ 00101e68 f i atcmd.obj
 0001:00000ebc       ?GetDevice@CRilInstanceHandle@@QBAPAVCRilHandle@@XZ 00101ebc f i atcmd.obj
 0001:00000fc0       ?GetCmdList@CRilInstanceHandle@@QBAPAV?$CDblList@VCCommand@@@@XZ 00101fc0 f i atcmd.obj
 0001:0000107c       ??_GCCommand@@QAAPAXI@Z    0010207c f i atcmd.obj
 0001:000010bc       GetCurrentThread           001020bc f i atcmd.obj
 0001:000010d4       ?GetHandle@CCommand@@QBAPAVCRilInstanceHandle@@XZ 001020d4 f i atcmd.obj
 0001:00001100       ?GetCheckPoint@CRilHandle@@QBAPAVCCheckPoint@@XZ 00102100 f i atcmd.obj
 0001:00001134       ?Add@?$CDblList@VCCommand@@@@QAAHQAVCCommand@@@Z 00102134 f i atcmd.obj
 0001:00001210       ?GetNext@CListElem@@QBAPAV1@XZ 00102210 f i atcmd.obj
 0001:00001238       ?SetNext@CListElem@@QAAXPAV1@@Z 00102238 f i atcmd.obj
 0001:00001254       ?SetPrev@CListElem@@QAAXPAV1@@Z 00102254 f i atcmd.obj
 0001:0000127c       ?Remove@?$CDblList@VCCommand@@@@QAAHQBVCCommand@@@Z 0010227c f i atcmd.obj
 0001:000013f8       ?GetPrev@CListElem@@QBAPAV1@XZ 001023f8 f i atcmd.obj
 0001:00001424       ?IsEmpty@?$CThreadSafeQueue@PAVCCommand@@@@QBA_NXZ 00102424 f i atcmd.obj
 0001:00001454       ?Front@?$CThreadSafeQueue@PAVCCommand@@@@QAAAAPAVCCommand@@XZ 00102454 f i atcmd.obj
 0001:00001484       ?Push_Back@?$CThreadSafeQueue@PAVCCommand@@@@QAAXABQAVCCommand@@@Z 00102484 f i atcmd.obj
 0001:000014f0       ?Lock@CriticalSection@@QAA_NXZ 001024f0 f i atcmd.obj
 0001:00001520       ?Unlock@CriticalSection@@QAA_NXZ 00102520 f i atcmd.obj
 0001:00001550       ?SetEvent@Event@@QAAHXZ    00102550 f i atcmd.obj
 0001:00001588       SetEvent                   00102588 f i atcmd.obj
 0001:000015bc       ?Pop_Front@?$CThreadSafeQueue@PAVCCommand@@@@QAAPAVCCommand@@XZ 001025bc f i atcmd.obj
 0001:00001664       ?ResetEvent@Event@@QAAHXZ  00102664 f i atcmd.obj
 0001:0000169c       ResetEvent                 0010269c f i atcmd.obj
 0001:000016d0       ?empty@?$queue@PAVCCommand@@V?$deque@PAVCCommand@@V?$allocator@PAVCCommand@@@std@@@std@@@std@@QBA_NXZ 001026d0 f i atcmd.obj
 0001:00001700       ?size@?$queue@PAVCCommand@@V?$deque@PAVCCommand@@V?$allocator@PAVCCommand@@@std@@@std@@@std@@QBAIXZ 00102700 f i atcmd.obj
 0001:00001730       ?front@?$queue@PAVCCommand@@V?$deque@PAVCCommand@@V?$allocator@PAVCCommand@@@std@@@std@@@std@@QAAAAPAVCCommand@@XZ 00102730 f i atcmd.obj
 0001:00001760       ?push@?$queue@PAVCCommand@@V?$deque@PAVCCommand@@V?$allocator@PAVCCommand@@@std@@@std@@@std@@QAAXABQAVCCommand@@@Z 00102760 f i atcmd.obj
 0001:0000177c       ?pop@?$queue@PAVCCommand@@V?$deque@PAVCCommand@@V?$allocator@PAVCCommand@@@std@@@std@@@std@@QAAXXZ 0010277c f i atcmd.obj
 0001:00001794       ?size@?$deque@PAVCCommand@@V?$allocator@PAVCCommand@@@std@@@std@@QBAIXZ 00102794 f i atcmd.obj
 0001:000017c0       ?empty@?$deque@PAVCCommand@@V?$allocator@PAVCCommand@@@std@@@std@@QBA_NXZ 001027c0 f i atcmd.obj
 0001:00001818       ?front@?$deque@PAVCCommand@@V?$allocator@PAVCCommand@@@std@@@std@@QAAAAPAVCCommand@@XZ 00102818 f i atcmd.obj
 0001:0000188c       ?pop_front@?$deque@PAVCCommand@@V?$allocator@PAVCCommand@@@std@@@std@@QAAXXZ 0010288c f i atcmd.obj
 0001:00001a04       ?push_back@?$deque@PAVCCommand@@V?$allocator@PAVCCommand@@@std@@@std@@QAAXABQAVCCommand@@@Z 00102a04 f i atcmd.obj
 0001:00001be4       ?_Orphan_all@_Container_base@std@@QBAXXZ 00102be4 f i atcmd.obj
 0001:00001c78       ??1?$_Deque_iterator@PAVCCommand@@V?$allocator@PAVCCommand@@@std@@$00@std@@QAA@XZ 00102c78 f i atcmd.obj
 0001:00001c90       ??1?$_Deque_const_iterator@PAVCCommand@@V?$allocator@PAVCCommand@@@std@@$00@std@@QAA@XZ 00102c90 f i atcmd.obj
 0001:00001ca8       ??1?$_Ranit@PAVCCommand@@HPBQAV1@ABQAV1@@std@@QAA@XZ 00102ca8 f i atcmd.obj
 0001:00001cc8       ??1_Iterator_base@std@@QAA@XZ 00102cc8 f i atcmd.obj
 0001:00001d1c       ?_Orphan_me@_Iterator_base@std@@QAAXXZ 00102d1c f i atcmd.obj
 0001:00001de4       ?begin@?$deque@PAVCCommand@@V?$allocator@PAVCCommand@@@std@@@std@@QAA?AV?$_Deque_iterator@PAVCCommand@@V?$allocator@PAVCCommand@@@std@@$00@2@XZ 00102de4 f i atcmd.obj
 0001:00001e38       ?_Growmap@?$deque@PAVCCommand@@V?$allocator@PAVCCommand@@@std@@@std@@IAAXI@Z 00102e38 f i atcmd.obj
 0001:000021ec       ?_Orphan_off@?$deque@PAVCCommand@@V?$allocator@PAVCCommand@@@std@@@std@@IBAXI@Z 001031ec f i atcmd.obj
 0001:00002344       ?allocate@?$allocator@PAVCCommand@@@std@@QAAPAPAVCCommand@@I@Z 00103344 f i atcmd.obj
 0001:00002378       ?construct@?$allocator@PAVCCommand@@@std@@QAAXPAPAVCCommand@@ABQAV3@@Z 00103378 f i atcmd.obj
 0001:00002394       ?destroy@?$allocator@PAVCCommand@@@std@@QAAXPAPAVCCommand@@@Z 00103394 f i atcmd.obj
 0001:000023ac       ??D?$_Deque_iterator@PAVCCommand@@V?$allocator@PAVCCommand@@@std@@$00@std@@QBAAAPAVCCommand@@XZ 001033ac f i atcmd.obj
 0001:000023dc       ?max_size@?$deque@PAVCCommand@@V?$allocator@PAVCCommand@@@std@@@std@@QBAIXZ 001033dc f i atcmd.obj
 0001:00002418       ?_Xlen@?$deque@PAVCCommand@@V?$allocator@PAVCCommand@@@std@@@std@@KAXXZ 00103418 f i atcmd.obj
 0001:00002490       ??0length_error@std@@QAA@ABV?$basic_string@DU?$char_traits@D@std@@V?$allocator@D@2@@1@@Z 00103490 f i atcmd.obj
 0001:000024dc       ??0logic_error@std@@QAA@ABV?$basic_string@DU?$char_traits@D@std@@V?$allocator@D@2@@1@@Z 001034dc f i atcmd.obj
 0001:0000254c       ?what@logic_error@std@@UBAPBDXZ 0010354c f i atcmd.obj
 0001:00002580       ??_Elogic_error@std@@UAAPAXI@Z 00103580 f i atcmd.obj
 0001:00002580       ??_Glogic_error@std@@UAAPAXI@Z 00103580 f i atcmd.obj
 0001:000025c0       ??1logic_error@std@@UAA@XZ 001035c0 f i atcmd.obj
 0001:000025f4       ??1length_error@std@@UAA@XZ 001035f4 f i atcmd.obj
 0001:0000261c       ??_Elength_error@std@@UAAPAXI@Z 0010361c f i atcmd.obj
 0001:0000261c       ??_Glength_error@std@@UAAPAXI@Z 0010361c f i atcmd.obj
 0001:00002664       ??0?$basic_string@DU?$char_traits@D@std@@V?$allocator@D@2@@std@@QAA@ABV01@@Z 00103664 f i atcmd.obj
 0001:00002704       ??1?$basic_string@DU?$char_traits@D@std@@V?$allocator@D@2@@std@@QAA@XZ 00103704 f i atcmd.obj
 0001:0000274c       ?c_str@?$basic_string@DU?$char_traits@D@std@@V?$allocator@D@2@@std@@QBAPBDXZ 0010374c f i atcmd.obj
 0001:0000277c       ??1?$_String_val@DV?$allocator@D@std@@@std@@QAA@XZ 0010377c f i atcmd.obj
 0001:00002794       ??1_String_base@std@@QAA@XZ 00103794 f i atcmd.obj
 0001:000027ac       ??1_Container_base@std@@QAA@XZ 001037ac f i atcmd.obj
 0001:000027c4       ?assign@?$basic_string@DU?$char_traits@D@std@@V?$allocator@D@2@@std@@QAAAAV12@ABV12@II@Z 001037c4 f i atcmd.obj
 0001:000028e8       ?_Tidy@?$basic_string@DU?$char_traits@D@std@@V?$allocator@D@2@@std@@IAAX_NI@Z 001038e8 f i atcmd.obj
 0001:00002994       ?_Myptr@?$basic_string@DU?$char_traits@D@std@@V?$allocator@D@2@@std@@IBAPBDXZ 00103994 f i atcmd.obj
 0001:000029ec       ??0?$_String_val@DV?$allocator@D@std@@@std@@IAA@V?$allocator@D@1@@Z 001039ec f i atcmd.obj
 0001:00002a2c       ??0?$allocator@D@std@@QAA@ABV01@@Z 00103a2c f i atcmd.obj
 0001:00002a50       ??0_String_base@std@@QAA@XZ 00103a50 f i atcmd.obj
 0001:00002a80       ??0_Container_base@std@@QAA@XZ 00103a80 f i atcmd.obj
 0001:00002ab0       ?erase@?$basic_string@DU?$char_traits@D@std@@V?$allocator@D@2@@std@@QAAAAV12@II@Z 00103ab0 f i atcmd.obj
 0001:00002bc4       ?size@?$basic_string@DU?$char_traits@D@std@@V?$allocator@D@2@@std@@QBAIXZ 00103bc4 f i atcmd.obj
 0001:00002bf0       ?_Eos@?$basic_string@DU?$char_traits@D@std@@V?$allocator@D@2@@std@@IAAXI@Z 00103bf0 f i atcmd.obj
 0001:00002c40       ?assign@?$char_traits@D@std@@SAXAADABD@Z 00103c40 f i atcmd.obj
 0001:00002c60       ?_Grow@?$basic_string@DU?$char_traits@D@std@@V?$allocator@D@2@@std@@IAA_NI_N@Z 00103c60 f i atcmd.obj
 0001:00002d74       ?_Myptr@?$basic_string@DU?$char_traits@D@std@@V?$allocator@D@2@@std@@IAAPADXZ 00103d74 f i atcmd.obj
 0001:00002dcc       ?deallocate@?$allocator@D@std@@QAAXPADI@Z 00103dcc f i atcmd.obj
 0001:00002de4       ??0length_error@std@@QAA@ABV01@@Z 00103de4 f i atcmd.obj
 0001:00002e30       ??0logic_error@std@@QAA@ABV01@@Z 00103e30 f i atcmd.obj
 0001:00002eb0       ??0?$basic_string@DU?$char_traits@D@std@@V?$allocator@D@2@@std@@QAA@PBD@Z 00103eb0 f i atcmd.obj
 0001:00002f30       ?max_size@?$basic_string@DU?$char_traits@D@std@@V?$allocator@D@2@@std@@QBAIXZ 00103f30 f i atcmd.obj
 0001:00002f98       ?_Copy@?$basic_string@DU?$char_traits@D@std@@V?$allocator@D@2@@std@@IAAXII@Z 00103f98 f i atcmd.obj
 0001:000031cc       ?assign@?$basic_string@DU?$char_traits@D@std@@V?$allocator@D@2@@std@@QAAAAV12@PBD@Z 001041cc f i atcmd.obj
 0001:00003210       ?length@?$char_traits@D@std@@SAIPBD@Z 00104210 f i atcmd.obj
 0001:00003240       ??0?$allocator@D@std@@QAA@XZ 00104240 f i atcmd.obj
 0001:00003264       ?allocate@?$allocator@D@std@@QAAPADI@Z 00104264 f i atcmd.obj
 0001:00003298       ?max_size@?$allocator@D@std@@QBAIXZ 00104298 f i atcmd.obj
 0001:000032e4       ?assign@?$basic_string@DU?$char_traits@D@std@@V?$allocator@D@2@@std@@QAAAAV12@PBDI@Z 001042e4 f i atcmd.obj
 0001:000033b0       ?_Inside@?$basic_string@DU?$char_traits@D@std@@V?$allocator@D@2@@std@@IAA_NPBD@Z 001043b0 f i atcmd.obj
 0001:00003444       ??$_Debug_pointer@D@std@@YAXPBDPBGI@Z 00104444 f i atcmd.obj
 0001:00003474       ??$copy_s@U?$char_traits@D@std@@@_Traits_helper@std@@YAPADPADIPBDI@Z 00104474 f i atcmd.obj
 0001:000034dc       ??$move_s@U?$char_traits@D@std@@@_Traits_helper@std@@YAPADPADIPBDI@Z 001044dc f i atcmd.obj
 0001:00003544       ??$_Allocate@D@std@@YAPADIPAD@Z 00104544 f i atcmd.obj
 0001:000035cc       ??0bad_alloc@std@@QAA@PBD@Z 001045cc f i atcmd.obj
 0001:00003610       ??1bad_alloc@std@@UAA@XZ   00104610 f i atcmd.obj
 0001:00003638       ??_Gbad_alloc@std@@UAAPAXI@Z 00104638 f i atcmd.obj
 0001:00003638       ??_Ebad_alloc@std@@UAAPAXI@Z 00104638 f i atcmd.obj
 0001:00003678       ??0bad_alloc@std@@QAA@ABV01@@Z 00104678 f i atcmd.obj
 0001:000036bc       ?deallocate@?$allocator@PAPAVCCommand@@@std@@QAAXPAPAPAVCCommand@@I@Z 001046bc f i atcmd.obj
 0001:000036d4       ?allocate@?$allocator@PAPAVCCommand@@@std@@QAAPAPAPAVCCommand@@I@Z 001046d4 f i atcmd.obj
 0001:00003708       ??0?$_Deque_iterator@PAVCCommand@@V?$allocator@PAVCCommand@@@std@@$00@std@@QAA@IPBV_Container_base@1@@Z 00104708 f i atcmd.obj
 0001:00003740       ??D?$_Deque_const_iterator@PAVCCommand@@V?$allocator@PAVCCommand@@@std@@$00@std@@QBAABQAVCCommand@@XZ 00104740 f i atcmd.obj
 0001:000038e4       ?max_size@?$allocator@PAVCCommand@@@std@@QBAIXZ 001048e4 f i atcmd.obj
 0001:00003938       ??0?$_Deque_const_iterator@PAVCCommand@@V?$allocator@PAVCCommand@@@std@@$00@std@@QAA@IPBV_Container_base@1@@Z 00104938 f i atcmd.obj
 0001:00003a58       ?_Adopt@_Iterator_base@std@@QAAXPBV_Container_base@2@@Z 00104a58 f i atcmd.obj
 0001:00003b08       ??0?$_Ranit@PAVCCommand@@HPBQAV1@ABQAV1@@std@@QAA@XZ 00104b08 f i atcmd.obj
 0001:00003b38       ??0_Iterator_base@std@@QAA@XZ 00104b38 f i atcmd.obj
 0001:00003b78       ??$_Char_traits_cat@U?$char_traits@D@std@@@std@@YA?AU_Secure_char_traits_tag@0@XZ 00104b78 f i atcmd.obj
 0001:00003bac       ??$copy_s@U?$char_traits@D@std@@@_Traits_helper@std@@YAPADPADIPBDIU_Secure_char_traits_tag@1@@Z 00104bac f i atcmd.obj
 0001:00003be8       ?_Copy_s@?$char_traits@D@std@@SAPADPADIPBDI@Z 00104be8 f i atcmd.obj
 0001:00003c20       ??$move_s@U?$char_traits@D@std@@@_Traits_helper@std@@YAPADPADIPBDIU_Secure_char_traits_tag@1@@Z 00104c20 f i atcmd.obj
 0001:00003c5c       ?_Move_s@?$char_traits@D@std@@SAPADPADIPBDI@Z 00104c5c f i atcmd.obj
 0001:00003c94       ??$unchecked_uninitialized_copy@PAPAPAVCCommand@@PAPAPAV1@V?$allocator@PAPAVCCommand@@@std@@@stdext@@YAPAPAPAVCCommand@@PAPAPAV1@00AAV?$allocator@PAPAVCCommand@@@std@@@Z 00104c94 f i atcmd.obj
 0001:00003d3c       ??$unchecked_uninitialized_fill_n@PAPAPAVCCommand@@IPAPAV1@V?$allocator@PAPAVCCommand@@@std@@@stdext@@YAXPAPAPAVCCommand@@IABQAPAV1@AAV?$allocator@PAPAVCCommand@@@std@@@Z 00104d3c f i atcmd.obj
 0001:00003dbc       ??$_Destroy_range@PAPAVCCommand@@V?$allocator@PAPAVCCommand@@@std@@@std@@YAXPAPAPAVCCommand@@0AAV?$allocator@PAPAVCCommand@@@0@@Z 00104dbc f i atcmd.obj
 0001:00003e0c       ??$_Allocate@PAVCCommand@@@std@@YAPAPAVCCommand@@IPAPAV1@@Z 00104e0c f i atcmd.obj
 0001:00003e9c       ??$_Construct@PAVCCommand@@PAV1@@std@@YAXPAPAVCCommand@@ABQAV1@@Z 00104e9c f i atcmd.obj
 0001:00003f04       ??2@YAPAXIPAX@Z            00104f04 f i atcmd.obj
 0001:00003f28       ??$_Destroy@PAVCCommand@@@std@@YAXPAPAVCCommand@@@Z 00104f28 f i atcmd.obj
 0001:00003f38       ??$_Allocate@PAPAVCCommand@@@std@@YAPAPAPAVCCommand@@IPAPAPAV1@@Z 00104f38 f i atcmd.obj
 0001:00003fc8       ??$_Checked_base@PAPAPAVCCommand@@@std@@YAPAPAPAVCCommand@@AAPAPAPAV1@@Z 00104fc8 f i atcmd.obj
 0001:00003ffc       ??$_Ptr_cat@PAPAPAVCCommand@@PAPAPAV1@@std@@YA?AU_Scalar_ptr_iterator_tag@0@AAPAPAPAVCCommand@@0@Z 00104ffc f i atcmd.obj
 0001:00004030       ??$_Uninit_copy@PAPAPAVCCommand@@PAPAPAV1@V?$allocator@PAPAVCCommand@@@std@@@std@@YAPAPAPAVCCommand@@PAPAPAV1@00AAV?$allocator@PAPAVCCommand@@@0@U_Scalar_ptr_iterator_tag@0@U_Range_checked_iterator_tag@0@@Z 00105030 f i atcmd.obj
 0001:000040d8       ??$_Uninit_fill_n@PAPAPAVCCommand@@IPAPAV1@V?$allocator@PAPAVCCommand@@@std@@@std@@YAXPAPAPAVCCommand@@IABQAPAV1@AAV?$allocator@PAPAVCCommand@@@0@U_Scalar_ptr_iterator_tag@0@U_Range_checked_iterator_tag@0@@Z 001050d8 f i atcmd.obj
 0001:000040f8       ??$_Destroy_range@PAPAVCCommand@@V?$allocator@PAPAVCCommand@@@std@@@std@@YAXPAPAPAVCCommand@@0AAV?$allocator@PAPAVCCommand@@@0@U_Scalar_ptr_iterator_tag@0@@Z 001050f8 f i atcmd.obj
 0001:00004108       ??$_Checked_base@PAPAPAVCCommand@@@std@@YAPAPAPAVCCommand@@AAPAPAPAV1@U_Unchanged_checked_iterator_base_type_tag@0@@Z 00105108 f i atcmd.obj
 0001:00004130       ??$_Debug_range@PAPAPAVCCommand@@@std@@YAXPAPAPAVCCommand@@0PBGI@Z 00105130 f i atcmd.obj
 0001:00004184       ??$_Debug_pointer@PAPAVCCommand@@@std@@YAXPAPAPAVCCommand@@PBGI@Z 00105184 f i atcmd.obj
 0001:000041b4       ??$unchecked_fill_n@PAPAPAVCCommand@@IPAPAV1@@stdext@@YAXPAPAPAVCCommand@@IABQAPAV1@@Z 001051b4 f i atcmd.obj
 0001:0000421c       ??$_Iter_cat@PAPAPAVCCommand@@@std@@YA?AUrandom_access_iterator_tag@0@ABQAPAPAVCCommand@@@Z 0010521c f i atcmd.obj
 0001:00004240       ??$_Debug_range2@PAPAPAVCCommand@@@std@@YAXPAPAPAVCCommand@@0PBGIUrandom_access_iterator_tag@0@@Z 00105240 f i atcmd.obj
 0001:000042a4       ??$_Fill_n@PAPAPAVCCommand@@IPAPAV1@@std@@YAXPAPAPAVCCommand@@IABQAPAV1@Urandom_access_iterator_tag@0@U_Range_checked_iterator_tag@0@@Z 001052a4 f i atcmd.obj
 0001:00004304       ??$_Fill_n@PAPAPAVCCommand@@IPAPAV1@@std@@YAXPAPAPAVCCommand@@IABQAPAV1@U_Range_checked_iterator_tag@0@@Z 00105304 f i atcmd.obj
 0001:00004350       ?Wait4ATConnectThreadProc@@YAKPAX@Z 00105350 f   callctrl.obj
 0001:00004384       ?ConvertToRILDisconnectCode@@YAKW4SWI_TYPE_EndReason@@@Z 00105384 f   callctrl.obj
 0001:000044fc       ?IsDataCall@CRadio@@QAAHW4SWI_TYPE_CDMA_CallState@@@Z 001054fc f   callctrl.obj
 0001:00004574       ?IsVoiceCall@CRadio@@QAAHW4SWI_TYPE_CDMA_CallState@@@Z 00105574 f   callctrl.obj
 0001:000045f4       ?IsEmergencyNumber@CRadio@@AAAHPBG@Z 001055f4 f   callctrl.obj
 0001:0000483c       ?GetEmergencyNumberCategory@CRadio@@AAAEPBG@Z 0010583c f   callctrl.obj
 0001:00004ab8       ?IsSpecialNumber@@YAHPAG@Z 00105ab8 f   callctrl.obj
 0001:00004ae4       ?RILDrv_Dial@@YAJKPBDKK@Z  00105ae4 f   callctrl.obj
 0001:00005090       ?RILDrv_Answer@@YAJK@Z     00106090 f   callctrl.obj
 0001:00005184       ?RILDrv_Hangup@@YAJK@Z     00106184 f   callctrl.obj
 0001:000052c0       ?RILDrv_DataDormant@@YAJK@Z 001062c0 f   callctrl.obj
 0001:000053ac       ?RILDrv_SendDTMF@@YAJKPBDK@Z 001063ac f   callctrl.obj
 0001:000056ec       ?RILDrv_GetCallList@@YAJK@Z 001066ec f   callctrl.obj
 0001:00005810       ?RILDrv_ManageCalls@@YAJKKK@Z 00106810 f   callctrl.obj
 0001:000059cc       ?RILDrv_TransferCall@@YAJKPBUriladdress_tag@@PBUrilsubaddress_tag@@@Z 001069cc f   callctrl.obj
 0001:00005b4c       ?RILDrv_GetLineStatus@@YAJK@Z 00106b4c f   callctrl.obj
 0001:00005c6c       ?RILDrv_GetCurrentPrivacyStatus@@YAJK@Z 00106c6c f   callctrl.obj
 0001:00005d50       ?RILDrv_SendAKey@@YAJKPBD@Z 00106d50 f   callctrl.obj
 0001:00005f68       ?RILDrv_SendFlash@@YAJKPAUriladdress_tag@@@Z 00106f68 f   callctrl.obj
 0001:00006290       ?RILDrv_SetCurrentAddressId@@YAJKK@Z 00107290 f   callctrl.obj
 0001:0000637c       ?RILDrv_GetCurrentAddressId@@YAJK@Z 0010737c f   callctrl.obj
 0001:00006460       ?FillCallInfoStruct@@YAXPAUrilcallinfo_tag@@KKKPAGK@Z 00107460 f   callctrl.obj
 0001:00006640       ?Dial@CRadio@@QAAJPAVCResponse@@PAX@Z 00107640 f   callctrl.obj
 0001:000077a4       ?Answer@CRadio@@QAAJPAVCResponse@@@Z 001087a4 f   callctrl.obj
 0001:0000796c       ?HangUp@CRadio@@QAAJPAVCResponse@@@Z 0010896c f   callctrl.obj
 0001:0000804c       ?DataDormant@CRadio@@QAAJPAVCResponse@@@Z 0010904c f   callctrl.obj
 0001:000081bc       ?GetCallList@CRadio@@QAAJPAVCResponse@@@Z 001091bc f   callctrl.obj
 0001:0000859c       ?ManageCall@CRadio@@QAAJPAVCResponse@@PAX@Z 0010959c f   callctrl.obj
 0001:00008694       ?ManageCDMACall@CRadio@@QAAJPAVCResponse@@PAX@Z 00109694 f   callctrl.obj
 0001:000089b4       ?ManageGSMCall@CRadio@@QAAJPAVCResponse@@PAX@Z 001099b4 f   callctrl.obj
 0001:00009430       ?GetLineStatus@CRadio@@QAAJPAVCResponse@@@Z 0010a430 f   callctrl.obj
 0001:00009628       ?ReadCurrentPrivacyStatus@CRadio@@QAAJXZ 0010a628 f   callctrl.obj
 0001:00009698       ?GetCurrentPrivacyStatus@CRadio@@QAAJPAVCResponse@@@Z 0010a698 f   callctrl.obj
 0001:00009788       ?SendAKey@CRadio@@QAAJPAVCResponse@@PAX@Z 0010a788 f   callctrl.obj
 0001:00009938       ?SendFlash@CRadio@@QAAJPAVCResponse@@PAX@Z 0010a938 f   callctrl.obj
 0001:00009dec       ?SendDTMF@CRadio@@QAAJPAVCResponse@@PAX@Z 0010adec f   callctrl.obj
 0001:0000a344       ?SetCurrentAddressId@CRadio@@QAAJPAVCResponse@@PAX@Z 0010b344 f   callctrl.obj
 0001:0000a63c       ?GetCurrentAddressId@CRadio@@QAAJPAVCResponse@@@Z 0010b63c f   callctrl.obj
 0001:0000a760       ?RILDrv_SetBearerServiceOptions@@YAJKPBUrilbearersvcinfo_tag@@@Z 0010b760 f   callctrl.obj
 0001:0000a8a8       ?SetBearerServiceInfo@CRadio@@QAAJPAVCResponse@@PAX@Z 0010b8a8 f   callctrl.obj
 0001:0000a934       ?FillRemotePartyInfo@@YAXPAUrilremotepartyinfo_tag@@PBUriladdress_tag@@@Z 0010b934 f   callctrl.obj
 0001:0000abdc       ?BroadcastRemotePartyInfo@CRadio@@QAAXKPBUriladdress_tag@@@Z 0010bbdc f   callctrl.obj
 0001:0000ac90       ?LookupCallIdByCallStatus@CRadio@@QAAHKAAK@Z 0010bc90 f   callctrl.obj
 0001:0000addc       ?SetCallStatus@CRadio@@QAAHKKKH@Z 0010bddc f   callctrl.obj
 0001:0000afe8       ?CallExists@CRadio@@QAAKK@Z 0010bfe8 f   callctrl.obj
 0001:0000b164       ?GetNumOfActiveCalls@CRadio@@QAAIXZ 0010c164 f   callctrl.obj
 0001:0000b228       ?GetNumOfActiveVoiceCalls@CRadio@@QAAIXZ 0010c228 f   callctrl.obj
 0001:0000b2ec       ?PacketDataCallOnEVDOsystem@CRadio@@QAAHXZ 0010c2ec f   callctrl.obj
 0001:0000b33c       ?LookupCallIDByQmiID@CRadio@@QAAHEAAK@Z 0010c33c f   callctrl.obj
 0001:0000b3f4       ?AddNewVoiceCall@CRadio@@QAAHAAKEKKKKPAGKK@Z 0010c3f4 f   callctrl.obj
 0001:0000b4e8       ?AddCall@CRadio@@QAAHKEKKKKPAGKK@Z 0010c4e8 f   callctrl.obj
 0001:0000b8a8       ?RemCall@CRadio@@QAAHK@Z   0010c8a8 f   callctrl.obj
 0001:0000ba24       ?GetCallType@CRadio@@QAAHKAAK@Z 0010ca24 f   callctrl.obj
 0001:0000bb68       ?GetMultiParty@CRadio@@QAAHKAAK@Z 0010cb68 f   callctrl.obj
 0001:0000bcac       ?SetMultiParty@CRadio@@QAAHKK@Z 0010ccac f   callctrl.obj
 0001:0000bdcc       ?UpdateLineStatus@CRadio@@QAAXXZ 0010cdcc f   callctrl.obj
 0001:0000c068       ?SetLineStatus@CRadio@@QAAXK@Z 0010d068 f   callctrl.obj
 0001:0000c110       ?GetCallInfo@CRadio@@QAAPBUrilcallinfo_tag@@K@Z 0010d110 f   callctrl.obj
 0001:0000c200       ?GetCallDestAddress@CRadio@@QAAPAGK@Z 0010d200 f   callctrl.obj
 0001:0000c320       ?InitiateDataCall@CRadio@@AAAJPAU__Dial_Data@@PAVCResponse@@@Z 0010d320 f   callctrl.obj
 0001:0000cb30       ?CloseDataPort@CRadio@@QAAHH@Z 0010db30 f   callctrl.obj
 0001:0000ccbc       ?HandleSWI_NOTIFY_CallConnecting@CRadio@@QAAXPAUSwiNotifyVariant@@@Z 0010dcbc f   callctrl.obj
 0001:0000d068       ?HandleSWI_NOTIFY_CallConnected@CRadio@@QAAXPAUSwiNotifyVariant@@@Z 0010e068 f   callctrl.obj
 0001:0000d7e0       ?HandleSWI_NOTIFY_CallDisconnected@CRadio@@QAAXPAUSwiNotifyVariant@@@Z 0010e7e0 f   callctrl.obj
 0001:0000dff8       ?HandleSWI_NOTIFY_CallIncomming@CRadio@@QAAXPAUSwiNotifyVariant@@@Z 0010eff8 f   callctrl.obj
 0001:0000ee68       ?HandleSWI_NOTIFY_COLP@CRadio@@QAAXPAUSwiNotifyVariant@@@Z 0010fe68 f   callctrl.obj
 0001:0000f164       ?HandleSWI_NOTIFY_CallCallerID@CRadio@@QAAXPAUSwiNotifyVariant@@@Z 00110164 f   callctrl.obj
 0001:0000f45c       ?HandleSWI_NOTIFY_OTASPState@CRadio@@QAAXPAUSwiNotifyVariant@@@Z 0011045c f   callctrl.obj
 0001:0000f74c       ?HandleSWI_NOTIFY_CallDormant@CRadio@@QAAXPAUSwiNotifyVariant@@@Z 0011074c f   callctrl.obj
 0001:0000f824       ?HandleSWI_NOTIFY_PktSessionCall@CRadio@@QAAXPAUSwiNotifyVariant@@@Z 00110824 f   callctrl.obj
 0001:0000fa34       ?HandleSWI_NOTIFY_USSD@CRadio@@QAAXPAUSwiNotifyVariant@@@Z 00110a34 f   callctrl.obj
 0001:0000fe64       ?UpdateAndBroadcastOnSWICallNotification@CRadio@@QAAXPAUSwiNotifyVariant@@@Z 00110e64 f   callctrl.obj
 0001:000101e4       ?GetRILCallTypeFromCMCallType@CRadio@@QAAKW4SWI_TYPE_CDMA_CallType@@@Z 001111e4 f   callctrl.obj
 0001:00010360       ?BroadcastCallStateChangedNotification@CRadio@@QAAXXZ 00111360 f   callctrl.obj
 0001:00010560       ?PacketDataStatusNotification@CRadio@@QAAXW4SWI_TYPE_CDMA_CallState@@@Z 00111560 f   callctrl.obj
 0001:000106b0       ?DataCallDisconnected@CRadio@@QAAHW4SWI_TYPE_EndReason@@@Z 001116b0 f   callctrl.obj
 0001:00010984       ??1?$_Iterator@$00@?$list@UtagEMERGENCY_NUM_INFO@@V?$allocator@UtagEMERGENCY_NUM_INFO@@@std@@@std@@QAA@XZ 00111984 f i callctrl.obj
 0001:0001099c       ??4?$_Iterator@$00@?$list@UtagEMERGENCY_NUM_INFO@@V?$allocator@UtagEMERGENCY_NUM_INFO@@@std@@@std@@QAAAAV012@ABV012@@Z 0011199c f i callctrl.obj
 0001:000109cc       ??1?$_Const_iterator@$00@?$list@UtagEMERGENCY_NUM_INFO@@V?$allocator@UtagEMERGENCY_NUM_INFO@@@std@@@std@@QAA@XZ 001119cc f i callctrl.obj
 0001:000109e4       ??4?$_Const_iterator@$00@?$list@UtagEMERGENCY_NUM_INFO@@V?$allocator@UtagEMERGENCY_NUM_INFO@@@std@@@std@@QAAAAV012@ABV012@@Z 001119e4 f i callctrl.obj
 0001:00010a2c       ??1?$_Bidit@UtagEMERGENCY_NUM_INFO@@HPBU1@ABU1@@std@@QAA@XZ 00111a2c f i callctrl.obj
 0001:00010a44       ??4?$_Bidit@UtagEMERGENCY_NUM_INFO@@HPBU1@ABU1@@std@@QAAAAU01@ABU01@@Z 00111a44 f i callctrl.obj
 0001:00010a7c       ??4_Iterator_base@std@@QAAAAV01@ABV01@@Z 00111a7c f i callctrl.obj
 0001:00010b04       ??BWideString@@QAAPAGXZ    00111b04 f i callctrl.obj
 0001:00010b50       ?GetRadioHandle@CRilHandle@@QAAPAVCRadio@@XZ 00111b50 f i callctrl.obj
 0001:00010bd4       ??BAnsiString@@QAAPADXZ    00111bd4 f i callctrl.obj
 0001:00010c20       ?wcsstr@@YAPAGPAGPBG@Z     00111c20 f i callctrl.obj
 0001:00010c54       ?SetNotifyCode@CResponse@@QAAXK@Z 00111c54 f i callctrl.obj
 0001:00010c74       ?GetRILCarrierIndex@CRilHandle@@QAAIXZ 00111c74 f i callctrl.obj
 0001:00010ca4       ?GetDevCapsHandle@CRadio@@QAAPAVCRadioCaps@@XZ 00111ca4 f i callctrl.obj
 0001:00010cd4       ?IsVoiceSupported@CRadioCaps@@QAAHXZ 00111cd4 f i callctrl.obj
 0001:00010d04       ?IsMOVoiceAllowed@CRadioCaps@@QAAHXZ 00111d04 f i callctrl.obj
 0001:00010d34       ?IsAllowedEmergencyCallsOnly@CRadioCaps@@QAAHXZ 00111d34 f i callctrl.obj
 0001:00010d64       ?IsAllowedSpecialCallsOnly@CRadioCaps@@QAAHXZ 00111d64 f i callctrl.obj
 0001:00010d94       ?IsDataSupported@CRadioCaps@@QAAHXZ 00111d94 f i callctrl.obj
 0001:00010dc4       ?MakeOK@CResponse@@QAAXXZ  00111dc4 f i callctrl.obj
 0001:00010de4       ?IsMTDataAllowed@CRadioCaps@@QAAHXZ 00111de4 f i callctrl.obj
 0001:00010e14       ?IsMTVoiceAllowed@CRadioCaps@@QAAHXZ 00111e14 f i callctrl.obj
 0001:00010e44       ?IsMODataAllowed@CRadioCaps@@QAAHXZ 00111e44 f i callctrl.obj
 0001:00010e74       ?PacketDataCallStatus@CRadio@@QAA?AW4RIL_PACKETDATASTATUS_ADV_STATE@@XZ 00111e74 f i callctrl.obj
 0001:00010ea4       ?GetLastError@CRadio@@QAAKXZ 00111ea4 f i callctrl.obj
 0001:00010ed4       ?GetSwiWirelessTech@CRadio@@QAAKXZ 00111ed4 f i callctrl.obj
 0001:00010f04       ?GetOldCarrierIndex@CRilHandle@@QAAIXZ 00111f04 f i callctrl.obj
 0001:00010f34       ?begin@?$list@UtagEMERGENCY_NUM_INFO@@V?$allocator@UtagEMERGENCY_NUM_INFO@@@std@@@std@@QAA?AV?$_Iterator@$00@12@XZ 00111f34 f i callctrl.obj
 0001:00010f98       ?end@?$list@UtagEMERGENCY_NUM_INFO@@V?$allocator@UtagEMERGENCY_NUM_INFO@@@std@@@std@@QAA?AV?$_Iterator@$00@12@XZ 00111f98 f i callctrl.obj
 0001:00010fec       ??0?$_Iterator@$00@?$list@UtagEMERGENCY_NUM_INFO@@V?$allocator@UtagEMERGENCY_NUM_INFO@@@std@@@std@@QAA@XZ 00111fec f i callctrl.obj
 0001:0001101c       ??D?$_Iterator@$00@?$list@UtagEMERGENCY_NUM_INFO@@V?$allocator@UtagEMERGENCY_NUM_INFO@@@std@@@std@@QBAAAUtagEMERGENCY_NUM_INFO@@XZ 0011201c f i callctrl.obj
 0001:0001104c       ??E?$_Iterator@$00@?$list@UtagEMERGENCY_NUM_INFO@@V?$allocator@UtagEMERGENCY_NUM_INFO@@@std@@@std@@QAAAAV012@XZ 0011204c f i callctrl.obj
 0001:00011078       ??9?$_Const_iterator@$00@?$list@UtagEMERGENCY_NUM_INFO@@V?$allocator@UtagEMERGENCY_NUM_INFO@@@std@@@std@@QBA_NABV012@@Z 00112078 f i callctrl.obj
 0001:000110d0       ?_Nextnode@?$list@UtagEMERGENCY_NUM_INFO@@V?$allocator@UtagEMERGENCY_NUM_INFO@@@std@@@std@@KAAAPAU_Node@?$_List_nod@UtagEMERGENCY_NUM_INFO@@V?$allocator@UtagEMERGENCY_NUM_INFO@@@std@@@2@PAU342@@Z 001120d0 f i callctrl.obj
 0001:000110f4       ??0?$_Iterator@$00@?$list@UtagEMERGENCY_NUM_INFO@@V?$allocator@UtagEMERGENCY_NUM_INFO@@@std@@@std@@QAA@PAU_Node@?$_List_nod@UtagEMERGENCY_NUM_INFO@@V?$allocator@UtagEMERGENCY_NUM_INFO@@@std@@@2@PBV12@@Z 001120f4 f i callctrl.obj
 0001:0001112c       ??0?$_Const_iterator@$00@?$list@UtagEMERGENCY_NUM_INFO@@V?$allocator@UtagEMERGENCY_NUM_INFO@@@std@@@std@@QAA@XZ 0011212c f i callctrl.obj
 0001:0001116c       ??D?$_Const_iterator@$00@?$list@UtagEMERGENCY_NUM_INFO@@V?$allocator@UtagEMERGENCY_NUM_INFO@@@std@@@std@@QBAABUtagEMERGENCY_NUM_INFO@@XZ 0011216c f i callctrl.obj
 0001:00011248       ??E?$_Const_iterator@$00@?$list@UtagEMERGENCY_NUM_INFO@@V?$allocator@UtagEMERGENCY_NUM_INFO@@@std@@@std@@QAAAAV012@XZ 00112248 f i callctrl.obj
 0001:00011338       ??8?$_Const_iterator@$00@?$list@UtagEMERGENCY_NUM_INFO@@V?$allocator@UtagEMERGENCY_NUM_INFO@@@std@@@std@@QBA_NABV012@@Z 00112338 f i callctrl.obj
 0001:000113a0       ??0?$_Bidit@UtagEMERGENCY_NUM_INFO@@HPBU1@ABU1@@std@@QAA@XZ 001123a0 f i callctrl.obj
 0001:000113d0       ?_Myval@?$list@UtagEMERGENCY_NUM_INFO@@V?$allocator@UtagEMERGENCY_NUM_INFO@@@std@@@std@@KAAAUtagEMERGENCY_NUM_INFO@@PAU_Node@?$_List_nod@UtagEMERGENCY_NUM_INFO@@V?$allocator@UtagEMERGENCY_NUM_INFO@@@std@@@2@@Z 001123d0 f i callctrl.obj
 0001:00011400       ??0?$_Const_iterator@$00@?$list@UtagEMERGENCY_NUM_INFO@@V?$allocator@UtagEMERGENCY_NUM_INFO@@@std@@@std@@QAA@PAU_Node@?$_List_nod@UtagEMERGENCY_NUM_INFO@@V?$allocator@UtagEMERGENCY_NUM_INFO@@@std@@@2@PBV12@@Z 00112400 f i callctrl.obj
 0001:00011468       ?_Compat@?$_Const_iterator@$00@?$list@UtagEMERGENCY_NUM_INFO@@V?$allocator@UtagEMERGENCY_NUM_INFO@@@std@@@std@@QBAXABV123@@Z 00112468 f i callctrl.obj
 0001:00011524       ?RILDrv_GetDevCaps@@YAJKK@Z 00112524 f   caps.obj
 0001:00011690       ?GetDevCaps@CRadio@@QAAJPAVCResponse@@PAX@Z 00112690 f   caps.obj
 0001:00011acc       ?GetDevCapsDial@CRadioCaps@@QAAXAAPAXAAI@Z 00112acc f i caps.obj
 0001:00011af4       ?GetDevCapsEquipmentStates@CRadioCaps@@QAAXAAPAXAAI@Z 00112af4 f i caps.obj
 0001:00011b20       ?GetSignalQualityImplemenation@CRadioCaps@@QAAXAAPAXAAI@Z 00112b20 f i caps.obj
 0001:00011b4c       ?GetDevCapsSimSupport@CRadioCaps@@QAAXAAPAXAAI@Z 00112b4c f i caps.obj
 0001:00011b78       ?GetDevCapsNitzNotification@CRadioCaps@@QAAXAAPAXAAI@Z 00112b78 f i caps.obj
 0001:00011ba4       ?GetDevCapsPhoneCapability@CRadioCaps@@QAAXAAPAXAAI@Z 00112ba4 f i caps.obj
 0001:00011bd0       ?GetDevCapsPBStoreLocs@CRadioCaps@@QAAXAAPAXAAI@Z 00112bd0 f i caps.obj
 0001:00011bfc       ?GetDevCapsPBIndexRange@CRadioCaps@@QAAXAAPAXAAI@Z 00112bfc f i caps.obj
 0001:00011c28       ?GetRilCapsPBEntryLength@CRadioCaps@@QAAXAAPAXAAI@Z 00112c28 f i caps.obj
 0001:00011c54       ?GetDevCapsLockFacilities@CRadioCaps@@QAAXAAPAXAAI@Z 00112c54 f i caps.obj
 0001:00011c80       ?GetDevCapsLockPwdLengths@CRadioCaps@@QAAXAAPAXAAI@Z 00112c80 f i caps.obj
 0001:00011cac       ?GetAvailStoreMem@@YAKXZ   00112cac f   channel.obj
 0001:00011ce4       ??0CChannel@@QAA@IJ@Z      00112ce4 f   channel.obj
 0001:00011df4       ??0CChannel@@QAA@PAGJ@Z    00112df4 f   channel.obj
 0001:00011ee8       ??1CChannel@@UAA@XZ        00112ee8 f   channel.obj
 0001:00011f20       ?IsChannelOpen@CChannel@@QAAHXZ 00112f20 f   channel.obj
 0001:00011f78       ?SetupChannel@CChannel@@QAAXXZ 00112f78 f   channel.obj
 0001:00012194       ?RecvThread@@YAXPAX@Z      00113194 f   channel.obj
 0001:000122f4       ?CreateChannel@CChannel@@QAAPAXP6AKKPAE@Z@Z 001132f4 f   channel.obj
 0001:000124dc       ?CloseChannel@CChannel@@QAAXXZ 001134dc f   channel.obj
 0001:000125d8       ?ResetChannel@CChannel@@QAAXXZ 001135d8 f   channel.obj
 0001:0001261c       ?ClearChannelError@CChannel@@QAAXPAX@Z 0011361c f   channel.obj
 0001:00012640       ?SendData@CChannel@@QAAKKPAE@Z 00113640 f   channel.obj
 0001:000126b4       ?PublicSendDataToEMPort@ChannelLinker@@SAKKPAE@Z 001136b4 f   channel.obj
 0001:00012740       ?PublicSendDataToEXPort@ChannelLinker@@SAKKPAE@Z 00113740 f   channel.obj
 0001:000127cc       ?ConfigChannel@CChannel@@QAAXIJ@Z 001137cc f   channel.obj
 0001:000127fc       ?DeviceIOCtrl@CChannel@@QAAHKPAXK0KPAKPAU_OVERLAPPED@@@Z 001137fc f   channel.obj
 0001:000128c0       ??0ChannelLinker@@QAA@PAGJ0J@Z 001138c0 f   channel.obj
 0001:00012c9c       ??1ChannelLinker@@UAA@XZ   00113c9c f   channel.obj
 0001:00013000       ?StartEMPort@ChannelLinker@@QAAXXZ 00114000 f   channel.obj
 0001:0001308c       ?StartEXPort@ChannelLinker@@QAAXXZ 0011408c f   channel.obj
 0001:00013118       ?EMPortThread@ChannelLinker@@SAXPAX@Z 00114118 f   channel.obj
 0001:000131b0       ?EXPortThread@ChannelLinker@@SAXPAX@Z 001141b0 f   channel.obj
 0001:00013254       ?DisplayRawData@CChannel@@QAAXEIPAE@Z 00114254 f   channel.obj
 0001:00013418       ??_ECChannel@@UAAPAXI@Z    00114418 f i channel.obj
 0001:00013418       ??_GCChannel@@UAAPAXI@Z    00114418 f i channel.obj
 0001:00013458       ?GetChannelError@CChannel@@QAAIXZ 00114458 f i channel.obj
 0001:00013484       ?GetMySelf@ChannelLinker@@SAPAV1@XZ 00114484 f i channel.obj
 0001:000134a4       ?InternalSend@CChannel@@QAAHPAXJPAE@Z 001144a4 f i channel.obj
 0001:00013638       ?InternalRecv@CChannel@@QAAHPAJPAE@Z 00114638 f i channel.obj
 0001:000138a4       ??_EChannelLinker@@UAAPAXI@Z 001148a4 f i channel.obj
 0001:000138a4       ??_GChannelLinker@@UAAPAXI@Z 001148a4 f i channel.obj
 0001:000138e4       ??0CCommand@@QAA@XZ        001148e4 f   command.obj
 0001:0001397c       ??1CCommand@@QAA@XZ        0011497c f   command.obj
 0001:00013abc       ?Init@CCommand@@QAAHQAVCRilInstanceHandle@@KKKW4APIID@@K@Z 00114abc f   command.obj
 0001:00013cd0       ?Init@CCommand@@QAAHQAVCRilInstanceHandle@@KKKPAXW4APIID@@K@Z 00114cd0 f   command.obj
 0001:00013ec0       ?Init@CCommand@@QAAHPAV1@@Z 00114ec0 f   command.obj
 0001:00013f94       ?GetPriority@CCommand@@QBAKXZ 00114f94 f   command.obj
 0001:0001402c       ?SendResponse@CCommand@@QBAHKQBXI@Z 0011502c f   command.obj
 0001:00014400       ?IsDataDialCommand@CCommand@@QAAHXZ 00115400 f   command.obj
 0001:0001447c       ??0CListElem@@QAA@XZ       0011547c f i command.obj
 0001:000144bc       ??1CListElem@@QAA@XZ       001154bc f i command.obj
 0001:000144cc       ?FInit@CCommand@@QBAHXZ    001154cc f i command.obj
 0001:000144fc       ?FIgnoreRsp@CCommand@@QBAHXZ 001154fc f i command.obj
 0001:0001452c       ?IsTimeout@CCommand@@QBAHK@Z 0011552c f i command.obj
 0001:0001458c       ?FReadyForNotifications@CRilInstanceHandle@@QBAHXZ 0011558c f i command.obj
 0001:000145f4       ?Ready@?$CUnboundedQueue@Urildrvnotification_tag@@@@QBAHXZ 001155f4 f i command.obj
 0001:0001465c       ?Ready@CEvent@@QBAHXZ      0011565c f i command.obj
 0001:000146a8       ?RILDrv_GetHSCSDCallSettings@@YAJK@Z 001156a8 f   data.obj
 0001:00014748       ?RILDrv_GetBearerServiceOptions@@YAJK@Z 00115748 f   data.obj
 0001:000147e8       ?RILDrv_GetRLPOptions@@YAJK@Z 001157e8 f   data.obj
 0001:00014890       ?RILDrv_SetRLPOptions@@YAJKPBUrilrlpinfo_tag@@@Z 00115890 f   data.obj
 0001:000152b4       ?RILDrv_GetDataCompression@@YAJK@Z 001162b4 f   data.obj
 0001:0001535c       ?RILDrv_SetDataCompression@@YAJKPBUrildatacompinfo_tag@@@Z 0011635c f   data.obj
 0001:00015ad8       ?RILDrv_GetErrorCorrection@@YAJK@Z 00116ad8 f   data.obj
 0001:00015b80       ?RILDrv_SetErrorCorrection@@YAJKPBUrilerrorcorrectioninfo_tag@@@Z 00116b80 f   data.obj
 0001:000161ac       ?RILDrv_GetSerialPortHandleFromContextID@@YAJKPAGKPAK@Z 001171ac f   data.obj
 0001:00016274       ?RILDrv_GetVTSerialPortHandle@@YAJPAGKPAK@Z 00117274 f   data.obj
 0001:000162ac       ??0CDatERI@@QAA@XZ         001172ac f   DatERI.obj
 0001:00016354       ??1CDatERI@@QAA@XZ         00117354 f   DatERI.obj
 0001:000163cc       ?Reset@CDatERI@@QAAXXZ     001173cc f   DatERI.obj
 0001:0001666c       ?Load@CDatERI@@QAAHPAEG@Z  0011766c f   DatERI.obj
 0001:00016cac       ?ParseCallPrompt@CDatERI@@IAA_NPAUSWI_STRUCT_CallPrompt@1@PAEGAAG@Z 00117cac f   DatERI.obj
 0001:00016f0c       ?ParseRoamInd@CDatERI@@IAA_NPAUSWI_STRUCT_RoamInd@1@PAEGAAG@Z 00117f0c f   DatERI.obj
 0001:000171b8       ?ParseString@CDatERI@@IAAXPAEG_NPAG@Z 001181b8 f   DatERI.obj
 0001:000172e8       ?GetVersion@CDatERI@@QAAGXZ 001182e8 f   DatERI.obj
 0001:00017318       ?Save@CDatERI@@QAA_NPAEGAAG1@Z 00118318 f   DatERI.obj
 0001:000178f4       ?SaveCallPrompt@CDatERI@@IAA_NPAUSWI_STRUCT_CallPrompt@1@PAEGAAG@Z 001188f4 f   DatERI.obj
 0001:00017b10       ?SaveRoamInd@CDatERI@@IAA_NPAUSWI_STRUCT_RoamInd@1@PAEGAAG@Z 00118b10 f   DatERI.obj
 0001:00017da0       ?SaveString@CDatERI@@IAAXPAGPAE_N@Z 00118da0 f   DatERI.obj
 0001:00017eac       ?GetRoamDetails@CDatERI@@QAA_NHAAUSWI_STRUCT_ERI@@@Z 00118eac f   DatERI.obj
 0001:000180ac       ?RoamIDExists@CDatERI@@QAAHH@Z 001190ac f   DatERI.obj
 0001:000181a0       ?CalcCRC16@CDatERI@@IAAGPAEG@Z 001191a0 f   DatERI.obj
 0001:00018318       ??1?$map@GPAUSWI_STRUCT_RoamInd@CDatERI@@U?$less@G@std@@V?$allocator@U?$pair@$$CBGPAUSWI_STRUCT_RoamInd@CDatERI@@@std@@@4@@std@@QAA@XZ 00119318 f i DatERI.obj
 0001:00018330       ??1?$map@GPAUSWI_STRUCT_CallPrompt@CDatERI@@U?$less@G@std@@V?$allocator@U?$pair@$$CBGPAUSWI_STRUCT_CallPrompt@CDatERI@@@std@@@4@@std@@QAA@XZ 00119330 f i DatERI.obj
 0001:00018348       ??1iterator@?$_Tree@V?$_Tmap_traits@GPAUSWI_STRUCT_RoamInd@CDatERI@@U?$less@G@std@@V?$allocator@U?$pair@$$CBGPAUSWI_STRUCT_RoamInd@CDatERI@@@std@@@4@$0A@@std@@@std@@QAA@XZ 00119348 f i DatERI.obj
 0001:00018360       ??1iterator@?$_Tree@V?$_Tmap_traits@GPAUSWI_STRUCT_CallPrompt@CDatERI@@U?$less@G@std@@V?$allocator@U?$pair@$$CBGPAUSWI_STRUCT_CallPrompt@CDatERI@@@std@@@4@$0A@@std@@@std@@QAA@XZ 00119360 f i DatERI.obj
 0001:00018378       ??1const_iterator@?$_Tree@V?$_Tmap_traits@GPAUSWI_STRUCT_RoamInd@CDatERI@@U?$less@G@std@@V?$allocator@U?$pair@$$CBGPAUSWI_STRUCT_RoamInd@CDatERI@@@std@@@4@$0A@@std@@@std@@QAA@XZ 00119378 f i DatERI.obj
 0001:00018390       ??1const_iterator@?$_Tree@V?$_Tmap_traits@GPAUSWI_STRUCT_CallPrompt@CDatERI@@U?$less@G@std@@V?$allocator@U?$pair@$$CBGPAUSWI_STRUCT_CallPrompt@CDatERI@@@std@@@4@$0A@@std@@@std@@QAA@XZ 00119390 f i DatERI.obj
 0001:000183a8       ??1?$_Bidit@U?$pair@$$CBGPAUSWI_STRUCT_RoamInd@CDatERI@@@std@@HPBU12@ABU12@@std@@QAA@XZ 001193a8 f i DatERI.obj
 0001:000183c0       ??1?$_Bidit@U?$pair@$$CBGPAUSWI_STRUCT_CallPrompt@CDatERI@@@std@@HPBU12@ABU12@@std@@QAA@XZ 001193c0 f i DatERI.obj
 0001:000183d8       ??0?$map@GPAUSWI_STRUCT_RoamInd@CDatERI@@U?$less@G@std@@V?$allocator@U?$pair@$$CBGPAUSWI_STRUCT_RoamInd@CDatERI@@@std@@@4@@std@@QAA@XZ 001193d8 f i DatERI.obj
 0001:00018424       ??A?$map@GPAUSWI_STRUCT_RoamInd@CDatERI@@U?$less@G@std@@V?$allocator@U?$pair@$$CBGPAUSWI_STRUCT_RoamInd@CDatERI@@@std@@@4@@std@@QAAAAPAUSWI_STRUCT_RoamInd@CDatERI@@ABG@Z 00119424 f i DatERI.obj
 0001:00018630       ??1?$_Tree@V?$_Tmap_traits@GPAUSWI_STRUCT_RoamInd@CDatERI@@U?$less@G@std@@V?$allocator@U?$pair@$$CBGPAUSWI_STRUCT_RoamInd@CDatERI@@@std@@@4@$0A@@std@@@std@@QAA@XZ 00119630 f i DatERI.obj
 0001:00018670       ?begin@?$_Tree@V?$_Tmap_traits@GPAUSWI_STRUCT_RoamInd@CDatERI@@U?$less@G@std@@V?$allocator@U?$pair@$$CBGPAUSWI_STRUCT_RoamInd@CDatERI@@@std@@@4@$0A@@std@@@std@@QAA?AViterator@12@XZ 00119670 f i DatERI.obj
 0001:000186cc       ?end@?$_Tree@V?$_Tmap_traits@GPAUSWI_STRUCT_RoamInd@CDatERI@@U?$less@G@std@@V?$allocator@U?$pair@$$CBGPAUSWI_STRUCT_RoamInd@CDatERI@@@std@@@4@$0A@@std@@@std@@QAA?AViterator@12@XZ 001196cc f i DatERI.obj
 0001:00018720       ?clear@?$_Tree@V?$_Tmap_traits@GPAUSWI_STRUCT_RoamInd@CDatERI@@U?$less@G@std@@V?$allocator@U?$pair@$$CBGPAUSWI_STRUCT_RoamInd@CDatERI@@@std@@@4@$0A@@std@@@std@@QAAXXZ 00119720 f i DatERI.obj
 0001:000187dc       ?find@?$_Tree@V?$_Tmap_traits@GPAUSWI_STRUCT_RoamInd@CDatERI@@U?$less@G@std@@V?$allocator@U?$pair@$$CBGPAUSWI_STRUCT_RoamInd@CDatERI@@@std@@@4@$0A@@std@@@std@@QAA?AViterator@12@ABG@Z 001197dc f i DatERI.obj
 0001:00018a3c       ??0?$map@GPAUSWI_STRUCT_CallPrompt@CDatERI@@U?$less@G@std@@V?$allocator@U?$pair@$$CBGPAUSWI_STRUCT_CallPrompt@CDatERI@@@std@@@4@@std@@QAA@XZ 00119a3c f i DatERI.obj
 0001:00018a88       ??A?$map@GPAUSWI_STRUCT_CallPrompt@CDatERI@@U?$less@G@std@@V?$allocator@U?$pair@$$CBGPAUSWI_STRUCT_CallPrompt@CDatERI@@@std@@@4@@std@@QAAAAPAUSWI_STRUCT_CallPrompt@CDatERI@@ABG@Z 00119a88 f i DatERI.obj
 0001:00018c94       ??1?$_Tree@V?$_Tmap_traits@GPAUSWI_STRUCT_CallPrompt@CDatERI@@U?$less@G@std@@V?$allocator@U?$pair@$$CBGPAUSWI_STRUCT_CallPrompt@CDatERI@@@std@@@4@$0A@@std@@@std@@QAA@XZ 00119c94 f i DatERI.obj
 0001:00018cd4       ?begin@?$_Tree@V?$_Tmap_traits@GPAUSWI_STRUCT_CallPrompt@CDatERI@@U?$less@G@std@@V?$allocator@U?$pair@$$CBGPAUSWI_STRUCT_CallPrompt@CDatERI@@@std@@@4@$0A@@std@@@std@@QAA?AViterator@12@XZ 00119cd4 f i DatERI.obj
 0001:00018d30       ?end@?$_Tree@V?$_Tmap_traits@GPAUSWI_STRUCT_CallPrompt@CDatERI@@U?$less@G@std@@V?$allocator@U?$pair@$$CBGPAUSWI_STRUCT_CallPrompt@CDatERI@@@std@@@4@$0A@@std@@@std@@QAA?AViterator@12@XZ 00119d30 f i DatERI.obj
 0001:00018d84       ?size@?$_Tree@V?$_Tmap_traits@GPAUSWI_STRUCT_CallPrompt@CDatERI@@U?$less@G@std@@V?$allocator@U?$pair@$$CBGPAUSWI_STRUCT_CallPrompt@CDatERI@@@std@@@4@$0A@@std@@@std@@QBAIXZ 00119d84 f i DatERI.obj
 0001:00018db0       ?clear@?$_Tree@V?$_Tmap_traits@GPAUSWI_STRUCT_CallPrompt@CDatERI@@U?$less@G@std@@V?$allocator@U?$pair@$$CBGPAUSWI_STRUCT_CallPrompt@CDatERI@@@std@@@4@$0A@@std@@@std@@QAAXXZ 00119db0 f i DatERI.obj
 0001:00018e64       ??Citerator@?$_Tree@V?$_Tmap_traits@GPAUSWI_STRUCT_RoamInd@CDatERI@@U?$less@G@std@@V?$allocator@U?$pair@$$CBGPAUSWI_STRUCT_RoamInd@CDatERI@@@std@@@4@$0A@@std@@@std@@QBAPAU?$pair@$$CBGPAUSWI_STRUCT_RoamInd@CDatERI@@@2@XZ 00119e64 f i DatERI.obj
 0001:00018e9c       ??Eiterator@?$_Tree@V?$_Tmap_traits@GPAUSWI_STRUCT_RoamInd@CDatERI@@U?$less@G@std@@V?$allocator@U?$pair@$$CBGPAUSWI_STRUCT_RoamInd@CDatERI@@@std@@@4@$0A@@std@@@std@@QAA?AV012@H@Z 00119e9c f i DatERI.obj
 0001:00018f54       ??9const_iterator@?$_Tree@V?$_Tmap_traits@GPAUSWI_STRUCT_RoamInd@CDatERI@@U?$less@G@std@@V?$allocator@U?$pair@$$CBGPAUSWI_STRUCT_RoamInd@CDatERI@@@std@@@4@$0A@@std@@@std@@QBA_NABV012@@Z 00119f54 f i DatERI.obj
 0001:00018fac       ??Citerator@?$_Tree@V?$_Tmap_traits@GPAUSWI_STRUCT_CallPrompt@CDatERI@@U?$less@G@std@@V?$allocator@U?$pair@$$CBGPAUSWI_STRUCT_CallPrompt@CDatERI@@@std@@@4@$0A@@std@@@std@@QBAPAU?$pair@$$CBGPAUSWI_STRUCT_CallPrompt@CDatERI@@@2@XZ 00119fac f i DatERI.obj
 0001:00018fe4       ??Eiterator@?$_Tree@V?$_Tmap_traits@GPAUSWI_STRUCT_CallPrompt@CDatERI@@U?$less@G@std@@V?$allocator@U?$pair@$$CBGPAUSWI_STRUCT_CallPrompt@CDatERI@@@std@@@4@$0A@@std@@@std@@QAA?AV012@H@Z 00119fe4 f i DatERI.obj
 0001:0001909c       ??9const_iterator@?$_Tree@V?$_Tmap_traits@GPAUSWI_STRUCT_CallPrompt@CDatERI@@U?$less@G@std@@V?$allocator@U?$pair@$$CBGPAUSWI_STRUCT_CallPrompt@CDatERI@@@std@@@4@$0A@@std@@@std@@QBA_NABV012@@Z 0011a09c f i DatERI.obj
 0001:000190f4       ??0iterator@?$_Tree@V?$_Tmap_traits@GPAUSWI_STRUCT_RoamInd@CDatERI@@U?$less@G@std@@V?$allocator@U?$pair@$$CBGPAUSWI_STRUCT_RoamInd@CDatERI@@@std@@@4@$0A@@std@@@std@@QAA@ABV012@@Z 0011a0f4 f i DatERI.obj
 0001:00019128       ??4iterator@?$_Tree@V?$_Tmap_traits@GPAUSWI_STRUCT_RoamInd@CDatERI@@U?$less@G@std@@V?$allocator@U?$pair@$$CBGPAUSWI_STRUCT_RoamInd@CDatERI@@@std@@@4@$0A@@std@@@std@@QAAAAV012@ABV012@@Z 0011a128 f i DatERI.obj
 0001:00019158       ??1?$_Tree_val@V?$_Tmap_traits@GPAUSWI_STRUCT_RoamInd@CDatERI@@U?$less@G@std@@V?$allocator@U?$pair@$$CBGPAUSWI_STRUCT_RoamInd@CDatERI@@@std@@@4@$0A@@std@@@std@@QAA@XZ 0011a158 f i DatERI.obj
 0001:00019170       ??0iterator@?$_Tree@V?$_Tmap_traits@GPAUSWI_STRUCT_CallPrompt@CDatERI@@U?$less@G@std@@V?$allocator@U?$pair@$$CBGPAUSWI_STRUCT_CallPrompt@CDatERI@@@std@@@4@$0A@@std@@@std@@QAA@ABV012@@Z 0011a170 f i DatERI.obj
 0001:000191a4       ??4iterator@?$_Tree@V?$_Tmap_traits@GPAUSWI_STRUCT_CallPrompt@CDatERI@@U?$less@G@std@@V?$allocator@U?$pair@$$CBGPAUSWI_STRUCT_CallPrompt@CDatERI@@@std@@@4@$0A@@std@@@std@@QAAAAV012@ABV012@@Z 0011a1a4 f i DatERI.obj
 0001:000191d4       ??1?$_Tree_val@V?$_Tmap_traits@GPAUSWI_STRUCT_CallPrompt@CDatERI@@U?$less@G@std@@V?$allocator@U?$pair@$$CBGPAUSWI_STRUCT_CallPrompt@CDatERI@@@std@@@4@$0A@@std@@@std@@QAA@XZ 0011a1d4 f i DatERI.obj
 0001:000191ec       ??0const_iterator@?$_Tree@V?$_Tmap_traits@GPAUSWI_STRUCT_RoamInd@CDatERI@@U?$less@G@std@@V?$allocator@U?$pair@$$CBGPAUSWI_STRUCT_RoamInd@CDatERI@@@std@@@4@$0A@@std@@@std@@QAA@ABV012@@Z 0011a1ec f i DatERI.obj
 0001:00019238       ??4const_iterator@?$_Tree@V?$_Tmap_traits@GPAUSWI_STRUCT_RoamInd@CDatERI@@U?$less@G@std@@V?$allocator@U?$pair@$$CBGPAUSWI_STRUCT_RoamInd@CDatERI@@@std@@@4@$0A@@std@@@std@@QAAAAV012@ABV012@@Z 0011a238 f i DatERI.obj
 0001:00019280       ??1?$_Tree_ptr@V?$_Tmap_traits@GPAUSWI_STRUCT_RoamInd@CDatERI@@U?$less@G@std@@V?$allocator@U?$pair@$$CBGPAUSWI_STRUCT_RoamInd@CDatERI@@@std@@@4@$0A@@std@@@std@@QAA@XZ 0011a280 f i DatERI.obj
 0001:00019298       ??0const_iterator@?$_Tree@V?$_Tmap_traits@GPAUSWI_STRUCT_CallPrompt@CDatERI@@U?$less@G@std@@V?$allocator@U?$pair@$$CBGPAUSWI_STRUCT_CallPrompt@CDatERI@@@std@@@4@$0A@@std@@@std@@QAA@ABV012@@Z 0011a298 f i DatERI.obj
 0001:000192e4       ??4const_iterator@?$_Tree@V?$_Tmap_traits@GPAUSWI_STRUCT_CallPrompt@CDatERI@@U?$less@G@std@@V?$allocator@U?$pair@$$CBGPAUSWI_STRUCT_CallPrompt@CDatERI@@@std@@@4@$0A@@std@@@std@@QAAAAV012@ABV012@@Z 0011a2e4 f i DatERI.obj
 0001:0001932c       ??1?$_Tree_ptr@V?$_Tmap_traits@GPAUSWI_STRUCT_CallPrompt@CDatERI@@U?$less@G@std@@V?$allocator@U?$pair@$$CBGPAUSWI_STRUCT_CallPrompt@CDatERI@@@std@@@4@$0A@@std@@@std@@QAA@XZ 0011a32c f i DatERI.obj
 0001:00019344       ??0?$_Bidit@U?$pair@$$CBGPAUSWI_STRUCT_RoamInd@CDatERI@@@std@@HPBU12@ABU12@@std@@QAA@ABU01@@Z 0011a344 f i DatERI.obj
 0001:00019378       ??0_Iterator_base@std@@QAA@ABV01@@Z 0011a378 f i DatERI.obj
 0001:000193c4       ??4?$_Bidit@U?$pair@$$CBGPAUSWI_STRUCT_RoamInd@CDatERI@@@std@@HPBU12@ABU12@@std@@QAAAAU01@ABU01@@Z 0011a3c4 f i DatERI.obj
 0001:000193f4       ??1?$_Tree_nod@V?$_Tmap_traits@GPAUSWI_STRUCT_RoamInd@CDatERI@@U?$less@G@std@@V?$allocator@U?$pair@$$CBGPAUSWI_STRUCT_RoamInd@CDatERI@@@std@@@4@$0A@@std@@@std@@QAA@XZ 0011a3f4 f i DatERI.obj
 0001:0001940c       ??0?$_Bidit@U?$pair@$$CBGPAUSWI_STRUCT_CallPrompt@CDatERI@@@std@@HPBU12@ABU12@@std@@QAA@ABU01@@Z 0011a40c f i DatERI.obj
 0001:00019440       ??4?$_Bidit@U?$pair@$$CBGPAUSWI_STRUCT_CallPrompt@CDatERI@@@std@@HPBU12@ABU12@@std@@QAAAAU01@ABU01@@Z 0011a440 f i DatERI.obj
 0001:00019470       ??1?$_Tree_nod@V?$_Tmap_traits@GPAUSWI_STRUCT_CallPrompt@CDatERI@@U?$less@G@std@@V?$allocator@U?$pair@$$CBGPAUSWI_STRUCT_CallPrompt@CDatERI@@@std@@@4@$0A@@std@@@std@@QAA@XZ 0011a470 f i DatERI.obj
 0001:00019488       ??1?$_Tmap_traits@GPAUSWI_STRUCT_RoamInd@CDatERI@@U?$less@G@std@@V?$allocator@U?$pair@$$CBGPAUSWI_STRUCT_RoamInd@CDatERI@@@std@@@4@$0A@@std@@QAA@XZ 0011a488 f i DatERI.obj
 0001:000194a0       ??1?$_Tmap_traits@GPAUSWI_STRUCT_CallPrompt@CDatERI@@U?$less@G@std@@V?$allocator@U?$pair@$$CBGPAUSWI_STRUCT_CallPrompt@CDatERI@@@std@@@4@$0A@@std@@QAA@XZ 0011a4a0 f i DatERI.obj
 0001:000194b8       ?_Key@?$_Tree@V?$_Tmap_traits@GPAUSWI_STRUCT_RoamInd@CDatERI@@U?$less@G@std@@V?$allocator@U?$pair@$$CBGPAUSWI_STRUCT_RoamInd@CDatERI@@@std@@@4@$0A@@std@@@std@@KAABGPAU_Node@?$_Tree_nod@V?$_Tmap_traits@GPAUSWI_STRUCT_RoamInd@CDatERI@@U?$less@G@std@@V?$allocator@U?$pair@$$CBGPAUSWI_STRUCT_RoamInd@CDatERI@@@std@@@4@$0A@@std@@@2@@Z 0011a4b8 f i DatERI.obj
 0001:000194fc       ??0?$_Tree@V?$_Tmap_traits@GPAUSWI_STRUCT_RoamInd@CDatERI@@U?$less@G@std@@V?$allocator@U?$pair@$$CBGPAUSWI_STRUCT_RoamInd@CDatERI@@@std@@@4@$0A@@std@@@std@@QAA@ABU?$less@G@1@ABV?$allocator@U?$pair@$$CBGPAUSWI_STRUCT_RoamInd@CDatERI@@@std@@@1@@Z 0011a4fc f i DatERI.obj
 0001:00019578       ?insert@?$_Tree@V?$_Tmap_traits@GPAUSWI_STRUCT_RoamInd@CDatERI@@U?$less@G@std@@V?$allocator@U?$pair@$$CBGPAUSWI_STRUCT_RoamInd@CDatERI@@@std@@@4@$0A@@std@@@std@@QAA?AViterator@12@V312@ABU?$pair@$$CBGPAUSWI_STRUCT_RoamInd@CDatERI@@@2@@Z 0011a578 f i DatERI.obj
 0001:0001a494       ?lower_bound@?$_Tree@V?$_Tmap_traits@GPAUSWI_STRUCT_RoamInd@CDatERI@@U?$less@G@std@@V?$allocator@U?$pair@$$CBGPAUSWI_STRUCT_RoamInd@CDatERI@@@std@@@4@$0A@@std@@@std@@QAA?AViterator@12@ABG@Z 0011b494 f i DatERI.obj
 0001:0001a4f0       ?_Erase@?$_Tree@V?$_Tmap_traits@GPAUSWI_STRUCT_RoamInd@CDatERI@@U?$less@G@std@@V?$allocator@U?$pair@$$CBGPAUSWI_STRUCT_RoamInd@CDatERI@@@std@@@4@$0A@@std@@@std@@IAAXPAU_Node@?$_Tree_nod@V?$_Tmap_traits@GPAUSWI_STRUCT_RoamInd@CDatERI@@U?$less@G@std@@V?$allocator@U?$pair@$$CBGPAUSWI_STRUCT_RoamInd@CDatERI@@@std@@@4@$0A@@std@@@2@@Z 0011b4f0 f i DatERI.obj
 0001:0001a594       ?_Lmost@?$_Tree@V?$_Tmap_traits@GPAUSWI_STRUCT_RoamInd@CDatERI@@U?$less@G@std@@V?$allocator@U?$pair@$$CBGPAUSWI_STRUCT_RoamInd@CDatERI@@@std@@@4@$0A@@std@@@std@@IBAAAPAU_Node@?$_Tree_nod@V?$_Tmap_traits@GPAUSWI_STRUCT_RoamInd@CDatERI@@U?$less@G@std@@V?$allocator@U?$pair@$$CBGPAUSWI_STRUCT_RoamInd@CDatERI@@@std@@@4@$0A@@std@@@2@XZ 0011b594 f i DatERI.obj
 0001:0001a5cc       ?_Rmost@?$_Tree@V?$_Tmap_traits@GPAUSWI_STRUCT_RoamInd@CDatERI@@U?$less@G@std@@V?$allocator@U?$pair@$$CBGPAUSWI_STRUCT_RoamInd@CDatERI@@@std@@@4@$0A@@std@@@std@@IBAAAPAU_Node@?$_Tree_nod@V?$_Tmap_traits@GPAUSWI_STRUCT_RoamInd@CDatERI@@U?$less@G@std@@V?$allocator@U?$pair@$$CBGPAUSWI_STRUCT_RoamInd@CDatERI@@@std@@@4@$0A@@std@@@2@XZ 0011b5cc f i DatERI.obj
 0001:0001a604       ?_Root@?$_Tree@V?$_Tmap_traits@GPAUSWI_STRUCT_RoamInd@CDatERI@@U?$less@G@std@@V?$allocator@U?$pair@$$CBGPAUSWI_STRUCT_RoamInd@CDatERI@@@std@@@4@$0A@@std@@@std@@IBAAAPAU_Node@?$_Tree_nod@V?$_Tmap_traits@GPAUSWI_STRUCT_RoamInd@CDatERI@@U?$less@G@std@@V?$allocator@U?$pair@$$CBGPAUSWI_STRUCT_RoamInd@CDatERI@@@std@@@4@$0A@@std@@@2@XZ 0011b604 f i DatERI.obj
 0001:0001a63c       ?_Orphan_ptr@?$_Tree@V?$_Tmap_traits@GPAUSWI_STRUCT_RoamInd@CDatERI@@U?$less@G@std@@V?$allocator@U?$pair@$$CBGPAUSWI_STRUCT_RoamInd@CDatERI@@@std@@@4@$0A@@std@@@std@@IBAXAAV12@PAU_Node@?$_Tree_nod@V?$_Tmap_traits@GPAUSWI_STRUCT_RoamInd@CDatERI@@U?$less@G@std@@V?$allocator@U?$pair@$$CBGPAUSWI_STRUCT_RoamInd@CDatERI@@@std@@@4@$0A@@std@@@2@@Z 0011b63c f i DatERI.obj
 0001:0001a718       ?_Tidy@?$_Tree@V?$_Tmap_traits@GPAUSWI_STRUCT_RoamInd@CDatERI@@U?$less@G@std@@V?$allocator@U?$pair@$$CBGPAUSWI_STRUCT_RoamInd@CDatERI@@@std@@@4@$0A@@std@@@std@@IAAXXZ 0011b718 f i DatERI.obj
 0001:0001a854       ??0?$allocator@U?$pair@$$CBGPAUSWI_STRUCT_RoamInd@CDatERI@@@std@@@std@@QAA@XZ 0011b854 f i DatERI.obj
 0001:0001a878       ??R?$less@G@std@@QBA_NABG0@Z 0011b878 f i DatERI.obj
 0001:0001a8d0       ?_Key@?$_Tree@V?$_Tmap_traits@GPAUSWI_STRUCT_CallPrompt@CDatERI@@U?$less@G@std@@V?$allocator@U?$pair@$$CBGPAUSWI_STRUCT_CallPrompt@CDatERI@@@std@@@4@$0A@@std@@@std@@KAABGPAU_Node@?$_Tree_nod@V?$_Tmap_traits@GPAUSWI_STRUCT_CallPrompt@CDatERI@@U?$less@G@std@@V?$allocator@U?$pair@$$CBGPAUSWI_STRUCT_CallPrompt@CDatERI@@@std@@@4@$0A@@std@@@2@@Z 0011b8d0 f i DatERI.obj
 0001:0001a914       ??0?$_Tree@V?$_Tmap_traits@GPAUSWI_STRUCT_CallPrompt@CDatERI@@U?$less@G@std@@V?$allocator@U?$pair@$$CBGPAUSWI_STRUCT_CallPrompt@CDatERI@@@std@@@4@$0A@@std@@@std@@QAA@ABU?$less@G@1@ABV?$allocator@U?$pair@$$CBGPAUSWI_STRUCT_CallPrompt@CDatERI@@@std@@@1@@Z 0011b914 f i DatERI.obj
 0001:0001a990       ?insert@?$_Tree@V?$_Tmap_traits@GPAUSWI_STRUCT_CallPrompt@CDatERI@@U?$less@G@std@@V?$allocator@U?$pair@$$CBGPAUSWI_STRUCT_CallPrompt@CDatERI@@@std@@@4@$0A@@std@@@std@@QAA?AViterator@12@V312@ABU?$pair@$$CBGPAUSWI_STRUCT_CallPrompt@CDatERI@@@2@@Z 0011b990 f i DatERI.obj
 0001:0001b8ac       ?lower_bound@?$_Tree@V?$_Tmap_traits@GPAUSWI_STRUCT_CallPrompt@CDatERI@@U?$less@G@std@@V?$allocator@U?$pair@$$CBGPAUSWI_STRUCT_CallPrompt@CDatERI@@@std@@@4@$0A@@std@@@std@@QAA?AViterator@12@ABG@Z 0011c8ac f i DatERI.obj
 0001:0001b908       ?_Erase@?$_Tree@V?$_Tmap_traits@GPAUSWI_STRUCT_CallPrompt@CDatERI@@U?$less@G@std@@V?$allocator@U?$pair@$$CBGPAUSWI_STRUCT_CallPrompt@CDatERI@@@std@@@4@$0A@@std@@@std@@IAAXPAU_Node@?$_Tree_nod@V?$_Tmap_traits@GPAUSWI_STRUCT_CallPrompt@CDatERI@@U?$less@G@std@@V?$allocator@U?$pair@$$CBGPAUSWI_STRUCT_CallPrompt@CDatERI@@@std@@@4@$0A@@std@@@2@@Z 0011c908 f i DatERI.obj
 0001:0001b9ac       ?_Lmost@?$_Tree@V?$_Tmap_traits@GPAUSWI_STRUCT_CallPrompt@CDatERI@@U?$less@G@std@@V?$allocator@U?$pair@$$CBGPAUSWI_STRUCT_CallPrompt@CDatERI@@@std@@@4@$0A@@std@@@std@@IBAAAPAU_Node@?$_Tree_nod@V?$_Tmap_traits@GPAUSWI_STRUCT_CallPrompt@CDatERI@@U?$less@G@std@@V?$allocator@U?$pair@$$CBGPAUSWI_STRUCT_CallPrompt@CDatERI@@@std@@@4@$0A@@std@@@2@XZ 0011c9ac f i DatERI.obj
 0001:0001b9e4       ?_Rmost@?$_Tree@V?$_Tmap_traits@GPAUSWI_STRUCT_CallPrompt@CDatERI@@U?$less@G@std@@V?$allocator@U?$pair@$$CBGPAUSWI_STRUCT_CallPrompt@CDatERI@@@std@@@4@$0A@@std@@@std@@IBAAAPAU_Node@?$_Tree_nod@V?$_Tmap_traits@GPAUSWI_STRUCT_CallPrompt@CDatERI@@U?$less@G@std@@V?$allocator@U?$pair@$$CBGPAUSWI_STRUCT_CallPrompt@CDatERI@@@std@@@4@$0A@@std@@@2@XZ 0011c9e4 f i DatERI.obj
 0001:0001ba1c       ?_Root@?$_Tree@V?$_Tmap_traits@GPAUSWI_STRUCT_CallPrompt@CDatERI@@U?$less@G@std@@V?$allocator@U?$pair@$$CBGPAUSWI_STRUCT_CallPrompt@CDatERI@@@std@@@4@$0A@@std@@@std@@IBAAAPAU_Node@?$_Tree_nod@V?$_Tmap_traits@GPAUSWI_STRUCT_CallPrompt@CDatERI@@U?$less@G@std@@V?$allocator@U?$pair@$$CBGPAUSWI_STRUCT_CallPrompt@CDatERI@@@std@@@4@$0A@@std@@@2@XZ 0011ca1c f i DatERI.obj
 0001:0001ba54       ?_Orphan_ptr@?$_Tree@V?$_Tmap_traits@GPAUSWI_STRUCT_CallPrompt@CDatERI@@U?$less@G@std@@V?$allocator@U?$pair@$$CBGPAUSWI_STRUCT_CallPrompt@CDatERI@@@std@@@4@$0A@@std@@@std@@IBAXAAV12@PAU_Node@?$_Tree_nod@V?$_Tmap_traits@GPAUSWI_STRUCT_CallPrompt@CDatERI@@U?$less@G@std@@V?$allocator@U?$pair@$$CBGPAUSWI_STRUCT_CallPrompt@CDatERI@@@std@@@4@$0A@@std@@@2@@Z 0011ca54 f i DatERI.obj
 0001:0001bb30       ?_Tidy@?$_Tree@V?$_Tmap_traits@GPAUSWI_STRUCT_CallPrompt@CDatERI@@U?$less@G@std@@V?$allocator@U?$pair@$$CBGPAUSWI_STRUCT_CallPrompt@CDatERI@@@std@@@4@$0A@@std@@@std@@IAAXXZ 0011cb30 f i DatERI.obj
 0001:0001bc6c       ??0?$allocator@U?$pair@$$CBGPAUSWI_STRUCT_CallPrompt@CDatERI@@@std@@@std@@QAA@XZ 0011cc6c f i DatERI.obj
 0001:0001bc90       ??0iterator@?$_Tree@V?$_Tmap_traits@GPAUSWI_STRUCT_RoamInd@CDatERI@@U?$less@G@std@@V?$allocator@U?$pair@$$CBGPAUSWI_STRUCT_RoamInd@CDatERI@@@std@@@4@$0A@@std@@@std@@QAA@PAU_Node@?$_Tree_nod@V?$_Tmap_traits@GPAUSWI_STRUCT_RoamInd@CDatERI@@U?$less@G@std@@V?$allocator@U?$pair@$$CBGPAUSWI_STRUCT_RoamInd@CDatERI@@@std@@@4@$0A@@std@@@2@PBV12@@Z 0011cc90 f i DatERI.obj
 0001:0001bcc8       ??Diterator@?$_Tree@V?$_Tmap_traits@GPAUSWI_STRUCT_RoamInd@CDatERI@@U?$less@G@std@@V?$allocator@U?$pair@$$CBGPAUSWI_STRUCT_RoamInd@CDatERI@@@std@@@4@$0A@@std@@@std@@QBAAAU?$pair@$$CBGPAUSWI_STRUCT_RoamInd@CDatERI@@@2@XZ 0011ccc8 f i DatERI.obj
 0001:0001bcf8       ??Eiterator@?$_Tree@V?$_Tmap_traits@GPAUSWI_STRUCT_RoamInd@CDatERI@@U?$less@G@std@@V?$allocator@U?$pair@$$CBGPAUSWI_STRUCT_RoamInd@CDatERI@@@std@@@4@$0A@@std@@@std@@QAAAAV012@XZ 0011ccf8 f i DatERI.obj
 0001:0001bd24       ??8const_iterator@?$_Tree@V?$_Tmap_traits@GPAUSWI_STRUCT_RoamInd@CDatERI@@U?$less@G@std@@V?$allocator@U?$pair@$$CBGPAUSWI_STRUCT_RoamInd@CDatERI@@@std@@@4@$0A@@std@@@std@@QBA_NABV012@@Z 0011cd24 f i DatERI.obj
 0001:0001be1c       ?_Mynode@const_iterator@?$_Tree@V?$_Tmap_traits@GPAUSWI_STRUCT_RoamInd@CDatERI@@U?$less@G@std@@V?$allocator@U?$pair@$$CBGPAUSWI_STRUCT_RoamInd@CDatERI@@@std@@@4@$0A@@std@@@std@@QBAPAU_Node@?$_Tree_nod@V?$_Tmap_traits@GPAUSWI_STRUCT_RoamInd@CDatERI@@U?$less@G@std@@V?$allocator@U?$pair@$$CBGPAUSWI_STRUCT_RoamInd@CDatERI@@@std@@@4@$0A@@std@@@3@XZ 0011ce1c f i DatERI.obj
 0001:0001be48       ??0?$pair@$$CBGPAUSWI_STRUCT_RoamInd@CDatERI@@@std@@QAA@ABGABQAUSWI_STRUCT_RoamInd@CDatERI@@@Z 0011ce48 f i DatERI.obj
 0001:0001be90       ??0iterator@?$_Tree@V?$_Tmap_traits@GPAUSWI_STRUCT_CallPrompt@CDatERI@@U?$less@G@std@@V?$allocator@U?$pair@$$CBGPAUSWI_STRUCT_CallPrompt@CDatERI@@@std@@@4@$0A@@std@@@std@@QAA@PAU_Node@?$_Tree_nod@V?$_Tmap_traits@GPAUSWI_STRUCT_CallPrompt@CDatERI@@U?$less@G@std@@V?$allocator@U?$pair@$$CBGPAUSWI_STRUCT_CallPrompt@CDatERI@@@std@@@4@$0A@@std@@@2@PBV12@@Z 0011ce90 f i DatERI.obj
 0001:0001bec8       ??Diterator@?$_Tree@V?$_Tmap_traits@GPAUSWI_STRUCT_CallPrompt@CDatERI@@U?$less@G@std@@V?$allocator@U?$pair@$$CBGPAUSWI_STRUCT_CallPrompt@CDatERI@@@std@@@4@$0A@@std@@@std@@QBAAAU?$pair@$$CBGPAUSWI_STRUCT_CallPrompt@CDatERI@@@2@XZ 0011cec8 f i DatERI.obj
 0001:0001bef8       ??Eiterator@?$_Tree@V?$_Tmap_traits@GPAUSWI_STRUCT_CallPrompt@CDatERI@@U?$less@G@std@@V?$allocator@U?$pair@$$CBGPAUSWI_STRUCT_CallPrompt@CDatERI@@@std@@@4@$0A@@std@@@std@@QAAAAV012@XZ 0011cef8 f i DatERI.obj
 0001:0001bf24       ??8const_iterator@?$_Tree@V?$_Tmap_traits@GPAUSWI_STRUCT_CallPrompt@CDatERI@@U?$less@G@std@@V?$allocator@U?$pair@$$CBGPAUSWI_STRUCT_CallPrompt@CDatERI@@@std@@@4@$0A@@std@@@std@@QBA_NABV012@@Z 0011cf24 f i DatERI.obj
 0001:0001c01c       ?_Mynode@const_iterator@?$_Tree@V?$_Tmap_traits@GPAUSWI_STRUCT_CallPrompt@CDatERI@@U?$less@G@std@@V?$allocator@U?$pair@$$CBGPAUSWI_STRUCT_CallPrompt@CDatERI@@@std@@@4@$0A@@std@@@std@@QBAPAU_Node@?$_Tree_nod@V?$_Tmap_traits@GPAUSWI_STRUCT_CallPrompt@CDatERI@@U?$less@G@std@@V?$allocator@U?$pair@$$CBGPAUSWI_STRUCT_CallPrompt@CDatERI@@@std@@@4@$0A@@std@@@3@XZ 0011d01c f i DatERI.obj
 0001:0001c048       ??0?$pair@$$CBGPAUSWI_STRUCT_CallPrompt@CDatERI@@@std@@QAA@ABGABQAUSWI_STRUCT_CallPrompt@CDatERI@@@Z 0011d048 f i DatERI.obj
 0001:0001c090       ??1?$pair@Viterator@?$_Tree@V?$_Tmap_traits@GPAUSWI_STRUCT_RoamInd@CDatERI@@U?$less@G@std@@V?$allocator@U?$pair@$$CBGPAUSWI_STRUCT_RoamInd@CDatERI@@@std@@@4@$0A@@std@@@std@@_N@std@@QAA@XZ 0011d090 f i DatERI.obj
 0001:0001c0a8       ??1?$pair@Viterator@?$_Tree@V?$_Tmap_traits@GPAUSWI_STRUCT_CallPrompt@CDatERI@@U?$less@G@std@@V?$allocator@U?$pair@$$CBGPAUSWI_STRUCT_CallPrompt@CDatERI@@@std@@@4@$0A@@std@@@std@@_N@std@@QAA@XZ 0011d0a8 f i DatERI.obj
 0001:0001c0c0       ?_Isnil@?$_Tree@V?$_Tmap_traits@GPAUSWI_STRUCT_RoamInd@CDatERI@@U?$less@G@std@@V?$allocator@U?$pair@$$CBGPAUSWI_STRUCT_RoamInd@CDatERI@@@std@@@4@$0A@@std@@@std@@KAAADPAU_Node@?$_Tree_nod@V?$_Tmap_traits@GPAUSWI_STRUCT_RoamInd@CDatERI@@U?$less@G@std@@V?$allocator@U?$pair@$$CBGPAUSWI_STRUCT_RoamInd@CDatERI@@@std@@@4@$0A@@std@@@2@@Z 0011d0c0 f i DatERI.obj
 0001:0001c0e8       ?_Left@?$_Tree@V?$_Tmap_traits@GPAUSWI_STRUCT_RoamInd@CDatERI@@U?$less@G@std@@V?$allocator@U?$pair@$$CBGPAUSWI_STRUCT_RoamInd@CDatERI@@@std@@@4@$0A@@std@@@std@@KAAAPAU_Node@?$_Tree_nod@V?$_Tmap_traits@GPAUSWI_STRUCT_RoamInd@CDatERI@@U?$less@G@std@@V?$allocator@U?$pair@$$CBGPAUSWI_STRUCT_RoamInd@CDatERI@@@std@@@4@$0A@@std@@@2@PAU342@@Z 0011d0e8 f i DatERI.obj
 0001:0001c10c       ?_Parent@?$_Tree@V?$_Tmap_traits@GPAUSWI_STRUCT_RoamInd@CDatERI@@U?$less@G@std@@V?$allocator@U?$pair@$$CBGPAUSWI_STRUCT_RoamInd@CDatERI@@@std@@@4@$0A@@std@@@std@@KAAAPAU_Node@?$_Tree_nod@V?$_Tmap_traits@GPAUSWI_STRUCT_RoamInd@CDatERI@@U?$less@G@std@@V?$allocator@U?$pair@$$CBGPAUSWI_STRUCT_RoamInd@CDatERI@@@std@@@4@$0A@@std@@@2@PAU342@@Z 0011d10c f i DatERI.obj
 0001:0001c134       ?_Right@?$_Tree@V?$_Tmap_traits@GPAUSWI_STRUCT_RoamInd@CDatERI@@U?$less@G@std@@V?$allocator@U?$pair@$$CBGPAUSWI_STRUCT_RoamInd@CDatERI@@@std@@@4@$0A@@std@@@std@@KAAAPAU_Node@?$_Tree_nod@V?$_Tmap_traits@GPAUSWI_STRUCT_RoamInd@CDatERI@@U?$less@G@std@@V?$allocator@U?$pair@$$CBGPAUSWI_STRUCT_RoamInd@CDatERI@@@std@@@4@$0A@@std@@@2@PAU342@@Z 0011d134 f i DatERI.obj
 0001:0001c15c       ?_Myval@?$_Tree@V?$_Tmap_traits@GPAUSWI_STRUCT_RoamInd@CDatERI@@U?$less@G@std@@V?$allocator@U?$pair@$$CBGPAUSWI_STRUCT_RoamInd@CDatERI@@@std@@@4@$0A@@std@@@std@@KAAAU?$pair@$$CBGPAUSWI_STRUCT_RoamInd@CDatERI@@@2@PAU_Node@?$_Tree_nod@V?$_Tmap_traits@GPAUSWI_STRUCT_RoamInd@CDatERI@@U?$less@G@std@@V?$allocator@U?$pair@$$CBGPAUSWI_STRUCT_RoamInd@CDatERI@@@std@@@4@$0A@@std@@@2@@Z 0011d15c f i DatERI.obj
 0001:0001c184       ?size@?$_Tree@V?$_Tmap_traits@GPAUSWI_STRUCT_RoamInd@CDatERI@@U?$less@G@std@@V?$allocator@U?$pair@$$CBGPAUSWI_STRUCT_RoamInd@CDatERI@@@std@@@4@$0A@@std@@@std@@QBAIXZ 0011d184 f i DatERI.obj
 0001:0001c1b8       ?insert@?$_Tree@V?$_Tmap_traits@GPAUSWI_STRUCT_RoamInd@CDatERI@@U?$less@G@std@@V?$allocator@U?$pair@$$CBGPAUSWI_STRUCT_RoamInd@CDatERI@@@std@@@4@$0A@@std@@@std@@QAA?AU?$pair@Viterator@?$_Tree@V?$_Tmap_traits@GPAUSWI_STRUCT_RoamInd@CDatERI@@U?$less@G@std@@V?$allocator@U?$pair@$$CBGPAUSWI_STRUCT_RoamInd@CDatERI@@@std@@@4@$0A@@std@@@std@@_N@2@ABU?$pair@$$CBGPAUSWI_STRUCT_RoamInd@CDatERI@@@2@@Z 0011d1b8 f i DatERI.obj
 0001:0001c620       ?erase@?$_Tree@V?$_Tmap_traits@GPAUSWI_STRUCT_RoamInd@CDatERI@@U?$less@G@std@@V?$allocator@U?$pair@$$CBGPAUSWI_STRUCT_RoamInd@CDatERI@@@std@@@4@$0A@@std@@@std@@QAA?AViterator@12@V312@0@Z 0011d620 f i DatERI.obj
 0001:0001c8f4       ?_Init@?$_Tree@V?$_Tmap_traits@GPAUSWI_STRUCT_RoamInd@CDatERI@@U?$less@G@std@@V?$allocator@U?$pair@$$CBGPAUSWI_STRUCT_RoamInd@CDatERI@@@std@@@4@$0A@@std@@@std@@IAAXXZ 0011d8f4 f i DatERI.obj
 0001:0001c9c0       ?_Insert@?$_Tree@V?$_Tmap_traits@GPAUSWI_STRUCT_RoamInd@CDatERI@@U?$less@G@std@@V?$allocator@U?$pair@$$CBGPAUSWI_STRUCT_RoamInd@CDatERI@@@std@@@4@$0A@@std@@@std@@IAA?AViterator@12@_NPAU_Node@?$_Tree_nod@V?$_Tmap_traits@GPAUSWI_STRUCT_RoamInd@CDatERI@@U?$less@G@std@@V?$allocator@U?$pair@$$CBGPAUSWI_STRUCT_RoamInd@CDatERI@@@std@@@4@$0A@@std@@@2@ABU?$pair@$$CBGPAUSWI_STRUCT_RoamInd@CDatERI@@@2@@Z 0011d9c0 f i DatERI.obj
 0001:0001d07c       ?_Lbound@?$_Tree@V?$_Tmap_traits@GPAUSWI_STRUCT_RoamInd@CDatERI@@U?$less@G@std@@V?$allocator@U?$pair@$$CBGPAUSWI_STRUCT_RoamInd@CDatERI@@@std@@@4@$0A@@std@@@std@@IBAPAU_Node@?$_Tree_nod@V?$_Tmap_traits@GPAUSWI_STRUCT_RoamInd@CDatERI@@U?$less@G@std@@V?$allocator@U?$pair@$$CBGPAUSWI_STRUCT_RoamInd@CDatERI@@@std@@@4@$0A@@std@@@2@ABG@Z 0011e07c f i DatERI.obj
 0001:0001d174       ??0?$_Tree_val@V?$_Tmap_traits@GPAUSWI_STRUCT_RoamInd@CDatERI@@U?$less@G@std@@V?$allocator@U?$pair@$$CBGPAUSWI_STRUCT_RoamInd@CDatERI@@@std@@@4@$0A@@std@@@std@@IAA@ABU?$less@G@1@V?$allocator@U?$pair@$$CBGPAUSWI_STRUCT_RoamInd@CDatERI@@@std@@@1@@Z 0011e174 f i DatERI.obj
 0001:0001d1d4       ?_Kfn@?$_Tmap_traits@GPAUSWI_STRUCT_RoamInd@CDatERI@@U?$less@G@std@@V?$allocator@U?$pair@$$CBGPAUSWI_STRUCT_RoamInd@CDatERI@@@std@@@4@$0A@@std@@SAABGABU?$pair@$$CBGPAUSWI_STRUCT_RoamInd@CDatERI@@@2@@Z 0011e1d4 f i DatERI.obj
 0001:0001d1f8       ??0?$allocator@U?$pair@$$CBGPAUSWI_STRUCT_RoamInd@CDatERI@@@std@@@std@@QAA@ABV01@@Z 0011e1f8 f i DatERI.obj
 0001:0001d21c       ?deallocate@?$allocator@U_Node@?$_Tree_nod@V?$_Tmap_traits@GPAUSWI_STRUCT_RoamInd@CDatERI@@U?$less@G@std@@V?$allocator@U?$pair@$$CBGPAUSWI_STRUCT_RoamInd@CDatERI@@@std@@@4@$0A@@std@@@std@@@std@@QAAXPAU_Node@?$_Tree_nod@V?$_Tmap_traits@GPAUSWI_STRUCT_RoamInd@CDatERI@@U?$less@G@std@@V?$allocator@U?$pair@$$CBGPAUSWI_STRUCT_RoamInd@CDatERI@@@std@@@4@$0A@@std@@@2@I@Z 0011e21c f i DatERI.obj
 0001:0001d234       ?destroy@?$allocator@U_Node@?$_Tree_nod@V?$_Tmap_traits@GPAUSWI_STRUCT_RoamInd@CDatERI@@U?$less@G@std@@V?$allocator@U?$pair@$$CBGPAUSWI_STRUCT_RoamInd@CDatERI@@@std@@@4@$0A@@std@@@std@@@std@@QAAXPAU_Node@?$_Tree_nod@V?$_Tmap_traits@GPAUSWI_STRUCT_RoamInd@CDatERI@@U?$less@G@std@@V?$allocator@U?$pair@$$CBGPAUSWI_STRUCT_RoamInd@CDatERI@@@std@@@4@$0A@@std@@@2@@Z 0011e234 f i DatERI.obj
 0001:0001d24c       ?destroy@?$allocator@PAU_Node@?$_Tree_nod@V?$_Tmap_traits@GPAUSWI_STRUCT_RoamInd@CDatERI@@U?$less@G@std@@V?$allocator@U?$pair@$$CBGPAUSWI_STRUCT_RoamInd@CDatERI@@@std@@@4@$0A@@std@@@std@@@std@@QAAXPAPAU_Node@?$_Tree_nod@V?$_Tmap_traits@GPAUSWI_STRUCT_RoamInd@CDatERI@@U?$less@G@std@@V?$allocator@U?$pair@$$CBGPAUSWI_STRUCT_RoamInd@CDatERI@@@std@@@4@$0A@@std@@@2@@Z 0011e24c f i DatERI.obj
 0001:0001d264       ?_Isnil@?$_Tree@V?$_Tmap_traits@GPAUSWI_STRUCT_CallPrompt@CDatERI@@U?$less@G@std@@V?$allocator@U?$pair@$$CBGPAUSWI_STRUCT_CallPrompt@CDatERI@@@std@@@4@$0A@@std@@@std@@KAAADPAU_Node@?$_Tree_nod@V?$_Tmap_traits@GPAUSWI_STRUCT_CallPrompt@CDatERI@@U?$less@G@std@@V?$allocator@U?$pair@$$CBGPAUSWI_STRUCT_CallPrompt@CDatERI@@@std@@@4@$0A@@std@@@2@@Z 0011e264 f i DatERI.obj
 0001:0001d28c       ?_Left@?$_Tree@V?$_Tmap_traits@GPAUSWI_STRUCT_CallPrompt@CDatERI@@U?$less@G@std@@V?$allocator@U?$pair@$$CBGPAUSWI_STRUCT_CallPrompt@CDatERI@@@std@@@4@$0A@@std@@@std@@KAAAPAU_Node@?$_Tree_nod@V?$_Tmap_traits@GPAUSWI_STRUCT_CallPrompt@CDatERI@@U?$less@G@std@@V?$allocator@U?$pair@$$CBGPAUSWI_STRUCT_CallPrompt@CDatERI@@@std@@@4@$0A@@std@@@2@PAU342@@Z 0011e28c f i DatERI.obj
 0001:0001d2b0       ?_Parent@?$_Tree@V?$_Tmap_traits@GPAUSWI_STRUCT_CallPrompt@CDatERI@@U?$less@G@std@@V?$allocator@U?$pair@$$CBGPAUSWI_STRUCT_CallPrompt@CDatERI@@@std@@@4@$0A@@std@@@std@@KAAAPAU_Node@?$_Tree_nod@V?$_Tmap_traits@GPAUSWI_STRUCT_CallPrompt@CDatERI@@U?$less@G@std@@V?$allocator@U?$pair@$$CBGPAUSWI_STRUCT_CallPrompt@CDatERI@@@std@@@4@$0A@@std@@@2@PAU342@@Z 0011e2b0 f i DatERI.obj
 0001:0001d2d8       ?_Right@?$_Tree@V?$_Tmap_traits@GPAUSWI_STRUCT_CallPrompt@CDatERI@@U?$less@G@std@@V?$allocator@U?$pair@$$CBGPAUSWI_STRUCT_CallPrompt@CDatERI@@@std@@@4@$0A@@std@@@std@@KAAAPAU_Node@?$_Tree_nod@V?$_Tmap_traits@GPAUSWI_STRUCT_CallPrompt@CDatERI@@U?$less@G@std@@V?$allocator@U?$pair@$$CBGPAUSWI_STRUCT_CallPrompt@CDatERI@@@std@@@4@$0A@@std@@@2@PAU342@@Z 0011e2d8 f i DatERI.obj
 0001:0001d300       ?_Myval@?$_Tree@V?$_Tmap_traits@GPAUSWI_STRUCT_CallPrompt@CDatERI@@U?$less@G@std@@V?$allocator@U?$pair@$$CBGPAUSWI_STRUCT_CallPrompt@CDatERI@@@std@@@4@$0A@@std@@@std@@KAAAU?$pair@$$CBGPAUSWI_STRUCT_CallPrompt@CDatERI@@@2@PAU_Node@?$_Tree_nod@V?$_Tmap_traits@GPAUSWI_STRUCT_CallPrompt@CDatERI@@U?$less@G@std@@V?$allocator@U?$pair@$$CBGPAUSWI_STRUCT_CallPrompt@CDatERI@@@std@@@4@$0A@@std@@@2@@Z 0011e300 f i DatERI.obj
 0001:0001d330       ?insert@?$_Tree@V?$_Tmap_traits@GPAUSWI_STRUCT_CallPrompt@CDatERI@@U?$less@G@std@@V?$allocator@U?$pair@$$CBGPAUSWI_STRUCT_CallPrompt@CDatERI@@@std@@@4@$0A@@std@@@std@@QAA?AU?$pair@Viterator@?$_Tree@V?$_Tmap_traits@GPAUSWI_STRUCT_CallPrompt@CDatERI@@U?$less@G@std@@V?$allocator@U?$pair@$$CBGPAUSWI_STRUCT_CallPrompt@CDatERI@@@std@@@4@$0A@@std@@@std@@_N@2@ABU?$pair@$$CBGPAUSWI_STRUCT_CallPrompt@CDatERI@@@2@@Z 0011e330 f i DatERI.obj
 0001:0001d798       ?erase@?$_Tree@V?$_Tmap_traits@GPAUSWI_STRUCT_CallPrompt@CDatERI@@U?$less@G@std@@V?$allocator@U?$pair@$$CBGPAUSWI_STRUCT_CallPrompt@CDatERI@@@std@@@4@$0A@@std@@@std@@QAA?AViterator@12@V312@0@Z 0011e798 f i DatERI.obj
 0001:0001da6c       ?_Init@?$_Tree@V?$_Tmap_traits@GPAUSWI_STRUCT_CallPrompt@CDatERI@@U?$less@G@std@@V?$allocator@U?$pair@$$CBGPAUSWI_STRUCT_CallPrompt@CDatERI@@@std@@@4@$0A@@std@@@std@@IAAXXZ 0011ea6c f i DatERI.obj
 0001:0001db38       ?_Insert@?$_Tree@V?$_Tmap_traits@GPAUSWI_STRUCT_CallPrompt@CDatERI@@U?$less@G@std@@V?$allocator@U?$pair@$$CBGPAUSWI_STRUCT_CallPrompt@CDatERI@@@std@@@4@$0A@@std@@@std@@IAA?AViterator@12@_NPAU_Node@?$_Tree_nod@V?$_Tmap_traits@GPAUSWI_STRUCT_CallPrompt@CDatERI@@U?$less@G@std@@V?$allocator@U?$pair@$$CBGPAUSWI_STRUCT_CallPrompt@CDatERI@@@std@@@4@$0A@@std@@@2@ABU?$pair@$$CBGPAUSWI_STRUCT_CallPrompt@CDatERI@@@2@@Z 0011eb38 f i DatERI.obj
 0001:0001e1f4       ?_Lbound@?$_Tree@V?$_Tmap_traits@GPAUSWI_STRUCT_CallPrompt@CDatERI@@U?$less@G@std@@V?$allocator@U?$pair@$$CBGPAUSWI_STRUCT_CallPrompt@CDatERI@@@std@@@4@$0A@@std@@@std@@IBAPAU_Node@?$_Tree_nod@V?$_Tmap_traits@GPAUSWI_STRUCT_CallPrompt@CDatERI@@U?$less@G@std@@V?$allocator@U?$pair@$$CBGPAUSWI_STRUCT_CallPrompt@CDatERI@@@std@@@4@$0A@@std@@@2@ABG@Z 0011f1f4 f i DatERI.obj
 0001:0001e2ec       ??0?$_Tree_val@V?$_Tmap_traits@GPAUSWI_STRUCT_CallPrompt@CDatERI@@U?$less@G@std@@V?$allocator@U?$pair@$$CBGPAUSWI_STRUCT_CallPrompt@CDatERI@@@std@@@4@$0A@@std@@@std@@IAA@ABU?$less@G@1@V?$allocator@U?$pair@$$CBGPAUSWI_STRUCT_CallPrompt@CDatERI@@@std@@@1@@Z 0011f2ec f i DatERI.obj
 0001:0001e34c       ?_Kfn@?$_Tmap_traits@GPAUSWI_STRUCT_CallPrompt@CDatERI@@U?$less@G@std@@V?$allocator@U?$pair@$$CBGPAUSWI_STRUCT_CallPrompt@CDatERI@@@std@@@4@$0A@@std@@SAABGABU?$pair@$$CBGPAUSWI_STRUCT_CallPrompt@CDatERI@@@2@@Z 0011f34c f i DatERI.obj
 0001:0001e370       ??0?$allocator@U?$pair@$$CBGPAUSWI_STRUCT_CallPrompt@CDatERI@@@std@@@std@@QAA@ABV01@@Z 0011f370 f i DatERI.obj
 0001:0001e394       ?deallocate@?$allocator@U_Node@?$_Tree_nod@V?$_Tmap_traits@GPAUSWI_STRUCT_CallPrompt@CDatERI@@U?$less@G@std@@V?$allocator@U?$pair@$$CBGPAUSWI_STRUCT_CallPrompt@CDatERI@@@std@@@4@$0A@@std@@@std@@@std@@QAAXPAU_Node@?$_Tree_nod@V?$_Tmap_traits@GPAUSWI_STRUCT_CallPrompt@CDatERI@@U?$less@G@std@@V?$allocator@U?$pair@$$CBGPAUSWI_STRUCT_CallPrompt@CDatERI@@@std@@@4@$0A@@std@@@2@I@Z 0011f394 f i DatERI.obj
 0001:0001e3ac       ?destroy@?$allocator@U_Node@?$_Tree_nod@V?$_Tmap_traits@GPAUSWI_STRUCT_CallPrompt@CDatERI@@U?$less@G@std@@V?$allocator@U?$pair@$$CBGPAUSWI_STRUCT_CallPrompt@CDatERI@@@std@@@4@$0A@@std@@@std@@@std@@QAAXPAU_Node@?$_Tree_nod@V?$_Tmap_traits@GPAUSWI_STRUCT_CallPrompt@CDatERI@@U?$less@G@std@@V?$allocator@U?$pair@$$CBGPAUSWI_STRUCT_CallPrompt@CDatERI@@@std@@@4@$0A@@std@@@2@@Z 0011f3ac f i DatERI.obj
 0001:0001e3c4       ?destroy@?$allocator@PAU_Node@?$_Tree_nod@V?$_Tmap_traits@GPAUSWI_STRUCT_CallPrompt@CDatERI@@U?$less@G@std@@V?$allocator@U?$pair@$$CBGPAUSWI_STRUCT_CallPrompt@CDatERI@@@std@@@4@$0A@@std@@@std@@@std@@QAAXPAPAU_Node@?$_Tree_nod@V?$_Tmap_traits@GPAUSWI_STRUCT_CallPrompt@CDatERI@@U?$less@G@std@@V?$allocator@U?$pair@$$CBGPAUSWI_STRUCT_CallPrompt@CDatERI@@@std@@@4@$0A@@std@@@2@@Z 0011f3c4 f i DatERI.obj
 0001:0001e3dc       ??0iterator@?$_Tree@V?$_Tmap_traits@GPAUSWI_STRUCT_RoamInd@CDatERI@@U?$less@G@std@@V?$allocator@U?$pair@$$CBGPAUSWI_STRUCT_RoamInd@CDatERI@@@std@@@4@$0A@@std@@@std@@QAA@XZ 0011f3dc f i DatERI.obj
 0001:0001e40c       ??Fiterator@?$_Tree@V?$_Tmap_traits@GPAUSWI_STRUCT_RoamInd@CDatERI@@U?$less@G@std@@V?$allocator@U?$pair@$$CBGPAUSWI_STRUCT_RoamInd@CDatERI@@@std@@@4@$0A@@std@@@std@@QAAAAV012@XZ 0011f40c f i DatERI.obj
 0001:0001e440       ??0const_iterator@?$_Tree@V?$_Tmap_traits@GPAUSWI_STRUCT_RoamInd@CDatERI@@U?$less@G@std@@V?$allocator@U?$pair@$$CBGPAUSWI_STRUCT_RoamInd@CDatERI@@@std@@@4@$0A@@std@@@std@@QAA@PAU_Node@?$_Tree_nod@V?$_Tmap_traits@GPAUSWI_STRUCT_RoamInd@CDatERI@@U?$less@G@std@@V?$allocator@U?$pair@$$CBGPAUSWI_STRUCT_RoamInd@CDatERI@@@std@@@4@$0A@@std@@@2@PBV12@@Z 0011f440 f i DatERI.obj
 0001:0001e4a8       ??Dconst_iterator@?$_Tree@V?$_Tmap_traits@GPAUSWI_STRUCT_RoamInd@CDatERI@@U?$less@G@std@@V?$allocator@U?$pair@$$CBGPAUSWI_STRUCT_RoamInd@CDatERI@@@std@@@4@$0A@@std@@@std@@QBAABU?$pair@$$CBGPAUSWI_STRUCT_RoamInd@CDatERI@@@2@XZ 0011f4a8 f i DatERI.obj
 0001:0001e584       ??Econst_iterator@?$_Tree@V?$_Tmap_traits@GPAUSWI_STRUCT_RoamInd@CDatERI@@U?$less@G@std@@V?$allocator@U?$pair@$$CBGPAUSWI_STRUCT_RoamInd@CDatERI@@@std@@@4@$0A@@std@@@std@@QAAAAV012@XZ 0011f584 f i DatERI.obj
 0001:0001e5b0       ??0iterator@?$_Tree@V?$_Tmap_traits@GPAUSWI_STRUCT_CallPrompt@CDatERI@@U?$less@G@std@@V?$allocator@U?$pair@$$CBGPAUSWI_STRUCT_CallPrompt@CDatERI@@@std@@@4@$0A@@std@@@std@@QAA@XZ 0011f5b0 f i DatERI.obj
 0001:0001e5e0       ??Fiterator@?$_Tree@V?$_Tmap_traits@GPAUSWI_STRUCT_CallPrompt@CDatERI@@U?$less@G@std@@V?$allocator@U?$pair@$$CBGPAUSWI_STRUCT_CallPrompt@CDatERI@@@std@@@4@$0A@@std@@@std@@QAAAAV012@XZ 0011f5e0 f i DatERI.obj
 0001:0001e614       ??0const_iterator@?$_Tree@V?$_Tmap_traits@GPAUSWI_STRUCT_CallPrompt@CDatERI@@U?$less@G@std@@V?$allocator@U?$pair@$$CBGPAUSWI_STRUCT_CallPrompt@CDatERI@@@std@@@4@$0A@@std@@@std@@QAA@PAU_Node@?$_Tree_nod@V?$_Tmap_traits@GPAUSWI_STRUCT_CallPrompt@CDatERI@@U?$less@G@std@@V?$allocator@U?$pair@$$CBGPAUSWI_STRUCT_CallPrompt@CDatERI@@@std@@@4@$0A@@std@@@2@PBV12@@Z 0011f614 f i DatERI.obj
 0001:0001e67c       ??Dconst_iterator@?$_Tree@V?$_Tmap_traits@GPAUSWI_STRUCT_CallPrompt@CDatERI@@U?$less@G@std@@V?$allocator@U?$pair@$$CBGPAUSWI_STRUCT_CallPrompt@CDatERI@@@std@@@4@$0A@@std@@@std@@QBAABU?$pair@$$CBGPAUSWI_STRUCT_CallPrompt@CDatERI@@@2@XZ 0011f67c f i DatERI.obj
 0001:0001e758       ??Econst_iterator@?$_Tree@V?$_Tmap_traits@GPAUSWI_STRUCT_CallPrompt@CDatERI@@U?$less@G@std@@V?$allocator@U?$pair@$$CBGPAUSWI_STRUCT_CallPrompt@CDatERI@@@std@@@4@$0A@@std@@@std@@QAAAAV012@XZ 0011f758 f i DatERI.obj
 0001:0001e784       ??0?$_Bidit@U?$pair@$$CBGPAUSWI_STRUCT_RoamInd@CDatERI@@@std@@HPBU12@ABU12@@std@@QAA@XZ 0011f784 f i DatERI.obj
 0001:0001e7b4       ??0?$_Bidit@U?$pair@$$CBGPAUSWI_STRUCT_CallPrompt@CDatERI@@@std@@HPBU12@ABU12@@std@@QAA@XZ 0011f7b4 f i DatERI.obj
 0001:0001e7e4       ?_Color@?$_Tree@V?$_Tmap_traits@GPAUSWI_STRUCT_RoamInd@CDatERI@@U?$less@G@std@@V?$allocator@U?$pair@$$CBGPAUSWI_STRUCT_RoamInd@CDatERI@@@std@@@4@$0A@@std@@@std@@KAAADPAU_Node@?$_Tree_nod@V?$_Tmap_traits@GPAUSWI_STRUCT_RoamInd@CDatERI@@U?$less@G@std@@V?$allocator@U?$pair@$$CBGPAUSWI_STRUCT_RoamInd@CDatERI@@@std@@@4@$0A@@std@@@2@@Z 0011f7e4 f i DatERI.obj
 0001:0001e80c       ?max_size@?$_Tree@V?$_Tmap_traits@GPAUSWI_STRUCT_RoamInd@CDatERI@@U?$less@G@std@@V?$allocator@U?$pair@$$CBGPAUSWI_STRUCT_RoamInd@CDatERI@@@std@@@4@$0A@@std@@@std@@QBAIXZ 0011f80c f i DatERI.obj
 0001:0001e848       ?erase@?$_Tree@V?$_Tmap_traits@GPAUSWI_STRUCT_RoamInd@CDatERI@@U?$less@G@std@@V?$allocator@U?$pair@$$CBGPAUSWI_STRUCT_RoamInd@CDatERI@@@std@@@4@$0A@@std@@@std@@QAA?AViterator@12@V312@@Z 0011f848 f i DatERI.obj
 0001:0001f3b4       ?_Lrotate@?$_Tree@V?$_Tmap_traits@GPAUSWI_STRUCT_RoamInd@CDatERI@@U?$less@G@std@@V?$allocator@U?$pair@$$CBGPAUSWI_STRUCT_RoamInd@CDatERI@@@std@@@4@$0A@@std@@@std@@IAAXPAU_Node@?$_Tree_nod@V?$_Tmap_traits@GPAUSWI_STRUCT_RoamInd@CDatERI@@U?$less@G@std@@V?$allocator@U?$pair@$$CBGPAUSWI_STRUCT_RoamInd@CDatERI@@@std@@@4@$0A@@std@@@2@@Z 001203b4 f i DatERI.obj
 0001:0001f578       ?_Rrotate@?$_Tree@V?$_Tmap_traits@GPAUSWI_STRUCT_RoamInd@CDatERI@@U?$less@G@std@@V?$allocator@U?$pair@$$CBGPAUSWI_STRUCT_RoamInd@CDatERI@@@std@@@4@$0A@@std@@@std@@IAAXPAU_Node@?$_Tree_nod@V?$_Tmap_traits@GPAUSWI_STRUCT_RoamInd@CDatERI@@U?$less@G@std@@V?$allocator@U?$pair@$$CBGPAUSWI_STRUCT_RoamInd@CDatERI@@@std@@@4@$0A@@std@@@2@@Z 00120578 f i DatERI.obj
 0001:0001f744       ?_Buynode@?$_Tree@V?$_Tmap_traits@GPAUSWI_STRUCT_RoamInd@CDatERI@@U?$less@G@std@@V?$allocator@U?$pair@$$CBGPAUSWI_STRUCT_RoamInd@CDatERI@@@std@@@4@$0A@@std@@@std@@IAAPAU_Node@?$_Tree_nod@V?$_Tmap_traits@GPAUSWI_STRUCT_RoamInd@CDatERI@@U?$less@G@std@@V?$allocator@U?$pair@$$CBGPAUSWI_STRUCT_RoamInd@CDatERI@@@std@@@4@$0A@@std@@@2@XZ 00120744 f i DatERI.obj
 0001:0001f8ec       ?_Buynode@?$_Tree@V?$_Tmap_traits@GPAUSWI_STRUCT_RoamInd@CDatERI@@U?$less@G@std@@V?$allocator@U?$pair@$$CBGPAUSWI_STRUCT_RoamInd@CDatERI@@@std@@@4@$0A@@std@@@std@@IAAPAU_Node@?$_Tree_nod@V?$_Tmap_traits@GPAUSWI_STRUCT_RoamInd@CDatERI@@U?$less@G@std@@V?$allocator@U?$pair@$$CBGPAUSWI_STRUCT_RoamInd@CDatERI@@@std@@@4@$0A@@std@@@2@PAU342@00ABU?$pair@$$CBGPAUSWI_STRUCT_RoamInd@CDatERI@@@2@D@Z 001208ec f i DatERI.obj
 0001:0001fa08       ??3@YAXPAX0@Z              00120a08 f i DatERI.obj
 0001:0001fa18       ??0?$_Tree_ptr@V?$_Tmap_traits@GPAUSWI_STRUCT_RoamInd@CDatERI@@U?$less@G@std@@V?$allocator@U?$pair@$$CBGPAUSWI_STRUCT_RoamInd@CDatERI@@@std@@@4@$0A@@std@@@std@@QAA@ABU?$less@G@1@V?$allocator@U?$pair@$$CBGPAUSWI_STRUCT_RoamInd@CDatERI@@@std@@@1@@Z 00120a18 f i DatERI.obj
 0001:0001fa78       ?_Color@?$_Tree@V?$_Tmap_traits@GPAUSWI_STRUCT_CallPrompt@CDatERI@@U?$less@G@std@@V?$allocator@U?$pair@$$CBGPAUSWI_STRUCT_CallPrompt@CDatERI@@@std@@@4@$0A@@std@@@std@@KAAADPAU_Node@?$_Tree_nod@V?$_Tmap_traits@GPAUSWI_STRUCT_CallPrompt@CDatERI@@U?$less@G@std@@V?$allocator@U?$pair@$$CBGPAUSWI_STRUCT_CallPrompt@CDatERI@@@std@@@4@$0A@@std@@@2@@Z 00120a78 f i DatERI.obj
 0001:0001faa0       ?max_size@?$_Tree@V?$_Tmap_traits@GPAUSWI_STRUCT_CallPrompt@CDatERI@@U?$less@G@std@@V?$allocator@U?$pair@$$CBGPAUSWI_STRUCT_CallPrompt@CDatERI@@@std@@@4@$0A@@std@@@std@@QBAIXZ 00120aa0 f i DatERI.obj
 0001:0001fadc       ?erase@?$_Tree@V?$_Tmap_traits@GPAUSWI_STRUCT_CallPrompt@CDatERI@@U?$less@G@std@@V?$allocator@U?$pair@$$CBGPAUSWI_STRUCT_CallPrompt@CDatERI@@@std@@@4@$0A@@std@@@std@@QAA?AViterator@12@V312@@Z 00120adc f i DatERI.obj
 0001:00020648       ?_Lrotate@?$_Tree@V?$_Tmap_traits@GPAUSWI_STRUCT_CallPrompt@CDatERI@@U?$less@G@std@@V?$allocator@U?$pair@$$CBGPAUSWI_STRUCT_CallPrompt@CDatERI@@@std@@@4@$0A@@std@@@std@@IAAXPAU_Node@?$_Tree_nod@V?$_Tmap_traits@GPAUSWI_STRUCT_CallPrompt@CDatERI@@U?$less@G@std@@V?$allocator@U?$pair@$$CBGPAUSWI_STRUCT_CallPrompt@CDatERI@@@std@@@4@$0A@@std@@@2@@Z 00121648 f i DatERI.obj
 0001:0002080c       ?_Rrotate@?$_Tree@V?$_Tmap_traits@GPAUSWI_STRUCT_CallPrompt@CDatERI@@U?$less@G@std@@V?$allocator@U?$pair@$$CBGPAUSWI_STRUCT_CallPrompt@CDatERI@@@std@@@4@$0A@@std@@@std@@IAAXPAU_Node@?$_Tree_nod@V?$_Tmap_traits@GPAUSWI_STRUCT_CallPrompt@CDatERI@@U?$less@G@std@@V?$allocator@U?$pair@$$CBGPAUSWI_STRUCT_CallPrompt@CDatERI@@@std@@@4@$0A@@std@@@2@@Z 0012180c f i DatERI.obj
 0001:000209d8       ?_Buynode@?$_Tree@V?$_Tmap_traits@GPAUSWI_STRUCT_CallPrompt@CDatERI@@U?$less@G@std@@V?$allocator@U?$pair@$$CBGPAUSWI_STRUCT_CallPrompt@CDatERI@@@std@@@4@$0A@@std@@@std@@IAAPAU_Node@?$_Tree_nod@V?$_Tmap_traits@GPAUSWI_STRUCT_CallPrompt@CDatERI@@U?$less@G@std@@V?$allocator@U?$pair@$$CBGPAUSWI_STRUCT_CallPrompt@CDatERI@@@std@@@4@$0A@@std@@@2@XZ 001219d8 f i DatERI.obj
 0001:00020b80       ?_Buynode@?$_Tree@V?$_Tmap_traits@GPAUSWI_STRUCT_CallPrompt@CDatERI@@U?$less@G@std@@V?$allocator@U?$pair@$$CBGPAUSWI_STRUCT_CallPrompt@CDatERI@@@std@@@4@$0A@@std@@@std@@IAAPAU_Node@?$_Tree_nod@V?$_Tmap_traits@GPAUSWI_STRUCT_CallPrompt@CDatERI@@U?$less@G@std@@V?$allocator@U?$pair@$$CBGPAUSWI_STRUCT_CallPrompt@CDatERI@@@std@@@4@$0A@@std@@@2@PAU342@00ABU?$pair@$$CBGPAUSWI_STRUCT_CallPrompt@CDatERI@@@2@D@Z 00121b80 f i DatERI.obj
 0001:00020c9c       ??0?$_Tree_ptr@V?$_Tmap_traits@GPAUSWI_STRUCT_CallPrompt@CDatERI@@U?$less@G@std@@V?$allocator@U?$pair@$$CBGPAUSWI_STRUCT_CallPrompt@CDatERI@@@std@@@4@$0A@@std@@@std@@QAA@ABU?$less@G@1@V?$allocator@U?$pair@$$CBGPAUSWI_STRUCT_CallPrompt@CDatERI@@@std@@@1@@Z 00121c9c f i DatERI.obj
 0001:00020cfc       ??0const_iterator@?$_Tree@V?$_Tmap_traits@GPAUSWI_STRUCT_RoamInd@CDatERI@@U?$less@G@std@@V?$allocator@U?$pair@$$CBGPAUSWI_STRUCT_RoamInd@CDatERI@@@std@@@4@$0A@@std@@@std@@QAA@XZ 00121cfc f i DatERI.obj
 0001:00020d3c       ??Fconst_iterator@?$_Tree@V?$_Tmap_traits@GPAUSWI_STRUCT_RoamInd@CDatERI@@U?$less@G@std@@V?$allocator@U?$pair@$$CBGPAUSWI_STRUCT_RoamInd@CDatERI@@@std@@@4@$0A@@std@@@std@@QAAAAV012@XZ 00121d3c f i DatERI.obj
 0001:00020d68       ?_Inc@const_iterator@?$_Tree@V?$_Tmap_traits@GPAUSWI_STRUCT_RoamInd@CDatERI@@U?$less@G@std@@V?$allocator@U?$pair@$$CBGPAUSWI_STRUCT_RoamInd@CDatERI@@@std@@@4@$0A@@std@@@std@@QAAXXZ 00121d68 f i DatERI.obj
 0001:00020f24       ??0const_iterator@?$_Tree@V?$_Tmap_traits@GPAUSWI_STRUCT_CallPrompt@CDatERI@@U?$less@G@std@@V?$allocator@U?$pair@$$CBGPAUSWI_STRUCT_CallPrompt@CDatERI@@@std@@@4@$0A@@std@@@std@@QAA@XZ 00121f24 f i DatERI.obj
 0001:00020f64       ??Fconst_iterator@?$_Tree@V?$_Tmap_traits@GPAUSWI_STRUCT_CallPrompt@CDatERI@@U?$less@G@std@@V?$allocator@U?$pair@$$CBGPAUSWI_STRUCT_CallPrompt@CDatERI@@@std@@@4@$0A@@std@@@std@@QAAAAV012@XZ 00121f64 f i DatERI.obj
 0001:00020f90       ?_Inc@const_iterator@?$_Tree@V?$_Tmap_traits@GPAUSWI_STRUCT_CallPrompt@CDatERI@@U?$less@G@std@@V?$allocator@U?$pair@$$CBGPAUSWI_STRUCT_CallPrompt@CDatERI@@@std@@@4@$0A@@std@@@std@@QAAXXZ 00121f90 f i DatERI.obj
 0001:0002114c       ??0?$pair@Viterator@?$_Tree@V?$_Tmap_traits@GPAUSWI_STRUCT_RoamInd@CDatERI@@U?$less@G@std@@V?$allocator@U?$pair@$$CBGPAUSWI_STRUCT_RoamInd@CDatERI@@@std@@@4@$0A@@std@@@std@@_N@std@@QAA@ABViterator@?$_Tree@V?$_Tmap_traits@GPAUSWI_STRUCT_RoamInd@CDatERI@@U?$less@G@std@@V?$allocator@U?$pair@$$CBGPAUSWI_STRUCT_RoamInd@CDatERI@@@std@@@4@$0A@@std@@@1@AB_N@Z 0012214c f i DatERI.obj
 0001:00021194       ??0?$pair@Viterator@?$_Tree@V?$_Tmap_traits@GPAUSWI_STRUCT_CallPrompt@CDatERI@@U?$less@G@std@@V?$allocator@U?$pair@$$CBGPAUSWI_STRUCT_CallPrompt@CDatERI@@@std@@@4@$0A@@std@@@std@@_N@std@@QAA@ABViterator@?$_Tree@V?$_Tmap_traits@GPAUSWI_STRUCT_CallPrompt@CDatERI@@U?$less@G@std@@V?$allocator@U?$pair@$$CBGPAUSWI_STRUCT_CallPrompt@CDatERI@@@std@@@4@$0A@@std@@@1@AB_N@Z 00122194 f i DatERI.obj
 0001:000211dc       ?_Max@?$_Tree@V?$_Tmap_traits@GPAUSWI_STRUCT_RoamInd@CDatERI@@U?$less@G@std@@V?$allocator@U?$pair@$$CBGPAUSWI_STRUCT_RoamInd@CDatERI@@@std@@@4@$0A@@std@@@std@@KAPAU_Node@?$_Tree_nod@V?$_Tmap_traits@GPAUSWI_STRUCT_RoamInd@CDatERI@@U?$less@G@std@@V?$allocator@U?$pair@$$CBGPAUSWI_STRUCT_RoamInd@CDatERI@@@std@@@4@$0A@@std@@@2@PAU342@@Z 001221dc f i DatERI.obj
 0001:00021248       ?_Min@?$_Tree@V?$_Tmap_traits@GPAUSWI_STRUCT_RoamInd@CDatERI@@U?$less@G@std@@V?$allocator@U?$pair@$$CBGPAUSWI_STRUCT_RoamInd@CDatERI@@@std@@@4@$0A@@std@@@std@@KAPAU_Node@?$_Tree_nod@V?$_Tmap_traits@GPAUSWI_STRUCT_RoamInd@CDatERI@@U?$less@G@std@@V?$allocator@U?$pair@$$CBGPAUSWI_STRUCT_RoamInd@CDatERI@@@std@@@4@$0A@@std@@@2@PAU342@@Z 00122248 f i DatERI.obj
 0001:000212b4       ??0?$_Tree_nod@V?$_Tmap_traits@GPAUSWI_STRUCT_RoamInd@CDatERI@@U?$less@G@std@@V?$allocator@U?$pair@$$CBGPAUSWI_STRUCT_RoamInd@CDatERI@@@std@@@4@$0A@@std@@@std@@IAA@ABU?$less@G@1@V?$allocator@U?$pair@$$CBGPAUSWI_STRUCT_RoamInd@CDatERI@@@std@@@1@@Z 001222b4 f i DatERI.obj
 0001:00021304       ?max_size@?$allocator@U?$pair@$$CBGPAUSWI_STRUCT_RoamInd@CDatERI@@@std@@@std@@QBAIXZ 00122304 f i DatERI.obj
 0001:00021350       ?allocate@?$allocator@U_Node@?$_Tree_nod@V?$_Tmap_traits@GPAUSWI_STRUCT_RoamInd@CDatERI@@U?$less@G@std@@V?$allocator@U?$pair@$$CBGPAUSWI_STRUCT_RoamInd@CDatERI@@@std@@@4@$0A@@std@@@std@@@std@@QAAPAU_Node@?$_Tree_nod@V?$_Tmap_traits@GPAUSWI_STRUCT_RoamInd@CDatERI@@U?$less@G@std@@V?$allocator@U?$pair@$$CBGPAUSWI_STRUCT_RoamInd@CDatERI@@@std@@@4@$0A@@std@@@2@I@Z 00122350 f i DatERI.obj
 0001:00021384       ?construct@?$allocator@PAU_Node@?$_Tree_nod@V?$_Tmap_traits@GPAUSWI_STRUCT_RoamInd@CDatERI@@U?$less@G@std@@V?$allocator@U?$pair@$$CBGPAUSWI_STRUCT_RoamInd@CDatERI@@@std@@@4@$0A@@std@@@std@@@std@@QAAXPAPAU_Node@?$_Tree_nod@V?$_Tmap_traits@GPAUSWI_STRUCT_RoamInd@CDatERI@@U?$less@G@std@@V?$allocator@U?$pair@$$CBGPAUSWI_STRUCT_RoamInd@CDatERI@@@std@@@4@$0A@@std@@@2@ABQAU342@@Z 00122384 f i DatERI.obj
 0001:000213a0       ?_Max@?$_Tree@V?$_Tmap_traits@GPAUSWI_STRUCT_CallPrompt@CDatERI@@U?$less@G@std@@V?$allocator@U?$pair@$$CBGPAUSWI_STRUCT_CallPrompt@CDatERI@@@std@@@4@$0A@@std@@@std@@KAPAU_Node@?$_Tree_nod@V?$_Tmap_traits@GPAUSWI_STRUCT_CallPrompt@CDatERI@@U?$less@G@std@@V?$allocator@U?$pair@$$CBGPAUSWI_STRUCT_CallPrompt@CDatERI@@@std@@@4@$0A@@std@@@2@PAU342@@Z 001223a0 f i DatERI.obj
 0001:0002140c       ?_Min@?$_Tree@V?$_Tmap_traits@GPAUSWI_STRUCT_CallPrompt@CDatERI@@U?$less@G@std@@V?$allocator@U?$pair@$$CBGPAUSWI_STRUCT_CallPrompt@CDatERI@@@std@@@4@$0A@@std@@@std@@KAPAU_Node@?$_Tree_nod@V?$_Tmap_traits@GPAUSWI_STRUCT_CallPrompt@CDatERI@@U?$less@G@std@@V?$allocator@U?$pair@$$CBGPAUSWI_STRUCT_CallPrompt@CDatERI@@@std@@@4@$0A@@std@@@2@PAU342@@Z 0012240c f i DatERI.obj
 0001:00021478       ??0?$_Tree_nod@V?$_Tmap_traits@GPAUSWI_STRUCT_CallPrompt@CDatERI@@U?$less@G@std@@V?$allocator@U?$pair@$$CBGPAUSWI_STRUCT_CallPrompt@CDatERI@@@std@@@4@$0A@@std@@@std@@IAA@ABU?$less@G@1@V?$allocator@U?$pair@$$CBGPAUSWI_STRUCT_CallPrompt@CDatERI@@@std@@@1@@Z 00122478 f i DatERI.obj
 0001:000214c8       ?max_size@?$allocator@U?$pair@$$CBGPAUSWI_STRUCT_CallPrompt@CDatERI@@@std@@@std@@QBAIXZ 001224c8 f i DatERI.obj
 0001:00021514       ?allocate@?$allocator@U_Node@?$_Tree_nod@V?$_Tmap_traits@GPAUSWI_STRUCT_CallPrompt@CDatERI@@U?$less@G@std@@V?$allocator@U?$pair@$$CBGPAUSWI_STRUCT_CallPrompt@CDatERI@@@std@@@4@$0A@@std@@@std@@@std@@QAAPAU_Node@?$_Tree_nod@V?$_Tmap_traits@GPAUSWI_STRUCT_CallPrompt@CDatERI@@U?$less@G@std@@V?$allocator@U?$pair@$$CBGPAUSWI_STRUCT_CallPrompt@CDatERI@@@std@@@4@$0A@@std@@@2@I@Z 00122514 f i DatERI.obj
 0001:00021548       ?construct@?$allocator@PAU_Node@?$_Tree_nod@V?$_Tmap_traits@GPAUSWI_STRUCT_CallPrompt@CDatERI@@U?$less@G@std@@V?$allocator@U?$pair@$$CBGPAUSWI_STRUCT_CallPrompt@CDatERI@@@std@@@4@$0A@@std@@@std@@@std@@QAAXPAPAU_Node@?$_Tree_nod@V?$_Tmap_traits@GPAUSWI_STRUCT_CallPrompt@CDatERI@@U?$less@G@std@@V?$allocator@U?$pair@$$CBGPAUSWI_STRUCT_CallPrompt@CDatERI@@@std@@@4@$0A@@std@@@2@ABQAU342@@Z 00122548 f i DatERI.obj
 0001:00021564       ?_Dec@const_iterator@?$_Tree@V?$_Tmap_traits@GPAUSWI_STRUCT_RoamInd@CDatERI@@U?$less@G@std@@V?$allocator@U?$pair@$$CBGPAUSWI_STRUCT_RoamInd@CDatERI@@@std@@@4@$0A@@std@@@std@@QAAXXZ 00122564 f i DatERI.obj
 0001:00021864       ?_Dec@const_iterator@?$_Tree@V?$_Tmap_traits@GPAUSWI_STRUCT_CallPrompt@CDatERI@@U?$less@G@std@@V?$allocator@U?$pair@$$CBGPAUSWI_STRUCT_CallPrompt@CDatERI@@@std@@@4@$0A@@std@@@std@@QAAXXZ 00122864 f i DatERI.obj
 0001:00021b64       ??0_Node@?$_Tree_nod@V?$_Tmap_traits@GPAUSWI_STRUCT_RoamInd@CDatERI@@U?$less@G@std@@V?$allocator@U?$pair@$$CBGPAUSWI_STRUCT_RoamInd@CDatERI@@@std@@@4@$0A@@std@@@std@@QAA@PAU012@00ABU?$pair@$$CBGPAUSWI_STRUCT_RoamInd@CDatERI@@@2@D@Z 00122b64 f i DatERI.obj
 0001:00021be8       ??0_Node@?$_Tree_nod@V?$_Tmap_traits@GPAUSWI_STRUCT_CallPrompt@CDatERI@@U?$less@G@std@@V?$allocator@U?$pair@$$CBGPAUSWI_STRUCT_CallPrompt@CDatERI@@@std@@@4@$0A@@std@@@std@@QAA@PAU012@00ABU?$pair@$$CBGPAUSWI_STRUCT_CallPrompt@CDatERI@@@2@D@Z 00122be8 f i DatERI.obj
 0001:00021c6c       ??0?$_Tmap_traits@GPAUSWI_STRUCT_RoamInd@CDatERI@@U?$less@G@std@@V?$allocator@U?$pair@$$CBGPAUSWI_STRUCT_RoamInd@CDatERI@@@std@@@4@$0A@@std@@QAA@U?$less@G@1@@Z 00122c6c f i DatERI.obj
 0001:00021c9c       ??0?$_Tmap_traits@GPAUSWI_STRUCT_CallPrompt@CDatERI@@U?$less@G@std@@V?$allocator@U?$pair@$$CBGPAUSWI_STRUCT_CallPrompt@CDatERI@@@std@@@4@$0A@@std@@QAA@U?$less@G@1@@Z 00122c9c f i DatERI.obj
 0001:00021ccc       ??$_Debug_lt_pred@U?$less@G@std@@GG@std@@YA_NU?$less@G@0@ABG1PBGI@Z 00122ccc f i DatERI.obj
 0001:00021d54       ??$_Destroy@U_Node@?$_Tree_nod@V?$_Tmap_traits@GPAUSWI_STRUCT_RoamInd@CDatERI@@U?$less@G@std@@V?$allocator@U?$pair@$$CBGPAUSWI_STRUCT_RoamInd@CDatERI@@@std@@@4@$0A@@std@@@std@@@std@@YAXPAU_Node@?$_Tree_nod@V?$_Tmap_traits@GPAUSWI_STRUCT_RoamInd@CDatERI@@U?$less@G@std@@V?$allocator@U?$pair@$$CBGPAUSWI_STRUCT_RoamInd@CDatERI@@@std@@@4@$0A@@std@@@0@@Z 00122d54 f i DatERI.obj
 0001:00021d64       ??$_Destroy@PAU_Node@?$_Tree_nod@V?$_Tmap_traits@GPAUSWI_STRUCT_RoamInd@CDatERI@@U?$less@G@std@@V?$allocator@U?$pair@$$CBGPAUSWI_STRUCT_RoamInd@CDatERI@@@std@@@4@$0A@@std@@@std@@@std@@YAXPAPAU_Node@?$_Tree_nod@V?$_Tmap_traits@GPAUSWI_STRUCT_RoamInd@CDatERI@@U?$less@G@std@@V?$allocator@U?$pair@$$CBGPAUSWI_STRUCT_RoamInd@CDatERI@@@std@@@4@$0A@@std@@@0@@Z 00122d64 f i DatERI.obj
 0001:00021d74       ??$_Destroy@U_Node@?$_Tree_nod@V?$_Tmap_traits@GPAUSWI_STRUCT_CallPrompt@CDatERI@@U?$less@G@std@@V?$allocator@U?$pair@$$CBGPAUSWI_STRUCT_CallPrompt@CDatERI@@@std@@@4@$0A@@std@@@std@@@std@@YAXPAU_Node@?$_Tree_nod@V?$_Tmap_traits@GPAUSWI_STRUCT_CallPrompt@CDatERI@@U?$less@G@std@@V?$allocator@U?$pair@$$CBGPAUSWI_STRUCT_CallPrompt@CDatERI@@@std@@@4@$0A@@std@@@0@@Z 00122d74 f i DatERI.obj
 0001:00021d84       ??$_Destroy@PAU_Node@?$_Tree_nod@V?$_Tmap_traits@GPAUSWI_STRUCT_CallPrompt@CDatERI@@U?$less@G@std@@V?$allocator@U?$pair@$$CBGPAUSWI_STRUCT_CallPrompt@CDatERI@@@std@@@4@$0A@@std@@@std@@@std@@YAXPAPAU_Node@?$_Tree_nod@V?$_Tmap_traits@GPAUSWI_STRUCT_CallPrompt@CDatERI@@U?$less@G@std@@V?$allocator@U?$pair@$$CBGPAUSWI_STRUCT_CallPrompt@CDatERI@@@std@@@4@$0A@@std@@@0@@Z 00122d84 f i DatERI.obj
 0001:00021d94       ??$swap@D@std@@YAXAAD0@Z   00122d94 f i DatERI.obj
 0001:00021dd4       ??$?0U?$pair@$$CBGPAUSWI_STRUCT_RoamInd@CDatERI@@@std@@@?$allocator@PAU_Node@?$_Tree_nod@V?$_Tmap_traits@GPAUSWI_STRUCT_RoamInd@CDatERI@@U?$less@G@std@@V?$allocator@U?$pair@$$CBGPAUSWI_STRUCT_RoamInd@CDatERI@@@std@@@4@$0A@@std@@@std@@@std@@QAA@ABV?$allocator@U?$pair@$$CBGPAUSWI_STRUCT_RoamInd@CDatERI@@@std@@@1@@Z 00122dd4 f i DatERI.obj
 0001:00021df8       ??$?0U?$pair@$$CBGPAUSWI_STRUCT_CallPrompt@CDatERI@@@std@@@?$allocator@PAU_Node@?$_Tree_nod@V?$_Tmap_traits@GPAUSWI_STRUCT_CallPrompt@CDatERI@@U?$less@G@std@@V?$allocator@U?$pair@$$CBGPAUSWI_STRUCT_CallPrompt@CDatERI@@@std@@@4@$0A@@std@@@std@@@std@@QAA@ABV?$allocator@U?$pair@$$CBGPAUSWI_STRUCT_CallPrompt@CDatERI@@@std@@@1@@Z 00122df8 f i DatERI.obj
 0001:00021e1c       ??$?0U?$pair@$$CBGPAUSWI_STRUCT_RoamInd@CDatERI@@@std@@@?$allocator@U_Node@?$_Tree_nod@V?$_Tmap_traits@GPAUSWI_STRUCT_RoamInd@CDatERI@@U?$less@G@std@@V?$allocator@U?$pair@$$CBGPAUSWI_STRUCT_RoamInd@CDatERI@@@std@@@4@$0A@@std@@@std@@@std@@QAA@ABV?$allocator@U?$pair@$$CBGPAUSWI_STRUCT_RoamInd@CDatERI@@@std@@@1@@Z 00122e1c f i DatERI.obj
 0001:00021e40       ??$_Allocate@U_Node@?$_Tree_nod@V?$_Tmap_traits@GPAUSWI_STRUCT_RoamInd@CDatERI@@U?$less@G@std@@V?$allocator@U?$pair@$$CBGPAUSWI_STRUCT_RoamInd@CDatERI@@@std@@@4@$0A@@std@@@std@@@std@@YAPAU_Node@?$_Tree_nod@V?$_Tmap_traits@GPAUSWI_STRUCT_RoamInd@CDatERI@@U?$less@G@std@@V?$allocator@U?$pair@$$CBGPAUSWI_STRUCT_RoamInd@CDatERI@@@std@@@4@$0A@@std@@@0@IPAU120@@Z 00122e40 f i DatERI.obj
 0001:00021ed0       ??$_Construct@PAU_Node@?$_Tree_nod@V?$_Tmap_traits@GPAUSWI_STRUCT_RoamInd@CDatERI@@U?$less@G@std@@V?$allocator@U?$pair@$$CBGPAUSWI_STRUCT_RoamInd@CDatERI@@@std@@@4@$0A@@std@@@std@@PAU123@@std@@YAXPAPAU_Node@?$_Tree_nod@V?$_Tmap_traits@GPAUSWI_STRUCT_RoamInd@CDatERI@@U?$less@G@std@@V?$allocator@U?$pair@$$CBGPAUSWI_STRUCT_RoamInd@CDatERI@@@std@@@4@$0A@@std@@@0@ABQAU120@@Z 00122ed0 f i DatERI.obj
 0001:00021f38       ??$?0U?$pair@$$CBGPAUSWI_STRUCT_CallPrompt@CDatERI@@@std@@@?$allocator@U_Node@?$_Tree_nod@V?$_Tmap_traits@GPAUSWI_STRUCT_CallPrompt@CDatERI@@U?$less@G@std@@V?$allocator@U?$pair@$$CBGPAUSWI_STRUCT_CallPrompt@CDatERI@@@std@@@4@$0A@@std@@@std@@@std@@QAA@ABV?$allocator@U?$pair@$$CBGPAUSWI_STRUCT_CallPrompt@CDatERI@@@std@@@1@@Z 00122f38 f i DatERI.obj
 0001:00021f5c       ??$_Allocate@U_Node@?$_Tree_nod@V?$_Tmap_traits@GPAUSWI_STRUCT_CallPrompt@CDatERI@@U?$less@G@std@@V?$allocator@U?$pair@$$CBGPAUSWI_STRUCT_CallPrompt@CDatERI@@@std@@@4@$0A@@std@@@std@@@std@@YAPAU_Node@?$_Tree_nod@V?$_Tmap_traits@GPAUSWI_STRUCT_CallPrompt@CDatERI@@U?$less@G@std@@V?$allocator@U?$pair@$$CBGPAUSWI_STRUCT_CallPrompt@CDatERI@@@std@@@4@$0A@@std@@@0@IPAU120@@Z 00122f5c f i DatERI.obj
 0001:00021fec       ??$_Construct@PAU_Node@?$_Tree_nod@V?$_Tmap_traits@GPAUSWI_STRUCT_CallPrompt@CDatERI@@U?$less@G@std@@V?$allocator@U?$pair@$$CBGPAUSWI_STRUCT_CallPrompt@CDatERI@@@std@@@4@$0A@@std@@@std@@PAU123@@std@@YAXPAPAU_Node@?$_Tree_nod@V?$_Tmap_traits@GPAUSWI_STRUCT_CallPrompt@CDatERI@@U?$less@G@std@@V?$allocator@U?$pair@$$CBGPAUSWI_STRUCT_CallPrompt@CDatERI@@@std@@@4@$0A@@std@@@0@ABQAU120@@Z 00122fec f i DatERI.obj
 0001:00022054       ?EnableNotifications@CRadio@@QAAX_N@Z 00123054 f   FakeResponse.obj
 0001:00023570       ?EnableTechHDRNotifications@CRadio@@QAAX_N@Z 00124570 f   FakeResponse.obj
 0001:000235c8       ?InitThreadProc@@YAKPAX@Z  001245c8 f   FakeResponse.obj
 0001:000239d8       ?HandleCommand@CRilHandle@@QAAHPAVCCommand@@@Z 001249d8 f   FakeResponse.obj
 0001:00024238       ?HandleRsp@CRilHandle@@QAAHAAPAVCCommand@@AAPAVCResponse@@@Z 00125238 f   FakeResponse.obj
 0001:00024538       ?ResponseThread@CRilHandle@@QAAKXZ 00125538 f   FakeResponse.obj
 0001:00024788       ?QueueCommandForDelayedResponse@CRilHandle@@QAAHPAVCCommand@@PAVCResponse@@@Z 00125788 f   FakeResponse.obj
 0001:00024a5c       ?IsSMSSupported@CRadioCaps@@QAAHXZ 00125a5c f i FakeResponse.obj
 0001:00024a8c       ?IsMOSMSAllowed@CRadioCaps@@QAAHXZ 00125a8c f i FakeResponse.obj
 0001:00024abc       ?IsMTSMSAllowed@CRadioCaps@@QAAHXZ 00125abc f i FakeResponse.obj
 0001:00024aec       ??0CSafeEntry@@QAA@PA_N@Z  00125aec f i FakeResponse.obj
 0001:00024b68       ??1CSafeEntry@@QAA@XZ      00125b68 f i FakeResponse.obj
 0001:00024b94       ?Lock@CSafeEntry@@QAA_NXZ  00125b94 f i FakeResponse.obj
 0001:00024c38       ?Unlock@CSafeEntry@@IAAXXZ 00125c38 f i FakeResponse.obj
 0001:00024ca0       ?IsDMMode@CRadio@@QAAHXZ   00125ca0 f i FakeResponse.obj
 0001:00024cd0       ?CmdOptIsSet@CCommand@@QAAHK@Z 00125cd0 f i FakeResponse.obj
 0001:00024d04       ?GetCmdData@CCommand@@QBAPAXXZ 00125d04 f i FakeResponse.obj
 0001:00024d30       ?GetNotifyCode@CResponse@@QBAKXZ 00125d30 f i FakeResponse.obj
 0001:00024d5c       ?SetCurrAPIID@CRilHandle@@QAAXK@Z 00125d5c f i FakeResponse.obj
 0001:00024da4       ?IsRILSuspended@CRilHandle@@QAAHXZ 00125da4 f i FakeResponse.obj
 0001:00024df4       ??_GCResponse@@QAAPAXI@Z   00125df4 f i FakeResponse.obj
 0001:00024e34       ?DeleteBlob@CResponse@@QAAXXZ 00125e34 f i FakeResponse.obj
 0001:00024e84       ?GetBlob@CResponse@@QBAXAAPAXAAI@Z 00125e84 f i FakeResponse.obj
 0001:00024ebc       ??_GCNotificationData@@QAAPAXI@Z 00125ebc f i FakeResponse.obj
 0001:00024efc       ?FDelayRsp@CCommand@@QBAHXZ 00125efc f i FakeResponse.obj
 0001:00024f2c       ?push_back@?$list@PAVCCommand@@V?$allocator@PAVCCommand@@@std@@@std@@QAAXABQAVCCommand@@@Z 00125f2c f i FakeResponse.obj
 0001:00024f74       ?end@?$list@PAVCCommand@@V?$allocator@PAVCCommand@@@std@@@std@@QAA?AV?$_Iterator@$00@12@XZ 00125f74 f i FakeResponse.obj
 0001:00024fd0       ?_Insert@?$list@PAVCCommand@@V?$allocator@PAVCCommand@@@std@@@std@@QAAXV?$_Iterator@$00@12@ABQAVCCommand@@@Z 00125fd0 f i FakeResponse.obj
 0001:000250cc       ??1?$_Iterator@$00@?$list@PAVCCommand@@V?$allocator@PAVCCommand@@@std@@@std@@QAA@XZ 001260cc f i FakeResponse.obj
 0001:000250e4       ??1?$_Const_iterator@$00@?$list@PAVCCommand@@V?$allocator@PAVCCommand@@@std@@@std@@QAA@XZ 001260e4 f i FakeResponse.obj
 0001:000250fc       ??1?$_Bidit@PAVCCommand@@HPBQAV1@ABQAV1@@std@@QAA@XZ 001260fc f i FakeResponse.obj
 0001:00025114       ?_Nextnode@?$list@PAVCCommand@@V?$allocator@PAVCCommand@@@std@@@std@@KAAAPAU_Node@?$_List_nod@PAVCCommand@@V?$allocator@PAVCCommand@@@std@@@2@PAU342@@Z 00126114 f i FakeResponse.obj
 0001:00025138       ?_Prevnode@?$list@PAVCCommand@@V?$allocator@PAVCCommand@@@std@@@std@@KAAAPAU_Node@?$_List_nod@PAVCCommand@@V?$allocator@PAVCCommand@@@std@@@2@PAU342@@Z 00126138 f i FakeResponse.obj
 0001:00025168       ?_Buynode@?$list@PAVCCommand@@V?$allocator@PAVCCommand@@@std@@@std@@IAAPAU_Node@?$_List_nod@PAVCCommand@@V?$allocator@PAVCCommand@@@std@@@2@PAU342@0ABQAVCCommand@@@Z 00126168 f i FakeResponse.obj
 0001:000252c8       ?_Incsize@?$list@PAVCCommand@@V?$allocator@PAVCCommand@@@std@@@std@@IAAXI@Z 001262c8 f i FakeResponse.obj
 0001:00025398       ??0?$_Iterator@$00@?$list@PAVCCommand@@V?$allocator@PAVCCommand@@@std@@@std@@QAA@PAU_Node@?$_List_nod@PAVCCommand@@V?$allocator@PAVCCommand@@@std@@@2@PBV12@@Z 00126398 f i FakeResponse.obj
 0001:000253d0       ?_Mynode@?$_Const_iterator@$00@?$list@PAVCCommand@@V?$allocator@PAVCCommand@@@std@@@std@@QBAPAU_Node@?$_List_nod@PAVCCommand@@V?$allocator@PAVCCommand@@@std@@@3@XZ 001263d0 f i FakeResponse.obj
 0001:000253fc       ?_Myval@?$list@PAVCCommand@@V?$allocator@PAVCCommand@@@std@@@std@@KAAAPAVCCommand@@PAU_Node@?$_List_nod@PAVCCommand@@V?$allocator@PAVCCommand@@@std@@@2@@Z 001263fc f i FakeResponse.obj
 0001:00025424       ?max_size@?$list@PAVCCommand@@V?$allocator@PAVCCommand@@@std@@@std@@QBAIXZ 00126424 f i FakeResponse.obj
 0001:00025458       ?deallocate@?$allocator@U_Node@?$_List_nod@PAVCCommand@@V?$allocator@PAVCCommand@@@std@@@std@@@std@@QAAXPAU_Node@?$_List_nod@PAVCCommand@@V?$allocator@PAVCCommand@@@std@@@2@I@Z 00126458 f i FakeResponse.obj
 0001:00025470       ?allocate@?$allocator@U_Node@?$_List_nod@PAVCCommand@@V?$allocator@PAVCCommand@@@std@@@std@@@std@@QAAPAU_Node@?$_List_nod@PAVCCommand@@V?$allocator@PAVCCommand@@@std@@@2@I@Z 00126470 f i FakeResponse.obj
 0001:000254a4       ?construct@?$allocator@PAU_Node@?$_List_nod@PAVCCommand@@V?$allocator@PAVCCommand@@@std@@@std@@@std@@QAAXPAPAU_Node@?$_List_nod@PAVCCommand@@V?$allocator@PAVCCommand@@@std@@@2@ABQAU342@@Z 001264a4 f i FakeResponse.obj
 0001:000254c0       ?destroy@?$allocator@PAU_Node@?$_List_nod@PAVCCommand@@V?$allocator@PAVCCommand@@@std@@@std@@@std@@QAAXPAPAU_Node@?$_List_nod@PAVCCommand@@V?$allocator@PAVCCommand@@@std@@@2@@Z 001264c0 f i FakeResponse.obj
 0001:000254e0       ??0?$_Const_iterator@$00@?$list@PAVCCommand@@V?$allocator@PAVCCommand@@@std@@@std@@QAA@PAU_Node@?$_List_nod@PAVCCommand@@V?$allocator@PAVCCommand@@@std@@@2@PBV12@@Z 001264e0 f i FakeResponse.obj
 0001:00025548       ??0?$_Bidit@PAVCCommand@@HPBQAV1@ABQAV1@@std@@QAA@XZ 00126548 f i FakeResponse.obj
 0001:00025578       ?Pop_Front@?$CThreadSafeQueue@PAUSwiNotifyVariant@@@@QAAPAUSwiNotifyVariant@@XZ 00126578 f i FakeResponse.obj
 0001:00025620       ?GetAlertEvent@?$CThreadSafeQueue@PAUSwiNotifyVariant@@@@QAAPAXXZ 00126620 f i FakeResponse.obj
 0001:00025654       ??BEvent@@QBAPAXXZ         00126654 f i FakeResponse.obj
 0001:00025680       ??$_Allocate@U_Node@?$_List_nod@PAVCCommand@@V?$allocator@PAVCCommand@@@std@@@std@@@std@@YAPAU_Node@?$_List_nod@PAVCCommand@@V?$allocator@PAVCCommand@@@std@@@0@IPAU120@@Z 00126680 f i FakeResponse.obj
 0001:00025710       ??$_Construct@PAU_Node@?$_List_nod@PAVCCommand@@V?$allocator@PAVCCommand@@@std@@@std@@PAU123@@std@@YAXPAPAU_Node@?$_List_nod@PAVCCommand@@V?$allocator@PAVCCommand@@@std@@@0@ABQAU120@@Z 00126710 f i FakeResponse.obj
 0001:00025778       ??$_Destroy@PAU_Node@?$_List_nod@PAVCCommand@@V?$allocator@PAVCCommand@@@std@@@std@@@std@@YAXPAPAU_Node@?$_List_nod@PAVCCommand@@V?$allocator@PAVCCommand@@@std@@@0@@Z 00126778 f i FakeResponse.obj
 0001:00025788       ?empty@?$queue@PAUSwiNotifyVariant@@V?$deque@PAUSwiNotifyVariant@@V?$allocator@PAUSwiNotifyVariant@@@std@@@std@@@std@@QBA_NXZ 00126788 f i FakeResponse.obj
 0001:000257b8       ?size@?$queue@PAUSwiNotifyVariant@@V?$deque@PAUSwiNotifyVariant@@V?$allocator@PAUSwiNotifyVariant@@@std@@@std@@@std@@QBAIXZ 001267b8 f i FakeResponse.obj
 0001:000257e8       ?front@?$queue@PAUSwiNotifyVariant@@V?$deque@PAUSwiNotifyVariant@@V?$allocator@PAUSwiNotifyVariant@@@std@@@std@@@std@@QAAAAPAUSwiNotifyVariant@@XZ 001267e8 f i FakeResponse.obj
 0001:00025818       ?pop@?$queue@PAUSwiNotifyVariant@@V?$deque@PAUSwiNotifyVariant@@V?$allocator@PAUSwiNotifyVariant@@@std@@@std@@@std@@QAAXXZ 00126818 f i FakeResponse.obj
 0001:00025830       ?size@?$deque@PAUSwiNotifyVariant@@V?$allocator@PAUSwiNotifyVariant@@@std@@@std@@QBAIXZ 00126830 f i FakeResponse.obj
 0001:0002585c       ?empty@?$deque@PAUSwiNotifyVariant@@V?$allocator@PAUSwiNotifyVariant@@@std@@@std@@QBA_NXZ 0012685c f i FakeResponse.obj
 0001:000258b4       ?front@?$deque@PAUSwiNotifyVariant@@V?$allocator@PAUSwiNotifyVariant@@@std@@@std@@QAAAAPAUSwiNotifyVariant@@XZ 001268b4 f i FakeResponse.obj
 0001:00025928       ?pop_front@?$deque@PAUSwiNotifyVariant@@V?$allocator@PAUSwiNotifyVariant@@@std@@@std@@QAAXXZ 00126928 f i FakeResponse.obj
 0001:00025aa0       ??1?$_Deque_iterator@PAUSwiNotifyVariant@@V?$allocator@PAUSwiNotifyVariant@@@std@@$00@std@@QAA@XZ 00126aa0 f i FakeResponse.obj
 0001:00025ab8       ??1?$_Deque_const_iterator@PAUSwiNotifyVariant@@V?$allocator@PAUSwiNotifyVariant@@@std@@$00@std@@QAA@XZ 00126ab8 f i FakeResponse.obj
 0001:00025ad0       ??1?$_Ranit@PAUSwiNotifyVariant@@HPBQAU1@ABQAU1@@std@@QAA@XZ 00126ad0 f i FakeResponse.obj
 0001:00025ae8       ?begin@?$deque@PAUSwiNotifyVariant@@V?$allocator@PAUSwiNotifyVariant@@@std@@@std@@QAA?AV?$_Deque_iterator@PAUSwiNotifyVariant@@V?$allocator@PAUSwiNotifyVariant@@@std@@$00@2@XZ 00126ae8 f i FakeResponse.obj
 0001:00025b3c       ?_Orphan_off@?$deque@PAUSwiNotifyVariant@@V?$allocator@PAUSwiNotifyVariant@@@std@@@std@@IBAXI@Z 00126b3c f i FakeResponse.obj
 0001:00025c94       ?destroy@?$allocator@PAUSwiNotifyVariant@@@std@@QAAXPAPAUSwiNotifyVariant@@@Z 00126c94 f i FakeResponse.obj
 0001:00025cac       ??D?$_Deque_iterator@PAUSwiNotifyVariant@@V?$allocator@PAUSwiNotifyVariant@@@std@@$00@std@@QBAAAPAUSwiNotifyVariant@@XZ 00126cac f i FakeResponse.obj
 0001:00025cdc       ??0?$_Deque_iterator@PAUSwiNotifyVariant@@V?$allocator@PAUSwiNotifyVariant@@@std@@$00@std@@QAA@IPBV_Container_base@1@@Z 00126cdc f i FakeResponse.obj
 0001:00025d14       ??D?$_Deque_const_iterator@PAUSwiNotifyVariant@@V?$allocator@PAUSwiNotifyVariant@@@std@@$00@std@@QBAABQAUSwiNotifyVariant@@XZ 00126d14 f i FakeResponse.obj
 0001:00025ec0       ??0?$_Deque_const_iterator@PAUSwiNotifyVariant@@V?$allocator@PAUSwiNotifyVariant@@@std@@$00@std@@QAA@IPBV_Container_base@1@@Z 00126ec0 f i FakeResponse.obj
 0001:00025fd8       ??0?$_Ranit@PAUSwiNotifyVariant@@HPBQAU1@ABQAU1@@std@@QAA@XZ 00126fd8 f i FakeResponse.obj
 0001:00026008       ??$_Destroy@PAUSwiNotifyVariant@@@std@@YAXPAPAUSwiNotifyVariant@@@Z 00127008 f i FakeResponse.obj
 0001:00026018       ?RILDrv_GetGPRSContextList@@YAJK@Z 00127018 f   gprs.obj
 0001:000260c0       ?RILDrv_SetGPRSContext@@YAJKPBUrilgprscontext_tag@@@Z 001270c0 f   gprs.obj
 0001:0002617c       ?RILDrv_NdisSetGPRSContextActivated@@YAJKPBUrilndisgprscontext_tag@@@Z 0012717c f   gprs.obj
 0001:0002620c       ?RILDrv_NdisReceivePacketDone@@YAJKPAUrilndispacket_tag@@@Z 0012720c f   gprs.obj
 0001:00026288       ?RILDrv_NdisSendPacket@@YAJKPAUrilndispacket_tag@@@Z 00127288 f   gprs.obj
 0001:00026304       ?RILDrv_DeleteGPRSContext@@YAJKK@Z 00127304 f   gprs.obj
 0001:000263a4       ?RILDrv_GetRequestedQualityOfServiceList@@YAJK@Z 001273a4 f   gprs.obj
 0001:0002643c       ?RILDrv_GetMinimumQualityOfServiceList@@YAJK@Z 0012743c f   gprs.obj
 0001:000264dc       ?SetQOS@@YAJKPBUrilgprsqosprofile_tag@@PBDW4APIID@@@Z 001274dc f   gprs.obj
 0001:00026e54       ?RILDrv_SetRequestedQualityOfService@@YAJKPBUrilgprsqosprofile_tag@@@Z 00127e54 f   gprs.obj
 0001:00026e94       ?RILDrv_SetMinimumQualityOfService@@YAJKPBUrilgprsqosprofile_tag@@@Z 00127e94 f   gprs.obj
 0001:00026edc       ?DeleteQOS@@YAJKKPBDW4APIID@@@Z 00127edc f   gprs.obj
 0001:00026fac       ?RILDrv_DeleteRequestedQualityOfService@@YAJKK@Z 00127fac f   gprs.obj
 0001:00026fec       ?RILDrv_DeleteMinimumQualityOfService@@YAJKK@Z 00127fec f   gprs.obj
 0001:00027034       ?RILDrv_SetGPRSAttached@@YAJKH@Z 00128034 f   gprs.obj
 0001:0002711c       ?RILDrv_GetGPRSAttached@@YAJK@Z 0012811c f   gprs.obj
 0001:000271b4       ?RILDrv_SetGPRSContextActivated@@YAJKKH@Z 001281b4 f   gprs.obj
 0001:000272d0       ?RILDrv_GetGPRSContextActivatedList@@YAJK@Z 001282d0 f   gprs.obj
 0001:00027368       ?ParseForceFailureResponse@@YAJPBDAAPAXAAI@Z 00128368 f   gprs.obj
 0001:00027398       ?RILDrv_EnterGPRSDataMode@@YAJKPBUrilentergprsdatamode_tag@@@Z 00128398 f   gprs.obj
 0001:000276ac       ?RILDrv_GetGPRSAddress@@YAJKK@Z 001286ac f   gprs.obj
 0001:0002777c       ?RILDrv_GPRSAnswer@@YAJKPBUrilgprsanswer_tag@@@Z 0012877c f   gprs.obj
 0001:00027b20       ?RILDrv_SendSimCmd@@YAJKPBEK@Z 00128b20 f   gprs.obj
 0001:00027ca4       ?RILDrv_SendRestrictedSimCmd@@YAJKKPBUrilsimcmdparameters_tag@@PBEK@Z 00128ca4 f   gprs.obj
 0001:00027e7c       ?RILDrv_GetSimRecordStatus@@YAJKK@Z 00128e7c f   gprs.obj
 0001:00027f14       ?RILDrv_GetGPRSRegistrationStatus@@YAJK@Z 00128f14 f   gprs.obj
 0001:00027fac       ?RILDrv_GetGPRSClass@@YAJK@Z 00128fac f   gprs.obj
 0001:0002804c       ?RILDrv_SetGPRSClass@@YAJKK@Z 0012904c f   gprs.obj
 0001:00028144       ?RILDrv_GetMOSMSService@@YAJK@Z 00129144 f   gprs.obj
 0001:000281e4       ?RILDrv_SetMOSMSService@@YAJKK@Z 001291e4 f   gprs.obj
 0001:000282dc       ?GetGPRSRegistrationStatus@CRadio@@QAAJPAVCResponse@@@Z 001292dc f   gprs.obj
 0001:00028440       ?DeleteGPRSContext@CRadio@@QAAJPAVCResponse@@PAX@Z 00129440 f   gprs.obj
 0001:00028520       ?GetGPRSAttached@CRadio@@QAAJPAVCResponse@@@Z 00129520 f   gprs.obj
 0001:000285ec       ?SetGPRSContextActivated@CRadio@@QAAJPAVCResponse@@PAX@Z 001295ec f   gprs.obj
 0001:00028764       ?SendSimCmd@CRadio@@QAAJPAVCResponse@@PAX@Z 00129764 f   gprs.obj
 0001:00028a9c       ?SendRestrictedSimCmd@CRadio@@QAAJPAVCResponse@@PAX@Z 00129a9c f   gprs.obj
 0001:000291d4       ?GetSimRecordStatus@CRadio@@QAAJPAVCResponse@@PAX@Z 0012a1d4 f   gprs.obj
 0001:0002943c       ?GetGPRSContextList@CRadio@@QAAJPAVCResponse@@@Z 0012a43c f   gprs.obj
 0001:000297ac       ?GPRSActivate@CRadio@@QAAJKH@Z 0012a7ac f   gprs.obj
 0001:00029988       ?SetGPRSContext@CRadio@@QAAJPAVCResponse@@PAX@Z 0012a988 f   gprs.obj
 0001:00029eac       ?RILDrv_HandleSuspend@@YAJKJW4_CEDEVICE_POWER_STATE@@@Z 0012aeac f   misc.obj
 0001:0002a004       ?RILDrv_HandleResume@@YAJKW4_CEDEVICE_POWER_STATE@@@Z 0012b004 f   misc.obj
 0001:0002a1f8       ?RILDrv_AuxPowerSet@@YAJKPAW4_CEDEVICE_POWER_STATE@@@Z 0012b1f8 f   misc.obj
 0001:0002a420       ?RILDrv_AuxPowerGet@@YAJKPAW4_CEDEVICE_POWER_STATE@@@Z 0012b420 f   misc.obj
 0001:0002a4d0       ?RILDrv_GetEquipmentInfo@@YAJK@Z 0012b4d0 f   misc.obj
 0001:0002a5b0       ?RILDrv_GetEquipmentState@@YAJK@Z 0012b5b0 f   misc.obj
 0001:0002a72c       ?RILDrv_SetEquipmentState@@YAJKK@Z 0012b72c f   misc.obj
 0001:0002a940       ?RILDrv_GetSignalQuality@@YAJK@Z 0012b940 f   misc.obj
 0001:0002aa24       ?RILDrv_GetCellTowerInfo@@YAJK@Z 0012ba24 f   misc.obj
 0001:0002ab08       ?RILDrv_GetPacketByteCount@@YAJK@Z 0012bb08 f   misc.obj
 0001:0002abe8       ?RILDrv_ResetPacketByteCount@@YAJK@Z 0012bbe8 f   misc.obj
 0001:0002accc       ?RILDrv_GetSystemTime@@YAJK@Z 0012bccc f   misc.obj
 0001:0002adb0       ?RILDrv_DevSpecific@@YAJKPBEK@Z 0012bdb0 f   misc.obj
 0001:0002b4bc       ?SetEquipmentCachedState@CRadio@@QAAXK@Z 0012c4bc f   misc.obj
 0001:0002b6ac       ?GetEquipmentState@CRadio@@QAAJPAVCResponse@@@Z 0012c6ac f   misc.obj
 0001:0002b7d0       ?ForceModemPowerOff@CRadio@@QAAXXZ 0012c7d0 f   misc.obj
 0001:0002b874       ?HardResetModem@CRadio@@QAAXXZ 0012c874 f   misc.obj
 0001:0002b8ac       ?NotifyHardResetModemRequired@CRadio@@QAAXXZ 0012c8ac f   misc.obj
 0001:0002b900       ?SetEquipmentState@CRadio@@QAAJPAVCResponse@@PAX@Z 0012c900 f   misc.obj
 0001:0002c034       ?FillSignalQualityStruct@CRadio@@QAAXPAUrilsignalquality_tag@@II@Z 0012d034 f   misc.obj
 0001:0002c8f0       ?GetSignalQuality@CRadio@@QAAJPAVCResponse@@@Z 0012d8f0 f   misc.obj
 0001:0002cbb8       ?GetCellTowerInfo@CRadio@@QAAJPAVCResponse@@@Z 0012dbb8 f   misc.obj
 0001:0002cf30       ?GetPacketByteCount@CRadio@@QAAJPAVCResponse@@@Z 0012df30 f   misc.obj
 0001:0002d0e8       ?ResetPacketByteCount@CRadio@@QAAJPAVCResponse@@@Z 0012e0e8 f   misc.obj
 0001:0002d1b0       ?GetSystemTime@CRadio@@QAAJPAVCResponse@@@Z 0012e1b0 f   misc.obj
 0001:0002d2fc       ?GetEquipmentInfo@CRadio@@QAAJPAVCResponse@@@Z 0012e2fc f   misc.obj
 0001:0002d914       ?GetLocationStatus@CRadio@@QAAJXZ 0012e914 f   misc.obj
 0001:0002d9a0       ?DevSpecific@CRadio@@QAAJPAVCResponse@@PAX@Z 0012e9a0 f   misc.obj
 0001:00033e58       ?UpdateAndBroadcastOnSWIGPSNotifications@CRadio@@QAAXPAUSwiNotifyVariant@@@Z 00134e58 f   misc.obj
 0001:00033e68       ?StartDMMode@CRadio@@QAAJW4eDM_MODE@@@Z 00134e68 f   misc.obj
 0001:000341d8       ?StopDMMode@CRadio@@QAAJXZ 001351d8 f   misc.obj
 0001:000343a0       ?StartPTMode@CRadio@@QAAJXZ 001353a0 f   misc.obj
 0001:000344d8       ?StopPTMode@CRadio@@QAAJXZ 001354d8 f   misc.obj
 0001:00034630       ?SetGpsOneXtra@CRadio@@QAAJK@Z 00135630 f   misc.obj
 0001:00034744       ?SetGpsDefault@CRadio@@QAAJKEKK@Z 00135744 f   misc.obj
 0001:000348a4       ?SetNMEAConfig@CRadio@@QAAJEEEPAG@Z 001358a4 f   misc.obj
 0001:00034a08       ?GetNMEAConfig@CRadio@@QAAJPAE00PAG@Z 00135a08 f   misc.obj
 0001:00034b6c       ?ForceGPSOneXtraDownload@CRadio@@QAAJXZ 00135b6c f   misc.obj
 0001:00034c24       ?RILDrv_GetPhonebookOptions@@YAJK@Z 00135c24 f   misc.obj
 0001:00034d08       ?RilToQmiSimPbStoreLocation@@YAKK@Z 00135d08 f   misc.obj
 0001:00034e38       ?GetPhonebookOptions@CRadio@@QAAJPAVCResponse@@@Z 00135e38 f   misc.obj
 0001:000350ec       ?RILDrv_SetPhonebookOptions@@YAJKPBUrilphonebookinfo_tag@@@Z 001360ec f   misc.obj
 0001:00035298       ?SetPhonebookOptions@CRadio@@QAAJPAVCResponse@@PAX@Z 00136298 f   misc.obj
 0001:00035380       ?RILDrv_ReadPhonebookEntries@@YAJKKK@Z 00136380 f   misc.obj
 0001:000354b8       ?ReadPhonebookEntries@CRadio@@QAAJPAVCResponse@@PAX@Z 001364b8 f   misc.obj
 0001:00035b70       ?UpdateAndBroadcastOnSWIPhoneBookNotification@CRadio@@QAAXPAUSwiNotifyVariant@@@Z 00136b70 f   misc.obj
 0001:00035f2c       ?cmp_emergency_num_info@@YA_NABUtagEMERGENCY_NUM_INFO@@0@Z 00136f2c f   misc.obj
 0001:00035f8c       ?cmp_emergency_num_info_equal@@YA_NABUtagEMERGENCY_NUM_INFO@@0@Z 00136f8c f   misc.obj
 0001:00035ff4       ?HandleSWIEmergencyListNotification@CRadio@@QAAXPAUSwiNotifyVariant@@@Z 00136ff4 f   misc.obj
 0001:00036288       ?RILDrv_WritePhonebookEntry@@YAJKPBUrilphonebookentry_tag@@@Z 00137288 f   misc.obj
 0001:00036394       ?WritePhonebookEntry@CRadio@@QAAJPAVCResponse@@PAX@Z 00137394 f   misc.obj
 0001:000366b4       ?RILDrv_DeletePhonebookEntry@@YAJKK@Z 001376b4 f   misc.obj
 0001:000367a0       ?DeletePhonebookEntry@CRadio@@QAAJPAVCResponse@@PAX@Z 001377a0 f   misc.obj
 0001:00036940       ?IsSafeImage@CRadio@@QAAHXZ 00137940 f   misc.obj
 0001:00036d34       ?GetFwImagePreference@CRadio@@QAAHPAKQAE@Z 00137d34 f   misc.obj
 0001:00036f64       ?SetFwImagePreference@CRadio@@QAAHPAKQAE@Z 00137f64 f   misc.obj
 0001:0003713c       ?SuspendResume@CRilHandle@@QAAXH@Z 0013813c f i misc.obj
 0001:0003719c       ?GetEquipmentCachedState@CRadio@@QAAKXZ 0013819c f i misc.obj
 0001:000371cc       ?IsSwiAPIOpenned@CRilHandle@@QAAHXZ 001381cc f i misc.obj
 0001:000371f8       ?wcschr@@YAPAGPAGG@Z       001381f8 f i misc.obj
 0001:0003722c       ?IsERIPresent@CDatERI@@QAA_NXZ 0013822c f i misc.obj
 0001:00037258       ?IsActivated@CRadio@@QAAHXZ 00138258 f i misc.obj
 0001:000372b0       ??0?$list@UtagEMERGENCY_NUM_INFO@@V?$allocator@UtagEMERGENCY_NUM_INFO@@@std@@@std@@QAA@XZ 001382b0 f i misc.obj
 0001:00037348       ??1?$list@UtagEMERGENCY_NUM_INFO@@V?$allocator@UtagEMERGENCY_NUM_INFO@@@std@@@std@@QAA@XZ 00138348 f i misc.obj
 0001:00037388       ?push_back@?$list@UtagEMERGENCY_NUM_INFO@@V?$allocator@UtagEMERGENCY_NUM_INFO@@@std@@@std@@QAAXABUtagEMERGENCY_NUM_INFO@@@Z 00138388 f i misc.obj
 0001:000373d0       ?clear@?$list@UtagEMERGENCY_NUM_INFO@@V?$allocator@UtagEMERGENCY_NUM_INFO@@@std@@@std@@QAAXXZ 001383d0 f i misc.obj
 0001:000374dc       ??1?$_List_val@UtagEMERGENCY_NUM_INFO@@V?$allocator@UtagEMERGENCY_NUM_INFO@@@std@@@std@@QAA@XZ 001384dc f i misc.obj
 0001:000374f4       ??1?$_List_ptr@UtagEMERGENCY_NUM_INFO@@V?$allocator@UtagEMERGENCY_NUM_INFO@@@std@@@std@@QAA@XZ 001384f4 f i misc.obj
 0001:0003750c       ??1?$_List_nod@UtagEMERGENCY_NUM_INFO@@V?$allocator@UtagEMERGENCY_NUM_INFO@@@std@@@std@@QAA@XZ 0013850c f i misc.obj
 0001:00037524       ?_Prevnode@?$list@UtagEMERGENCY_NUM_INFO@@V?$allocator@UtagEMERGENCY_NUM_INFO@@@std@@@std@@KAAAPAU_Node@?$_List_nod@UtagEMERGENCY_NUM_INFO@@V?$allocator@UtagEMERGENCY_NUM_INFO@@@std@@@2@PAU342@@Z 00138524 f i misc.obj
 0001:00037554       ?_Insert@?$list@UtagEMERGENCY_NUM_INFO@@V?$allocator@UtagEMERGENCY_NUM_INFO@@@std@@@std@@QAAXV?$_Iterator@$00@12@ABUtagEMERGENCY_NUM_INFO@@@Z 00138554 f i misc.obj
 0001:00037658       ?_Buynode@?$list@UtagEMERGENCY_NUM_INFO@@V?$allocator@UtagEMERGENCY_NUM_INFO@@@std@@@std@@IAAPAU_Node@?$_List_nod@UtagEMERGENCY_NUM_INFO@@V?$allocator@UtagEMERGENCY_NUM_INFO@@@std@@@2@XZ 00138658 f i misc.obj
 0001:0003775c       ?_Tidy@?$list@UtagEMERGENCY_NUM_INFO@@V?$allocator@UtagEMERGENCY_NUM_INFO@@@std@@@std@@IAAXXZ 0013875c f i misc.obj
 0001:000377f0       ?_Orphan_ptr@?$list@UtagEMERGENCY_NUM_INFO@@V?$allocator@UtagEMERGENCY_NUM_INFO@@@std@@@std@@IBAXAAV12@PAU_Node@?$_List_nod@UtagEMERGENCY_NUM_INFO@@V?$allocator@UtagEMERGENCY_NUM_INFO@@@std@@@2@@Z 001387f0 f i misc.obj
 0001:000378c4       ??0?$_List_val@UtagEMERGENCY_NUM_INFO@@V?$allocator@UtagEMERGENCY_NUM_INFO@@@std@@@std@@QAA@V?$allocator@UtagEMERGENCY_NUM_INFO@@@1@@Z 001388c4 f i misc.obj
 0001:00037920       ??0?$allocator@UtagEMERGENCY_NUM_INFO@@@std@@QAA@XZ 00138920 f i misc.obj
 0001:00037944       ?deallocate@?$allocator@U_Node@?$_List_nod@UtagEMERGENCY_NUM_INFO@@V?$allocator@UtagEMERGENCY_NUM_INFO@@@std@@@std@@@std@@QAAXPAU_Node@?$_List_nod@UtagEMERGENCY_NUM_INFO@@V?$allocator@UtagEMERGENCY_NUM_INFO@@@std@@@2@I@Z 00138944 f i misc.obj
 0001:0003795c       ?destroy@?$allocator@U_Node@?$_List_nod@UtagEMERGENCY_NUM_INFO@@V?$allocator@UtagEMERGENCY_NUM_INFO@@@std@@@std@@@std@@QAAXPAU_Node@?$_List_nod@UtagEMERGENCY_NUM_INFO@@V?$allocator@UtagEMERGENCY_NUM_INFO@@@std@@@2@@Z 0013895c f i misc.obj
 0001:0003797c       ?_Buynode@?$list@UtagEMERGENCY_NUM_INFO@@V?$allocator@UtagEMERGENCY_NUM_INFO@@@std@@@std@@IAAPAU_Node@?$_List_nod@UtagEMERGENCY_NUM_INFO@@V?$allocator@UtagEMERGENCY_NUM_INFO@@@std@@@2@PAU342@0ABUtagEMERGENCY_NUM_INFO@@@Z 0013897c f i misc.obj
 0001:00037adc       ?_Incsize@?$list@UtagEMERGENCY_NUM_INFO@@V?$allocator@UtagEMERGENCY_NUM_INFO@@@std@@@std@@IAAXI@Z 00138adc f i misc.obj
 0001:00037bac       ??0?$_List_ptr@UtagEMERGENCY_NUM_INFO@@V?$allocator@UtagEMERGENCY_NUM_INFO@@@std@@@std@@IAA@V?$allocator@UtagEMERGENCY_NUM_INFO@@@1@@Z 00138bac f i misc.obj
 0001:00037c08       ??0?$allocator@UtagEMERGENCY_NUM_INFO@@@std@@QAA@ABV01@@Z 00138c08 f i misc.obj
 0001:00037c2c       ?allocate@?$allocator@U_Node@?$_List_nod@UtagEMERGENCY_NUM_INFO@@V?$allocator@UtagEMERGENCY_NUM_INFO@@@std@@@std@@@std@@QAAPAU_Node@?$_List_nod@UtagEMERGENCY_NUM_INFO@@V?$allocator@UtagEMERGENCY_NUM_INFO@@@std@@@2@I@Z 00138c2c f i misc.obj
 0001:00037c60       ?construct@?$allocator@PAU_Node@?$_List_nod@UtagEMERGENCY_NUM_INFO@@V?$allocator@UtagEMERGENCY_NUM_INFO@@@std@@@std@@@std@@QAAXPAPAU_Node@?$_List_nod@UtagEMERGENCY_NUM_INFO@@V?$allocator@UtagEMERGENCY_NUM_INFO@@@std@@@2@ABQAU342@@Z 00138c60 f i misc.obj
 0001:00037c7c       ?destroy@?$allocator@PAU_Node@?$_List_nod@UtagEMERGENCY_NUM_INFO@@V?$allocator@UtagEMERGENCY_NUM_INFO@@@std@@@std@@@std@@QAAXPAPAU_Node@?$_List_nod@UtagEMERGENCY_NUM_INFO@@V?$allocator@UtagEMERGENCY_NUM_INFO@@@std@@@2@@Z 00138c7c f i misc.obj
 0001:00037c94       ?_Mynode@?$_Const_iterator@$00@?$list@UtagEMERGENCY_NUM_INFO@@V?$allocator@UtagEMERGENCY_NUM_INFO@@@std@@@std@@QBAPAU_Node@?$_List_nod@UtagEMERGENCY_NUM_INFO@@V?$allocator@UtagEMERGENCY_NUM_INFO@@@std@@@3@XZ 00138c94 f i misc.obj
 0001:00037cc0       ?max_size@?$list@UtagEMERGENCY_NUM_INFO@@V?$allocator@UtagEMERGENCY_NUM_INFO@@@std@@@std@@QBAIXZ 00138cc0 f i misc.obj
 0001:00037cf4       ??0?$_List_nod@UtagEMERGENCY_NUM_INFO@@V?$allocator@UtagEMERGENCY_NUM_INFO@@@std@@@std@@IAA@V?$allocator@UtagEMERGENCY_NUM_INFO@@@1@@Z 00138cf4 f i misc.obj
 0001:00037d34       ?construct@?$allocator@UtagEMERGENCY_NUM_INFO@@@std@@QAAXPAUtagEMERGENCY_NUM_INFO@@ABU3@@Z 00138d34 f i misc.obj
 0001:00037d50       ?max_size@?$allocator@UtagEMERGENCY_NUM_INFO@@@std@@QBAIXZ 00138d50 f i misc.obj
 0001:00037da8       ??$sort@P6A_NABUtagEMERGENCY_NUM_INFO@@0@Z@?$list@UtagEMERGENCY_NUM_INFO@@V?$allocator@UtagEMERGENCY_NUM_INFO@@@std@@@std@@QAAXP6A_NABUtagEMERGENCY_NUM_INFO@@0@Z@Z 00138da8 f i misc.obj
 0001:00038164       ??$merge@P6A_NABUtagEMERGENCY_NUM_INFO@@0@Z@?$list@UtagEMERGENCY_NUM_INFO@@V?$allocator@UtagEMERGENCY_NUM_INFO@@@std@@@std@@QAAXAAV01@P6A_NABUtagEMERGENCY_NUM_INFO@@1@Z@Z 00139164 f i misc.obj
 0001:00038614       ??$unique@P6A_NABUtagEMERGENCY_NUM_INFO@@0@Z@?$list@UtagEMERGENCY_NUM_INFO@@V?$allocator@UtagEMERGENCY_NUM_INFO@@@std@@@std@@QAAXP6A_NABUtagEMERGENCY_NUM_INFO@@0@Z@Z 00139614 f i misc.obj
 0001:000387fc       ??$_Destroy@U_Node@?$_List_nod@UtagEMERGENCY_NUM_INFO@@V?$allocator@UtagEMERGENCY_NUM_INFO@@@std@@@std@@@std@@YAXPAU_Node@?$_List_nod@UtagEMERGENCY_NUM_INFO@@V?$allocator@UtagEMERGENCY_NUM_INFO@@@std@@@0@@Z 001397fc f i misc.obj
 0001:0003880c       ??$?0UtagEMERGENCY_NUM_INFO@@@?$allocator@PAU_Node@?$_List_nod@UtagEMERGENCY_NUM_INFO@@V?$allocator@UtagEMERGENCY_NUM_INFO@@@std@@@std@@@std@@QAA@ABV?$allocator@UtagEMERGENCY_NUM_INFO@@@1@@Z 0013980c f i misc.obj
 0001:00038830       ??$_Allocate@U_Node@?$_List_nod@UtagEMERGENCY_NUM_INFO@@V?$allocator@UtagEMERGENCY_NUM_INFO@@@std@@@std@@@std@@YAPAU_Node@?$_List_nod@UtagEMERGENCY_NUM_INFO@@V?$allocator@UtagEMERGENCY_NUM_INFO@@@std@@@0@IPAU120@@Z 00139830 f i misc.obj
 0001:000388c0       ??$_Construct@PAU_Node@?$_List_nod@UtagEMERGENCY_NUM_INFO@@V?$allocator@UtagEMERGENCY_NUM_INFO@@@std@@@std@@PAU123@@std@@YAXPAPAU_Node@?$_List_nod@UtagEMERGENCY_NUM_INFO@@V?$allocator@UtagEMERGENCY_NUM_INFO@@@std@@@0@ABQAU120@@Z 001398c0 f i misc.obj
 0001:00038928       ??$_Destroy@PAU_Node@?$_List_nod@UtagEMERGENCY_NUM_INFO@@V?$allocator@UtagEMERGENCY_NUM_INFO@@@std@@@std@@@std@@YAXPAPAU_Node@?$_List_nod@UtagEMERGENCY_NUM_INFO@@V?$allocator@UtagEMERGENCY_NUM_INFO@@@std@@@0@@Z 00139928 f i misc.obj
 0001:00038938       ??$?0UtagEMERGENCY_NUM_INFO@@@?$allocator@U_Node@?$_List_nod@UtagEMERGENCY_NUM_INFO@@V?$allocator@UtagEMERGENCY_NUM_INFO@@@std@@@std@@@std@@QAA@ABV?$allocator@UtagEMERGENCY_NUM_INFO@@@1@@Z 00139938 f i misc.obj
 0001:0003895c       ??$_Construct@UtagEMERGENCY_NUM_INFO@@U1@@std@@YAXPAUtagEMERGENCY_NUM_INFO@@ABU1@@Z 0013995c f i misc.obj
 0001:000389c4       ??0?$_Iterator@$00@?$list@UtagEMERGENCY_NUM_INFO@@V?$allocator@UtagEMERGENCY_NUM_INFO@@@std@@@std@@QAA@ABV012@@Z 001399c4 f i misc.obj
 0001:000389f8       ??0?$_Const_iterator@$00@?$list@UtagEMERGENCY_NUM_INFO@@V?$allocator@UtagEMERGENCY_NUM_INFO@@@std@@@std@@QAA@ABV012@@Z 001399f8 f i misc.obj
 0001:00038a44       ??0?$_Bidit@UtagEMERGENCY_NUM_INFO@@HPBU1@ABU1@@std@@QAA@ABU01@@Z 00139a44 f i misc.obj
 0001:00038a80       ??0?$list@UtagEMERGENCY_NUM_INFO@@V?$allocator@UtagEMERGENCY_NUM_INFO@@@std@@@std@@QAA@ABV?$allocator@UtagEMERGENCY_NUM_INFO@@@1@@Z 00139a80 f i misc.obj
 0001:00038b14       ?empty@?$list@UtagEMERGENCY_NUM_INFO@@V?$allocator@UtagEMERGENCY_NUM_INFO@@@std@@@std@@QBA_NXZ 00139b14 f i misc.obj
 0001:00038b6c       ?erase@?$list@UtagEMERGENCY_NUM_INFO@@V?$allocator@UtagEMERGENCY_NUM_INFO@@@std@@@std@@QAA?AV?$_Iterator@$00@12@V312@@Z 00139b6c f i misc.obj
 0001:00038d88       ?swap@?$list@UtagEMERGENCY_NUM_INFO@@V?$allocator@UtagEMERGENCY_NUM_INFO@@@std@@@std@@QAAXAAV12@@Z 00139d88 f i misc.obj
 0001:00038f24       ?_Swap_all@_Container_base@std@@QBAXAAV12@@Z 00139f24 f i misc.obj
 0001:0003901c       ?splice@?$list@UtagEMERGENCY_NUM_INFO@@V?$allocator@UtagEMERGENCY_NUM_INFO@@@std@@@std@@QAAXV?$_Iterator@$00@12@AAV12@@Z 0013a01c f i misc.obj
 0001:00039164       ?_Splice@?$list@UtagEMERGENCY_NUM_INFO@@V?$allocator@UtagEMERGENCY_NUM_INFO@@@std@@@std@@QAAXV?$_Iterator@$00@12@AAV12@00I_N@Z 0013a164 f i misc.obj
 0001:000395e0       ??E?$_Iterator@$00@?$list@UtagEMERGENCY_NUM_INFO@@V?$allocator@UtagEMERGENCY_NUM_INFO@@@std@@@std@@QAA?AV012@H@Z 0013a5e0 f i misc.obj
 0001:000396a0       ?erase@?$list@UtagEMERGENCY_NUM_INFO@@V?$allocator@UtagEMERGENCY_NUM_INFO@@@std@@@std@@QAA?AV?$_Iterator@$00@12@V312@0@Z 0013a6a0 f i misc.obj
 0001:000399a4       ?splice@?$list@UtagEMERGENCY_NUM_INFO@@V?$allocator@UtagEMERGENCY_NUM_INFO@@@std@@@std@@QAAXV?$_Iterator@$00@12@AAV12@00@Z 0013a9a4 f i misc.obj
 0001:00039d68       ??$_Debug_order@V?$_Iterator@$00@?$list@UtagEMERGENCY_NUM_INFO@@V?$allocator@UtagEMERGENCY_NUM_INFO@@@std@@@std@@P6A_NABUtagEMERGENCY_NUM_INFO@@0@Z@std@@YAXV?$_Iterator@$00@?$list@UtagEMERGENCY_NUM_INFO@@V?$allocator@UtagEMERGENCY_NUM_INFO@@@std@@@0@0P6A_NABUtagEMERGENCY_NUM_INFO@@1@ZPBGI@Z 0013ad68 f i misc.obj
 0001:00039ef0       ??$_Debug_lt_pred@P6A_NABUtagEMERGENCY_NUM_INFO@@0@ZU1@U1@@std@@YA_NP6A_NABUtagEMERGENCY_NUM_INFO@@0@ZAAU1@2PBGI@Z 0013aef0 f i misc.obj
 0001:00039f80       ??$?8UtagEMERGENCY_NUM_INFO@@U0@@std@@YA_NABV?$allocator@UtagEMERGENCY_NUM_INFO@@@0@0@Z 0013af80 f i misc.obj
 0001:00039fa4       ??$swap@PAU_Node@?$_List_nod@UtagEMERGENCY_NUM_INFO@@V?$allocator@UtagEMERGENCY_NUM_INFO@@@std@@@std@@@std@@YAXAAPAU_Node@?$_List_nod@UtagEMERGENCY_NUM_INFO@@V?$allocator@UtagEMERGENCY_NUM_INFO@@@std@@@0@0@Z 0013afa4 f i misc.obj
 0001:00039fe4       ??$swap@I@std@@YAXAAI0@Z   0013afe4 f i misc.obj
 0001:0003a02c       ??$insert@V?$_Iterator@$00@?$list@UtagEMERGENCY_NUM_INFO@@V?$allocator@UtagEMERGENCY_NUM_INFO@@@std@@@std@@@?$list@UtagEMERGENCY_NUM_INFO@@V?$allocator@UtagEMERGENCY_NUM_INFO@@@std@@@std@@QAAXV?$_Iterator@$00@01@00@Z 0013b02c f i misc.obj
 0001:0003a198       ??$_Distance@V?$_Iterator@$00@?$list@UtagEMERGENCY_NUM_INFO@@V?$allocator@UtagEMERGENCY_NUM_INFO@@@std@@@std@@I@std@@YAXV?$_Iterator@$00@?$list@UtagEMERGENCY_NUM_INFO@@V?$allocator@UtagEMERGENCY_NUM_INFO@@@std@@@0@0AAI@Z 0013b198 f i misc.obj
 0001:0003a284       ??$_Debug_range@V?$_Iterator@$00@?$list@UtagEMERGENCY_NUM_INFO@@V?$allocator@UtagEMERGENCY_NUM_INFO@@@std@@@std@@@std@@YAXV?$_Iterator@$00@?$list@UtagEMERGENCY_NUM_INFO@@V?$allocator@UtagEMERGENCY_NUM_INFO@@@std@@@0@0PBGI@Z 0013b284 f i misc.obj
 0001:0003a380       ??$_Debug_pointer@$$A6A_NABUtagEMERGENCY_NUM_INFO@@0@Z@std@@YAXP6A_NABUtagEMERGENCY_NUM_INFO@@0@ZPBGI@Z 0013b380 f i misc.obj
 0001:0003a3b0       ??$_Iter_cat@V?$_Iterator@$00@?$list@UtagEMERGENCY_NUM_INFO@@V?$allocator@UtagEMERGENCY_NUM_INFO@@@std@@@std@@@std@@YA?AUbidirectional_iterator_tag@0@ABV?$_Iterator@$00@?$list@UtagEMERGENCY_NUM_INFO@@V?$allocator@UtagEMERGENCY_NUM_INFO@@@std@@@0@@Z 0013b3b0 f i misc.obj
 0001:0003a3dc       ??$_Debug_order2@V?$_Iterator@$00@?$list@UtagEMERGENCY_NUM_INFO@@V?$allocator@UtagEMERGENCY_NUM_INFO@@@std@@@std@@P6A_NABUtagEMERGENCY_NUM_INFO@@0@Z@std@@YAXV?$_Iterator@$00@?$list@UtagEMERGENCY_NUM_INFO@@V?$allocator@UtagEMERGENCY_NUM_INFO@@@std@@@0@0P6A_NABUtagEMERGENCY_NUM_INFO@@1@ZPBGIUforward_iterator_tag@0@@Z 0013b3dc f i misc.obj
 0001:0003a53c       ??$_Insert@V?$_Iterator@$00@?$list@UtagEMERGENCY_NUM_INFO@@V?$allocator@UtagEMERGENCY_NUM_INFO@@@std@@@std@@@?$list@UtagEMERGENCY_NUM_INFO@@V?$allocator@UtagEMERGENCY_NUM_INFO@@@std@@@std@@QAAXV?$_Iterator@$00@01@00Uforward_iterator_tag@1@@Z 0013b53c f i misc.obj
 0001:0003a7d4       ??$_Distance2@V?$_Iterator@$00@?$list@UtagEMERGENCY_NUM_INFO@@V?$allocator@UtagEMERGENCY_NUM_INFO@@@std@@@std@@I@std@@YAXV?$_Iterator@$00@?$list@UtagEMERGENCY_NUM_INFO@@V?$allocator@UtagEMERGENCY_NUM_INFO@@@std@@@0@0AAIUbidirectional_iterator_tag@0@@Z 0013b7d4 f i misc.obj
 0001:0003a870       ??F?$_Iterator@$00@?$list@UtagEMERGENCY_NUM_INFO@@V?$allocator@UtagEMERGENCY_NUM_INFO@@@std@@@std@@QAAAAV012@XZ 0013b870 f i misc.obj
 0001:0003a89c       ??F?$_Const_iterator@$00@?$list@UtagEMERGENCY_NUM_INFO@@V?$allocator@UtagEMERGENCY_NUM_INFO@@@std@@@std@@QAAAAV012@XZ 0013b89c f i misc.obj
 0001:0003a9a0       ??$_Debug_range2@V?$_Iterator@$00@?$list@UtagEMERGENCY_NUM_INFO@@V?$allocator@UtagEMERGENCY_NUM_INFO@@@std@@@std@@@std@@YAXV?$_Iterator@$00@?$list@UtagEMERGENCY_NUM_INFO@@V?$allocator@UtagEMERGENCY_NUM_INFO@@@std@@@0@0PBGIUinput_iterator_tag@0@@Z 0013b9a0 f i misc.obj
 0001:0003a9e0       ??$_Debug_get_cont@V?$_Iterator@$00@?$list@UtagEMERGENCY_NUM_INFO@@V?$allocator@UtagEMERGENCY_NUM_INFO@@@std@@@std@@@std@@YAPBV_Container_base@0@ABV?$_Iterator@$00@?$list@UtagEMERGENCY_NUM_INFO@@V?$allocator@UtagEMERGENCY_NUM_INFO@@@std@@@0@@Z 0013b9e0 f i misc.obj
 0001:0003aa04       ?MonitorThreadProc@@YAKPAX@Z 0013ba04 f   monitor.obj
 0001:0003abfc       ??0CMonitor@@QAA@XZ        0013bbfc f   monitor.obj
 0001:0003ac8c       ??1CMonitor@@QAA@XZ        0013bc8c f   monitor.obj
 0001:0003add8       ?Init@CMonitor@@QAAHQAXKK@Z 0013bdd8 f   monitor.obj
 0001:0003b218       ??_GCCheckPoint@@QAAPAXI@Z 0013c218 f i monitor.obj
 0001:0003b260       ?Hex2Dec@@YAGE@Z           0013c260 f   msg.obj
 0001:0003b2d0       ?ValidateMsgDCS@@YAJABUrilmsgdcs_tag@@@Z 0013c2d0 f   msg.obj
 0001:0003b570       ?ValidateMsgValidityPeriod@@YAJABU_SYSTEMTIME@@K@Z 0013c570 f   msg.obj
 0001:0003b61c       ?ValidateMsgAddress@@YAJABUriladdress_tag@@@Z 0013c61c f   msg.obj
 0001:0003b754       ?ValidateMsgProtocolID@@YAJK@Z 0013c754 f   msg.obj
 0001:0003b7dc       ?ValidateMsgDlvStatus@@YAJK@Z 0013c7dc f   msg.obj
 0001:0003b864       ?ValidateSubmitMsg@@YAJABUrilmessage_tag@@@Z 0013c864 f   msg.obj
 0001:0003ba80       ?ValidateIS637SubmitMsg@@YAJABUrilmessage_tag@@@Z 0013ca80 f   msg.obj
 0001:0003bb24       ?ValidateCmdMsg@@YAJABUrilmessage_tag@@@Z 0013cb24 f   msg.obj
 0001:0003bce0       ?ValidateDeliverMsg@@YAJABUrilmessage_tag@@@Z 0013cce0 f   msg.obj
 0001:0003be68       ?ValidateStatusMsg@@YAJABUrilmessage_tag@@@Z 0013ce68 f   msg.obj
 0001:0003c060       ?ValidateRawMsg@@YAJABUrilmessage_tag@@@Z 0013d060 f   msg.obj
 0001:0003c104       ?ValidateMessage@@YAJABUrilmessage_tag@@@Z 0013d104 f   msg.obj
 0001:0003c2dc       ?RILDrv_GetMsgServiceOptions@@YAJK@Z 0013d2dc f   msg.obj
 0001:0003c3c8       ?RILDrv_SetMsgServiceOptions@@YAJKPBUrilmsgserviceinfo_tag@@@Z 0013d3c8 f   msg.obj
 0001:0003c96c       ?RILDrv_GetMsgConfig@@YAJK@Z 0013d96c f   msg.obj
 0001:0003ca50       ?RILDrv_SetMsgConfig@@YAJKPBUrilmsgconfig_tag@@@Z 0013da50 f   msg.obj
 0001:0003cc40       ?RILDrv_GetCellBroadcastMsgConfig@@YAJK@Z 0013dc40 f   msg.obj
 0001:0003cd20       ?RILDrv_SetCellBroadcastMsgConfig@@YAJKPBUrilcbmsgconfig_tag@@@Z 0013dd20 f   msg.obj
 0001:0003cea4       ?RILDrv_ReadMsg@@YAJKK@Z   0013dea4 f   msg.obj
 0001:0003cf94       ?RILDrv_DeleteMsg@@YAJKK@Z 0013df94 f   msg.obj
 0001:0003d1c4       ?RILDrv_SendMsg@@YAJKPBUrilmessage_tag@@K@Z 0013e1c4 f   msg.obj
 0001:0003d444       ?RILDrv_SendStoredMsg@@YAJKKK@Z 0013e444 f   msg.obj
 0001:0003d530       ?RILDrv_SendMsgAcknowledgement@@YAJKH@Z 0013e530 f   msg.obj
 0001:0003d614       ?MsgReceiveThreadProc@@YAKPAX@Z 0013e614 f   msg.obj
 0001:0003d7ac       ?MsgSendThreadProc@@YAKPAX@Z 0013e7ac f   msg.obj
 0001:0003d99c       ?MsgReceiveOnNotifyThreadProcGsm@@YAKPAX@Z 0013e99c f   msg.obj
 0001:0003e958       ?MsgReceiveOnNotifyThreadProc@@YAKPAX@Z 0013f958 f   msg.obj
 0001:0003fa54       ?SendMsg@CRadio@@QAAJPAVCResponse@@PAX@Z 00140a54 f   msg.obj
 0001:00041bcc       ?GenerateMsgRefNum@CRadio@@QAAKXZ 00142bcc f   msg.obj
 0001:00041c00       ?UpdateAndBroadcastOnSWISMSNotification@CRadio@@QAAXPAUSwiNotifyVariant@@@Z 00142c00 f   msg.obj
 0001:000423b8       ?ReceiveMsg@CRadio@@QAAXPAUrilmessage_tag@@@Z 001433b8 f   msg.obj
 0001:00042b4c       ?DivertMsg@CRadio@@QAAJPAUrilmessage_tag@@K@Z 00143b4c f   msg.obj
 0001:0004437c       ?isLocalMsg@CRadio@@QAAHPAUrilmessage_tag@@@Z 0014537c f   msg.obj
 0001:00044524       ?CompareAddresses@CRadio@@QAAHPBUriladdress_tag@@0@Z 00145524 f   msg.obj
 0001:00044638       ?GetMsgServiceOptions@CRadio@@QAAJPAVCResponse@@@Z 00145638 f   msg.obj
 0001:0004475c       ?GetMsgConfig@CRadio@@QAAJPAVCResponse@@@Z 0014575c f   msg.obj
 0001:00044a94       ?SetMsgConfig@CRadio@@QAAJPAVCResponse@@PAX@Z 00145a94 f   msg.obj
 0001:00044cc4       ?GetCellBroadcastMsgConfig@CRadio@@QAAJPAVCResponse@@@Z 00145cc4 f   msg.obj
 0001:00044da4       ?SetCellBroadcastMsgConfig@CRadio@@QAAJPAVCResponse@@PAX@Z 00145da4 f   msg.obj
 0001:00044f68       ?SmsMtSetRilAddressNumberType@CRadio@@QAAKE@Z 00145f68 f   msg.obj
 0001:0004504c       ?SmsMtSetRilAddressNumberPlan@CRadio@@QAAKE@Z 0014604c f   msg.obj
 0001:0004512c       ?CovertNumberToBCD@CRadio@@QAAEG@Z 0014612c f   msg.obj
 0001:0004519c       ?IsEmailAddr@CRadio@@IAAHPAG@Z 0014619c f   msg.obj
 0001:000452c4       ?InitSMSSendHdr@CRadio@@QAAXPAUSWI_STRUCT_SMS_CdmaHeader@@@Z 001462c4 f   msg.obj
 0001:00045474       ?RILDrv_WriteMsg@@YAJKPBUrilmessage_tag@@K@Z 00146474 f   msg.obj
 0001:00045538       ??0SWISYNCBLOCK@@QAA@PAVCriticalSection@@@Z 00146538 f i msg.obj
 0001:00045574       ??1SWISYNCBLOCK@@QAA@XZ    00146574 f i msg.obj
 0001:00045590       ?MakeDelayRsp@CResponse@@QAAXXZ 00146590 f i msg.obj
 0001:000455b0       ?MemRealloc@@YAPAXPAXII@Z  001465b0 f i msg.obj
 0001:0004567c       ??0CriticalSection@@QAA@XZ 0014667c f i msg.obj
 0001:000456bc       ??_GCriticalSection@@UAAPAXI@Z 001466bc f i msg.obj
 0001:000456bc       ??_ECriticalSection@@UAAPAXI@Z 001466bc f i msg.obj
 0001:000456fc       ??1CriticalSection@@UAA@XZ 001466fc f i msg.obj
 0001:00045728       ?RILDrv_GetSubscriberNumbers@@YAJK@Z 00146728 f   network.obj
 0001:00045808       ?RILDrv_GetCurrentOperator@@YAJKK@Z 00146808 f   network.obj
 0001:000458e8       ?RILDrv_GetOperatorList@@YAJK@Z 001468e8 f   network.obj
 0001:000459c8       ?RILDrv_GetRegistrationStatus@@YAJK@Z 001469c8 f   network.obj
 0001:00045aa8       ?RILDrv_GetCurrentSystemType@@YAJK@Z 00146aa8 f   network.obj
 0001:00045b88       ?RILDrv_GetRoamingMode@@YAJK@Z 00146b88 f   network.obj
 0001:00045c68       ?RILDrv_SetRoamingMode@@YAJKK@Z 00146c68 f   network.obj
 0001:00045d48       ?RILDrv_GetPreferredPrivacyMode@@YAJK@Z 00146d48 f   network.obj
 0001:00045e28       ?RILDrv_SetPreferredPrivacyMode@@YAJKK@Z 00146e28 f   network.obj
 0001:00045f14       ?GetSubscriberNumbers@CRadio@@QAAJPAVCResponse@@@Z 00146f14 f   network.obj
 0001:00046068       ?GetCurrentOperator@CRadio@@QAAJPAVCResponse@@@Z 00147068 f   network.obj
 0001:00046230       ?AddPreferredOperator@CRadio@@QAAJPAVCResponse@@PAX@Z 00147230 f   network.obj
 0001:00046574       ?RemovePreferredOperator@CRadio@@QAAJPAVCResponse@@PAX@Z 00147574 f   network.obj
 0001:00046758       ?GetPreferredOperatorList@CRadio@@QAAJPAVCResponse@@PAX@Z 00147758 f   network.obj
 0001:00047308       ?GetOperatorList@CRadio@@QAAJPAVCResponse@@@Z 00148308 f   network.obj
 0001:00047598       ?UnRegisterFromNetwork@CRadio@@QAAJPAVCResponse@@@Z 00148598 f   network.obj
 0001:0004775c       ?RegisterOnNetwork@CRadio@@QAAJPAVCResponse@@PAX@Z 0014875c f   network.obj
 0001:00048244       ?UpdateEVDONetworkType@CRadio@@QAAXK@Z 00149244 f   network.obj
 0001:00048318       ?GetRegistrationStatus@CRadio@@QAAJPAVCResponse@@@Z 00149318 f   network.obj
 0001:000484f4       ?SetRegistrationStatus@CRadio@@QAAXK@Z 001494f4 f   network.obj
 0001:00048584       ?GetCurrentSystemType@CRadio@@QAAJPAVCResponse@@@Z 00149584 f   network.obj
 0001:0004878c       ?GetRoamingMode@CRadio@@QAAJPAVCResponse@@@Z 0014978c f   network.obj
 0001:00048978       ?SetRoamingMode@CRadio@@QAAJPAVCResponse@@PAX@Z 00149978 f   network.obj
 0001:00048c5c       ?GetPreferredPrivacyMode@CRadio@@QAAJPAVCResponse@@@Z 00149c5c f   network.obj
 0001:00048cd8       ?SetPreferredPrivacyMode@CRadio@@QAAJPAVCResponse@@PAX@Z 00149cd8 f   network.obj
 0001:00048d54       ?SetHomeAndCurrentOperator@CRadio@@QAAXK@Z 00149d54 f   network.obj
 0001:000490b4       ?RILDrv_RegisterOnNetwork@@YAJKKPBUriloperatornames_tag@@@Z 0014a0b4 f   network.obj
 0001:000491f0       ?RILDrv_GetPreferredOperatorList@@YAJKK@Z 0014a1f0 f   network.obj
 0001:00049290       ?RILDrv_AddPreferredOperator@@YAJKKPBUriloperatornames_tag@@@Z 0014a290 f   network.obj
 0001:00049404       ?RILDrv_RemovePreferredOperator@@YAJKK@Z 0014a404 f   network.obj
 0001:000494ac       ?GetAllOperatorsList@CRadio@@QAAJPAVCResponse@@@Z 0014a4ac f   network.obj
 0001:00049718       ?RILDrv_GetAllOperatorsList@@YAJK@Z 0014a718 f   network.obj
 0001:000497b8       ?RILDrv_UnregisterFromNetwork@@YAJK@Z 0014a7b8 f   network.obj
 0001:000498a0       ?CheckCurrentRUIM@CRadio@@QAAHXZ 0014a8a0 f   network.obj
 0001:000499bc       GetCurrentThreadId         0014a9bc f i network.obj
 0001:000499dc       ?DataDormancyPollingThreadProc@@YAKPAX@Z 0014a9dc f   Radio.obj
 0001:00049a10       ?ConvertToRILSystem@CRadio@@QAAKK@Z 0014aa10 f   Radio.obj
 0001:00049b84       ??0CRadio@@QAA@PAVCRilHandle@@@Z 0014ab84 f   Radio.obj
 0001:0004a1dc       ??1CRadio@@QAA@XZ          0014b1dc f   Radio.obj
 0001:0004a404       ?LoadSwiAux@CRadio@@QAAXXZ 0014b404 f   Radio.obj
 0001:0004abe0       ?UnloadSwiAux@CRadio@@QAAXXZ 0014bbe0 f   Radio.obj
 0001:0004ad08       ?Init@CRadio@@QAAJXZ       0014bd08 f   Radio.obj
 0001:0004b360       ?GetUserNetworkPreference@CRadio@@QAAHXZ 0014c360 f   Radio.obj
 0001:0004b3e8       ?GetRuimLockStatus@CRadio@@QAAKXZ 0014c3e8 f   Radio.obj
 0001:0004b8dc       ?UpdateUserNetworkPreference@CRadio@@QAAXH@Z 0014c8dc f   Radio.obj
 0001:0004b96c       ?SetSwiWirelessTech@CRadio@@QAAXK@Z 0014c96c f   Radio.obj
 0001:0004bae0       ?ExecuteCommand@CRadio@@QAAJPAVCCommand@@PAVCResponse@@@Z 0014cae0 f   Radio.obj
 0001:0004c9b0       ?PreExecCmd@CRadio@@QAAJPAVCCommand@@PAVCResponse@@@Z 0014d9b0 f   Radio.obj
 0001:0004cc6c       ?LaunchWapIOTA@CRadio@@QAAXG@Z 0014dc6c f   Radio.obj
 0001:0004cde8       ?ReceiveNotification@CRadio@@QAAXKPAXI@Z 0014dde8 f   Radio.obj
 0001:0004ce1c       ?UpdateCombinedServiceStatus@CRadio@@QAAHKK@Z 0014de1c f   Radio.obj
 0001:0004da28       ?SendDelayedNITZThreadProc@@YAKPAX@Z 0014ea28 f   Radio.obj
 0001:0004dc28       ?UpdateAndBroadcastOnSWINotification@CRadio@@QAAXPAUSwiNotifyVariant@@@Z 0014ec28 f   Radio.obj
 0001:00051ab0       ?SWIEventCallback@@YAXPAUSwiNotifyVariant@@@Z 00152ab0 f   Radio.obj
 0001:00051b44       ?GetDataDialCmd@CRadio@@QAAPAVCCommand@@XZ 00152b44 f   Radio.obj
 0001:00051d3c       ?Wait4ATConnect@CRadio@@QAAXXZ 00152d3c f   Radio.obj
 0001:00052910       ?DataDormancyPollingThread@CRadio@@QAAXXZ 00153910 f   Radio.obj
 0001:00052c38       ?OnIdle@CRadio@@QAAXXZ     00153c38 f   Radio.obj
 0001:00052e00       ?DecBasedOrder@@YAKK@Z     00153e00 f   Radio.obj
 0001:00052e68       ?HandleRssi@CRadio@@QAAXH@Z 00153e68 f   Radio.obj
 0001:00052fe8       ?HandleGsmSystemStatus@CRadio@@QAAXPAUSWI_STRUCT_GsmSystemStatus@@@Z 00153fe8 f   Radio.obj
 0001:00053ae0       ?UpdateSIMStatus@CRadio@@QAAXK@Z 00154ae0 f   Radio.obj
 0001:00053b2c       ?GetSIMStatus@CRadio@@QAAKXZ 00154b2c f   Radio.obj
 0001:00053b5c       ?UpdatePhLockedState@CRadio@@QAAXK@Z 00154b5c f   Radio.obj
 0001:00053c18       ?GetPhLockedState@CRadio@@QAAKXZ 00154c18 f   Radio.obj
 0001:00053c50       ?GetPhoneBookEntry@CRadio@@QAAHXZ 00154c50 f   Radio.obj
 0001:000541c0       ?UpdateMDNNumber@CRadio@@QAAHXZ 001551c0 f   Radio.obj
 0001:00054554       ?InitializeRadioStateMachine@CRadio@@QAAXH@Z 00155554 f   Radio.obj
 0001:000554ac       ?BroadcastMinActiveStateNotification@CRadio@@QAAXXZ 001564ac f   Radio.obj
 0001:000554fc       ?BroadcastEquipmentStateNotification@CRadio@@QAAXKK@Z 001564fc f   Radio.obj
 0001:000555c8       ?InitializeEmergencyList@CRadio@@AAAXXZ 001565c8 f   Radio.obj
 0001:00055b70       ?UpdateEmergencyRegistry@CRadio@@AAAXXZ 00156b70 f   Radio.obj
 0001:0005610c       ?ResetCallState@CRadio@@AAAXXZ 0015710c f   Radio.obj
 0001:000562d4       ?RIL_CALLSTAT_2_STR@@YAPAGK@Z 001572d4 f   Radio.obj
 0001:00056310       ??1?$map@KU__Fail_Cmd_Data_tag@@U?$less@K@std@@V?$allocator@U?$pair@$$CBKU__Fail_Cmd_Data_tag@@@std@@@3@@std@@QAA@XZ 00157310 f i Radio.obj
 0001:00056328       ??1?$map@KKU?$less@K@std@@V?$allocator@U?$pair@$$CBKK@std@@@2@@std@@QAA@XZ 00157328 f i Radio.obj
 0001:00056340       ??_GCRadioCaps@@QAAPAXI@Z  00157340 f i Radio.obj
 0001:00056380       ?FInited@CRilHandle@@QBAHXZ 00157380 f i Radio.obj
 0001:000563b4       ?GetpCSWaitingCommands@CRilHandle@@QAAPAUCRITICAL_SECTION@@XZ 001573b4 f i Radio.obj
 0001:000563dc       ??4?$_Iterator@$00@?$list@PAVCCommand@@V?$allocator@PAVCCommand@@@std@@@std@@QAAAAV012@ABV012@@Z 001573dc f i Radio.obj
 0001:0005640c       ??4?$_Const_iterator@$00@?$list@PAVCCommand@@V?$allocator@PAVCCommand@@@std@@@std@@QAAAAV012@ABV012@@Z 0015740c f i Radio.obj
 0001:00056454       ??4?$_Bidit@PAVCCommand@@HPBQAV1@ABQAV1@@std@@QAAAAU01@ABU01@@Z 00157454 f i Radio.obj
 0001:00056484       ??0?$map@KU__Fail_Cmd_Data_tag@@U?$less@K@std@@V?$allocator@U?$pair@$$CBKU__Fail_Cmd_Data_tag@@@std@@@3@@std@@QAA@XZ 00157484 f i Radio.obj
 0001:000564d0       ??1?$_Tree@V?$_Tmap_traits@KU__Fail_Cmd_Data_tag@@U?$less@K@std@@V?$allocator@U?$pair@$$CBKU__Fail_Cmd_Data_tag@@@std@@@3@$0A@@std@@@std@@QAA@XZ 001574d0 f i Radio.obj
 0001:00056510       ??0?$map@KKU?$less@K@std@@V?$allocator@U?$pair@$$CBKK@std@@@2@@std@@QAA@XZ 00157510 f i Radio.obj
 0001:0005655c       ??A?$map@KKU?$less@K@std@@V?$allocator@U?$pair@$$CBKK@std@@@2@@std@@QAAAAKABK@Z 0015755c f i Radio.obj
 0001:00056768       ??1?$_Tree@V?$_Tmap_traits@KKU?$less@K@std@@V?$allocator@U?$pair@$$CBKK@std@@@2@$0A@@std@@@std@@QAA@XZ 00157768 f i Radio.obj
 0001:000567a8       ?begin@?$list@PAVCCommand@@V?$allocator@PAVCCommand@@@std@@@std@@QAA?AV?$_Iterator@$00@12@XZ 001577a8 f i Radio.obj
 0001:00056814       ?remove@?$list@PAVCCommand@@V?$allocator@PAVCCommand@@@std@@@std@@QAAXABQAVCCommand@@@Z 00157814 f i Radio.obj
 0001:00056948       ??0?$_Iterator@$00@?$list@PAVCCommand@@V?$allocator@PAVCCommand@@@std@@@std@@QAA@XZ 00157948 f i Radio.obj
 0001:00056978       ??D?$_Iterator@$00@?$list@PAVCCommand@@V?$allocator@PAVCCommand@@@std@@@std@@QBAAAPAVCCommand@@XZ 00157978 f i Radio.obj
 0001:000569a8       ??E?$_Iterator@$00@?$list@PAVCCommand@@V?$allocator@PAVCCommand@@@std@@@std@@QAAAAV012@XZ 001579a8 f i Radio.obj
 0001:000569d4       ??8?$_Const_iterator@$00@?$list@PAVCCommand@@V?$allocator@PAVCCommand@@@std@@@std@@QBA_NABV012@@Z 001579d4 f i Radio.obj
 0001:00056a3c       ??9?$_Const_iterator@$00@?$list@PAVCCommand@@V?$allocator@PAVCCommand@@@std@@@std@@QBA_NABV012@@Z 00157a3c f i Radio.obj
 0001:00056a94       ??1?$_Tree_val@V?$_Tmap_traits@KU__Fail_Cmd_Data_tag@@U?$less@K@std@@V?$allocator@U?$pair@$$CBKU__Fail_Cmd_Data_tag@@@std@@@3@$0A@@std@@@std@@QAA@XZ 00157a94 f i Radio.obj
 0001:00056aac       ??1iterator@?$_Tree@V?$_Tmap_traits@KKU?$less@K@std@@V?$allocator@U?$pair@$$CBKK@std@@@2@$0A@@std@@@std@@QAA@XZ 00157aac f i Radio.obj
 0001:00056ac4       ??0iterator@?$_Tree@V?$_Tmap_traits@KKU?$less@K@std@@V?$allocator@U?$pair@$$CBKK@std@@@2@$0A@@std@@@std@@QAA@ABV012@@Z 00157ac4 f i Radio.obj
 0001:00056af8       ??4iterator@?$_Tree@V?$_Tmap_traits@KKU?$less@K@std@@V?$allocator@U?$pair@$$CBKK@std@@@2@$0A@@std@@@std@@QAAAAV012@ABV012@@Z 00157af8 f i Radio.obj
 0001:00056b28       ??1?$_Tree_val@V?$_Tmap_traits@KKU?$less@K@std@@V?$allocator@U?$pair@$$CBKK@std@@@2@$0A@@std@@@std@@QAA@XZ 00157b28 f i Radio.obj
 0001:00056b40       ??0?$_Iterator@$00@?$list@PAVCCommand@@V?$allocator@PAVCCommand@@@std@@@std@@QAA@ABV012@@Z 00157b40 f i Radio.obj
 0001:00056b74       ??1?$_Tree_ptr@V?$_Tmap_traits@KU__Fail_Cmd_Data_tag@@U?$less@K@std@@V?$allocator@U?$pair@$$CBKU__Fail_Cmd_Data_tag@@@std@@@3@$0A@@std@@@std@@QAA@XZ 00157b74 f i Radio.obj
 0001:00056b8c       ??1const_iterator@?$_Tree@V?$_Tmap_traits@KKU?$less@K@std@@V?$allocator@U?$pair@$$CBKK@std@@@2@$0A@@std@@@std@@QAA@XZ 00157b8c f i Radio.obj
 0001:00056ba4       ??0const_iterator@?$_Tree@V?$_Tmap_traits@KKU?$less@K@std@@V?$allocator@U?$pair@$$CBKK@std@@@2@$0A@@std@@@std@@QAA@ABV012@@Z 00157ba4 f i Radio.obj
 0001:00056bf0       ??4const_iterator@?$_Tree@V?$_Tmap_traits@KKU?$less@K@std@@V?$allocator@U?$pair@$$CBKK@std@@@2@$0A@@std@@@std@@QAAAAV012@ABV012@@Z 00157bf0 f i Radio.obj
 0001:00056c38       ??1?$_Tree_ptr@V?$_Tmap_traits@KKU?$less@K@std@@V?$allocator@U?$pair@$$CBKK@std@@@2@$0A@@std@@@std@@QAA@XZ 00157c38 f i Radio.obj
 0001:00056c50       ??0?$_Const_iterator@$00@?$list@PAVCCommand@@V?$allocator@PAVCCommand@@@std@@@std@@QAA@ABV012@@Z 00157c50 f i Radio.obj
 0001:00056c9c       ??1?$_Tree_nod@V?$_Tmap_traits@KU__Fail_Cmd_Data_tag@@U?$less@K@std@@V?$allocator@U?$pair@$$CBKU__Fail_Cmd_Data_tag@@@std@@@3@$0A@@std@@@std@@QAA@XZ 00157c9c f i Radio.obj
 0001:00056cb4       ??1?$_Bidit@U?$pair@$$CBKK@std@@HPBU12@ABU12@@std@@QAA@XZ 00157cb4 f i Radio.obj
 0001:00056ccc       ??0?$_Bidit@U?$pair@$$CBKK@std@@HPBU12@ABU12@@std@@QAA@ABU01@@Z 00157ccc f i Radio.obj
 0001:00056d00       ??4?$_Bidit@U?$pair@$$CBKK@std@@HPBU12@ABU12@@std@@QAAAAU01@ABU01@@Z 00157d00 f i Radio.obj
 0001:00056d30       ??1?$_Tree_nod@V?$_Tmap_traits@KKU?$less@K@std@@V?$allocator@U?$pair@$$CBKK@std@@@2@$0A@@std@@@std@@QAA@XZ 00157d30 f i Radio.obj
 0001:00056d48       ??0?$_Bidit@PAVCCommand@@HPBQAV1@ABQAV1@@std@@QAA@ABU01@@Z 00157d48 f i Radio.obj
 0001:00056d7c       ??1?$_Tmap_traits@KU__Fail_Cmd_Data_tag@@U?$less@K@std@@V?$allocator@U?$pair@$$CBKU__Fail_Cmd_Data_tag@@@std@@@3@$0A@@std@@QAA@XZ 00157d7c f i Radio.obj
 0001:00056d94       ??1?$_Tmap_traits@KKU?$less@K@std@@V?$allocator@U?$pair@$$CBKK@std@@@2@$0A@@std@@QAA@XZ 00157d94 f i Radio.obj
 0001:00056db4       ??0?$_Tree@V?$_Tmap_traits@KU__Fail_Cmd_Data_tag@@U?$less@K@std@@V?$allocator@U?$pair@$$CBKU__Fail_Cmd_Data_tag@@@std@@@3@$0A@@std@@@std@@QAA@ABU?$less@K@1@ABV?$allocator@U?$pair@$$CBKU__Fail_Cmd_Data_tag@@@std@@@1@@Z 00157db4 f i Radio.obj
 0001:00056e30       ?_Tidy@?$_Tree@V?$_Tmap_traits@KU__Fail_Cmd_Data_tag@@U?$less@K@std@@V?$allocator@U?$pair@$$CBKU__Fail_Cmd_Data_tag@@@std@@@3@$0A@@std@@@std@@IAAXXZ 00157e30 f i Radio.obj
 0001:00056f6c       ??1iterator@?$_Tree@V?$_Tmap_traits@KU__Fail_Cmd_Data_tag@@U?$less@K@std@@V?$allocator@U?$pair@$$CBKU__Fail_Cmd_Data_tag@@@std@@@3@$0A@@std@@@std@@QAA@XZ 00157f6c f i Radio.obj
 0001:00056f84       ??1const_iterator@?$_Tree@V?$_Tmap_traits@KU__Fail_Cmd_Data_tag@@U?$less@K@std@@V?$allocator@U?$pair@$$CBKU__Fail_Cmd_Data_tag@@@std@@@3@$0A@@std@@@std@@QAA@XZ 00157f84 f i Radio.obj
 0001:00056f9c       ??1?$_Bidit@U?$pair@$$CBKU__Fail_Cmd_Data_tag@@@std@@HPBU12@ABU12@@std@@QAA@XZ 00157f9c f i Radio.obj
 0001:00056fb4       ?end@?$_Tree@V?$_Tmap_traits@KU__Fail_Cmd_Data_tag@@U?$less@K@std@@V?$allocator@U?$pair@$$CBKU__Fail_Cmd_Data_tag@@@std@@@3@$0A@@std@@@std@@QAA?AViterator@12@XZ 00157fb4 f i Radio.obj
 0001:00057008       ??0?$allocator@U?$pair@$$CBKU__Fail_Cmd_Data_tag@@@std@@@std@@QAA@XZ 00158008 f i Radio.obj
 0001:0005702c       ??R?$less@K@std@@QBA_NABK0@Z 0015802c f i Radio.obj
 0001:00057080       ?_Key@?$_Tree@V?$_Tmap_traits@KKU?$less@K@std@@V?$allocator@U?$pair@$$CBKK@std@@@2@$0A@@std@@@std@@KAABKPAU_Node@?$_Tree_nod@V?$_Tmap_traits@KKU?$less@K@std@@V?$allocator@U?$pair@$$CBKK@std@@@2@$0A@@std@@@2@@Z 00158080 f i Radio.obj
 0001:000570c4       ??0?$_Tree@V?$_Tmap_traits@KKU?$less@K@std@@V?$allocator@U?$pair@$$CBKK@std@@@2@$0A@@std@@@std@@QAA@ABU?$less@K@1@ABV?$allocator@U?$pair@$$CBKK@std@@@1@@Z 001580c4 f i Radio.obj
 0001:00057138       ?end@?$_Tree@V?$_Tmap_traits@KKU?$less@K@std@@V?$allocator@U?$pair@$$CBKK@std@@@2@$0A@@std@@@std@@QAA?AViterator@12@XZ 00158138 f i Radio.obj
 0001:00057194       ?insert@?$_Tree@V?$_Tmap_traits@KKU?$less@K@std@@V?$allocator@U?$pair@$$CBKK@std@@@2@$0A@@std@@@std@@QAA?AViterator@12@V312@ABU?$pair@$$CBKK@2@@Z 00158194 f i Radio.obj
 0001:000580b0       ?lower_bound@?$_Tree@V?$_Tmap_traits@KKU?$less@K@std@@V?$allocator@U?$pair@$$CBKK@std@@@2@$0A@@std@@@std@@QAA?AViterator@12@ABK@Z 001590b0 f i Radio.obj
 0001:00058114       ?_Tidy@?$_Tree@V?$_Tmap_traits@KKU?$less@K@std@@V?$allocator@U?$pair@$$CBKK@std@@@2@$0A@@std@@@std@@IAAXXZ 00159114 f i Radio.obj
 0001:00058250       ??0?$allocator@U?$pair@$$CBKK@std@@@std@@QAA@XZ 00159250 f i Radio.obj
 0001:0005827c       ?erase@?$list@PAVCCommand@@V?$allocator@PAVCCommand@@@std@@@std@@QAA?AV?$_Iterator@$00@12@V312@@Z 0015927c f i Radio.obj
 0001:00058490       ??0?$_Const_iterator@$00@?$list@PAVCCommand@@V?$allocator@PAVCCommand@@@std@@@std@@QAA@XZ 00159490 f i Radio.obj
 0001:000584d0       ??D?$_Const_iterator@$00@?$list@PAVCCommand@@V?$allocator@PAVCCommand@@@std@@@std@@QBAABQAVCCommand@@XZ 001594d0 f i Radio.obj
 0001:000585ac       ??E?$_Const_iterator@$00@?$list@PAVCCommand@@V?$allocator@PAVCCommand@@@std@@@std@@QAAAAV012@XZ 001595ac f i Radio.obj
 0001:0005869c       ?_Compat@?$_Const_iterator@$00@?$list@PAVCCommand@@V?$allocator@PAVCCommand@@@std@@@std@@QBAXABV123@@Z 0015969c f i Radio.obj
 0001:00058758       ??Diterator@?$_Tree@V?$_Tmap_traits@KKU?$less@K@std@@V?$allocator@U?$pair@$$CBKK@std@@@2@$0A@@std@@@std@@QBAAAU?$pair@$$CBKK@2@XZ 00159758 f i Radio.obj
 0001:00058788       ??8const_iterator@?$_Tree@V?$_Tmap_traits@KKU?$less@K@std@@V?$allocator@U?$pair@$$CBKK@std@@@2@$0A@@std@@@std@@QBA_NABV012@@Z 00159788 f i Radio.obj
 0001:00058880       ?_Mynode@const_iterator@?$_Tree@V?$_Tmap_traits@KKU?$less@K@std@@V?$allocator@U?$pair@$$CBKK@std@@@2@$0A@@std@@@std@@QBAPAU_Node@?$_Tree_nod@V?$_Tmap_traits@KKU?$less@K@std@@V?$allocator@U?$pair@$$CBKK@std@@@2@$0A@@std@@@3@XZ 00159880 f i Radio.obj
 0001:000588ac       ??0?$pair@$$CBKK@std@@QAA@ABK0@Z 001598ac f i Radio.obj
 0001:000588f4       ??1?$pair@Viterator@?$_Tree@V?$_Tmap_traits@KKU?$less@K@std@@V?$allocator@U?$pair@$$CBKK@std@@@2@$0A@@std@@@std@@_N@std@@QAA@XZ 001598f4 f i Radio.obj
 0001:0005890c       ?_Left@?$_Tree@V?$_Tmap_traits@KU__Fail_Cmd_Data_tag@@U?$less@K@std@@V?$allocator@U?$pair@$$CBKU__Fail_Cmd_Data_tag@@@std@@@3@$0A@@std@@@std@@KAAAPAU_Node@?$_Tree_nod@V?$_Tmap_traits@KU__Fail_Cmd_Data_tag@@U?$less@K@std@@V?$allocator@U?$pair@$$CBKU__Fail_Cmd_Data_tag@@@std@@@3@$0A@@std@@@2@PAU342@@Z 0015990c f i Radio.obj
 0001:00058930       ?_Parent@?$_Tree@V?$_Tmap_traits@KU__Fail_Cmd_Data_tag@@U?$less@K@std@@V?$allocator@U?$pair@$$CBKU__Fail_Cmd_Data_tag@@@std@@@3@$0A@@std@@@std@@KAAAPAU_Node@?$_Tree_nod@V?$_Tmap_traits@KU__Fail_Cmd_Data_tag@@U?$less@K@std@@V?$allocator@U?$pair@$$CBKU__Fail_Cmd_Data_tag@@@std@@@3@$0A@@std@@@2@PAU342@@Z 00159930 f i Radio.obj
 0001:00058958       ?_Right@?$_Tree@V?$_Tmap_traits@KU__Fail_Cmd_Data_tag@@U?$less@K@std@@V?$allocator@U?$pair@$$CBKU__Fail_Cmd_Data_tag@@@std@@@3@$0A@@std@@@std@@KAAAPAU_Node@?$_Tree_nod@V?$_Tmap_traits@KU__Fail_Cmd_Data_tag@@U?$less@K@std@@V?$allocator@U?$pair@$$CBKU__Fail_Cmd_Data_tag@@@std@@@3@$0A@@std@@@2@PAU342@@Z 00159958 f i Radio.obj
 0001:00058980       ?begin@?$_Tree@V?$_Tmap_traits@KU__Fail_Cmd_Data_tag@@U?$less@K@std@@V?$allocator@U?$pair@$$CBKU__Fail_Cmd_Data_tag@@@std@@@3@$0A@@std@@@std@@QAA?AViterator@12@XZ 00159980 f i Radio.obj
 0001:000589e4       ?erase@?$_Tree@V?$_Tmap_traits@KU__Fail_Cmd_Data_tag@@U?$less@K@std@@V?$allocator@U?$pair@$$CBKU__Fail_Cmd_Data_tag@@@std@@@3@$0A@@std@@@std@@QAA?AViterator@12@V312@0@Z 001599e4 f i Radio.obj
 0001:00058cb8       ??0iterator@?$_Tree@V?$_Tmap_traits@KU__Fail_Cmd_Data_tag@@U?$less@K@std@@V?$allocator@U?$pair@$$CBKU__Fail_Cmd_Data_tag@@@std@@@3@$0A@@std@@@std@@QAA@ABV012@@Z 00159cb8 f i Radio.obj
 0001:00058cec       ??0const_iterator@?$_Tree@V?$_Tmap_traits@KU__Fail_Cmd_Data_tag@@U?$less@K@std@@V?$allocator@U?$pair@$$CBKU__Fail_Cmd_Data_tag@@@std@@@3@$0A@@std@@@std@@QAA@ABV012@@Z 00159cec f i Radio.obj
 0001:00058d38       ??0?$_Bidit@U?$pair@$$CBKU__Fail_Cmd_Data_tag@@@std@@HPBU12@ABU12@@std@@QAA@ABU01@@Z 00159d38 f i Radio.obj
 0001:00058d6c       ??8const_iterator@?$_Tree@V?$_Tmap_traits@KU__Fail_Cmd_Data_tag@@U?$less@K@std@@V?$allocator@U?$pair@$$CBKU__Fail_Cmd_Data_tag@@@std@@@3@$0A@@std@@@std@@QBA_NABV012@@Z 00159d6c f i Radio.obj
 0001:00058e64       ?_Init@?$_Tree@V?$_Tmap_traits@KU__Fail_Cmd_Data_tag@@U?$less@K@std@@V?$allocator@U?$pair@$$CBKU__Fail_Cmd_Data_tag@@@std@@@3@$0A@@std@@@std@@IAAXXZ 00159e64 f i Radio.obj
 0001:00058f28       ?_Isnil@?$_Tree@V?$_Tmap_traits@KU__Fail_Cmd_Data_tag@@U?$less@K@std@@V?$allocator@U?$pair@$$CBKU__Fail_Cmd_Data_tag@@@std@@@3@$0A@@std@@@std@@KAAADPAU_Node@?$_Tree_nod@V?$_Tmap_traits@KU__Fail_Cmd_Data_tag@@U?$less@K@std@@V?$allocator@U?$pair@$$CBKU__Fail_Cmd_Data_tag@@@std@@@3@$0A@@std@@@2@@Z 00159f28 f i Radio.obj
 0001:00058f50       ?_Rmost@?$_Tree@V?$_Tmap_traits@KU__Fail_Cmd_Data_tag@@U?$less@K@std@@V?$allocator@U?$pair@$$CBKU__Fail_Cmd_Data_tag@@@std@@@3@$0A@@std@@@std@@IBAAAPAU_Node@?$_Tree_nod@V?$_Tmap_traits@KU__Fail_Cmd_Data_tag@@U?$less@K@std@@V?$allocator@U?$pair@$$CBKU__Fail_Cmd_Data_tag@@@std@@@3@$0A@@std@@@2@XZ 00159f50 f i Radio.obj
 0001:00058f88       ??0?$_Tree_val@V?$_Tmap_traits@KU__Fail_Cmd_Data_tag@@U?$less@K@std@@V?$allocator@U?$pair@$$CBKU__Fail_Cmd_Data_tag@@@std@@@3@$0A@@std@@@std@@IAA@ABU?$less@K@1@V?$allocator@U?$pair@$$CBKU__Fail_Cmd_Data_tag@@@std@@@1@@Z 00159f88 f i Radio.obj
 0001:00058fe8       ??0?$allocator@U?$pair@$$CBKU__Fail_Cmd_Data_tag@@@std@@@std@@QAA@ABV01@@Z 00159fe8 f i Radio.obj
 0001:0005900c       ?deallocate@?$allocator@U_Node@?$_Tree_nod@V?$_Tmap_traits@KU__Fail_Cmd_Data_tag@@U?$less@K@std@@V?$allocator@U?$pair@$$CBKU__Fail_Cmd_Data_tag@@@std@@@3@$0A@@std@@@std@@@std@@QAAXPAU_Node@?$_Tree_nod@V?$_Tmap_traits@KU__Fail_Cmd_Data_tag@@U?$less@K@std@@V?$allocator@U?$pair@$$CBKU__Fail_Cmd_Data_tag@@@std@@@3@$0A@@std@@@2@I@Z 0015a00c f i Radio.obj
 0001:00059024       ?destroy@?$allocator@PAU_Node@?$_Tree_nod@V?$_Tmap_traits@KU__Fail_Cmd_Data_tag@@U?$less@K@std@@V?$allocator@U?$pair@$$CBKU__Fail_Cmd_Data_tag@@@std@@@3@$0A@@std@@@std@@@std@@QAAXPAPAU_Node@?$_Tree_nod@V?$_Tmap_traits@KU__Fail_Cmd_Data_tag@@U?$less@K@std@@V?$allocator@U?$pair@$$CBKU__Fail_Cmd_Data_tag@@@std@@@3@$0A@@std@@@2@@Z 0015a024 f i Radio.obj
 0001:0005903c       ?_Isnil@?$_Tree@V?$_Tmap_traits@KKU?$less@K@std@@V?$allocator@U?$pair@$$CBKK@std@@@2@$0A@@std@@@std@@KAAADPAU_Node@?$_Tree_nod@V?$_Tmap_traits@KKU?$less@K@std@@V?$allocator@U?$pair@$$CBKK@std@@@2@$0A@@std@@@2@@Z 0015a03c f i Radio.obj
 0001:00059064       ?_Left@?$_Tree@V?$_Tmap_traits@KKU?$less@K@std@@V?$allocator@U?$pair@$$CBKK@std@@@2@$0A@@std@@@std@@KAAAPAU_Node@?$_Tree_nod@V?$_Tmap_traits@KKU?$less@K@std@@V?$allocator@U?$pair@$$CBKK@std@@@2@$0A@@std@@@2@PAU342@@Z 0015a064 f i Radio.obj
 0001:00059088       ?_Parent@?$_Tree@V?$_Tmap_traits@KKU?$less@K@std@@V?$allocator@U?$pair@$$CBKK@std@@@2@$0A@@std@@@std@@KAAAPAU_Node@?$_Tree_nod@V?$_Tmap_traits@KKU?$less@K@std@@V?$allocator@U?$pair@$$CBKK@std@@@2@$0A@@std@@@2@PAU342@@Z 0015a088 f i Radio.obj
 0001:000590b0       ?_Right@?$_Tree@V?$_Tmap_traits@KKU?$less@K@std@@V?$allocator@U?$pair@$$CBKK@std@@@2@$0A@@std@@@std@@KAAAPAU_Node@?$_Tree_nod@V?$_Tmap_traits@KKU?$less@K@std@@V?$allocator@U?$pair@$$CBKK@std@@@2@$0A@@std@@@2@PAU342@@Z 0015a0b0 f i Radio.obj
 0001:000590d8       ?_Myval@?$_Tree@V?$_Tmap_traits@KKU?$less@K@std@@V?$allocator@U?$pair@$$CBKK@std@@@2@$0A@@std@@@std@@KAAAU?$pair@$$CBKK@2@PAU_Node@?$_Tree_nod@V?$_Tmap_traits@KKU?$less@K@std@@V?$allocator@U?$pair@$$CBKK@std@@@2@$0A@@std@@@2@@Z 0015a0d8 f i Radio.obj
 0001:00059100       ?begin@?$_Tree@V?$_Tmap_traits@KKU?$less@K@std@@V?$allocator@U?$pair@$$CBKK@std@@@2@$0A@@std@@@std@@QAA?AViterator@12@XZ 0015a100 f i Radio.obj
 0001:0005915c       ?size@?$_Tree@V?$_Tmap_traits@KKU?$less@K@std@@V?$allocator@U?$pair@$$CBKK@std@@@2@$0A@@std@@@std@@QBAIXZ 0015a15c f i Radio.obj
 0001:00059190       ?insert@?$_Tree@V?$_Tmap_traits@KKU?$less@K@std@@V?$allocator@U?$pair@$$CBKK@std@@@2@$0A@@std@@@std@@QAA?AU?$pair@Viterator@?$_Tree@V?$_Tmap_traits@KKU?$less@K@std@@V?$allocator@U?$pair@$$CBKK@std@@@2@$0A@@std@@@std@@_N@2@ABU?$pair@$$CBKK@2@@Z 0015a190 f i Radio.obj
 0001:000595f8       ?erase@?$_Tree@V?$_Tmap_traits@KKU?$less@K@std@@V?$allocator@U?$pair@$$CBKK@std@@@2@$0A@@std@@@std@@QAA?AViterator@12@V312@0@Z 0015a5f8 f i Radio.obj
 0001:000598cc       ?_Init@?$_Tree@V?$_Tmap_traits@KKU?$less@K@std@@V?$allocator@U?$pair@$$CBKK@std@@@2@$0A@@std@@@std@@IAAXXZ 0015a8cc f i Radio.obj
 0001:00059998       ?_Insert@?$_Tree@V?$_Tmap_traits@KKU?$less@K@std@@V?$allocator@U?$pair@$$CBKK@std@@@2@$0A@@std@@@std@@IAA?AViterator@12@_NPAU_Node@?$_Tree_nod@V?$_Tmap_traits@KKU?$less@K@std@@V?$allocator@U?$pair@$$CBKK@std@@@2@$0A@@std@@@2@ABU?$pair@$$CBKK@2@@Z 0015a998 f i Radio.obj
 0001:0005a054       ?_Lbound@?$_Tree@V?$_Tmap_traits@KKU?$less@K@std@@V?$allocator@U?$pair@$$CBKK@std@@@2@$0A@@std@@@std@@IBAPAU_Node@?$_Tree_nod@V?$_Tmap_traits@KKU?$less@K@std@@V?$allocator@U?$pair@$$CBKK@std@@@2@$0A@@std@@@2@ABK@Z 0015b054 f i Radio.obj
 0001:0005a14c       ?_Rmost@?$_Tree@V?$_Tmap_traits@KKU?$less@K@std@@V?$allocator@U?$pair@$$CBKK@std@@@2@$0A@@std@@@std@@IBAAAPAU_Node@?$_Tree_nod@V?$_Tmap_traits@KKU?$less@K@std@@V?$allocator@U?$pair@$$CBKK@std@@@2@$0A@@std@@@2@XZ 0015b14c f i Radio.obj
 0001:0005a184       ??0?$_Tree_val@V?$_Tmap_traits@KKU?$less@K@std@@V?$allocator@U?$pair@$$CBKK@std@@@2@$0A@@std@@@std@@IAA@ABU?$less@K@1@V?$allocator@U?$pair@$$CBKK@std@@@1@@Z 0015b184 f i Radio.obj
 0001:0005a1e4       ?_Kfn@?$_Tmap_traits@KKU?$less@K@std@@V?$allocator@U?$pair@$$CBKK@std@@@2@$0A@@std@@SAABKABU?$pair@$$CBKK@2@@Z 0015b1e4 f i Radio.obj
 0001:0005a208       ??0?$allocator@U?$pair@$$CBKK@std@@@std@@QAA@ABV01@@Z 0015b208 f i Radio.obj
 0001:0005a22c       ?deallocate@?$allocator@U_Node@?$_Tree_nod@V?$_Tmap_traits@KKU?$less@K@std@@V?$allocator@U?$pair@$$CBKK@std@@@2@$0A@@std@@@std@@@std@@QAAXPAU_Node@?$_Tree_nod@V?$_Tmap_traits@KKU?$less@K@std@@V?$allocator@U?$pair@$$CBKK@std@@@2@$0A@@std@@@2@I@Z 0015b22c f i Radio.obj
 0001:0005a244       ?destroy@?$allocator@PAU_Node@?$_Tree_nod@V?$_Tmap_traits@KKU?$less@K@std@@V?$allocator@U?$pair@$$CBKK@std@@@2@$0A@@std@@@std@@@std@@QAAXPAPAU_Node@?$_Tree_nod@V?$_Tmap_traits@KKU?$less@K@std@@V?$allocator@U?$pair@$$CBKK@std@@@2@$0A@@std@@@2@@Z 0015b244 f i Radio.obj
 0001:0005a25c       ?_Orphan_ptr@?$list@PAVCCommand@@V?$allocator@PAVCCommand@@@std@@@std@@IBAXAAV12@PAU_Node@?$_List_nod@PAVCCommand@@V?$allocator@PAVCCommand@@@std@@@2@@Z 0015b25c f i Radio.obj
 0001:0005a330       ?destroy@?$allocator@U_Node@?$_List_nod@PAVCCommand@@V?$allocator@PAVCCommand@@@std@@@std@@@std@@QAAXPAU_Node@?$_List_nod@PAVCCommand@@V?$allocator@PAVCCommand@@@std@@@2@@Z 0015b330 f i Radio.obj
 0001:0005a350       ??E?$_Iterator@$00@?$list@PAVCCommand@@V?$allocator@PAVCCommand@@@std@@@std@@QAA?AV012@H@Z 0015b350 f i Radio.obj
 0001:0005a408       ??0iterator@?$_Tree@V?$_Tmap_traits@KU__Fail_Cmd_Data_tag@@U?$less@K@std@@V?$allocator@U?$pair@$$CBKU__Fail_Cmd_Data_tag@@@std@@@3@$0A@@std@@@std@@QAA@PAU_Node@?$_Tree_nod@V?$_Tmap_traits@KU__Fail_Cmd_Data_tag@@U?$less@K@std@@V?$allocator@U?$pair@$$CBKU__Fail_Cmd_Data_tag@@@std@@@3@$0A@@std@@@2@PBV12@@Z 0015b408 f i Radio.obj
 0001:0005a440       ??0iterator@?$_Tree@V?$_Tmap_traits@KKU?$less@K@std@@V?$allocator@U?$pair@$$CBKK@std@@@2@$0A@@std@@@std@@QAA@XZ 0015b440 f i Radio.obj
 0001:0005a470       ??0iterator@?$_Tree@V?$_Tmap_traits@KKU?$less@K@std@@V?$allocator@U?$pair@$$CBKK@std@@@2@$0A@@std@@@std@@QAA@PAU_Node@?$_Tree_nod@V?$_Tmap_traits@KKU?$less@K@std@@V?$allocator@U?$pair@$$CBKK@std@@@2@$0A@@std@@@2@PBV12@@Z 0015b470 f i Radio.obj
 0001:0005a4a8       ??Eiterator@?$_Tree@V?$_Tmap_traits@KKU?$less@K@std@@V?$allocator@U?$pair@$$CBKK@std@@@2@$0A@@std@@@std@@QAAAAV012@XZ 0015b4a8 f i Radio.obj
 0001:0005a4d4       ??Fiterator@?$_Tree@V?$_Tmap_traits@KKU?$less@K@std@@V?$allocator@U?$pair@$$CBKK@std@@@2@$0A@@std@@@std@@QAAAAV012@XZ 0015b4d4 f i Radio.obj
 0001:0005a500       ??Dconst_iterator@?$_Tree@V?$_Tmap_traits@KKU?$less@K@std@@V?$allocator@U?$pair@$$CBKK@std@@@2@$0A@@std@@@std@@QBAABU?$pair@$$CBKK@2@XZ 0015b500 f i Radio.obj
 0001:0005a5e4       ?erase@?$_Tree@V?$_Tmap_traits@KU__Fail_Cmd_Data_tag@@U?$less@K@std@@V?$allocator@U?$pair@$$CBKU__Fail_Cmd_Data_tag@@@std@@@3@$0A@@std@@@std@@QAA?AViterator@12@V312@@Z 0015b5e4 f i Radio.obj
 0001:0005b150       ?_Mynode@const_iterator@?$_Tree@V?$_Tmap_traits@KU__Fail_Cmd_Data_tag@@U?$less@K@std@@V?$allocator@U?$pair@$$CBKU__Fail_Cmd_Data_tag@@@std@@@3@$0A@@std@@@std@@QBAPAU_Node@?$_Tree_nod@V?$_Tmap_traits@KU__Fail_Cmd_Data_tag@@U?$less@K@std@@V?$allocator@U?$pair@$$CBKU__Fail_Cmd_Data_tag@@@std@@@3@$0A@@std@@@3@XZ 0015c150 f i Radio.obj
 0001:0005b17c       ??Eiterator@?$_Tree@V?$_Tmap_traits@KU__Fail_Cmd_Data_tag@@U?$less@K@std@@V?$allocator@U?$pair@$$CBKU__Fail_Cmd_Data_tag@@@std@@@3@$0A@@std@@@std@@QAAAAV012@XZ 0015c17c f i Radio.obj
 0001:0005b1a8       ?_Color@?$_Tree@V?$_Tmap_traits@KU__Fail_Cmd_Data_tag@@U?$less@K@std@@V?$allocator@U?$pair@$$CBKU__Fail_Cmd_Data_tag@@@std@@@3@$0A@@std@@@std@@KAAADPAU_Node@?$_Tree_nod@V?$_Tmap_traits@KU__Fail_Cmd_Data_tag@@U?$less@K@std@@V?$allocator@U?$pair@$$CBKU__Fail_Cmd_Data_tag@@@std@@@3@$0A@@std@@@2@@Z 0015c1a8 f i Radio.obj
 0001:0005b1d0       ?clear@?$_Tree@V?$_Tmap_traits@KU__Fail_Cmd_Data_tag@@U?$less@K@std@@V?$allocator@U?$pair@$$CBKU__Fail_Cmd_Data_tag@@@std@@@3@$0A@@std@@@std@@QAAXXZ 0015c1d0 f i Radio.obj
 0001:0005b284       ?_Lmost@?$_Tree@V?$_Tmap_traits@KU__Fail_Cmd_Data_tag@@U?$less@K@std@@V?$allocator@U?$pair@$$CBKU__Fail_Cmd_Data_tag@@@std@@@3@$0A@@std@@@std@@IBAAAPAU_Node@?$_Tree_nod@V?$_Tmap_traits@KU__Fail_Cmd_Data_tag@@U?$less@K@std@@V?$allocator@U?$pair@$$CBKU__Fail_Cmd_Data_tag@@@std@@@3@$0A@@std@@@2@XZ 0015c284 f i Radio.obj
 0001:0005b2bc       ?_Lrotate@?$_Tree@V?$_Tmap_traits@KU__Fail_Cmd_Data_tag@@U?$less@K@std@@V?$allocator@U?$pair@$$CBKU__Fail_Cmd_Data_tag@@@std@@@3@$0A@@std@@@std@@IAAXPAU_Node@?$_Tree_nod@V?$_Tmap_traits@KU__Fail_Cmd_Data_tag@@U?$less@K@std@@V?$allocator@U?$pair@$$CBKU__Fail_Cmd_Data_tag@@@std@@@3@$0A@@std@@@2@@Z 0015c2bc f i Radio.obj
 0001:0005b480       ?_Root@?$_Tree@V?$_Tmap_traits@KU__Fail_Cmd_Data_tag@@U?$less@K@std@@V?$allocator@U?$pair@$$CBKU__Fail_Cmd_Data_tag@@@std@@@3@$0A@@std@@@std@@IBAAAPAU_Node@?$_Tree_nod@V?$_Tmap_traits@KU__Fail_Cmd_Data_tag@@U?$less@K@std@@V?$allocator@U?$pair@$$CBKU__Fail_Cmd_Data_tag@@@std@@@3@$0A@@std@@@2@XZ 0015c480 f i Radio.obj
 0001:0005b4b8       ?_Rrotate@?$_Tree@V?$_Tmap_traits@KU__Fail_Cmd_Data_tag@@U?$less@K@std@@V?$allocator@U?$pair@$$CBKU__Fail_Cmd_Data_tag@@@std@@@3@$0A@@std@@@std@@IAAXPAU_Node@?$_Tree_nod@V?$_Tmap_traits@KU__Fail_Cmd_Data_tag@@U?$less@K@std@@V?$allocator@U?$pair@$$CBKU__Fail_Cmd_Data_tag@@@std@@@3@$0A@@std@@@2@@Z 0015c4b8 f i Radio.obj
 0001:0005b684       ?_Buynode@?$_Tree@V?$_Tmap_traits@KU__Fail_Cmd_Data_tag@@U?$less@K@std@@V?$allocator@U?$pair@$$CBKU__Fail_Cmd_Data_tag@@@std@@@3@$0A@@std@@@std@@IAAPAU_Node@?$_Tree_nod@V?$_Tmap_traits@KU__Fail_Cmd_Data_tag@@U?$less@K@std@@V?$allocator@U?$pair@$$CBKU__Fail_Cmd_Data_tag@@@std@@@3@$0A@@std@@@2@XZ 0015c684 f i Radio.obj
 0001:0005b824       ??0?$_Tree_ptr@V?$_Tmap_traits@KU__Fail_Cmd_Data_tag@@U?$less@K@std@@V?$allocator@U?$pair@$$CBKU__Fail_Cmd_Data_tag@@@std@@@3@$0A@@std@@@std@@QAA@ABU?$less@K@1@V?$allocator@U?$pair@$$CBKU__Fail_Cmd_Data_tag@@@std@@@1@@Z 0015c824 f i Radio.obj
 0001:0005b884       ?_Color@?$_Tree@V?$_Tmap_traits@KKU?$less@K@std@@V?$allocator@U?$pair@$$CBKK@std@@@2@$0A@@std@@@std@@KAAADPAU_Node@?$_Tree_nod@V?$_Tmap_traits@KKU?$less@K@std@@V?$allocator@U?$pair@$$CBKK@std@@@2@$0A@@std@@@2@@Z 0015c884 f i Radio.obj
 0001:0005b8ac       ?max_size@?$_Tree@V?$_Tmap_traits@KKU?$less@K@std@@V?$allocator@U?$pair@$$CBKK@std@@@2@$0A@@std@@@std@@QBAIXZ 0015c8ac f i Radio.obj
 0001:0005b8e8       ?erase@?$_Tree@V?$_Tmap_traits@KKU?$less@K@std@@V?$allocator@U?$pair@$$CBKK@std@@@2@$0A@@std@@@std@@QAA?AViterator@12@V312@@Z 0015c8e8 f i Radio.obj
 0001:0005c454       ?clear@?$_Tree@V?$_Tmap_traits@KKU?$less@K@std@@V?$allocator@U?$pair@$$CBKK@std@@@2@$0A@@std@@@std@@QAAXXZ 0015d454 f i Radio.obj
 0001:0005c508       ?_Lmost@?$_Tree@V?$_Tmap_traits@KKU?$less@K@std@@V?$allocator@U?$pair@$$CBKK@std@@@2@$0A@@std@@@std@@IBAAAPAU_Node@?$_Tree_nod@V?$_Tmap_traits@KKU?$less@K@std@@V?$allocator@U?$pair@$$CBKK@std@@@2@$0A@@std@@@2@XZ 0015d508 f i Radio.obj
 0001:0005c540       ?_Lrotate@?$_Tree@V?$_Tmap_traits@KKU?$less@K@std@@V?$allocator@U?$pair@$$CBKK@std@@@2@$0A@@std@@@std@@IAAXPAU_Node@?$_Tree_nod@V?$_Tmap_traits@KKU?$less@K@std@@V?$allocator@U?$pair@$$CBKK@std@@@2@$0A@@std@@@2@@Z 0015d540 f i Radio.obj
 0001:0005c704       ?_Root@?$_Tree@V?$_Tmap_traits@KKU?$less@K@std@@V?$allocator@U?$pair@$$CBKK@std@@@2@$0A@@std@@@std@@IBAAAPAU_Node@?$_Tree_nod@V?$_Tmap_traits@KKU?$less@K@std@@V?$allocator@U?$pair@$$CBKK@std@@@2@$0A@@std@@@2@XZ 0015d704 f i Radio.obj
 0001:0005c73c       ?_Rrotate@?$_Tree@V?$_Tmap_traits@KKU?$less@K@std@@V?$allocator@U?$pair@$$CBKK@std@@@2@$0A@@std@@@std@@IAAXPAU_Node@?$_Tree_nod@V?$_Tmap_traits@KKU?$less@K@std@@V?$allocator@U?$pair@$$CBKK@std@@@2@$0A@@std@@@2@@Z 0015d73c f i Radio.obj
 0001:0005c908       ?_Buynode@?$_Tree@V?$_Tmap_traits@KKU?$less@K@std@@V?$allocator@U?$pair@$$CBKK@std@@@2@$0A@@std@@@std@@IAAPAU_Node@?$_Tree_nod@V?$_Tmap_traits@KKU?$less@K@std@@V?$allocator@U?$pair@$$CBKK@std@@@2@$0A@@std@@@2@XZ 0015d908 f i Radio.obj
 0001:0005cab0       ?_Buynode@?$_Tree@V?$_Tmap_traits@KKU?$less@K@std@@V?$allocator@U?$pair@$$CBKK@std@@@2@$0A@@std@@@std@@IAAPAU_Node@?$_Tree_nod@V?$_Tmap_traits@KKU?$less@K@std@@V?$allocator@U?$pair@$$CBKK@std@@@2@$0A@@std@@@2@PAU342@00ABU?$pair@$$CBKK@2@D@Z 0015dab0 f i Radio.obj
 0001:0005cbcc       ??0?$_Tree_ptr@V?$_Tmap_traits@KKU?$less@K@std@@V?$allocator@U?$pair@$$CBKK@std@@@2@$0A@@std@@@std@@QAA@ABU?$less@K@1@V?$allocator@U?$pair@$$CBKK@std@@@1@@Z 0015dbcc f i Radio.obj
 0001:0005cc34       ??Eiterator@?$_Tree@V?$_Tmap_traits@KU__Fail_Cmd_Data_tag@@U?$less@K@std@@V?$allocator@U?$pair@$$CBKU__Fail_Cmd_Data_tag@@@std@@@3@$0A@@std@@@std@@QAA?AV012@H@Z 0015dc34 f i Radio.obj
 0001:0005ccf4       ??0const_iterator@?$_Tree@V?$_Tmap_traits@KU__Fail_Cmd_Data_tag@@U?$less@K@std@@V?$allocator@U?$pair@$$CBKU__Fail_Cmd_Data_tag@@@std@@@3@$0A@@std@@@std@@QAA@PAU_Node@?$_Tree_nod@V?$_Tmap_traits@KU__Fail_Cmd_Data_tag@@U?$less@K@std@@V?$allocator@U?$pair@$$CBKU__Fail_Cmd_Data_tag@@@std@@@3@$0A@@std@@@2@PBV12@@Z 0015dcf4 f i Radio.obj
 0001:0005cd5c       ??Econst_iterator@?$_Tree@V?$_Tmap_traits@KU__Fail_Cmd_Data_tag@@U?$less@K@std@@V?$allocator@U?$pair@$$CBKU__Fail_Cmd_Data_tag@@@std@@@3@$0A@@std@@@std@@QAAAAV012@XZ 0015dd5c f i Radio.obj
 0001:0005cd88       ??9const_iterator@?$_Tree@V?$_Tmap_traits@KU__Fail_Cmd_Data_tag@@U?$less@K@std@@V?$allocator@U?$pair@$$CBKU__Fail_Cmd_Data_tag@@@std@@@3@$0A@@std@@@std@@QBA_NABV012@@Z 0015dd88 f i Radio.obj
 0001:0005cde8       ??Eiterator@?$_Tree@V?$_Tmap_traits@KKU?$less@K@std@@V?$allocator@U?$pair@$$CBKK@std@@@2@$0A@@std@@@std@@QAA?AV012@H@Z 0015dde8 f i Radio.obj
 0001:0005cea0       ??0const_iterator@?$_Tree@V?$_Tmap_traits@KKU?$less@K@std@@V?$allocator@U?$pair@$$CBKK@std@@@2@$0A@@std@@@std@@QAA@XZ 0015dea0 f i Radio.obj
 0001:0005cee8       ??0const_iterator@?$_Tree@V?$_Tmap_traits@KKU?$less@K@std@@V?$allocator@U?$pair@$$CBKK@std@@@2@$0A@@std@@@std@@QAA@PAU_Node@?$_Tree_nod@V?$_Tmap_traits@KKU?$less@K@std@@V?$allocator@U?$pair@$$CBKK@std@@@2@$0A@@std@@@2@PBV12@@Z 0015dee8 f i Radio.obj
 0001:0005cf50       ??Econst_iterator@?$_Tree@V?$_Tmap_traits@KKU?$less@K@std@@V?$allocator@U?$pair@$$CBKK@std@@@2@$0A@@std@@@std@@QAAAAV012@XZ 0015df50 f i Radio.obj
 0001:0005cf7c       ??Fconst_iterator@?$_Tree@V?$_Tmap_traits@KKU?$less@K@std@@V?$allocator@U?$pair@$$CBKK@std@@@2@$0A@@std@@@std@@QAAAAV012@XZ 0015df7c f i Radio.obj
 0001:0005cfa8       ??9const_iterator@?$_Tree@V?$_Tmap_traits@KKU?$less@K@std@@V?$allocator@U?$pair@$$CBKK@std@@@2@$0A@@std@@@std@@QBA_NABV012@@Z 0015dfa8 f i Radio.obj
 0001:0005d000       ??0?$pair@Viterator@?$_Tree@V?$_Tmap_traits@KKU?$less@K@std@@V?$allocator@U?$pair@$$CBKK@std@@@2@$0A@@std@@@std@@_N@std@@QAA@ABViterator@?$_Tree@V?$_Tmap_traits@KKU?$less@K@std@@V?$allocator@U?$pair@$$CBKK@std@@@2@$0A@@std@@@1@AB_N@Z 0015e000 f i Radio.obj
 0001:0005d048       ??0?$_Bidit@U?$pair@$$CBKU__Fail_Cmd_Data_tag@@@std@@HPBU12@ABU12@@std@@QAA@XZ 0015e048 f i Radio.obj
 0001:0005d078       ??0?$_Bidit@U?$pair@$$CBKK@std@@HPBU12@ABU12@@std@@QAA@XZ 0015e078 f i Radio.obj
 0001:0005d0a8       ?_Erase@?$_Tree@V?$_Tmap_traits@KU__Fail_Cmd_Data_tag@@U?$less@K@std@@V?$allocator@U?$pair@$$CBKU__Fail_Cmd_Data_tag@@@std@@@3@$0A@@std@@@std@@IAAXPAU_Node@?$_Tree_nod@V?$_Tmap_traits@KU__Fail_Cmd_Data_tag@@U?$less@K@std@@V?$allocator@U?$pair@$$CBKU__Fail_Cmd_Data_tag@@@std@@@3@$0A@@std@@@2@@Z 0015e0a8 f i Radio.obj
 0001:0005d14c       ?_Max@?$_Tree@V?$_Tmap_traits@KU__Fail_Cmd_Data_tag@@U?$less@K@std@@V?$allocator@U?$pair@$$CBKU__Fail_Cmd_Data_tag@@@std@@@3@$0A@@std@@@std@@KAPAU_Node@?$_Tree_nod@V?$_Tmap_traits@KU__Fail_Cmd_Data_tag@@U?$less@K@std@@V?$allocator@U?$pair@$$CBKU__Fail_Cmd_Data_tag@@@std@@@3@$0A@@std@@@2@PAU342@@Z 0015e14c f i Radio.obj
 0001:0005d1b8       ?_Min@?$_Tree@V?$_Tmap_traits@KU__Fail_Cmd_Data_tag@@U?$less@K@std@@V?$allocator@U?$pair@$$CBKU__Fail_Cmd_Data_tag@@@std@@@3@$0A@@std@@@std@@KAPAU_Node@?$_Tree_nod@V?$_Tmap_traits@KU__Fail_Cmd_Data_tag@@U?$less@K@std@@V?$allocator@U?$pair@$$CBKU__Fail_Cmd_Data_tag@@@std@@@3@$0A@@std@@@2@PAU342@@Z 0015e1b8 f i Radio.obj
 0001:0005d224       ?_Orphan_ptr@?$_Tree@V?$_Tmap_traits@KU__Fail_Cmd_Data_tag@@U?$less@K@std@@V?$allocator@U?$pair@$$CBKU__Fail_Cmd_Data_tag@@@std@@@3@$0A@@std@@@std@@IBAXAAV12@PAU_Node@?$_Tree_nod@V?$_Tmap_traits@KU__Fail_Cmd_Data_tag@@U?$less@K@std@@V?$allocator@U?$pair@$$CBKU__Fail_Cmd_Data_tag@@@std@@@3@$0A@@std@@@2@@Z 0015e224 f i Radio.obj
 0001:0005d2f8       ??0?$_Tree_nod@V?$_Tmap_traits@KU__Fail_Cmd_Data_tag@@U?$less@K@std@@V?$allocator@U?$pair@$$CBKU__Fail_Cmd_Data_tag@@@std@@@3@$0A@@std@@@std@@IAA@ABU?$less@K@1@V?$allocator@U?$pair@$$CBKU__Fail_Cmd_Data_tag@@@std@@@1@@Z 0015e2f8 f i Radio.obj
 0001:0005d348       ?allocate@?$allocator@U_Node@?$_Tree_nod@V?$_Tmap_traits@KU__Fail_Cmd_Data_tag@@U?$less@K@std@@V?$allocator@U?$pair@$$CBKU__Fail_Cmd_Data_tag@@@std@@@3@$0A@@std@@@std@@@std@@QAAPAU_Node@?$_Tree_nod@V?$_Tmap_traits@KU__Fail_Cmd_Data_tag@@U?$less@K@std@@V?$allocator@U?$pair@$$CBKU__Fail_Cmd_Data_tag@@@std@@@3@$0A@@std@@@2@I@Z 0015e348 f i Radio.obj
 0001:0005d37c       ?destroy@?$allocator@U_Node@?$_Tree_nod@V?$_Tmap_traits@KU__Fail_Cmd_Data_tag@@U?$less@K@std@@V?$allocator@U?$pair@$$CBKU__Fail_Cmd_Data_tag@@@std@@@3@$0A@@std@@@std@@@std@@QAAXPAU_Node@?$_Tree_nod@V?$_Tmap_traits@KU__Fail_Cmd_Data_tag@@U?$less@K@std@@V?$allocator@U?$pair@$$CBKU__Fail_Cmd_Data_tag@@@std@@@3@$0A@@std@@@2@@Z 0015e37c f i Radio.obj
 0001:0005d394       ?construct@?$allocator@PAU_Node@?$_Tree_nod@V?$_Tmap_traits@KU__Fail_Cmd_Data_tag@@U?$less@K@std@@V?$allocator@U?$pair@$$CBKU__Fail_Cmd_Data_tag@@@std@@@3@$0A@@std@@@std@@@std@@QAAXPAPAU_Node@?$_Tree_nod@V?$_Tmap_traits@KU__Fail_Cmd_Data_tag@@U?$less@K@std@@V?$allocator@U?$pair@$$CBKU__Fail_Cmd_Data_tag@@@std@@@3@$0A@@std@@@2@ABQAU342@@Z 0015e394 f i Radio.obj
 0001:0005d3b0       ?_Erase@?$_Tree@V?$_Tmap_traits@KKU?$less@K@std@@V?$allocator@U?$pair@$$CBKK@std@@@2@$0A@@std@@@std@@IAAXPAU_Node@?$_Tree_nod@V?$_Tmap_traits@KKU?$less@K@std@@V?$allocator@U?$pair@$$CBKK@std@@@2@$0A@@std@@@2@@Z 0015e3b0 f i Radio.obj
 0001:0005d454       ?_Max@?$_Tree@V?$_Tmap_traits@KKU?$less@K@std@@V?$allocator@U?$pair@$$CBKK@std@@@2@$0A@@std@@@std@@KAPAU_Node@?$_Tree_nod@V?$_Tmap_traits@KKU?$less@K@std@@V?$allocator@U?$pair@$$CBKK@std@@@2@$0A@@std@@@2@PAU342@@Z 0015e454 f i Radio.obj
 0001:0005d4c0       ?_Min@?$_Tree@V?$_Tmap_traits@KKU?$less@K@std@@V?$allocator@U?$pair@$$CBKK@std@@@2@$0A@@std@@@std@@KAPAU_Node@?$_Tree_nod@V?$_Tmap_traits@KKU?$less@K@std@@V?$allocator@U?$pair@$$CBKK@std@@@2@$0A@@std@@@2@PAU342@@Z 0015e4c0 f i Radio.obj
 0001:0005d52c       ?_Orphan_ptr@?$_Tree@V?$_Tmap_traits@KKU?$less@K@std@@V?$allocator@U?$pair@$$CBKK@std@@@2@$0A@@std@@@std@@IBAXAAV12@PAU_Node@?$_Tree_nod@V?$_Tmap_traits@KKU?$less@K@std@@V?$allocator@U?$pair@$$CBKK@std@@@2@$0A@@std@@@2@@Z 0015e52c f i Radio.obj
 0001:0005d600       ??0?$_Tree_nod@V?$_Tmap_traits@KKU?$less@K@std@@V?$allocator@U?$pair@$$CBKK@std@@@2@$0A@@std@@@std@@IAA@ABU?$less@K@1@V?$allocator@U?$pair@$$CBKK@std@@@1@@Z 0015e600 f i Radio.obj
 0001:0005d650       ?max_size@?$allocator@U?$pair@$$CBKK@std@@@std@@QBAIXZ 0015e650 f i Radio.obj
 0001:0005d69c       ?allocate@?$allocator@U_Node@?$_Tree_nod@V?$_Tmap_traits@KKU?$less@K@std@@V?$allocator@U?$pair@$$CBKK@std@@@2@$0A@@std@@@std@@@std@@QAAPAU_Node@?$_Tree_nod@V?$_Tmap_traits@KKU?$less@K@std@@V?$allocator@U?$pair@$$CBKK@std@@@2@$0A@@std@@@2@I@Z 0015e69c f i Radio.obj
 0001:0005d6d0       ?destroy@?$allocator@U_Node@?$_Tree_nod@V?$_Tmap_traits@KKU?$less@K@std@@V?$allocator@U?$pair@$$CBKK@std@@@2@$0A@@std@@@std@@@std@@QAAXPAU_Node@?$_Tree_nod@V?$_Tmap_traits@KKU?$less@K@std@@V?$allocator@U?$pair@$$CBKK@std@@@2@$0A@@std@@@2@@Z 0015e6d0 f i Radio.obj
 0001:0005d6e8       ?construct@?$allocator@PAU_Node@?$_Tree_nod@V?$_Tmap_traits@KKU?$less@K@std@@V?$allocator@U?$pair@$$CBKK@std@@@2@$0A@@std@@@std@@@std@@QAAXPAPAU_Node@?$_Tree_nod@V?$_Tmap_traits@KKU?$less@K@std@@V?$allocator@U?$pair@$$CBKK@std@@@2@$0A@@std@@@2@ABQAU342@@Z 0015e6e8 f i Radio.obj
 0001:0005d704       ?_Inc@const_iterator@?$_Tree@V?$_Tmap_traits@KU__Fail_Cmd_Data_tag@@U?$less@K@std@@V?$allocator@U?$pair@$$CBKU__Fail_Cmd_Data_tag@@@std@@@3@$0A@@std@@@std@@QAAXXZ 0015e704 f i Radio.obj
 0001:0005d8c0       ?_Dec@const_iterator@?$_Tree@V?$_Tmap_traits@KKU?$less@K@std@@V?$allocator@U?$pair@$$CBKK@std@@@2@$0A@@std@@@std@@QAAXXZ 0015e8c0 f i Radio.obj
 0001:0005dbc0       ?_Inc@const_iterator@?$_Tree@V?$_Tmap_traits@KKU?$less@K@std@@V?$allocator@U?$pair@$$CBKK@std@@@2@$0A@@std@@@std@@QAAXXZ 0015ebc0 f i Radio.obj
 0001:0005dd7c       ??0_Node@?$_Tree_nod@V?$_Tmap_traits@KKU?$less@K@std@@V?$allocator@U?$pair@$$CBKK@std@@@2@$0A@@std@@@std@@QAA@PAU012@00ABU?$pair@$$CBKK@2@D@Z 0015ed7c f i Radio.obj
 0001:0005de00       ??0?$_Tmap_traits@KU__Fail_Cmd_Data_tag@@U?$less@K@std@@V?$allocator@U?$pair@$$CBKU__Fail_Cmd_Data_tag@@@std@@@3@$0A@@std@@QAA@U?$less@K@1@@Z 0015ee00 f i Radio.obj
 0001:0005de30       ??0?$_Tmap_traits@KKU?$less@K@std@@V?$allocator@U?$pair@$$CBKK@std@@@2@$0A@@std@@QAA@U?$less@K@1@@Z 0015ee30 f i Radio.obj
 0001:0005de60       ?Push_Back@?$CThreadSafeQueue@PAUSwiNotifyVariant@@@@QAAXABQAUSwiNotifyVariant@@@Z 0015ee60 f i Radio.obj
 0001:0005decc       ??$_Debug_lt_pred@U?$less@K@std@@KK@std@@YA_NU?$less@K@0@ABK1PBGI@Z 0015eecc f i Radio.obj
 0001:0005df54       ??$_Destroy@PAU_Node@?$_Tree_nod@V?$_Tmap_traits@KU__Fail_Cmd_Data_tag@@U?$less@K@std@@V?$allocator@U?$pair@$$CBKU__Fail_Cmd_Data_tag@@@std@@@3@$0A@@std@@@std@@@std@@YAXPAPAU_Node@?$_Tree_nod@V?$_Tmap_traits@KU__Fail_Cmd_Data_tag@@U?$less@K@std@@V?$allocator@U?$pair@$$CBKU__Fail_Cmd_Data_tag@@@std@@@3@$0A@@std@@@0@@Z 0015ef54 f i Radio.obj
 0001:0005df64       ??$_Destroy@PAU_Node@?$_Tree_nod@V?$_Tmap_traits@KKU?$less@K@std@@V?$allocator@U?$pair@$$CBKK@std@@@2@$0A@@std@@@std@@@std@@YAXPAPAU_Node@?$_Tree_nod@V?$_Tmap_traits@KKU?$less@K@std@@V?$allocator@U?$pair@$$CBKK@std@@@2@$0A@@std@@@0@@Z 0015ef64 f i Radio.obj
 0001:0005df74       ??$_Destroy@U_Node@?$_List_nod@PAVCCommand@@V?$allocator@PAVCCommand@@@std@@@std@@@std@@YAXPAU_Node@?$_List_nod@PAVCCommand@@V?$allocator@PAVCCommand@@@std@@@0@@Z 0015ef74 f i Radio.obj
 0001:0005df84       ??$?0U?$pair@$$CBKU__Fail_Cmd_Data_tag@@@std@@@?$allocator@PAU_Node@?$_Tree_nod@V?$_Tmap_traits@KU__Fail_Cmd_Data_tag@@U?$less@K@std@@V?$allocator@U?$pair@$$CBKU__Fail_Cmd_Data_tag@@@std@@@3@$0A@@std@@@std@@@std@@QAA@ABV?$allocator@U?$pair@$$CBKU__Fail_Cmd_Data_tag@@@std@@@1@@Z 0015ef84 f i Radio.obj
 0001:0005dfa8       ??$?0U?$pair@$$CBKK@std@@@?$allocator@PAU_Node@?$_Tree_nod@V?$_Tmap_traits@KKU?$less@K@std@@V?$allocator@U?$pair@$$CBKK@std@@@2@$0A@@std@@@std@@@std@@QAA@ABV?$allocator@U?$pair@$$CBKK@std@@@1@@Z 0015efa8 f i Radio.obj
 0001:0005dfcc       ??$?0U?$pair@$$CBKU__Fail_Cmd_Data_tag@@@std@@@?$allocator@U_Node@?$_Tree_nod@V?$_Tmap_traits@KU__Fail_Cmd_Data_tag@@U?$less@K@std@@V?$allocator@U?$pair@$$CBKU__Fail_Cmd_Data_tag@@@std@@@3@$0A@@std@@@std@@@std@@QAA@ABV?$allocator@U?$pair@$$CBKU__Fail_Cmd_Data_tag@@@std@@@1@@Z 0015efcc f i Radio.obj
 0001:0005dff0       ??$_Allocate@U_Node@?$_Tree_nod@V?$_Tmap_traits@KU__Fail_Cmd_Data_tag@@U?$less@K@std@@V?$allocator@U?$pair@$$CBKU__Fail_Cmd_Data_tag@@@std@@@3@$0A@@std@@@std@@@std@@YAPAU_Node@?$_Tree_nod@V?$_Tmap_traits@KU__Fail_Cmd_Data_tag@@U?$less@K@std@@V?$allocator@U?$pair@$$CBKU__Fail_Cmd_Data_tag@@@std@@@3@$0A@@std@@@0@IPAU120@@Z 0015eff0 f i Radio.obj
 0001:0005e080       ??$_Destroy@U_Node@?$_Tree_nod@V?$_Tmap_traits@KU__Fail_Cmd_Data_tag@@U?$less@K@std@@V?$allocator@U?$pair@$$CBKU__Fail_Cmd_Data_tag@@@std@@@3@$0A@@std@@@std@@@std@@YAXPAU_Node@?$_Tree_nod@V?$_Tmap_traits@KU__Fail_Cmd_Data_tag@@U?$less@K@std@@V?$allocator@U?$pair@$$CBKU__Fail_Cmd_Data_tag@@@std@@@3@$0A@@std@@@0@@Z 0015f080 f i Radio.obj
 0001:0005e090       ??$_Construct@PAU_Node@?$_Tree_nod@V?$_Tmap_traits@KU__Fail_Cmd_Data_tag@@U?$less@K@std@@V?$allocator@U?$pair@$$CBKU__Fail_Cmd_Data_tag@@@std@@@3@$0A@@std@@@std@@PAU123@@std@@YAXPAPAU_Node@?$_Tree_nod@V?$_Tmap_traits@KU__Fail_Cmd_Data_tag@@U?$less@K@std@@V?$allocator@U?$pair@$$CBKU__Fail_Cmd_Data_tag@@@std@@@3@$0A@@std@@@0@ABQAU120@@Z 0015f090 f i Radio.obj
 0001:0005e0f8       ??$?0U?$pair@$$CBKK@std@@@?$allocator@U_Node@?$_Tree_nod@V?$_Tmap_traits@KKU?$less@K@std@@V?$allocator@U?$pair@$$CBKK@std@@@2@$0A@@std@@@std@@@std@@QAA@ABV?$allocator@U?$pair@$$CBKK@std@@@1@@Z 0015f0f8 f i Radio.obj
 0001:0005e11c       ??$_Allocate@U_Node@?$_Tree_nod@V?$_Tmap_traits@KKU?$less@K@std@@V?$allocator@U?$pair@$$CBKK@std@@@2@$0A@@std@@@std@@@std@@YAPAU_Node@?$_Tree_nod@V?$_Tmap_traits@KKU?$less@K@std@@V?$allocator@U?$pair@$$CBKK@std@@@2@$0A@@std@@@0@IPAU120@@Z 0015f11c f i Radio.obj
 0001:0005e1ac       ??$_Destroy@U_Node@?$_Tree_nod@V?$_Tmap_traits@KKU?$less@K@std@@V?$allocator@U?$pair@$$CBKK@std@@@2@$0A@@std@@@std@@@std@@YAXPAU_Node@?$_Tree_nod@V?$_Tmap_traits@KKU?$less@K@std@@V?$allocator@U?$pair@$$CBKK@std@@@2@$0A@@std@@@0@@Z 0015f1ac f i Radio.obj
 0001:0005e1bc       ??$_Construct@PAU_Node@?$_Tree_nod@V?$_Tmap_traits@KKU?$less@K@std@@V?$allocator@U?$pair@$$CBKK@std@@@2@$0A@@std@@@std@@PAU123@@std@@YAXPAPAU_Node@?$_Tree_nod@V?$_Tmap_traits@KKU?$less@K@std@@V?$allocator@U?$pair@$$CBKK@std@@@2@$0A@@std@@@0@ABQAU120@@Z 0015f1bc f i Radio.obj
 0001:0005e224       ?push@?$queue@PAUSwiNotifyVariant@@V?$deque@PAUSwiNotifyVariant@@V?$allocator@PAUSwiNotifyVariant@@@std@@@std@@@std@@QAAXABQAUSwiNotifyVariant@@@Z 0015f224 f i Radio.obj
 0001:0005e240       ?push_back@?$deque@PAUSwiNotifyVariant@@V?$allocator@PAUSwiNotifyVariant@@@std@@@std@@QAAXABQAUSwiNotifyVariant@@@Z 0015f240 f i Radio.obj
 0001:0005e420       ?_Growmap@?$deque@PAUSwiNotifyVariant@@V?$allocator@PAUSwiNotifyVariant@@@std@@@std@@IAAXI@Z 0015f420 f i Radio.obj
 0001:0005e7d4       ?allocate@?$allocator@PAUSwiNotifyVariant@@@std@@QAAPAPAUSwiNotifyVariant@@I@Z 0015f7d4 f i Radio.obj
 0001:0005e808       ?construct@?$allocator@PAUSwiNotifyVariant@@@std@@QAAXPAPAUSwiNotifyVariant@@ABQAU3@@Z 0015f808 f i Radio.obj
 0001:0005e824       ?max_size@?$deque@PAUSwiNotifyVariant@@V?$allocator@PAUSwiNotifyVariant@@@std@@@std@@QBAIXZ 0015f824 f i Radio.obj
 0001:0005e860       ?_Xlen@?$deque@PAUSwiNotifyVariant@@V?$allocator@PAUSwiNotifyVariant@@@std@@@std@@KAXXZ 0015f860 f i Radio.obj
 0001:0005e8d8       ?deallocate@?$allocator@PAPAUSwiNotifyVariant@@@std@@QAAXPAPAPAUSwiNotifyVariant@@I@Z 0015f8d8 f i Radio.obj
 0001:0005e8f0       ?allocate@?$allocator@PAPAUSwiNotifyVariant@@@std@@QAAPAPAPAUSwiNotifyVariant@@I@Z 0015f8f0 f i Radio.obj
 0001:0005e924       ?max_size@?$allocator@PAUSwiNotifyVariant@@@std@@QBAIXZ 0015f924 f i Radio.obj
 0001:0005e970       ??$unchecked_uninitialized_copy@PAPAPAUSwiNotifyVariant@@PAPAPAU1@V?$allocator@PAPAUSwiNotifyVariant@@@std@@@stdext@@YAPAPAPAUSwiNotifyVariant@@PAPAPAU1@00AAV?$allocator@PAPAUSwiNotifyVariant@@@std@@@Z 0015f970 f i Radio.obj
 0001:0005ea18       ??$unchecked_uninitialized_fill_n@PAPAPAUSwiNotifyVariant@@IPAPAU1@V?$allocator@PAPAUSwiNotifyVariant@@@std@@@stdext@@YAXPAPAPAUSwiNotifyVariant@@IABQAPAU1@AAV?$allocator@PAPAUSwiNotifyVariant@@@std@@@Z 0015fa18 f i Radio.obj
 0001:0005ea98       ??$_Destroy_range@PAPAUSwiNotifyVariant@@V?$allocator@PAPAUSwiNotifyVariant@@@std@@@std@@YAXPAPAPAUSwiNotifyVariant@@0AAV?$allocator@PAPAUSwiNotifyVariant@@@0@@Z 0015fa98 f i Radio.obj
 0001:0005eae8       ??$_Allocate@PAUSwiNotifyVariant@@@std@@YAPAPAUSwiNotifyVariant@@IPAPAU1@@Z 0015fae8 f i Radio.obj
 0001:0005eb78       ??$_Construct@PAUSwiNotifyVariant@@PAU1@@std@@YAXPAPAUSwiNotifyVariant@@ABQAU1@@Z 0015fb78 f i Radio.obj
 0001:0005ebe0       ??$_Allocate@PAPAUSwiNotifyVariant@@@std@@YAPAPAPAUSwiNotifyVariant@@IPAPAPAU1@@Z 0015fbe0 f i Radio.obj
 0001:0005ec70       ??$_Checked_base@PAPAPAUSwiNotifyVariant@@@std@@YAPAPAPAUSwiNotifyVariant@@AAPAPAPAU1@@Z 0015fc70 f i Radio.obj
 0001:0005eca4       ??$_Ptr_cat@PAPAPAUSwiNotifyVariant@@PAPAPAU1@@std@@YA?AU_Scalar_ptr_iterator_tag@0@AAPAPAPAUSwiNotifyVariant@@0@Z 0015fca4 f i Radio.obj
 0001:0005ecd8       ??$_Uninit_copy@PAPAPAUSwiNotifyVariant@@PAPAPAU1@V?$allocator@PAPAUSwiNotifyVariant@@@std@@@std@@YAPAPAPAUSwiNotifyVariant@@PAPAPAU1@00AAV?$allocator@PAPAUSwiNotifyVariant@@@0@U_Scalar_ptr_iterator_tag@0@U_Range_checked_iterator_tag@0@@Z 0015fcd8 f i Radio.obj
 0001:0005ed80       ??$_Uninit_fill_n@PAPAPAUSwiNotifyVariant@@IPAPAU1@V?$allocator@PAPAUSwiNotifyVariant@@@std@@@std@@YAXPAPAPAUSwiNotifyVariant@@IABQAPAU1@AAV?$allocator@PAPAUSwiNotifyVariant@@@0@U_Scalar_ptr_iterator_tag@0@U_Range_checked_iterator_tag@0@@Z 0015fd80 f i Radio.obj
 0001:0005eda0       ??$_Destroy_range@PAPAUSwiNotifyVariant@@V?$allocator@PAPAUSwiNotifyVariant@@@std@@@std@@YAXPAPAPAUSwiNotifyVariant@@0AAV?$allocator@PAPAUSwiNotifyVariant@@@0@U_Scalar_ptr_iterator_tag@0@@Z 0015fda0 f i Radio.obj
 0001:0005edb0       ??$_Checked_base@PAPAPAUSwiNotifyVariant@@@std@@YAPAPAPAUSwiNotifyVariant@@AAPAPAPAU1@U_Unchanged_checked_iterator_base_type_tag@0@@Z 0015fdb0 f i Radio.obj
 0001:0005edd8       ??$_Debug_range@PAPAPAUSwiNotifyVariant@@@std@@YAXPAPAPAUSwiNotifyVariant@@0PBGI@Z 0015fdd8 f i Radio.obj
 0001:0005ee2c       ??$_Debug_pointer@PAPAUSwiNotifyVariant@@@std@@YAXPAPAPAUSwiNotifyVariant@@PBGI@Z 0015fe2c f i Radio.obj
 0001:0005ee5c       ??$unchecked_fill_n@PAPAPAUSwiNotifyVariant@@IPAPAU1@@stdext@@YAXPAPAPAUSwiNotifyVariant@@IABQAPAU1@@Z 0015fe5c f i Radio.obj
 0001:0005eec4       ??$_Iter_cat@PAPAPAUSwiNotifyVariant@@@std@@YA?AUrandom_access_iterator_tag@0@ABQAPAPAUSwiNotifyVariant@@@Z 0015fec4 f i Radio.obj
 0001:0005eee8       ??$_Debug_range2@PAPAPAUSwiNotifyVariant@@@std@@YAXPAPAPAUSwiNotifyVariant@@0PBGIUrandom_access_iterator_tag@0@@Z 0015fee8 f i Radio.obj
 0001:0005ef4c       ??$_Fill_n@PAPAPAUSwiNotifyVariant@@IPAPAU1@@std@@YAXPAPAPAUSwiNotifyVariant@@IABQAPAU1@Urandom_access_iterator_tag@0@U_Range_checked_iterator_tag@0@@Z 0015ff4c f i Radio.obj
 0001:0005efac       ??$_Fill_n@PAPAPAUSwiNotifyVariant@@IPAPAU1@@std@@YAXPAPAPAUSwiNotifyVariant@@IABQAPAU1@U_Range_checked_iterator_tag@0@@Z 0015ffac f i Radio.obj
 0001:0005eff8       ??0CRadioCaps@@QAA@XZ      0015fff8 f   RadioCaps.obj
 0001:0005f03c       ??1CRadioCaps@@QAA@XZ      0016003c f   RadioCaps.obj
 0001:0005f080       ?Init@CRadioCaps@@QAAJXZ   00160080 f   RadioCaps.obj
 0001:0005fcd8       ?SetDevCapsLockFacilities@CRadioCaps@@QAAXKH@Z 00160cd8 f   RadioCaps.obj
 0001:0005fe84       ??0CResponse@@QAA@XZ       00160e84 f   response.obj
 0001:0005fee4       ??1CResponse@@QAA@XZ       00160ee4 f   response.obj
 0001:0005ff1c       ?SetBlob@CResponse@@QAAHQBXI@Z 00160f1c f   response.obj
 0001:00060190       ?MakeError@CResponse@@QAAHJ@Z 00161190 f   response.obj
 0001:00060250       ?GetError@CResponse@@QBAJXZ 00161250 f   response.obj
 0001:00060308       ??0CNotificationData@@QAA@XZ 00161308 f   response.obj
 0001:00060358       ??1CNotificationData@@QAA@XZ 00161358 f   response.obj
 0001:00060388       ?InitFromDWORDBlob@CNotificationData@@QAAHKK@Z 00161388 f   response.obj
 0001:00060554       ?InitFromRealBlob@CNotificationData@@QAAHKQBXI@Z 00161554 f   response.obj
 0001:00060734       ??0CRilHandle@@QAA@XZ      00161734 f   rilhand.obj
 0001:00060ac0       ?DeleteInstanceHandle@@YAHPAXK@Z 00161ac0 f   rilhand.obj
 0001:00060bb0       ??1CRilHandle@@QAA@XZ      00161bb0 f   rilhand.obj
 0001:00061168       ?SendReadyStateNotification@CRilHandle@@QAAXKH@Z 00162168 f   rilhand.obj
 0001:0006121c       ?StartInit@CRilHandle@@QAAHXZ 0016221c f   rilhand.obj
 0001:00061bb0       ?GeneralInitDone@CRilHandle@@QAAXH@Z 00162bb0 f   rilhand.obj
 0001:00061f4c       ?GenerateCancelledRsp@@YAHPAXK@Z 00162f4c f   rilhand.obj
 0001:00062138       ?PrepareForReinit@CRilHandle@@QAAXXZ 00163138 f   rilhand.obj
 0001:000621bc       ?LaunchThreads@CRilHandle@@QAAHXZ 001631bc f   rilhand.obj
 0001:000627a8       ?FCancelSet@CRilHandle@@QBAHXZ 001637a8 f   rilhand.obj
 0001:00062848       ?WaitForCommandOrCancel@CRilHandle@@QBAHXZ 00163848 f   rilhand.obj
 0001:00062a74       ?AddToList@CRilHandle@@QAAHQAVCRilInstanceHandle@@@Z 00163a74 f   rilhand.obj
 0001:00062af4       ?RemoveFromList@CRilHandle@@QAAHQAVCRilInstanceHandle@@@Z 00163af4 f   rilhand.obj
 0001:00062b74       ?GetNextCmdID@CRilHandle@@QAAJXZ 00163b74 f   rilhand.obj
 0001:00062c04       ?NotifyHandle@@YAHPAXK@Z   00163c04 f   rilhand.obj
 0001:00062d88       ?BroadcastNotification@CRilHandle@@QAAXPAVCNotificationData@@@Z 00163d88 f   rilhand.obj
 0001:00062f58       ?BroadcastRealBlobNotification@CRilHandle@@QAAHKQBXI@Z 00163f58 f   rilhand.obj
 0001:00063170       ?BroadcastDWORDBlobNotification@CRilHandle@@QAAHKK@Z 00164170 f   rilhand.obj
 0001:000632dc       ?RegisterWithCPM@CRilHandle@@QAAHXZ 001642dc f   rilhand.obj
 0001:00063490       ?GetAPIInfo@CRilHandle@@QAAXW4APIID@@AAUAPIINFO@@@Z 00164490 f   rilhand.obj
 0001:0006386c       ?NotificationItemDtor@@YAXPAX@Z 0016486c f   rilhand.obj
 0001:0006388c       ?PreBroadcastNotification@CRilHandle@@QAAHPAVCNotificationData@@@Z 0016488c f   rilhand.obj
 0001:000648a0       ??0CRilInstanceHandle@@QAA@XZ 001658a0 f   rilhand.obj
 0001:000649bc       ??1CRilInstanceHandle@@QAA@XZ 001659bc f   rilhand.obj
 0001:00064b20       ?Init@CRilInstanceHandle@@QAAHQAVCRilHandle@@@Z 00165b20 f   rilhand.obj
 0001:00064c50       ?Notify@CRilInstanceHandle@@QAAXKJQBXI@Z 00165c50 f   rilhand.obj
 0001:00064e24       ?FEnoughStorage@@YAHPAXK@Z 00165e24 f   rilhand.obj
 0001:00064f20       ?GetNextNotification@CRilInstanceHandle@@QAAHAAUrildrvnotification_tag@@@Z 00165f20 f   rilhand.obj
 0001:00065318       ?CreateNotificationQueue@CRilInstanceHandle@@QAAHPBGPAEKPAK@Z 00166318 f   rilhand.obj
 0001:000655bc       ?ImgPref2Ids@@YAXKQAEQAG111@Z 001665bc f   rilhand.obj
 0001:000657b8       ?Ids2ImgPref@@YAXPAKQAEQAG222@Z 001667b8 f   rilhand.obj
 0001:00065b18       ?InitializeSWI@CRilHandle@@QAAHXZ 00166b18 f   rilhand.obj
 0001:00068ce0       ?DeInitializeSWI@CRilHandle@@QAAHH@Z 00169ce0 f   rilhand.obj
 0001:0006900c       ?CheckVoiceMailBox@CRilHandle@@QAAXXZ 0016a00c f   rilhand.obj
 0001:000692b0       ?CloseSWI@CRilHandle@@QAAHXZ 0016a2b0 f   rilhand.obj
 0001:00069578       ?CheckDelayedRspCmdTimeout@CRilHandle@@QAAXXZ 0016a578 f   rilhand.obj
 0001:00069ae8       ?SwitchUnattendedMode@CRilHandle@@QAAXH@Z 0016aae8 f   rilhand.obj
 0001:00069ca4       ??_GCRilInstanceHandle@@QAAPAXI@Z 0016aca4 f i rilhand.obj
 0001:00069ce4       ??_GCRadio@@QAAPAXI@Z      0016ace4 f i rilhand.obj
 0001:00069d24       ??_GCMonitor@@QAAPAXI@Z    0016ad24 f i rilhand.obj
 0001:00069d64       ??_G?$CThreadSafeQueue@PAVCCommand@@@@QAAPAXI@Z 0016ad64 f i rilhand.obj
 0001:00069da4       ??_G?$CThreadSafeQueue@PAUSwiNotifyVariant@@@@QAAPAXI@Z 0016ada4 f i rilhand.obj
 0001:00069de4       ??_G?$CDblList@VCRilInstanceHandle@@@@QAAPAXI@Z 0016ade4 f i rilhand.obj
 0001:00069e24       ?GetCode@CNotificationData@@QBAKXZ 0016ae24 f i rilhand.obj
 0001:00069e4c       ?GetBlob@CNotificationData@@QBAQBXXZ 0016ae4c f i rilhand.obj
 0001:00069e78       ?GetSize@CNotificationData@@QBAIXZ 0016ae78 f i rilhand.obj
 0001:00069ea4       ?GetTimeout@CCommand@@QBAKXZ 0016aea4 f i rilhand.obj
 0001:00069ed0       ?GetExecTime@CCommand@@QBAKXZ 0016aed0 f i rilhand.obj
 0001:00069efc       ?CancelNotifications@CRilInstanceHandle@@QBAXXZ 0016aefc f i rilhand.obj
 0001:00069f30       ??_G?$CDblList@VCCommand@@@@QAAPAXI@Z 0016af30 f i rilhand.obj
 0001:00069f70       ?GetLocationState@CRadio@@QAAKXZ 0016af70 f i rilhand.obj
 0001:00069fa0       ?GetCurrentCallPrivacy@CRadio@@QAAKXZ 0016afa0 f i rilhand.obj
 0001:00069fd0       ?SaveRawCarrierID@CRadio@@QAAXW4SWI_TYPE_CarrierID@@@Z 0016afd0 f i rilhand.obj
 0001:00069ff4       ?SetSwiDeviceType@CRadio@@QAAXK@Z 0016aff4 f i rilhand.obj
 0001:0006a018       ?SetIsRUIM@CRadio@@QAAXH@Z 0016b018 f i rilhand.obj
 0001:0006a03c       ?GetIsRUIM@CRadio@@QAAHXZ  0016b03c f i rilhand.obj
 0001:0006a06c       ?GetItemsEventName@?$CUnboundedQueue@Urildrvnotification_tag@@@@QAAPBGXZ 0016b06c f i rilhand.obj
 0001:0006a0a0       ?GetName@CUniquelyNamedEvent@@QAAPBGXZ 0016b0a0 f i rilhand.obj
 0001:0006a0c8       ??0?$CDblList@VCRilInstanceHandle@@@@QAA@XZ 0016b0c8 f i rilhand.obj
 0001:0006a104       ??1?$CDblList@VCRilInstanceHandle@@@@QAA@XZ 0016b104 f i rilhand.obj
 0001:0006a128       ?Add@?$CDblList@VCRilInstanceHandle@@@@QAAHQAVCRilInstanceHandle@@@Z 0016b128 f i rilhand.obj
 0001:0006a20c       ?Remove@?$CDblList@VCRilInstanceHandle@@@@QAAHQBVCRilInstanceHandle@@@Z 0016b20c f i rilhand.obj
 0001:0006a390       ?Enum@?$CDblList@VCRilInstanceHandle@@@@QAAXQ6AHPAXK@ZK@Z 0016b390 f i rilhand.obj
 0001:0006a444       ??0?$CUnboundedQueue@Urildrvnotification_tag@@@@QAA@P6AXPAX@Z@Z 0016b444 f i rilhand.obj
 0001:0006a4e4       ??0CUniquelyNamedEvent@@QAA@XZ 0016b4e4 f i rilhand.obj
 0001:0006a534       ??0CEvent@@QAA@XZ          0016b534 f i rilhand.obj
 0001:0006a578       ??_ECEvent@@UAAPAXI@Z      0016b578 f i rilhand.obj
 0001:0006a578       ??_GCEvent@@UAAPAXI@Z      0016b578 f i rilhand.obj
 0001:0006a5b8       ??1CEvent@@UAA@XZ          0016b5b8 f i rilhand.obj
 0001:0006a5fc       ??_ECUniquelyNamedEvent@@UAAPAXI@Z 0016b5fc f i rilhand.obj
 0001:0006a5fc       ??_GCUniquelyNamedEvent@@UAAPAXI@Z 0016b5fc f i rilhand.obj
 0001:0006a63c       ??1CUniquelyNamedEvent@@UAA@XZ 0016b63c f i rilhand.obj
 0001:0006a65c       ??1?$CUnboundedQueue@Urildrvnotification_tag@@@@UAA@XZ 0016b65c f i rilhand.obj
 0001:0006a7c0       ?Reset@CEvent@@QBAXXZ      0016b7c0 f i rilhand.obj
 0001:0006a834       ?Init@?$CUnboundedQueue@Urildrvnotification_tag@@@@QAAHK@Z 0016b834 f i rilhand.obj
 0001:0006a950       ?Init@CUniquelyNamedEvent@@QAAHHHPAG@Z 0016b950 f i rilhand.obj
 0001:0006aa4c       ?Put@?$CUnboundedQueue@Urildrvnotification_tag@@@@QAAHQAUrildrvnotification_tag@@@Z 0016ba4c f i rilhand.obj
 0001:0006ac4c       ?Set@CEvent@@QBAXXZ        0016bc4c f i rilhand.obj
 0001:0006acc8       ?ConditionalGet@?$CUnboundedQueue@Urildrvnotification_tag@@@@QAAJQ6AHPAXK@ZKPAPAUrildrvnotification_tag@@@Z 0016bcc8 f i rilhand.obj
 0001:0006af10       ??0?$CDblList@VCCommand@@@@QAA@XZ 0016bf10 f i rilhand.obj
 0001:0006af4c       ??1?$CDblList@VCCommand@@@@QAA@XZ 0016bf4c f i rilhand.obj
 0001:0006af70       ??0?$CThreadSafeQueue@PAVCCommand@@@@QAA@XZ 0016bf70 f i rilhand.obj
 0001:0006b03c       ??0Event@@QAA@HHPBGPAU_SECURITY_ATTRIBUTES@@@Z 0016c03c f i rilhand.obj
 0001:0006b098       ??_EEvent@@UAAPAXI@Z       0016c098 f i rilhand.obj
 0001:0006b098       ??_GEvent@@UAAPAXI@Z       0016c098 f i rilhand.obj
 0001:0006b0d8       ??1Event@@UAA@XZ           0016c0d8 f i rilhand.obj
 0001:0006b110       ??1?$CThreadSafeQueue@PAVCCommand@@@@QAA@XZ 0016c110 f i rilhand.obj
 0001:0006b1a4       ?GetAlertEvent@?$CThreadSafeQueue@PAVCCommand@@@@QAAPAXXZ 0016c1a4 f i rilhand.obj
 0001:0006b1e0       ??0?$CThreadSafeQueue@PAUSwiNotifyVariant@@@@QAA@XZ 0016c1e0 f i rilhand.obj
 0001:0006b2b4       ??1?$CThreadSafeQueue@PAUSwiNotifyVariant@@@@QAA@XZ 0016c2b4 f i rilhand.obj
 0001:0006b348       ??_G?$CUnboundedQueue@Urildrvnotification_tag@@@@UAAPAXI@Z 0016c348 f i rilhand.obj
 0001:0006b348       ??_E?$CUnboundedQueue@Urildrvnotification_tag@@@@UAAPAXI@Z 0016c348 f i rilhand.obj
 0001:0006b388       ??1?$queue@PAVCCommand@@V?$deque@PAVCCommand@@V?$allocator@PAVCCommand@@@std@@@std@@@std@@QAA@XZ 0016c388 f i rilhand.obj
 0001:0006b3a0       ??1?$queue@PAUSwiNotifyVariant@@V?$deque@PAUSwiNotifyVariant@@V?$allocator@PAUSwiNotifyVariant@@@std@@@std@@@std@@QAA@XZ 0016c3a0 f i rilhand.obj
 0001:0006b3b8       ??0?$queue@PAVCCommand@@V?$deque@PAVCCommand@@V?$allocator@PAVCCommand@@@std@@@std@@@std@@QAA@XZ 0016c3b8 f i rilhand.obj
 0001:0006b3f0       ??1?$deque@PAVCCommand@@V?$allocator@PAVCCommand@@@std@@@std@@QAA@XZ 0016c3f0 f i rilhand.obj
 0001:0006b430       ??0?$queue@PAUSwiNotifyVariant@@V?$deque@PAUSwiNotifyVariant@@V?$allocator@PAUSwiNotifyVariant@@@std@@@std@@@std@@QAA@XZ 0016c430 f i rilhand.obj
 0001:0006b468       ??1?$deque@PAUSwiNotifyVariant@@V?$allocator@PAUSwiNotifyVariant@@@std@@@std@@QAA@XZ 0016c468 f i rilhand.obj
 0001:0006b4a8       ??1?$_Deque_val@PAVCCommand@@V?$allocator@PAVCCommand@@@std@@@std@@QAA@XZ 0016c4a8 f i rilhand.obj
 0001:0006b4c0       ??1?$_Deque_val@PAUSwiNotifyVariant@@V?$allocator@PAUSwiNotifyVariant@@@std@@@std@@QAA@XZ 0016c4c0 f i rilhand.obj
 0001:0006b4d8       ??1?$_Deque_map@PAVCCommand@@V?$allocator@PAVCCommand@@@std@@@std@@QAA@XZ 0016c4d8 f i rilhand.obj
 0001:0006b4f0       ??1?$_Deque_map@PAUSwiNotifyVariant@@V?$allocator@PAUSwiNotifyVariant@@@std@@@std@@QAA@XZ 0016c4f0 f i rilhand.obj
 0001:0006b508       ??0?$deque@PAVCCommand@@V?$allocator@PAVCCommand@@@std@@@std@@QAA@XZ 0016c508 f i rilhand.obj
 0001:0006b590       ??0?$allocator@PAVCCommand@@@std@@QAA@XZ 0016c590 f i rilhand.obj
 0001:0006b5b4       ?_Tidy@?$deque@PAVCCommand@@V?$allocator@PAVCCommand@@@std@@@std@@IAAXXZ 0016c5b4 f i rilhand.obj
 0001:0006b6f4       ??0?$deque@PAUSwiNotifyVariant@@V?$allocator@PAUSwiNotifyVariant@@@std@@@std@@QAA@XZ 0016c6f4 f i rilhand.obj
 0001:0006b77c       ?_Tidy@?$deque@PAUSwiNotifyVariant@@V?$allocator@PAUSwiNotifyVariant@@@std@@@std@@IAAXXZ 0016c77c f i rilhand.obj
 0001:0006b8bc       ?deallocate@?$allocator@PAVCCommand@@@std@@QAAXPAPAVCCommand@@I@Z 0016c8bc f i rilhand.obj
 0001:0006b8d4       ?pop_back@?$deque@PAVCCommand@@V?$allocator@PAVCCommand@@@std@@@std@@QAAXXZ 0016c8d4 f i rilhand.obj
 0001:0006ba50       ??0?$_Deque_val@PAVCCommand@@V?$allocator@PAVCCommand@@@std@@@std@@IAA@V?$allocator@PAVCCommand@@@1@@Z 0016ca50 f i rilhand.obj
 0001:0006baac       ??0?$allocator@PAVCCommand@@@std@@QAA@ABV01@@Z 0016caac f i rilhand.obj
 0001:0006bad0       ?destroy@?$allocator@PAPAVCCommand@@@std@@QAAXPAPAPAVCCommand@@@Z 0016cad0 f i rilhand.obj
 0001:0006bae8       ?pop_back@?$deque@PAUSwiNotifyVariant@@V?$allocator@PAUSwiNotifyVariant@@@std@@@std@@QAAXXZ 0016cae8 f i rilhand.obj
 0001:0006bc64       ??0?$_Deque_val@PAUSwiNotifyVariant@@V?$allocator@PAUSwiNotifyVariant@@@std@@@std@@IAA@V?$allocator@PAUSwiNotifyVariant@@@1@@Z 0016cc64 f i rilhand.obj
 0001:0006bcc0       ??0?$allocator@PAUSwiNotifyVariant@@@std@@QAA@XZ 0016ccc0 f i rilhand.obj
 0001:0006bce4       ?deallocate@?$allocator@PAUSwiNotifyVariant@@@std@@QAAXPAPAUSwiNotifyVariant@@I@Z 0016cce4 f i rilhand.obj
 0001:0006bcfc       ?destroy@?$allocator@PAPAUSwiNotifyVariant@@@std@@QAAXPAPAPAUSwiNotifyVariant@@@Z 0016ccfc f i rilhand.obj
 0001:0006bd14       ??0?$_Deque_map@PAVCCommand@@V?$allocator@PAVCCommand@@@std@@@std@@IAA@V?$allocator@PAVCCommand@@@1@@Z 0016cd14 f i rilhand.obj
 0001:0006bd54       ??0?$_Deque_map@PAUSwiNotifyVariant@@V?$allocator@PAUSwiNotifyVariant@@@std@@@std@@IAA@V?$allocator@PAUSwiNotifyVariant@@@1@@Z 0016cd54 f i rilhand.obj
 0001:0006bd94       ??0?$allocator@PAUSwiNotifyVariant@@@std@@QAA@ABV01@@Z 0016cd94 f i rilhand.obj
 0001:0006bdb8       ?GrowQueue@?$CUnboundedQueue@Urildrvnotification_tag@@@@IAAHXZ 0016cdb8 f i rilhand.obj
 0001:0006bf0c       ??$_Destroy@PAPAVCCommand@@@std@@YAXPAPAPAVCCommand@@@Z 0016cf0c f i rilhand.obj
 0001:0006bf1c       ??$_Destroy@PAPAUSwiNotifyVariant@@@std@@YAXPAPAPAUSwiNotifyVariant@@@Z 0016cf1c f i rilhand.obj
 0001:0006bf2c       ??$?0PAVCCommand@@@?$allocator@PAPAVCCommand@@@std@@QAA@ABV?$allocator@PAVCCommand@@@1@@Z 0016cf2c f i rilhand.obj
 0001:0006bf50       ??$?0PAUSwiNotifyVariant@@@?$allocator@PAPAUSwiNotifyVariant@@@std@@QAA@ABV?$allocator@PAUSwiNotifyVariant@@@1@@Z 0016cf50 f i rilhand.obj
 0001:0006bf7c       ??0?$list@PAVCCommand@@V?$allocator@PAVCCommand@@@std@@@std@@QAA@XZ 0016cf7c f i rilhand.obj
 0001:0006c00c       ??1?$_List_val@PAVCCommand@@V?$allocator@PAVCCommand@@@std@@@std@@QAA@XZ 0016d00c f i rilhand.obj
 0001:0006c024       ??1?$_List_ptr@PAVCCommand@@V?$allocator@PAVCCommand@@@std@@@std@@QAA@XZ 0016d024 f i rilhand.obj
 0001:0006c03c       ??1?$_List_nod@PAVCCommand@@V?$allocator@PAVCCommand@@@std@@@std@@QAA@XZ 0016d03c f i rilhand.obj
 0001:0006c05c       ?_Buynode@?$list@PAVCCommand@@V?$allocator@PAVCCommand@@@std@@@std@@IAAPAU_Node@?$_List_nod@PAVCCommand@@V?$allocator@PAVCCommand@@@std@@@2@XZ 0016d05c f i rilhand.obj
 0001:0006c160       ??0?$_List_val@PAVCCommand@@V?$allocator@PAVCCommand@@@std@@@std@@QAA@V?$allocator@PAVCCommand@@@1@@Z 0016d160 f i rilhand.obj
 0001:0006c1bc       ??0?$_List_ptr@PAVCCommand@@V?$allocator@PAVCCommand@@@std@@@std@@IAA@V?$allocator@PAVCCommand@@@1@@Z 0016d1bc f i rilhand.obj
 0001:0006c218       ??0?$_List_nod@PAVCCommand@@V?$allocator@PAVCCommand@@@std@@@std@@IAA@V?$allocator@PAVCCommand@@@1@@Z 0016d218 f i rilhand.obj
 0001:0006c258       ??$?0PAVCCommand@@@?$allocator@PAU_Node@?$_List_nod@PAVCCommand@@V?$allocator@PAVCCommand@@@std@@@std@@@std@@QAA@ABV?$allocator@PAVCCommand@@@1@@Z 0016d258 f i rilhand.obj
 0001:0006c27c       ??$?0PAVCCommand@@@?$allocator@U_Node@?$_List_nod@PAVCCommand@@V?$allocator@PAVCCommand@@@std@@@std@@@std@@QAA@ABV?$allocator@PAVCCommand@@@1@@Z 0016d27c f i rilhand.obj
 0001:0006c2a8       ??1?$list@PAVCCommand@@V?$allocator@PAVCCommand@@@std@@@std@@QAA@XZ 0016d2a8 f i rilhand.obj
 0001:0006c2e8       ?_Tidy@?$list@PAVCCommand@@V?$allocator@PAVCCommand@@@std@@@std@@IAAXXZ 0016d2e8 f i rilhand.obj
 0001:0006c37c       ?clear@?$list@PAVCCommand@@V?$allocator@PAVCCommand@@@std@@@std@@QAAXXZ 0016d37c f i rilhand.obj
 0001:0006c488       ?NdisRilInstanceFromHandle@CRilHandle@@QAAPBXPAX@Z 0016d488 f   rilhandndis.obj
 0001:0006c570       ?RilNdisSendPacket@@YAXQAUrilndispacket_tag@@@Z 0016d570 f   rilhandndis.obj
 0001:0006c60c       ?RilNdisRecievePacketDone@@YAXQAUrilndispacket_tag@@@Z 0016d60c f   rilhandndis.obj
 0001:0006c6a8       ?ValidChannelIndex@@YAHK@Z 0016d6a8 f   rilhandndis.obj
 0001:0006c6f8       ?NdisGetIPAddress@CRilHandle@@QAAHKPAUSWI_STRUCT_IPConfigurationGobi@@@Z 0016d6f8 f   rilhandndis.obj
 0001:0006c7e0       ?NdisStart@CRilHandle@@AAAHXZ 0016d7e0 f   rilhandndis.obj
 0001:0006c90c       ?NdisStop@CRilHandle@@AAAXXZ 0016d90c f   rilhandndis.obj
 0001:0006c9c8       ?NdisCountEvents@CRilHandle@@AAAKXZ 0016d9c8 f   rilhandndis.obj
 0001:0006ca54       ?NdisGetFreeNdisEntry@CRilHandle@@QAAJPAK@Z 0016da54 f   rilhandndis.obj
 0001:0006cb08       ?NdisRemoveNdisEntry@CRilHandle@@QAAXPAX@Z 0016db08 f   rilhandndis.obj
 0001:0006cbc8       ?NdisCidFromHandle@CRilHandle@@QAAJPAXPAK@Z 0016dbc8 f   rilhandndis.obj
 0001:0006cca8       ?NdisHandleFromCid@CRilHandle@@QAAJKPAPAX@Z 0016dca8 f   rilhandndis.obj
 0001:0006cda8       ?NdisFindValidCid@CRilHandle@@QAAJPAK@Z 0016dda8 f   rilhandndis.obj
 0001:0006ce78       ?NdisRilCallbacksFromCID@CRilHandle@@QAAXKPAPAXPAP6AXPAXPAUrilndispacket_tag@@@Z3PAP6AX1PAUrilndisstatus_tag@@@Z@Z 0016de78 f   rilhandndis.obj
 0001:0006cfec       ?NdisRemoveCallbacks@CRilHandle@@QAAXK@Z 0016dfec f   rilhandndis.obj
 0001:0006d140       ?NdisAddNdisEntry@CRilHandle@@QAAXKKPAXPBXPBUrilndisgprscontext_tag@@@Z 0016e140 f   rilhandndis.obj
 0001:0006d234       ?myinet_addr@@YAKPBEE@Z    0016e234 f   rilhandndis.obj
 0001:0006d2d8       ?myinet_ipv6addr@@YA?AUrilndisipv6addr_tag@@PBEE@Z 0016e2d8 f   rilhandndis.obj
 0001:0006d338       ?NdisConvertConfig@CRilHandle@@QAAXPBUoemndisconfiguration_tag@@PAUrilndisipconfig_tag@@@Z 0016e338 f   rilhandndis.obj
 0001:0006d848       ?NdisCloseAllConnections@CRilHandle@@QAAXH@Z 0016e848 f   rilhandndis.obj
 0001:0006d8e4       ?NdisShutdownConnection@CRilHandle@@QAAXPAXH@Z 0016e8e4 f   rilhandndis.obj
 0001:0006da40       ?ConsumeReadDataCallback@@YAKKPAE@Z 0016ea40 f   rilhandndis.obj
 0001:0006daa8       ?NdisConsumeReadData@CRilHandle@@QAAKKPAE@Z 0016eaa8 f   rilhandndis.obj
 0001:0006dbe8       ?NdisNotifyThread@CRilHandle@@QAAKXZ 0016ebe8 f   rilhandndis.obj
 0001:0006f390       ?NdisAddNotifyEvent@CRilHandle@@QAAJPAX@Z 00170390 f   rilhandndis.obj
 0001:0006f4bc       ?NdisRemoveNotifyEvent@CRilHandle@@QAAJPAX@Z 001704bc f   rilhandndis.obj
 0001:0006f758       ?NdisInterfaceInitialise@CRilHandle@@QAAPAXK@Z 00170758 f   rilhandndis.obj
 0001:0006f7dc       ?NdisInterfaceShutdown@CRilHandle@@QAAHPAX@Z 001707dc f   rilhandndis.obj
 0001:0006f814       ?NdisInterfaceReceiveEvent@CRilHandle@@QAAHPAXPAUoemndisevent_tag@@PAH@Z 00170814 f   rilhandndis.obj
 0001:0006f898       ?NdisInterfaceTransmitEvent@CRilHandle@@QAAHPAXPBUoemndisevent_tag@@@Z 00170898 f   rilhandndis.obj
 0001:0006fa8c       ?NdisAddRxPacket@CRilHandle@@QAAXPAUrilndispacket_tag@@@Z 00170a8c f   rilhandndis.obj
 0001:0006fab0       ?NdisRemoveRxPacket@CRilHandle@@QAAXPAUrilndispacket_tag@@@Z 00170ab0 f   rilhandndis.obj
 0001:0006fad4       ?NdisAllocateCommand@CRilHandle@@QAAJW4oemndiseventtype_tag@@PAX1@Z 00170ad4 f   rilhandndis.obj
 0001:0006fb74       ?NdisAllocateCommand@CRilHandle@@QAAJPAUrilndispacket_tag@@PAX1@Z 00170b74 f   rilhandndis.obj
 0001:0006fc14       ?NdisRemoveCommand@CRilHandle@@QAAJJ@Z 00170c14 f   rilhandndis.obj
 0001:0006fc70       ?NdisShutdown@CRilInstanceHandle@@QAAXXZ 00170c70 f   rilhandndis.obj
 0001:0006fc9c       GetIPForAdapter            00170c9c f   rilhandndis.obj
 0001:0006fe24       tcpxsum                    00170e24 f   rilhandndis.obj
 0001:00070098       UpdateIPCheckSum           00171098 f   rilhandndis.obj
 0001:000703a0       ?NdisPacketTest@@YAHPAUrilndispacket_tag@@@Z 001713a0 f   rilhandndis.obj
 0001:00070498       ?PreExecNDISCmd@CRilInstanceHandle@@AAAJK@Z 00171498 f   rilhandndis.obj
 0001:00070598       ?NdisSendPacket@CRilInstanceHandle@@QAAJPAUrilndispacket_tag@@@Z 00171598 f   rilhandndis.obj
 0001:00070874       ?NdisSetGPRSContextActivated@CRilInstanceHandle@@QAAJPBV1@PBUrilndisgprscontext_tag@@@Z 00171874 f   rilhandndis.obj
 0001:00070ff4       ?NdisReceivePacketDone@CRilInstanceHandle@@QAAJPAUrilndispacket_tag@@@Z 00171ff4 f   rilhandndis.obj
 0001:000710c8       ?NdisNotifyThreadProc@@YAKPAX@Z 001720c8 f   rilhandndis.obj
 0001:00071108       ??0AsyncResponse@@QAA@XZ   00172108 f   rilhandndis.obj
 0001:00071144       ??1AsyncResponse@@QAA@XZ   00172144 f   rilhandndis.obj
 0001:000711d4       ?AddCommand@AsyncResponse@@QAAJPAUoemndisapireference_tag@@@Z 001721d4 f   rilhandndis.obj
 0001:00071280       ?RemoveCommand@AsyncResponse@@QAAJJ@Z 00172280 f   rilhandndis.obj
 0001:00071364       ?ProcessCommand@AsyncResponse@@QAAHPBUoemndisapireference_tag@@@Z 00172364 f   rilhandndis.obj
 0001:000715fc       ?AddListItem@AsyncResponse@@AAAJPAUasyncresponse_tag@@@Z 001725fc f   rilhandndis.obj
 0001:000716f4       ?RemoveListItem@AsyncResponse@@AAAJPAUasyncresponse_tag@@@Z 001726f4 f   rilhandndis.obj
 0001:00071864       ?RemoveAllCommands@AsyncResponse@@QAAXXZ 00172864 f   rilhandndis.obj
 0001:000718e8       ??0NdisRxPacketQueue@@QAA@XZ 001728e8 f   rilhandndis.obj
 0001:00071924       ??1NdisRxPacketQueue@@QAA@XZ 00172924 f   rilhandndis.obj
 0001:000719b4       ?AddPacket@NdisRxPacketQueue@@QAAJPAUrilndispacket_tag@@@Z 001729b4 f   rilhandndis.obj
 0001:00071a5c       ?RemovePacket@NdisRxPacketQueue@@QAAXPAUrilndispacket_tag@@@Z 00172a5c f   rilhandndis.obj
 0001:00071b24       ?FindPacket@NdisRxPacketQueue@@QAAPAUrilndispacket_tag@@XZ 00172b24 f   rilhandndis.obj
 0001:00071bd4       ?AddListItem@NdisRxPacketQueue@@AAAJPAUndispacketqueueelement_tag@@@Z 00172bd4 f   rilhandndis.obj
 0001:00071ccc       ?RemoveListItem@NdisRxPacketQueue@@AAAJPAUndispacketqueueelement_tag@@@Z 00172ccc f   rilhandndis.obj
 0001:00071e3c       ?DumpPacket@@YAXPAUrilndispacket_tag@@@Z 00172e3c f   rilhandndis.obj
 0001:00072100       ?LocalPacketFree@@YAXPAUrilndispacket_tag@@@Z 00173100 f   rilhandndis.obj
 0001:00072110       ?DEBUG_TYPE@@YAXW4oemndiseventtype_tag@@@Z 00173110 f   rilhandndis.obj
 0001:00072388       ?GetAPIFailSetting@CRadio@@QAAPAU__Fail_Cmd_Data_tag@@K@Z 00173388 f i rilhandndis.obj
 0001:000723cc       ??A?$map@KU__Fail_Cmd_Data_tag@@U?$less@K@std@@V?$allocator@U?$pair@$$CBKU__Fail_Cmd_Data_tag@@@std@@@3@@std@@QAAAAU__Fail_Cmd_Data_tag@@ABK@Z 001733cc f i rilhandndis.obj
 0001:000725d8       ??4iterator@?$_Tree@V?$_Tmap_traits@KU__Fail_Cmd_Data_tag@@U?$less@K@std@@V?$allocator@U?$pair@$$CBKU__Fail_Cmd_Data_tag@@@std@@@3@$0A@@std@@@std@@QAAAAV012@ABV012@@Z 001735d8 f i rilhandndis.obj
 0001:00072608       ??4const_iterator@?$_Tree@V?$_Tmap_traits@KU__Fail_Cmd_Data_tag@@U?$less@K@std@@V?$allocator@U?$pair@$$CBKU__Fail_Cmd_Data_tag@@@std@@@3@$0A@@std@@@std@@QAAAAV012@ABV012@@Z 00173608 f i rilhandndis.obj
 0001:00072650       ??4?$_Bidit@U?$pair@$$CBKU__Fail_Cmd_Data_tag@@@std@@HPBU12@ABU12@@std@@QAAAAU01@ABU01@@Z 00173650 f i rilhandndis.obj
 0001:00072680       ?_Key@?$_Tree@V?$_Tmap_traits@KU__Fail_Cmd_Data_tag@@U?$less@K@std@@V?$allocator@U?$pair@$$CBKU__Fail_Cmd_Data_tag@@@std@@@3@$0A@@std@@@std@@KAABKPAU_Node@?$_Tree_nod@V?$_Tmap_traits@KU__Fail_Cmd_Data_tag@@U?$less@K@std@@V?$allocator@U?$pair@$$CBKU__Fail_Cmd_Data_tag@@@std@@@3@$0A@@std@@@2@@Z 00173680 f i rilhandndis.obj
 0001:000726c4       ?insert@?$_Tree@V?$_Tmap_traits@KU__Fail_Cmd_Data_tag@@U?$less@K@std@@V?$allocator@U?$pair@$$CBKU__Fail_Cmd_Data_tag@@@std@@@3@$0A@@std@@@std@@QAA?AViterator@12@V312@ABU?$pair@$$CBKU__Fail_Cmd_Data_tag@@@2@@Z 001736c4 f i rilhandndis.obj
 0001:000735e0       ?lower_bound@?$_Tree@V?$_Tmap_traits@KU__Fail_Cmd_Data_tag@@U?$less@K@std@@V?$allocator@U?$pair@$$CBKU__Fail_Cmd_Data_tag@@@std@@@3@$0A@@std@@@std@@QAA?AViterator@12@ABK@Z 001745e0 f i rilhandndis.obj
 0001:0007363c       ??Diterator@?$_Tree@V?$_Tmap_traits@KU__Fail_Cmd_Data_tag@@U?$less@K@std@@V?$allocator@U?$pair@$$CBKU__Fail_Cmd_Data_tag@@@std@@@3@$0A@@std@@@std@@QBAAAU?$pair@$$CBKU__Fail_Cmd_Data_tag@@@2@XZ 0017463c f i rilhandndis.obj
 0001:0007366c       ??0?$pair@$$CBKU__Fail_Cmd_Data_tag@@@std@@QAA@ABKABU__Fail_Cmd_Data_tag@@@Z 0017466c f i rilhandndis.obj
 0001:000736b4       ??1?$pair@Viterator@?$_Tree@V?$_Tmap_traits@KU__Fail_Cmd_Data_tag@@U?$less@K@std@@V?$allocator@U?$pair@$$CBKU__Fail_Cmd_Data_tag@@@std@@@3@$0A@@std@@@std@@_N@std@@QAA@XZ 001746b4 f i rilhandndis.obj
 0001:000736cc       ?_Myval@?$_Tree@V?$_Tmap_traits@KU__Fail_Cmd_Data_tag@@U?$less@K@std@@V?$allocator@U?$pair@$$CBKU__Fail_Cmd_Data_tag@@@std@@@3@$0A@@std@@@std@@KAAAU?$pair@$$CBKU__Fail_Cmd_Data_tag@@@2@PAU_Node@?$_Tree_nod@V?$_Tmap_traits@KU__Fail_Cmd_Data_tag@@U?$less@K@std@@V?$allocator@U?$pair@$$CBKU__Fail_Cmd_Data_tag@@@std@@@3@$0A@@std@@@2@@Z 001746cc f i rilhandndis.obj
 0001:000736f4       ?size@?$_Tree@V?$_Tmap_traits@KU__Fail_Cmd_Data_tag@@U?$less@K@std@@V?$allocator@U?$pair@$$CBKU__Fail_Cmd_Data_tag@@@std@@@3@$0A@@std@@@std@@QBAIXZ 001746f4 f i rilhandndis.obj
 0001:00073728       ?insert@?$_Tree@V?$_Tmap_traits@KU__Fail_Cmd_Data_tag@@U?$less@K@std@@V?$allocator@U?$pair@$$CBKU__Fail_Cmd_Data_tag@@@std@@@3@$0A@@std@@@std@@QAA?AU?$pair@Viterator@?$_Tree@V?$_Tmap_traits@KU__Fail_Cmd_Data_tag@@U?$less@K@std@@V?$allocator@U?$pair@$$CBKU__Fail_Cmd_Data_tag@@@std@@@3@$0A@@std@@@std@@_N@2@ABU?$pair@$$CBKU__Fail_Cmd_Data_tag@@@2@@Z 00174728 f i rilhandndis.obj
 0001:00073b90       ?_Insert@?$_Tree@V?$_Tmap_traits@KU__Fail_Cmd_Data_tag@@U?$less@K@std@@V?$allocator@U?$pair@$$CBKU__Fail_Cmd_Data_tag@@@std@@@3@$0A@@std@@@std@@IAA?AViterator@12@_NPAU_Node@?$_Tree_nod@V?$_Tmap_traits@KU__Fail_Cmd_Data_tag@@U?$less@K@std@@V?$allocator@U?$pair@$$CBKU__Fail_Cmd_Data_tag@@@std@@@3@$0A@@std@@@2@ABU?$pair@$$CBKU__Fail_Cmd_Data_tag@@@2@@Z 00174b90 f i rilhandndis.obj
 0001:0007424c       ?_Lbound@?$_Tree@V?$_Tmap_traits@KU__Fail_Cmd_Data_tag@@U?$less@K@std@@V?$allocator@U?$pair@$$CBKU__Fail_Cmd_Data_tag@@@std@@@3@$0A@@std@@@std@@IBAPAU_Node@?$_Tree_nod@V?$_Tmap_traits@KU__Fail_Cmd_Data_tag@@U?$less@K@std@@V?$allocator@U?$pair@$$CBKU__Fail_Cmd_Data_tag@@@std@@@3@$0A@@std@@@2@ABK@Z 0017524c f i rilhandndis.obj
 0001:00074344       ?_Kfn@?$_Tmap_traits@KU__Fail_Cmd_Data_tag@@U?$less@K@std@@V?$allocator@U?$pair@$$CBKU__Fail_Cmd_Data_tag@@@std@@@3@$0A@@std@@SAABKABU?$pair@$$CBKU__Fail_Cmd_Data_tag@@@2@@Z 00175344 f i rilhandndis.obj
 0001:00074368       ??0iterator@?$_Tree@V?$_Tmap_traits@KU__Fail_Cmd_Data_tag@@U?$less@K@std@@V?$allocator@U?$pair@$$CBKU__Fail_Cmd_Data_tag@@@std@@@3@$0A@@std@@@std@@QAA@XZ 00175368 f i rilhandndis.obj
 0001:00074398       ??Fiterator@?$_Tree@V?$_Tmap_traits@KU__Fail_Cmd_Data_tag@@U?$less@K@std@@V?$allocator@U?$pair@$$CBKU__Fail_Cmd_Data_tag@@@std@@@3@$0A@@std@@@std@@QAAAAV012@XZ 00175398 f i rilhandndis.obj
 0001:000743c4       ??Dconst_iterator@?$_Tree@V?$_Tmap_traits@KU__Fail_Cmd_Data_tag@@U?$less@K@std@@V?$allocator@U?$pair@$$CBKU__Fail_Cmd_Data_tag@@@std@@@3@$0A@@std@@@std@@QBAABU?$pair@$$CBKU__Fail_Cmd_Data_tag@@@2@XZ 001753c4 f i rilhandndis.obj
 0001:000744a0       ?max_size@?$_Tree@V?$_Tmap_traits@KU__Fail_Cmd_Data_tag@@U?$less@K@std@@V?$allocator@U?$pair@$$CBKU__Fail_Cmd_Data_tag@@@std@@@3@$0A@@std@@@std@@QBAIXZ 001754a0 f i rilhandndis.obj
 0001:000744dc       ?_Buynode@?$_Tree@V?$_Tmap_traits@KU__Fail_Cmd_Data_tag@@U?$less@K@std@@V?$allocator@U?$pair@$$CBKU__Fail_Cmd_Data_tag@@@std@@@3@$0A@@std@@@std@@IAAPAU_Node@?$_Tree_nod@V?$_Tmap_traits@KU__Fail_Cmd_Data_tag@@U?$less@K@std@@V?$allocator@U?$pair@$$CBKU__Fail_Cmd_Data_tag@@@std@@@3@$0A@@std@@@2@PAU342@00ABU?$pair@$$CBKU__Fail_Cmd_Data_tag@@@2@D@Z 001754dc f i rilhandndis.obj
 0001:000745f8       ??0const_iterator@?$_Tree@V?$_Tmap_traits@KU__Fail_Cmd_Data_tag@@U?$less@K@std@@V?$allocator@U?$pair@$$CBKU__Fail_Cmd_Data_tag@@@std@@@3@$0A@@std@@@std@@QAA@XZ 001755f8 f i rilhandndis.obj
 0001:00074638       ??Fconst_iterator@?$_Tree@V?$_Tmap_traits@KU__Fail_Cmd_Data_tag@@U?$less@K@std@@V?$allocator@U?$pair@$$CBKU__Fail_Cmd_Data_tag@@@std@@@3@$0A@@std@@@std@@QAAAAV012@XZ 00175638 f i rilhandndis.obj
 0001:00074664       ??0?$pair@Viterator@?$_Tree@V?$_Tmap_traits@KU__Fail_Cmd_Data_tag@@U?$less@K@std@@V?$allocator@U?$pair@$$CBKU__Fail_Cmd_Data_tag@@@std@@@3@$0A@@std@@@std@@_N@std@@QAA@ABViterator@?$_Tree@V?$_Tmap_traits@KU__Fail_Cmd_Data_tag@@U?$less@K@std@@V?$allocator@U?$pair@$$CBKU__Fail_Cmd_Data_tag@@@std@@@3@$0A@@std@@@1@AB_N@Z 00175664 f i rilhandndis.obj
 0001:000746ac       ?max_size@?$allocator@U?$pair@$$CBKU__Fail_Cmd_Data_tag@@@std@@@std@@QBAIXZ 001756ac f i rilhandndis.obj
 0001:000746fc       ?_Dec@const_iterator@?$_Tree@V?$_Tmap_traits@KU__Fail_Cmd_Data_tag@@U?$less@K@std@@V?$allocator@U?$pair@$$CBKU__Fail_Cmd_Data_tag@@@std@@@3@$0A@@std@@@std@@QAAXXZ 001756fc f i rilhandndis.obj
 0001:000749fc       ??0_Node@?$_Tree_nod@V?$_Tmap_traits@KU__Fail_Cmd_Data_tag@@U?$less@K@std@@V?$allocator@U?$pair@$$CBKU__Fail_Cmd_Data_tag@@@std@@@3@$0A@@std@@@std@@QAA@PAU012@00ABU?$pair@$$CBKU__Fail_Cmd_Data_tag@@@2@D@Z 001759fc f i rilhandndis.obj
 0001:00074a80       ?RILDrv_SetDTMFMonitoring@@YAJKH@Z 00175a80 f   rilmain.obj
 0001:00074b28       ?RILDrv_GetAudioDevices@@YAJK@Z 00175b28 f   rilmain.obj
 0001:00074bd0       ?RILDrv_FetchSimToolkitCmd@@YAJK@Z 00175bd0 f   rilmain.obj
 0001:00074c78       ?RILDrv_SetHideConnectedIdStatus@@YAJKK@Z 00175c78 f   rilmain.obj
 0001:00074d20       ?RILDrv_GetCCBSStatus@@YAJKK@Z 00175d20 f   rilmain.obj
 0001:00074dc8       ?RILDrv_ClearCCBSRegistration@@YAJKK@Z 00175dc8 f   rilmain.obj
 0001:00074e70       DllMain                    00175e70 f   rilmain.obj
 0001:00074fb8       ?RIL_Init@@YAKK@Z          00175fb8 f   rilmain.obj
 0001:0007558c       ?RIL_Deinit@@YAHK@Z        0017658c f   rilmain.obj
 0001:00075750       ?RIL_Open@@YAKKKK@Z        00176750 f   rilmain.obj
 0001:000759e4       ?RIL_Close@@YAHK@Z         001769e4 f   rilmain.obj
 0001:00075c50       ?RIL_Read@@YAKKPAXK@Z      00176c50 f   rilmain.obj
 0001:00075c74       ?RIL_Write@@YAKKPBXK@Z     00176c74 f   rilmain.obj
 0001:00075c98       ?RIL_Seek@@YAKKJK@Z        00176c98 f   rilmain.obj
 0001:00075cbc       ?RIL_PowerDown@@YAXK@Z     00176cbc f   rilmain.obj
 0001:00075ccc       ?RIL_PowerUp@@YAXK@Z       00176ccc f   rilmain.obj
 0001:00075ce4       ?RIL_IOControl@@YAHKKPAEK0KPAK@Z 00176ce4 f   rilmain.obj
 0001:0007b784       ?RILDrv_GetNextNotification@@YAJKPAUrildrvnotification_tag@@@Z 0017c784 f   rilmain.obj
 0001:0007b850       ?RILDrv_GetSerialPortStatistics@@YAJKPAUrilserialportstats_tag@@@Z 0017c850 f   rilmain.obj
 0001:0007b8d4       ?ClearCmdHandle@@YAHPAXK@Z 0017c8d4 f   rilmain.obj
 0001:0007baec       ?ExtractHandle@@YAQAVCRilInstanceHandle@@K@Z 0017caec f   rilmain.obj
 0001:0007bc04       ?SignalCriticalError@@YAXK@Z 0017cc04 f   rilmain.obj
 0001:0007bcc0       ?hex2bin@@YAEEE@Z          0017ccc0 f   rilmain.obj
 0001:0007bdb4       ?DoFirmwareUpgrade@CRadio@@QAAHH@Z 0017cdb4 f   rilmain.obj
 0001:0007cff0       ??_GCRilHandle@@QAAPAXI@Z  0017dff0 f i rilmain.obj
 0001:0007d030       ?ClearHandle@CCommand@@QAAXXZ 0017e030 f i rilmain.obj
 0001:0007d058       ?Enum@?$CDblList@VCCommand@@@@QAAXQ6AHPAXK@ZK@Z 0017e058 f i rilmain.obj
 0001:0007d114       ?SwiGetProcAddress@@YAP6AHXZPAUHINSTANCE__@@PBG@Z 0017e114 f   SDK7Wrapper.obj
 0001:0007d1a4       ??0CSDK7@@QAA@XZ           0017e1a4 f   SDK7Wrapper.obj
 0001:0007d208       ??1CSDK7@@QAA@XZ           0017e208 f   SDK7Wrapper.obj
 0001:0007d220       ?Cleanup@CSDK7@@QAAXXZ     0017e220 f   SDK7Wrapper.obj
 0001:0007ddc4       ?Initialize@CSDK7@@QAA_NXZ 0017edc4 f   SDK7Wrapper.obj
 0001:00080684       ?GetDLLVersion@CSDK7@@QAAKXZ 00181684 f   SDK7Wrapper.obj
 0001:000806b0       ?RILDrv_GetPhoneLockedState@@YAJK@Z 001816b0 f   secur.obj
 0001:00080790       ?GetPhoneLockedState@CRadio@@QAAJPAVCResponse@@@Z 00181790 f   secur.obj
 0001:00080a00       ?RILDrv_UnlockPhone@@YAJKPBD0@Z 00181a00 f   secur.obj
 0001:00080c6c       ?UnlockPhone@CRadio@@QAAJPAVCResponse@@PAX@Z 00181c6c f   secur.obj
 0001:00080ff8       ?RILDrv_ChangeLockingPassword@@YAJKKKPBD0@Z 00181ff8 f   secur.obj
 0001:00081418       ?ChangeLockingPassword@CRadio@@QAAJPAVCResponse@@PAX@Z 00182418 f   secur.obj
 0001:00081804       ?RILDrv_SetLockingStatus@@YAJKKPBDK@Z 00182804 f   secur.obj
 0001:000819d4       ?SetLockingStatus@CRadio@@QAAJPAVCResponse@@PAX@Z 001829d4 f   secur.obj
 0001:00081c88       ?RILDrv_GetLockingStatus@@YAJKKPBD@Z 00182c88 f   secur.obj
 0001:00081e44       ?GetLockingStatus@CRadio@@QAAJPAVCResponse@@PAX@Z 00182e44 f   secur.obj
 0001:0008211c       ?RILDrv_GetUserIdentity@@YAJK@Z 0018311c f   secur.obj
 0001:00082208       ?GetUserIdentity@CRadio@@QAAJPAVCResponse@@@Z 00183208 f   secur.obj
 0001:000826f4       ?RILDrv_GetCallBarringStatus@@YAJKKKPBD@Z 001836f4 f   secur.obj
 0001:000829f0       ?RILDrv_SetCallBarringStatus@@YAJKKKPBDK@Z 001839f0 f   secur.obj
 0001:00082dd4       ?RILDrv_ChangeCallBarringPassword@@YAJKKPBD0@Z 00183dd4 f   secur.obj
 0001:00083130       ?GetCallBarringStatus@CRadio@@QAAJPAVCResponse@@PAX@Z 00184130 f   secur.obj
 0001:00083394       ?SetCallBarringStatus@CRadio@@QAAJPAVCResponse@@PAX@Z 00184394 f   secur.obj
 0001:00083638       ?ChangeCallBarringPassword@CRadio@@QAAJPAVCResponse@@PAX@Z 00184638 f   secur.obj
 0001:000837fc       ?SemiByteCharsToByte@@YAEDD@Z 001847fc f   smscb.obj
 0001:000838b8       ?GSMHexToGSM@@YAHQBDIQADIAAI@Z 001848b8 f   smscb.obj
 0001:000839a0       ?ParseCellBroadcastMessage@@YAJPBEIAAUrilmessage_tag@@@Z 001849a0 f   smscb.obj
 0001:00084358       ?RILDrv_GetCallerIdSettings@@YAJK@Z 00185358 f   supsvc.obj
 0001:00084470       ?RILDrv_SetCallerIdStatus@@YAJKK@Z 00185470 f   supsvc.obj
 0001:00084670       ?RILDrv_GetHideIdSettings@@YAJK@Z 00185670 f   supsvc.obj
 0001:00084750       ?RILDrv_SetHideIdStatus@@YAJKK@Z 00185750 f   supsvc.obj
 0001:00084990       ?RILDrv_GetDialedIdSettings@@YAJK@Z 00185990 f   supsvc.obj
 0001:00084aac       ?RILDrv_SetDialedIdStatus@@YAJKK@Z 00185aac f   supsvc.obj
 0001:00084ce8       ?RILDrv_GetHideConnectedIdSettings@@YAJK@Z 00185ce8 f   supsvc.obj
 0001:00084dcc       ?RILDrv_GetCallForwardingSettings@@YAJKKK@Z 00185dcc f   supsvc.obj
 0001:000850a4       ?RILDrv_AddCallForwarding@@YAJKKPBUrilcallforwardingsettings_tag@@@Z 001860a4 f   supsvc.obj
 0001:00085440       ?RILDrv_RemoveCallForwarding@@YAJKKK@Z 00186440 f   supsvc.obj
 0001:00085714       ?RILDrv_SetCallForwardingStatus@@YAJKKKK@Z 00186714 f   supsvc.obj
 0001:00085a60       ?RILDrv_GetCallWaitingSettings@@YAJKK@Z 00186a60 f   supsvc.obj
 0001:00085ce0       ?RILDrv_SetCallWaitingStatus@@YAJKKK@Z 00186ce0 f   supsvc.obj
 0001:00086290       ?RILDrv_SendSupServiceData@@YAJKPBEK@Z 00187290 f   supsvc.obj
 0001:00086568       ?RILDrv_CancelSupServiceDataSession@@YAJK@Z 00187568 f   supsvc.obj
 0001:00086684       ?SendSupSvcsThreadProc@@YAKPAX@Z 00187684 f   supsvc.obj
 0001:0008680c       ?GetCallerIdSettings@CRadio@@QAAJPAVCResponse@@@Z 0018780c f   supsvc.obj
 0001:000869e0       ?SetCallerIdStatus@CRadio@@QAAJPAVCResponse@@PAX@Z 001879e0 f   supsvc.obj
 0001:00086b24       ?GetHideIdSettings@CRadio@@QAAJPAVCResponse@@@Z 00187b24 f   supsvc.obj
 0001:00086e1c       ?SetHideIdStatus@CRadio@@QAAJPAVCResponse@@PAX@Z 00187e1c f   supsvc.obj
 0001:00087034       ?GetDialedIdSettings@CRadio@@QAAJPAVCResponse@@@Z 00188034 f   supsvc.obj
 0001:00087228       ?SetDialedIdStatus@CRadio@@QAAJPAVCResponse@@PAX@Z 00188228 f   supsvc.obj
 0001:000872b0       ?GetCallForwardingSettings@CRadio@@QAAJPAVCResponse@@PAX@Z 001882b0 f   supsvc.obj
 0001:00087a68       ?AddCallForwarding@CRadio@@QAAJPAVCResponse@@PAX@Z 00188a68 f   supsvc.obj
 0001:00087e14       ?SetCallForwarding@CRadio@@QAAJPAVCResponse@@PAX@Z 00188e14 f   supsvc.obj
 0001:00088160       ?RemoveCallForwarding@CRadio@@QAAJPAVCResponse@@PAX@Z 00189160 f   supsvc.obj
 0001:00088394       ?GetCallWaitingSettings@CRadio@@QAAJPAVCResponse@@PAX@Z 00189394 f   supsvc.obj
 0001:00088798       ?SetCallWaitingStatus@CRadio@@QAAJPAVCResponse@@PAX@Z 00189798 f   supsvc.obj
 0001:000889f4       ?SendSupServiceData@CRadio@@QAAJPAVCResponse@@PAX@Z 001899f4 f   supsvc.obj
 0001:00088d58       ?SendUSSD@CRadio@@QAAXPAG@Z 00189d58 f   supsvc.obj
 0001:000891e4       ?CancelSupServiceDataSession@CRadio@@QAAJPAVCResponse@@@Z 0018a1e4 f   supsvc.obj
 0001:000892f0       ?GetHideConnectedIdSettings@CRadio@@QAAJPAVCResponse@@@Z 0018a2f0 f   supsvc.obj
 0001:000894e8       ?SetEnum@CRadio@@QAAJPAD@Z 0018a4e8 f   supsvc.obj
 0001:00089668       ?ClearEnum@CRadio@@QAAJXZ  0018a668 f   supsvc.obj
 0001:000897dc       ?GetDevCapsInfoClasses@CRadioCaps@@QAAXAAPAXAAI@Z 0018a7dc f i supsvc.obj
 0001:00089808       ??_G__Send_SupSvcs_USSD_Data_tag@@QAAPAXI@Z 0018a808 f i supsvc.obj
 0001:00089848       ??1__Send_SupSvcs_USSD_Data_tag@@QAA@XZ 0018a848 f i supsvc.obj
 0001:00089878       ?_tcsncpyz@@YAPAGQAGQBGI@Z 0018a878 f   toolbox.obj
 0001:00089920       ?_tcsncatz@@YAPAGQAGQBGI@Z 0018a920 f   toolbox.obj
 0001:000899fc       ?strncpyz@@YAPADQADQBDI@Z  0018a9fc f   toolbox.obj
 0001:00089a9c       ?strncatz@@YAPADQADQBDI@Z  0018aa9c f   toolbox.obj
 0001:00089b68       ?wcsncpyz@@YAPAGQAGQBGI@Z  0018ab68 f   toolbox.obj
 0001:00089c10       ?wcsncatz@@YAPAGQAGQBGI@Z  0018ac10 f   toolbox.obj
 0001:00089cec       ?_sntprintfz@@YAHQAGIQBGZZ 0018acec f   toolbox.obj
 0001:00089db4       ?_snprintfz@@YAHQADIQBDZZ  0018adb4 f   toolbox.obj
 0001:00089e74       ?_snwprintfz@@YAHQAGIQBGZZ 0018ae74 f   toolbox.obj
 0001:00089f3c       ?GetRegistryDWORD@@YA_NQAUHKEY__@@QBG1QAK@Z 0018af3c f   toolbox.obj
 0001:0008a050       ?SetRegistryDWORD@@YA_NQAUHKEY__@@QBG1K@Z 0018b050 f   toolbox.obj
 0001:0008a12c       ?GetRegistryBoolean@@YA_NQAUHKEY__@@QBG1QA_N@Z 0018b12c f   toolbox.obj
 0001:0008a1bc       ?SetRegistryBoolean@@YA_NQAUHKEY__@@QBG1_N@Z 0018b1bc f   toolbox.obj
 0001:0008a220       ?GetRegistryBINARY@@YA_NQAUHKEY__@@QBG1QAEK@Z 0018b220 f   toolbox.obj
 0001:0008a320       ?SetRegistryBINARY@@YA_NQAUHKEY__@@QBG1QBEK@Z 0018b320 f   toolbox.obj
 0001:0008a408       ?GetRegistrySZ@@YA_NQAUHKEY__@@QBG1QAGK@Z 0018b408 f   toolbox.obj
 0001:0008a520       ?SetRegistrySZ@@YA_NQAUHKEY__@@QBG11@Z 0018b520 f   toolbox.obj
 0001:0008a620       ?BoundedRandom@@YAHHH@Z    0018b620 f   toolbox.obj
 0001:0008a77c       ??0ResourceString@@QAA@XZ  0018b77c f   toolbox.obj
 0001:0008a7ac       ??0ResourceString@@QAA@PAUHINSTANCE__@@I@Z 0018b7ac f   toolbox.obj
 0001:0008a7ec       ?LoadResourceString@ResourceString@@QAAPBGPAUHINSTANCE__@@I@Z 0018b7ec f   toolbox.obj
 0001:0008a944       ??BResourceString@@QAAPBGXZ 0018b944 f   toolbox.obj
 0001:0008a994       ??1ResourceString@@QAA@XZ  0018b994 f   toolbox.obj
 0001:0008a9b0       ??0CommandLineTokenizer@@QAA@XZ 0018b9b0 f   toolbox.obj
 0001:0008a9f0       ??0CommandLineTokenizer@@QAA@PBG@Z 0018b9f0 f   toolbox.obj
 0001:0008aa2c       ??1CommandLineTokenizer@@QAA@XZ 0018ba2c f   toolbox.obj
 0001:0008aa58       ?SetCommandLine@CommandLineTokenizer@@QAA_NPBG@Z 0018ba58 f   toolbox.obj
 0001:0008ab6c       ?NextParameter@CommandLineTokenizer@@QAAPAGXZ 0018bb6c f   toolbox.obj
 0001:0008ae98       ??0CommandLineParameterHandler@@QAA@QBGQAPBGQAP6A_N0@ZQ6A_N0@Z@Z 0018be98 f   toolbox.obj
 0001:0008af20       ?ProcessParameters@CommandLineParameterHandler@@QAA_NXZ 0018bf20 f   toolbox.obj
 0001:0008b178       ??0AnsiString@@QAA@QBGG@Z  0018c178 f   toolbox.obj
 0001:0008b358       ??0AnsiString@@QAA@QBDD@Z  0018c358 f   toolbox.obj
 0001:0008b48c       ??1AnsiString@@QAA@XZ      0018c48c f   toolbox.obj
 0001:0008b4b8       ??0WideString@@QAA@QBDD@Z  0018c4b8 f   toolbox.obj
 0001:0008b684       ??0WideString@@QAA@QBGG@Z  0018c684 f   toolbox.obj
 0001:0008b7d0       ??1WideString@@QAA@XZ      0018c7d0 f   toolbox.obj
 0001:0008b7fc       ??0USAsciiString@@QAA@PBG@Z 0018c7fc f   toolbox.obj
 0001:0008b918       ??0USAsciiString@@QAA@QBD@Z 0018c918 f   toolbox.obj
 0001:0008b9c0       ??1USAsciiString@@QAA@XZ   0018c9c0 f   toolbox.obj
 0001:0008b9ec       ??0VerboseString@@QAA@QBGGG@Z 0018c9ec f   toolbox.obj
 0001:0008bce8       ??1VerboseString@@QAA@XZ   0018cce8 f   toolbox.obj
 0001:0008bd14       ??0PrintableString@@QAA@QBDI_NDD@Z 0018cd14 f   toolbox.obj
 0001:0008c084       ??1PrintableString@@QAA@XZ 0018d084 f   toolbox.obj
 0001:0008c0b0       ??0HexString@@QAA@QBDI@Z   0018d0b0 f   toolbox.obj
 0001:0008c1c8       ??1HexString@@QAA@XZ       0018d1c8 f   toolbox.obj
 0001:0008c1f4       ??0StringCollection@@QAA@XZ 0018d1f4 f   toolbox.obj
 0001:0008c23c       ??1StringCollection@@UAA@XZ 0018d23c f   toolbox.obj
 0001:0008c268       ?AddString@StringCollection@@UAA_NQBGQAH@Z 0018d268 f   toolbox.obj
 0001:0008c35c       ?GetString@StringCollection@@UAAPAGH@Z 0018d35c f   toolbox.obj
 0001:0008c394       ?GetSize@StringCollection@@UAAHXZ 0018d394 f   toolbox.obj
 0001:0008c3e0       ??0SortedStringCollection@@QAA@_N@Z 0018d3e0 f   toolbox.obj
 0001:0008c458       ??1SortedStringCollection@@UAA@XZ 0018d458 f   toolbox.obj
 0001:0008c480       ?AddString@SortedStringCollection@@UAA_NQBG_N@Z 0018d480 f   toolbox.obj
 0001:0008c68c       ?FindStringIndex@SortedStringCollection@@QAAHQBG@Z 0018d68c f   toolbox.obj
 0001:0008c820       ??0CCheckPoint@@QAA@XZ     0018d820 f   toolbox.obj
 0001:0008c88c       ??1CCheckPoint@@QAA@XZ     0018d88c f   toolbox.obj
 0001:0008c910       ?Init@CCheckPoint@@QAA_NI@Z 0018d910 f   toolbox.obj
 0001:0008ca80       ?Reached@CCheckPoint@@QAAXXZ 0018da80 f   toolbox.obj
 0001:0008cbb8       ?Wait@CCheckPoint@@QAA_NK@Z 0018dbb8 f   toolbox.obj
 0001:0008cce8       ?bsearch@@YAPAXPBX0IIP6AH00@Z@Z 0018dce8 f   toolbox.obj
 0001:0008cea8       ?MemoryReadable@@YA_NPBXI@Z 0018dea8 f   toolbox.obj
 0001:0008cf00       ?MemoryWriteable@@YA_NPAXI@Z 0018df00 f   toolbox.obj
 0001:0008cf60       ?_tcsReadable@@YA_NPBG@Z   0018df60 f   toolbox.obj
 0001:0008cfcc       ?_tcsWriteable@@YA_NPAG@Z  0018dfcc f   toolbox.obj
 0001:0008d060       ?strReadable@@YA_NPBD@Z    0018e060 f   toolbox.obj
 0001:0008d0cc       ?strWriteable@@YA_NPAD@Z   0018e0cc f   toolbox.obj
 0001:0008d158       ?wcsReadable@@YA_NPBG@Z    0018e158 f   toolbox.obj
 0001:0008d1c4       ?wcsWriteable@@YA_NPAG@Z   0018e1c4 f   toolbox.obj
 0001:0008d258       ??0TaskList@@QAA@I@Z       0018e258 f   toolbox.obj
 0001:0008d3f8       ??1TaskList@@QAA@XZ        0018e3f8 f   toolbox.obj
 0001:0008d5bc       ?AddTask@TaskList@@QAA_NPAIP6A_NPAX@Z1W4TaskListUrgency@1@@Z 0018e5bc f   toolbox.obj
 0001:0008d8a8       ?RemoveTask@TaskList@@QAA_NI@Z 0018e8a8 f   toolbox.obj
 0001:0008db94       ?TasksRemaining@TaskList@@QAAIXZ 0018eb94 f   toolbox.obj
 0001:0008dc98       ?AddWorkerThread@TaskList@@AAA_NXZ 0018ec98 f   toolbox.obj
 0001:0008dd94       ?TaskListThreadProc@@YAKPAX@Z 0018ed94 f   toolbox.obj
 0001:0008e0a4       ??0WorkerThread@@QAA@Q6AKPAX0@ZQAXK@Z 0018f0a4 f   toolbox.obj
 0001:0008e114       ??1WorkerThread@@QAA@XZ    0018f114 f   toolbox.obj
 0001:0008e12c       ?StartWorkerThread@WorkerThread@@QAA_NXZ 0018f12c f   toolbox.obj
 0001:0008e2b4       ?StopWorkerThread@WorkerThread@@QAA_NXZ 0018f2b4 f   toolbox.obj
 0001:0008e3b4       ?RunWorkerThreadProc@WorkerThread@@CAKPAX@Z 0018f3b4 f   toolbox.obj
 0001:0008e464       ??0MemoryMappedFileData@@QAA@XZ 0018f464 f   toolbox.obj
 0001:0008e4d4       ??1MemoryMappedFileData@@QAA@XZ 0018f4d4 f   toolbox.obj
 0001:0008e550       ?Initialize@MemoryMappedFileData@@QAA_NQBG@Z 0018f550 f   toolbox.obj
 0001:0008e704       ??0StringBuffer@@QAA@I@Z   0018f704 f   toolbox.obj
 0001:0008e764       ??1StringBuffer@@QAA@XZ    0018f764 f   toolbox.obj
 0001:0008e77c       ?Set@StringBuffer@@QAA_NQBG@Z 0018f77c f   toolbox.obj
 0001:0008e874       ?Append@StringBuffer@@QAA_NQBG@Z 0018f874 f   toolbox.obj
 0001:0008e988       ?Append@StringBuffer@@QAA_NQBGI@Z 0018f988 f   toolbox.obj
 0001:0008eab0       ?Empty@StringBuffer@@QAAXXZ 0018fab0 f   toolbox.obj
 0001:0008eb68       ?FreeMemory@StringBuffer@@QAAXXZ 0018fb68 f   toolbox.obj
 0001:0008ec4c       ?EnsureSpaceToAddStringLength@StringBuffer@@AAA_NI@Z 0018fc4c f   toolbox.obj
 0001:0008eed4       ?GetSystemTimeAsFileTime@@YAXPAU_FILETIME@@@Z 0018fed4 f   toolbox.obj
 0001:0008ef00       ?WaitForSingleObjectReset@@YAKPAXK@Z 0018ff00 f   toolbox.obj
 0001:0008f01c       ??_EStringCollection@@UAAPAXI@Z 0019001c f i toolbox.obj
 0001:0008f01c       ??_GStringCollection@@UAAPAXI@Z 0019001c f i toolbox.obj
 0001:0008f05c       ??_GSortedStringCollection@@UAAPAXI@Z 0019005c f i toolbox.obj
 0001:0008f05c       ??_ESortedStringCollection@@UAAPAXI@Z 0019005c f i toolbox.obj
 0001:0008f09c       ??0UNSYNCBLOCK_Implementation@@QAA@AAUCRITICAL_SECTION@@@Z 0019009c f i toolbox.obj
 0001:0008f0d8       ??1UNSYNCBLOCK_Implementation@@QAA@XZ 001900d8 f i toolbox.obj
 0001:0008f0f4       ??0?$GrowablePointerCollection@G@@QAA@H@Z 001900f4 f i toolbox.obj
 0001:0008f170       ??1?$GrowablePointerCollection@G@@UAA@XZ 00190170 f i toolbox.obj
 0001:0008f214       ?AddPointer@?$GrowablePointerCollection@G@@QAA_NQBG@Z 00190214 f i toolbox.obj
 0001:0008f290       ?InsertPointer@?$GrowablePointerCollection@G@@QAA_NQBGH@Z 00190290 f i toolbox.obj
 0001:0008f30c       ?RemoveThingAtIndex@?$GrowablePointerCollection@G@@UAA_NH@Z 0019030c f i toolbox.obj
 0001:0008f370       ?RemoveAllThings@?$GrowablePointerCollection@G@@UAA_NXZ 00190370 f i toolbox.obj
 0001:0008f3d0       ?SwapThingsAtIndices@?$GrowablePointerCollection@G@@UAA_NHH@Z 001903d0 f i toolbox.obj
 0001:0008f434       ?GetPointerAtIndex@?$GrowablePointerCollection@G@@QAAPAGH@Z 00190434 f i toolbox.obj
 0001:0008f51c       ?GetThingAtIndex@?$GrowablePointerCollection@G@@UAAPAGH@Z 0019051c f i toolbox.obj
 0001:0008f57c       ?GetPointerIndex@?$GrowablePointerCollection@G@@QAAHPBG@Z 0019057c f i toolbox.obj
 0001:0008f62c       ?GetFilteredThingIndex@?$GrowablePointerCollection@G@@UAAHP6A_NABQAGPAX@ZQAX@Z 0019062c f i toolbox.obj
 0001:0008f690       ?GetPointerToThingAtIndex@?$GrowablePointerCollection@G@@UAAPAPAGH@Z 00190690 f i toolbox.obj
 0001:0008f6f4       ??1?$GrowableThingCollection@PAG@@UAA@XZ 001906f4 f i toolbox.obj
 0001:0008f7a8       ?AddThing@?$GrowableThingCollection@PAG@@UAA_NQAG@Z 001907a8 f i toolbox.obj
 0001:0008f894       ?InsertThing@?$GrowableThingCollection@PAG@@UAA_NQAGH@Z 00190894 f i toolbox.obj
 0001:0008fa58       ?RemoveThingAtIndex@?$GrowableThingCollection@PAG@@UAA_NH@Z 00190a58 f i toolbox.obj
 0001:0008fbd0       ?RemoveThing@?$GrowableThingCollection@PAG@@UAA_NQAG@Z 00190bd0 f i toolbox.obj
 0001:0008fcfc       ?RemoveAllThings@?$GrowableThingCollection@PAG@@UAA_NXZ 00190cfc f i toolbox.obj
 0001:0008fd84       ?SwapThingsAtIndices@?$GrowableThingCollection@PAG@@UAA_NHH@Z 00190d84 f i toolbox.obj
 0001:0008ff4c       ?GetSize@?$GrowableThingCollection@PAG@@UAAHXZ 00190f4c f i toolbox.obj
 0001:0008ff98       ?Lock@?$GrowableThingCollection@PAG@@UAA_NXZ 00190f98 f i toolbox.obj
 0001:00090040       ?Unlock@?$GrowableThingCollection@PAG@@UAA_NXZ 00191040 f i toolbox.obj
 0001:00090124       ?BlockModificationByOtherThreads@?$GrowableThingCollection@PAG@@UAA_NXZ 00191124 f i toolbox.obj
 0001:00090154       ?AllowModificationByOtherThreads@?$GrowableThingCollection@PAG@@UAA_NXZ 00191154 f i toolbox.obj
 0001:00090184       ?GetThingAtIndex@?$GrowableThingCollection@PAG@@UAAPAGH@Z 00191184 f i toolbox.obj
 0001:00090278       ?SetThingAtIndex@?$GrowableThingCollection@PAG@@UAA_NQAGH@Z 00191278 f i toolbox.obj
 0001:0009036c       ?GetThingIndex@?$GrowableThingCollection@PAG@@UAAHQAG@Z 0019136c f i toolbox.obj
 0001:00090428       ?GetFilteredThingIndex@?$GrowableThingCollection@PAG@@UAAHP6A_NABQAGPAX@ZQAX@Z 00191428 f i toolbox.obj
 0001:00090538       ?GetPointerToThingAtIndex@?$GrowableThingCollection@PAG@@UAAPAPAGH@Z 00191538 f i toolbox.obj
 0001:00090678       ?GetPointerToThing@?$GrowableThingCollection@PAG@@UAAPAPAGQAG@Z 00191678 f i toolbox.obj
 0001:000907b8       ?MakeRoomForAnotherThing@?$GrowableThingCollection@PAG@@MAA_NXZ 001917b8 f i toolbox.obj
 0001:00090928       ??0?$GrowableThingCollection@PAX@@QAA@H@Z 00191928 f i toolbox.obj
 0001:00090a2c       ??1?$GrowableThingCollection@PAX@@UAA@XZ 00191a2c f i toolbox.obj
 0001:00090ae0       ?AddThing@?$GrowableThingCollection@PAX@@UAA_NQAX@Z 00191ae0 f i toolbox.obj
 0001:00090bcc       ?InsertThing@?$GrowableThingCollection@PAX@@UAA_NQAXH@Z 00191bcc f i toolbox.obj
 0001:00090d90       ?RemoveThingAtIndex@?$GrowableThingCollection@PAX@@UAA_NH@Z 00191d90 f i toolbox.obj
 0001:00090f08       ?RemoveThing@?$GrowableThingCollection@PAX@@UAA_NQAX@Z 00191f08 f i toolbox.obj
 0001:00091034       ?RemoveAllThings@?$GrowableThingCollection@PAX@@UAA_NXZ 00192034 f i toolbox.obj
 0001:000910bc       ?SwapThingsAtIndices@?$GrowableThingCollection@PAX@@UAA_NHH@Z 001920bc f i toolbox.obj
 0001:00091284       ?GetSize@?$GrowableThingCollection@PAX@@UAAHXZ 00192284 f i toolbox.obj
 0001:000912d0       ?Lock@?$GrowableThingCollection@PAX@@UAA_NXZ 001922d0 f i toolbox.obj
 0001:00091378       ?Unlock@?$GrowableThingCollection@PAX@@UAA_NXZ 00192378 f i toolbox.obj
 0001:0009145c       ?BlockModificationByOtherThreads@?$GrowableThingCollection@PAX@@UAA_NXZ 0019245c f i toolbox.obj
 0001:0009148c       ?AllowModificationByOtherThreads@?$GrowableThingCollection@PAX@@UAA_NXZ 0019248c f i toolbox.obj
 0001:000914bc       ?GetThingAtIndex@?$GrowableThingCollection@PAX@@UAAPAXH@Z 001924bc f i toolbox.obj
 0001:000915b0       ?SetThingAtIndex@?$GrowableThingCollection@PAX@@UAA_NQAXH@Z 001925b0 f i toolbox.obj
 0001:000916a4       ?GetThingIndex@?$GrowableThingCollection@PAX@@UAAHQAX@Z 001926a4 f i toolbox.obj
 0001:00091760       ?GetFilteredThingIndex@?$GrowableThingCollection@PAX@@UAAHP6A_NABQAXPAX@ZQAX@Z 00192760 f i toolbox.obj
 0001:00091870       ?GetPointerToThingAtIndex@?$GrowableThingCollection@PAX@@UAAPAPAXH@Z 00192870 f i toolbox.obj
 0001:000919b0       ?GetPointerToThing@?$GrowableThingCollection@PAX@@UAAPAPAXQAX@Z 001929b0 f i toolbox.obj
 0001:00091af0       ?MakeRoomForAnotherThing@?$GrowableThingCollection@PAX@@MAA_NXZ 00192af0 f i toolbox.obj
 0001:00091c60       ??0?$GrowableThingCollection@UTaskListTaskData@TaskList@@@@QAA@H@Z 00192c60 f i toolbox.obj
 0001:00091d64       ??1?$GrowableThingCollection@UTaskListTaskData@TaskList@@@@UAA@XZ 00192d64 f i toolbox.obj
 0001:00091e18       ?AddThing@?$GrowableThingCollection@UTaskListTaskData@TaskList@@@@UAA_NUTaskListTaskData@TaskList@@@Z 00192e18 f i toolbox.obj
 0001:00091f18       ?InsertThing@?$GrowableThingCollection@UTaskListTaskData@TaskList@@@@UAA_NUTaskListTaskData@TaskList@@H@Z 00192f18 f i toolbox.obj
 0001:000920f0       ?RemoveThingAtIndex@?$GrowableThingCollection@UTaskListTaskData@TaskList@@@@UAA_NH@Z 001930f0 f i toolbox.obj
 0001:00092268       ?RemoveThing@?$GrowableThingCollection@UTaskListTaskData@TaskList@@@@UAA_NUTaskListTaskData@TaskList@@@Z 00193268 f i toolbox.obj
 0001:0009239c       ?RemoveAllThings@?$GrowableThingCollection@UTaskListTaskData@TaskList@@@@UAA_NXZ 0019339c f i toolbox.obj
 0001:00092424       ?SwapThingsAtIndices@?$GrowableThingCollection@UTaskListTaskData@TaskList@@@@UAA_NHH@Z 00193424 f i toolbox.obj
 0001:000925f8       ?GetSize@?$GrowableThingCollection@UTaskListTaskData@TaskList@@@@UAAHXZ 001935f8 f i toolbox.obj
 0001:00092644       ?Lock@?$GrowableThingCollection@UTaskListTaskData@TaskList@@@@UAA_NXZ 00193644 f i toolbox.obj
 0001:000926ec       ?Unlock@?$GrowableThingCollection@UTaskListTaskData@TaskList@@@@UAA_NXZ 001936ec f i toolbox.obj
 0001:000927d0       ?BlockModificationByOtherThreads@?$GrowableThingCollection@UTaskListTaskData@TaskList@@@@UAA_NXZ 001937d0 f i toolbox.obj
 0001:00092800       ?AllowModificationByOtherThreads@?$GrowableThingCollection@UTaskListTaskData@TaskList@@@@UAA_NXZ 00193800 f i toolbox.obj
 0001:00092830       ?GetThingAtIndex@?$GrowableThingCollection@UTaskListTaskData@TaskList@@@@UAA?AUTaskListTaskData@TaskList@@H@Z 00193830 f i toolbox.obj
 0001:00092938       ?SetThingAtIndex@?$GrowableThingCollection@UTaskListTaskData@TaskList@@@@UAA_NUTaskListTaskData@TaskList@@H@Z 00193938 f i toolbox.obj
 0001:00092a30       ?GetThingIndex@?$GrowableThingCollection@UTaskListTaskData@TaskList@@@@UAAHUTaskListTaskData@TaskList@@@Z 00193a30 f i toolbox.obj
 0001:00092aec       ?GetFilteredThingIndex@?$GrowableThingCollection@UTaskListTaskData@TaskList@@@@UAAHP6A_NABUTaskListTaskData@TaskList@@PAX@ZQAX@Z 00193aec f i toolbox.obj
 0001:00092bfc       ?GetPointerToThingAtIndex@?$GrowableThingCollection@UTaskListTaskData@TaskList@@@@UAAPAUTaskListTaskData@TaskList@@H@Z 00193bfc f i toolbox.obj
 0001:00092d3c       ?GetPointerToThing@?$GrowableThingCollection@UTaskListTaskData@TaskList@@@@UAAPAUTaskListTaskData@TaskList@@U23@@Z 00193d3c f i toolbox.obj
 0001:00092e7c       ?MakeRoomForAnotherThing@?$GrowableThingCollection@UTaskListTaskData@TaskList@@@@MAA_NXZ 00193e7c f i toolbox.obj
 0001:00092fec       ??_E?$GrowablePointerCollection@G@@UAAPAXI@Z 00193fec f i toolbox.obj
 0001:00092fec       ??_G?$GrowablePointerCollection@G@@UAAPAXI@Z 00193fec f i toolbox.obj
 0001:0009302c       ??_G?$GrowableThingCollection@PAG@@UAAPAXI@Z 0019402c f i toolbox.obj
 0001:0009302c       ??_E?$GrowableThingCollection@PAG@@UAAPAXI@Z 0019402c f i toolbox.obj
 0001:0009306c       ??_G?$GrowableThingCollection@PAX@@UAAPAXI@Z 0019406c f i toolbox.obj
 0001:0009306c       ??_E?$GrowableThingCollection@PAX@@UAAPAXI@Z 0019406c f i toolbox.obj
 0001:000930ac       ??_E?$GrowableThingCollection@UTaskListTaskData@TaskList@@@@UAAPAXI@Z 001940ac f i toolbox.obj
 0001:000930ac       ??_G?$GrowableThingCollection@UTaskListTaskData@TaskList@@@@UAAPAXI@Z 001940ac f i toolbox.obj
 0001:000930ec       ??0?$GrowableThingCollection@PAG@@QAA@H@Z 001940ec f i toolbox.obj
 0001:000931f0       ?FlagFromValue@@YAHIQBULISTVALUEMAP@@IAAK@Z 001941f0 f   util.obj
 0001:00093300       ?FlagFromString@@YAHQBDQBULISTSTRINGMAP@@IAAK@Z 00194300 f   util.obj
 0001:000933e0       ?ValueFromFlag@@YAHIQBULISTVALUEMAP@@IAAI@Z 001943e0 f   util.obj
 0001:00093484       ?StringFromFlag@@YAHIQBULISTSTRINGMAP@@IAAPBD@Z 00194484 f   util.obj
 0001:00093528       ?StringFilterW@@YAJPAGI00@Z 00194528 f   util.obj
 0001:00093680       ?DetermineSimResponseError@@YAJKK@Z 00194680 f   util.obj
 0001:000937b4       ?IsElementarySimFile@@YAHK@Z 001947b4 f   util.obj
 0001:00093884       ?UpdateStatStore@@YAXXZ    00194884 f   util.obj
 0001:00093994       ??0CBuffer@@QAA@XZ         00194994 f   util.obj
 0001:000939e4       ??1CBuffer@@QAA@XZ         001949e4 f   util.obj
 0001:00093a10       ?Append@CBuffer@@QAAHQBDI@Z 00194a10 f   util.obj
 0001:00093c2c       ?GiveUpData@CBuffer@@QAAPADXZ 00194c2c f   util.obj
 0001:00093ccc       ?InheritData@CBuffer@@QAAXPAV1@@Z 00194ccc f   util.obj
 0001:00093db0       ??0CSharedResource@@QAA@XZ 00194db0 f   util.obj
 0001:00093e6c       ??1CSharedResource@@QAA@XZ 00194e6c f   util.obj
 0001:00093f40       ?Init@CSharedResource@@QAAHQAX@Z 00194f40 f   util.obj
 0001:00094070       ?EnterSharedUse@CSharedResource@@QAAHXZ 00195070 f   util.obj
 0001:00094368       ?ExitSharedUse@CSharedResource@@QAAHXZ 00195368 f   util.obj
 0001:00094474       ?EnterExclusiveUse@CSharedResource@@QBAHP6AXK@ZK@Z 00195474 f   util.obj
 0001:000946b0       ?ExitExclusiveUse@CSharedResource@@QBAHXZ 001956b0 f   util.obj
 0001:0009473c       ?InitializeCarrierIndex@CRilHandle@@QAAXXZ 0019573c f   util.obj
 0001:00094a64       ?UpdateLocalCarrierIndex@CRilHandle@@QAAXW4SWI_TYPE_CarrierID@@@Z 00195a64 f   util.obj
 0001:00095028       ?MessageBoxOnSeparateThread@@YAXPBG0I@Z 00196028 f   util.obj
 0001:0009514c       ?MessageBoxFunction@@YAIPAX@Z 0019614c f   util.obj
 0001:000951d4       ?DumpMem@@YAXPAXH@Z        001961d4 f   util.obj
 0001:00095eec       ?SetRILCarrierIndex@CRilHandle@@QAAXI@Z 00196eec f i util.obj
 0001:00095f30       ?ConvertToSwiAudioMode@@YAEK@Z 00196f30 f   voice.obj
 0001:000960c0       ?RILDrv_GetAudioGain@@YAJK@Z 001970c0 f   voice.obj
 0001:000961a0       ?RILDrv_SetAudioGain@@YAJKPBUrilgaininfo_tag@@@Z 001971a0 f   voice.obj
 0001:000963d0       ?RILDrv_SetAudioDevices@@YAJKPBUrilaudiodeviceinfo_tag@@@Z 001973d0 f   voice.obj
 0001:0009650c       ?RILDrv_GetAudioMuting@@YAJK@Z 0019750c f   voice.obj
 0001:000965ec       ?RILDrv_SetAudioMuting@@YAJKH@Z 001975ec f   voice.obj
 0001:000966d4       ?GetAudioGain@CRadio@@QAAJPAVCResponse@@@Z 001976d4 f   voice.obj
 0001:000967cc       ?SetAudioGain@CRadio@@QAAJPAVCResponse@@PAX@Z 001977cc f   voice.obj
 0001:00096df4       ?SetAudioDevices@CRadio@@QAAJPAVCResponse@@PAX@Z 00197df4 f   voice.obj
 0001:00097470       ?GetAudioMuting@CRadio@@QAAJPAVCResponse@@@Z 00198470 f   voice.obj
 0001:0009756c       ?SetAudioMuting@CRadio@@QAAJPAVCResponse@@PAX@Z 0019856c f   voice.obj
 0001:000976e0       ?ProgramAudioParameter@CRadio@@QAAJXZ 001986e0 f   voice.obj
 0001:000977b0       ?ProgramAudioParameter9090@CRadio@@QAAJXZ 001987b0 f   voice.obj
 0001:00099028       ?ProgramAudioParameterSwiM2MAV@CRadio@@QAAJXZ 0019a028 f   voice.obj
 0001:0009a09c       ?HWSetMicMute@CRadio@@QAAJH@Z 0019b09c f   voice.obj
 0001:0009a390       ?HWSetSpeakerMute@CRadio@@QAAJH@Z 0019b390 f   voice.obj
 0001:0009a65c       ?HWPlayAudioTone@CRadio@@QAAJPAEPAG@Z 0019b65c f   voice.obj
 0001:0009a914       ?TBD_Output@@YAXW4TBD_CLASS_TYPE@@W4TBD_OUTPUT_LEVEL@@QBGZZ 0019b914 f   sw_utilityG:sw_utilityG.dll
 0001:0009a924       ?LogC@@YAXPBGZZ            0019b924 f   sw_utilityG:sw_utilityG.dll
 0001:0009a934       ?LogW@@YAXPBGZZ            0019b934 f   sw_utilityG:sw_utilityG.dll
 0001:0009a944       ?LogStoreFileLine@@YAXPAGH@Z 0019b944 f   sw_utilityG:sw_utilityG.dll
 0001:0009a954       ?TBD_Assert@@YA_N_NQBG1H@Z 0019b954 f   sw_utilityG:sw_utilityG.dll
 0001:0009a964       ?WriteLog@@YAXKPBGZZ       0019b964 f   sw_utilityG:sw_utilityG.dll
 0001:0009a974       ?SW_AtoT@@YAPAGPAGPADK@Z   0019b974 f   sw_utilityG:sw_utilityG.dll
 0001:0009a984       ?GetDataPortDetails@@YAHPAGAAK@Z 0019b984 f   sw_utilityG:sw_utilityG.dll
 0001:0009a994       ?GetCarrierIndex@@YAKXZ    0019b994 f   sw_utilityG:sw_utilityG.dll
 0001:0009a9a4       ?DWORD2IP@@YAPBGK@Z        0019b9a4 f   sw_utilityG:sw_utilityG.dll
 0001:0009a9b4       ?IP2DWORD@@YAKPBG@Z        0019b9b4 f   sw_utilityG:sw_utilityG.dll
 0001:0009a9c4       ?LocalToUTCTime@@YAHPAU_SYSTEMTIME@@0@Z 0019b9c4 f   sw_utilityG:sw_utilityG.dll
 0001:0009a9d4       ?SW_TtoA@@YAPADPADPAGK@Z   0019b9d4 f   sw_utilityG:sw_utilityG.dll
 0001:0009a9e4       ??1CVerInfo@@QAA@XZ        0019b9e4 f   sw_utilityG:sw_utilityG.dll
 0001:0009a9f4       ?GetProductVersionStr@CVerInfo@@QAAPAGXZ 0019b9f4 f   sw_utilityG:sw_utilityG.dll
 0001:0009aa04       ??0CVerInfo@@QAA@PAG@Z     0019ba04 f   sw_utilityG:sw_utilityG.dll
 0001:0009aa14       ?GetRegValue@@YAJPAUHKEY__@@PBG1PAGPAK@Z 0019ba14 f   sw_utilityG:sw_utilityG.dll
 0001:0009aa24       ?ConvertPrefMode@@YAH_NH@Z 0019ba24 f   sw_utilityG:sw_utilityG.dll
 0001:0009aa34       ?DisplayRawData@@YAXIPAEHPBG@Z 0019ba34 f   sw_utilityG:sw_utilityG.dll
 0001:0009aa44       ?SWAI_GetRegValue@@YAJPAUHKEY__@@PBG1PAGPAK@Z 0019ba44 f   sw_utilityG:sw_utilityG.dll
 0001:0009aa54       ?SWAI_SetRegValue@@YAJPAUHKEY__@@PBG1K@Z 0019ba54 f   sw_utilityG:sw_utilityG.dll
 0001:0009aa64       ?SWAI_GetRegValue@@YAJPAUHKEY__@@PBG1AAK@Z 0019ba64 f   sw_utilityG:sw_utilityG.dll
 0001:0009aa74       ?SetRegValue@@YAJPAUHKEY__@@PBG1K@Z 0019ba74 f   sw_utilityG:sw_utilityG.dll
 0001:0009aa84       ?GetProductFeatures@@YAHAAK@Z 0019ba84 f   sw_utilityG:sw_utilityG.dll
 0001:0009aa94       ?GetRegValue@@YAJPAUHKEY__@@PBG1AAK@Z 0019ba94 f   sw_utilityG:sw_utilityG.dll
 0001:0009aaa4       ?SetRegValue@@YAJPAUHKEY__@@PBG11@Z 0019baa4 f   sw_utilityG:sw_utilityG.dll
 0001:0009aab4       ?LogV@@YAXPBGZZ            0019bab4 f   sw_utilityG:sw_utilityG.dll
 0001:0009aac4       ?GetVerInfo@@YAPAGPAUHINSTANCE__@@@Z 0019bac4 f   sw_utilityG:sw_utilityG.dll
 0001:0009aad4       ?InitLog@@YAXPAUHINSTANCE__@@@Z 0019bad4 f   sw_utilityG:sw_utilityG.dll
 0001:0009aae4       ?ChangeCarrierIndex@@YAJKK@Z 0019bae4 f   sw_utilityG:sw_utilityG.dll
 0001:0009aaf4       ValidateAPIPermission      0019baf4 f   ossvcs:ossvcs.dll
 0001:0009ab04       GetStatStore               0019bb04 f   ossvcs:ossvcs.dll
 0001:0009ab14       _DllMainCRTStartup         0019bb14 f   corelibc:pegdmain.obj
 0001:0009abac       __security_check_cookie    0019bbac     corelibc:armsecgs.obj
 0001:0009abc0       __gsfailure                0019bbc0     corelibc:armsecgs.obj
 0001:0009ac04       _onexit                    0019bc04 f   corelibc:onexit.obj
 0001:0009acb0       atexit                     0019bcb0 f   corelibc:onexit.obj
 0001:0009acd0       GetCurrentProcess          0019bcd0 f i corelibc:crt0dat.obj
 0001:0009ad0c       _cinit                     0019bd0c f   corelibc:crt0dat.obj
 0001:0009ae7c       exit                       0019be7c f   corelibc:crt0dat.obj
 0001:0009ae94       _exit                      0019be94 f   corelibc:crt0dat.obj
 0001:0009aeac       _cexit                     0019beac f   corelibc:crt0dat.obj
 0001:0009aec8       _c_exit                    0019bec8 f   corelibc:crt0dat.obj
 0001:0009af14       __security_init_cookie     0019bf14 f   corelibc:seccinit.obj
 0001:0009af64       PHGetFeatureLevel          0019bf64 f   ccoreutl:ccoreutl.dll
 0001:0009af74       htonl                      0019bf74 f   winsock:WINSOCK.dll
 0001:0009af84       inet_addr                  0019bf84 f   winsock:WINSOCK.dll
 0001:0009af94       ntohs                      0019bf94 f   winsock:WINSOCK.dll
 0001:0009afa4       GetAdaptersInfo            0019bfa4 f   Iphlpapi:iphlpapi.dll
 0001:0009afb4       ?DialCall@CSwiGobiDll@@QAAKPAUtDialReqParam@@PAEPAUalphaIDInfo@@1PAUccSUPSType@@@Z 0019bfb4 f   sdkril:SDKRIL.dll
 0001:0009afc4       SwiPstGetDsMipActiveProf   0019bfc4 f   sdkril:SDKRIL.dll
 0001:0009afd4       ?AnserCall@CSwiGobiDll@@QAAKPAE0@Z 0019bfd4 f   sdkril:SDKRIL.dll
 0001:0009afe4       ?EndCall@CSwiGobiDll@@QAAKPAE0@Z 0019bfe4 f   sdkril:SDKRIL.dll
 0001:0009aff4       ?ManageCalls@CSwiGobiDll@@QAAKPAE0PAG@Z 0019bff4 f   sdkril:SDKRIL.dll
 0001:0009b004       ?SendFlash@CSwiGobiDll@@QAAKPAEPAD00@Z 0019c004 f   sdkril:SDKRIL.dll
 0001:0009b014       ?StopDTMF@CSwiGobiDll@@QAAKPAE0@Z 0019c014 f   sdkril:SDKRIL.dll
 0001:0009b024       ?StartDTMF@CSwiGobiDll@@QAAKPAE00@Z 0019c024 f   sdkril:SDKRIL.dll
 0001:0009b034       ?GetCellLocationInfo@CSwiGobiDll@@QAAKPAUgeranCellInfo@@PAUumtsCellInfo@@PAUcdmaCellInfo@@PAK@Z 0019c034 f   sdkril:SDKRIL.dll
 0001:0009b044       ?SetXTRAEmbeddedClient@CSwiGobiDll@@QAAKEE@Z 0019c044 f   sdkril:SDKRIL.dll
 0001:0009b054       ?SetPDSDefaults@CSwiGobiDll@@QAAKKEKK@Z 0019c054 f   sdkril:SDKRIL.dll
 0001:0009b064       ?SetNMEAConfig@CSwiGobiDll@@QAAKEEEPAG@Z 0019c064 f   sdkril:SDKRIL.dll
 0001:0009b074       ?GetNMEAConfig@CSwiGobiDll@@QAAKPAE00PAG@Z 0019c074 f   sdkril:SDKRIL.dll
 0001:0009b084       ?ForceXTRADownload@CSwiGobiDll@@QAAKXZ 0019c084 f   sdkril:SDKRIL.dll
 0001:0009b094       ?GetPhonebookCapabilities@CSwiGobiDll@@QAAKPAEPAG1100@Z 0019c094 f   sdkril:SDKRIL.dll
 0001:0009b0a4       ?ReadPhonebookRecords@CSwiGobiDll@@QAAKPAEPAG111@Z 0019c0a4 f   sdkril:SDKRIL.dll
 0001:0009b0b4       ?WritePhonebookRecord@CSwiGobiDll@@QAAKPAEPAG1000000@Z 0019c0b4 f   sdkril:SDKRIL.dll
 0001:0009b0c4       ?DeletePhonebookRecord@CSwiGobiDll@@QAAKPAEPAG1@Z 0019c0c4 f   sdkril:SDKRIL.dll
 0001:0009b0d4       SwiSetPower                0019c0d4 f   sdkril:SDKRIL.dll
 0001:0009b0e4       ?GetRTREConfig@CSwiGobiDll@@QAAKPAE0@Z 0019c0e4 f   sdkril:SDKRIL.dll
 0001:0009b0f4       ??1CSwiGobiDll@@QAA@XZ     0019c0f4 f   sdkril:SDKRIL.dll
 0001:0009b104       ?UIMGetCardStatus@CSwiGobiDll@@QAAKPAHPAUQMI_UIM_GET_CARD_STATUS_RESP@@@Z 0019c104 f   sdkril:SDKRIL.dll
 0001:0009b114       ?GetDunCallInfo@CSwiGobiDll@@QAAKPAKPAE101111PA_KPAG221100002221@Z 0019c114 f   sdkril:SDKRIL.dll
 0001:0009b124       ?GetDormancyState@CSwiGobiDll@@QAAKPAK@Z 0019c124 f   sdkril:SDKRIL.dll
 0001:0009b134       ?Initialize@CSwiGobiDll@@QAA_NXZ 0019c134 f   sdkril:SDKRIL.dll
 0001:0009b144       ??0CSwiGobiDll@@QAA@XZ     0019c144 f   sdkril:SDKRIL.dll
 0001:0009b154       ?GetWaitingMessage@CSwiGobiDll@@QAAKPAUwaitingMsgInfo@@@Z 0019c154 f   sdkril:SDKRIL.dll
 0001:0009b164       SwiSetGsmProfileBasic      0019c164 f   sdkril:SDKRIL.dll
 0001:0009b174       SwiGetGsmProfileBasic      0019c174 f   sdkril:SDKRIL.dll
 0001:0009b184       ?GetCallBarring@CSwiGobiDll@@QAAKPAE00PAGPAUalphaIDInfo@@00PAUccSUPSType@@@Z 0019c184 f   sdkril:SDKRIL.dll
 0001:0009b194       ?SetSUPS@CSwiGobiDll@@QAAKPAUvoiceSetSUPSServiceReq@@PAGPAUalphaIDInfo@@PAE3PAUccSUPSType@@@Z 0019c194 f   sdkril:SDKRIL.dll
 0001:0009b1a4       ?ChangeBarringPwd@CSwiGobiDll@@QAAKPAUcallBarringPwd@@PAGPAUalphaIDInfo@@PAE3PAUccSUPSType@@@Z 0019c1a4 f   sdkril:SDKRIL.dll
 0001:0009b1b4       ?GetCallForwarding@CSwiGobiDll@@QAAKPAE0PAUgetCallFWInfo@@0PAUalphaIDInfo@@00PAUccSUPSType@@PAUgetExtCallFWInfo@@@Z 0019c1b4 f   sdkril:SDKRIL.dll
 0001:0009b1c4       ?GetCallWaiting@CSwiGobiDll@@QAAKPAE0PAGPAUalphaIDInfo@@00PAUccSUPSType@@@Z 0019c1c4 f   sdkril:SDKRIL.dll
 0001:0009b1d4       ?OrigUSSD@CSwiGobiDll@@QAAKPAUUSSInfo@@PAGPAUalphaIDInfo@@0PAE3PAUccSUPSType@@@Z 0019c1d4 f   sdkril:SDKRIL.dll
 0001:0009b1e4       ?AnswerUSSD@CSwiGobiDll@@QAAKPAUUSSInfo@@@Z 0019c1e4 f   sdkril:SDKRIL.dll
 0001:0009b1f4       ?CancelUSSD@CSwiGobiDll@@QAAKXZ 0019c1f4 f   sdkril:SDKRIL.dll
 0001:0009b204       ?SwiM2MAV_AudioSetProfile@CSwiGobiDll@@QAAKPAE00000@Z 0019c204 f   sdkril:SDKRIL.dll
 0001:0009b214       ?SwiM2MAV_AudioSetTxVolume@CSwiGobiDll@@QAAKPAEPAG@Z 0019c214 f   sdkril:SDKRIL.dll
 0001:0009b224       ?SwiM2MAV_AudioGetProfile@CSwiGobiDll@@QAAKPAE000000@Z 0019c224 f   sdkril:SDKRIL.dll
 0001:0009b234       ?SetReceiverVolume@CSwiGobiDll@@QAAKPAE@Z 0019c234 f   sdkril:SDKRIL.dll
 0001:0009b244       ?SetMicVolume@CSwiGobiDll@@QAAKPAG@Z 0019c244 f   sdkril:SDKRIL.dll
 0001:0009b254       ?SetSpeakerMuteStatus@CSwiGobiDll@@QAAKPAE@Z 0019c254 f   sdkril:SDKRIL.dll
 0001:0009b264       ?SetMICMuteStatus@CSwiGobiDll@@QAAKPAE@Z 0019c264 f   sdkril:SDKRIL.dll
 0001:0009b274       ?SetAudioProfile@CSwiGobiDll@@QAAKPAE@Z 0019c274 f   sdkril:SDKRIL.dll
 0001:0009b284       ?SetRXGainLevel@CSwiGobiDll@@QAAKPAEPAG1@Z 0019c284 f   sdkril:SDKRIL.dll
 0001:0009b294       ?SetRXPCMFilter@CSwiGobiDll@@QAAKPAG0PAK0@Z 0019c294 f   sdkril:SDKRIL.dll
 0001:0009b2a4       ?SetTXPCMFilter@CSwiGobiDll@@QAAKPAG0PAK0@Z 0019c2a4 f   sdkril:SDKRIL.dll
 0001:0009b2b4       ?SetAutoOutputGain@CSwiGobiDll@@QAAKPAE@Z 0019c2b4 f   sdkril:SDKRIL.dll
 0001:0009b2c4       ?SetAutoInputGain@CSwiGobiDll@@QAAKPAE@Z 0019c2c4 f   sdkril:SDKRIL.dll
 0001:0009b2d4       ?SetNoiseSuppression@CSwiGobiDll@@QAAKPAE@Z 0019c2d4 f   sdkril:SDKRIL.dll
 0001:0009b2e4       ?SetEchoCancelMode@CSwiGobiDll@@QAAKPAE@Z 0019c2e4 f   sdkril:SDKRIL.dll
 0001:0009b2f4       ?GetAudioProfile@CSwiGobiDll@@QAAKPAE@Z 0019c2f4 f   sdkril:SDKRIL.dll
 0001:0009b304       ?SwiM2MAV_AudioSetVolDB@CSwiGobiDll@@QAAKPAE00PAG@Z 0019c304 f   sdkril:SDKRIL.dll
 0001:0009b314       ?SwiM2MAV_AudioSetAVNS@CSwiGobiDll@@QAAKPAE0@Z 0019c314 f   sdkril:SDKRIL.dll
 0001:0009b324       ?SwiM2MAV_AudioSetVolume@CSwiGobiDll@@QAAKPAE00@Z 0019c324 f   sdkril:SDKRIL.dll
 0001:0009b334       ?SwiM2MAV_AudioSetSTG@CSwiGobiDll@@QAAKPAEPAG@Z 0019c334 f   sdkril:SDKRIL.dll
 0001:0009b344       ?SwiM2MAV_AudioSetAVEC@CSwiGobiDll@@QAAKPAE0@Z 0019c344 f   sdkril:SDKRIL.dll
 0001:0009b354       ?SwiM2MAV_AudioPlayTone@CSwiGobiDll@@QAAKPAE0PAG@Z 0019c354 f   sdkril:SDKRIL.dll
 0001:0009b364       ?PlayAudioTone@CSwiGobiDll@@QAAKPAE@Z 0019c364 f   sdkril:SDKRIL.dll
 0001:0009b374       ??3@YAXPAX@Z               0019c374 f   coredll:COREDLL.dll
 0001:0009b384       LeaveCriticalSection       0019c384 f   coredll:COREDLL.dll
 0001:0009b394       EnterCriticalSection       0019c394 f   coredll:COREDLL.dll
 0001:0009b3a4       GetTickCount               0019c3a4 f   coredll:COREDLL.dll
 0001:0009b3b4       ??2@YAPAXI@Z               0019c3b4 f   coredll:COREDLL.dll
 0001:0009b3c4       memset                     0019c3c4 f   coredll:COREDLL.dll
 0001:0009b3d4       SetThreadPriority          0019c3d4 f   coredll:COREDLL.dll
 0001:0009b3e4       EventModify                0019c3e4 f   coredll:COREDLL.dll
 0001:0009b3f4       __rt_udiv                  0019c3f4 f   coredll:COREDLL.dll
 0001:0009b404       __CxxThrowException        0019c404 f   coredll:COREDLL.dll
 0001:0009b414       ??_7type_info@@6B@         0019c414 f   coredll:COREDLL.dll
 0001:0009b424       ??0exception@std@@QAA@ABV01@@Z 0019c424 f   coredll:COREDLL.dll
 0001:0009b434       ??1exception@std@@UAA@XZ   0019c434 f   coredll:COREDLL.dll
 0001:0009b444       ??0exception@std@@QAA@XZ   0019c444 f   coredll:COREDLL.dll
 0001:0009b454       strlen                     0019c454 f   coredll:COREDLL.dll
 0001:0009b464       memcpy                     0019c464 f   coredll:COREDLL.dll
 0001:0009b474       ??0exception@std@@QAA@PBD@Z 0019c474 f   coredll:COREDLL.dll
 0001:0009b484       ?what@exception@std@@UBAPBDXZ 0019c484 f   coredll:COREDLL.dll
 0001:0009b494       wcscmp                     0019c494 f   coredll:COREDLL.dll
 0001:0009b4a4       wcslen                     0019c4a4 f   coredll:COREDLL.dll
 0001:0009b4b4       ??_V@YAXPAX@Z              0019c4b4 f   coredll:COREDLL.dll
 0001:0009b4c4       _isctype                   0019c4c4 f   coredll:COREDLL.dll
 0001:0009b4d4       ??_U@YAPAXI@Z              0019c4d4 f   coredll:COREDLL.dll
 0001:0009b4e4       Sleep                      0019c4e4 f   coredll:COREDLL.dll
 0001:0009b4f4       wcscpy                     0019c4f4 f   coredll:COREDLL.dll
 0001:0009b504       swprintf                   0019c504 f   coredll:COREDLL.dll
 0001:0009b514       strcpy                     0019c514 f   coredll:COREDLL.dll
 0001:0009b524       CreateProcessW             0019c524 f   coredll:COREDLL.dll
 0001:0009b534       wcsstr                     0019c534 f   coredll:COREDLL.dll
 0001:0009b544       CreateFileW                0019c544 f   coredll:COREDLL.dll
 0001:0009b554       CloseHandle                0019c554 f   coredll:COREDLL.dll
 0001:0009b564       EscapeCommFunction         0019c564 f   coredll:COREDLL.dll
 0001:0009b574       strchr                     0019c574 f   coredll:COREDLL.dll
 0001:0009b584       _wcsicmp                   0019c584 f   coredll:COREDLL.dll
 0001:0009b594       NKDbgPrintfW               0019c594 f   coredll:COREDLL.dll
 0001:0009b5a4       CreateThread               0019c5a4 f   coredll:COREDLL.dll
 0001:0009b5b4       WriteFile                  0019c5b4 f   coredll:COREDLL.dll
 0001:0009b5c4       strcat                     0019c5c4 f   coredll:COREDLL.dll
 0001:0009b5d4       PurgeComm                  0019c5d4 f   coredll:COREDLL.dll
 0001:0009b5e4       SetCommMask                0019c5e4 f   coredll:COREDLL.dll
 0001:0009b5f4       SetCommTimeouts            0019c5f4 f   coredll:COREDLL.dll
 0001:0009b604       GetCommModemStatus         0019c604 f   coredll:COREDLL.dll
 0001:0009b614       SetCommState               0019c614 f   coredll:COREDLL.dll
 0001:0009b624       MessageBoxW                0019c624 f   coredll:COREDLL.dll
 0001:0009b634       ShowWindow                 0019c634 f   coredll:COREDLL.dll
 0001:0009b644       FindWindowW                0019c644 f   coredll:COREDLL.dll
 0001:0009b654       SetSystemPowerState        0019c654 f   coredll:COREDLL.dll
 0001:0009b664       MultiByteToWideChar        0019c664 f   coredll:COREDLL.dll
 0001:0009b674       GetStoreInformation        0019c674 f   coredll:COREDLL.dll
 0001:0009b684       CreateMutexW               0019c684 f   coredll:COREDLL.dll
 0001:0009b694       wcscat                     0019c694 f   coredll:COREDLL.dll
 0001:0009b6a4       GetLastError               0019c6a4 f   coredll:COREDLL.dll
 0001:0009b6b4       TerminateThread            0019c6b4 f   coredll:COREDLL.dll
 0001:0009b6c4       WaitForSingleObject        0019c6c4 f   coredll:COREDLL.dll
 0001:0009b6d4       FlushFileBuffers           0019c6d4 f   coredll:COREDLL.dll
 0001:0009b6e4       ReadFile                   0019c6e4 f   coredll:COREDLL.dll
 0001:0009b6f4       WaitCommEvent              0019c6f4 f   coredll:COREDLL.dll
 0001:0009b704       DeviceIoControl            0019c704 f   coredll:COREDLL.dll
 0001:0009b714       OutputDebugStringW         0019c714 f   coredll:COREDLL.dll
 0001:0009b724       wsprintfW                  0019c724 f   coredll:COREDLL.dll
 0001:0009b734       __C_specific_handler       0019c734 f   coredll:COREDLL.dll
 0001:0009b744       __rt_sdiv                  0019c744 f   coredll:COREDLL.dll
 0001:0009b754       WaitForMultipleObjects     0019c754 f   coredll:COREDLL.dll
 0001:0009b764       wcsncpy                    0019c764 f   coredll:COREDLL.dll
 0001:0009b774       abs                        0019c774 f   coredll:COREDLL.dll
 0001:0009b784       _snwprintf                 0019c784 f   coredll:COREDLL.dll
 0001:0009b794       wcschr                     0019c794 f   coredll:COREDLL.dll
 0001:0009b7a4       strncat                    0019c7a4 f   coredll:COREDLL.dll
 0001:0009b7b4       strncpy                    0019c7b4 f   coredll:COREDLL.dll
 0001:0009b7c4       _snprintf                  0019c7c4 f   coredll:COREDLL.dll
 0001:0009b7d4       wcsncat                    0019c7d4 f   coredll:COREDLL.dll
 0001:0009b7e4       _wtol                      0019c7e4 f   coredll:COREDLL.dll
 0001:0009b7f4       WideCharToMultiByte        0019c7f4 f   coredll:COREDLL.dll
 0001:0009b804       ??_M@YAXPAXIHP6AX0@Z@Z     0019c804 f   coredll:COREDLL.dll
 0001:0009b814       ??_L@YAXPAXIHP6AX0@Z1@Z    0019c814 f   coredll:COREDLL.dll
 0001:0009b824       KernelIoControl            0019c824 f   coredll:COREDLL.dll
 0001:0009b834       FileTimeToSystemTime       0019c834 f   coredll:COREDLL.dll
 0001:0009b844       LocalFileTimeToFileTime    0019c844 f   coredll:COREDLL.dll
 0001:0009b854       SystemTimeToFileTime       0019c854 f   coredll:COREDLL.dll
 0001:0009b864       iswctype                   0019c864 f   coredll:COREDLL.dll
 0001:0009b874       InitializeCriticalSection  0019c874 f   coredll:COREDLL.dll
 0001:0009b884       DeleteCriticalSection      0019c884 f   coredll:COREDLL.dll
 0001:0009b894       sprintf                    0019c894 f   coredll:COREDLL.dll
 0001:0009b8a4       atoi                       0019c8a4 f   coredll:COREDLL.dll
 0001:0009b8b4       _itoa                      0019c8b4 f   coredll:COREDLL.dll
 0001:0009b8c4       GetProcAddressW            0019c8c4 f   coredll:COREDLL.dll
 0001:0009b8d4       LoadLibraryW               0019c8d4 f   coredll:COREDLL.dll
 0001:0009b8e4       FreeLibrary                0019c8e4 f   coredll:COREDLL.dll
 0001:0009b8f4       CreateEventW               0019c8f4 f   coredll:COREDLL.dll
 0001:0009b904       _wcsupr                    0019c904 f   coredll:COREDLL.dll
 0001:0009b914       CeSetThreadPriority        0019c914 f   coredll:COREDLL.dll
 0001:0009b924       SetSystemTime              0019c924 f   coredll:COREDLL.dll
 0001:0009b934       strstr                     0019c934 f   coredll:COREDLL.dll
 0001:0009b944       pow                        0019c944 f   coredll:COREDLL.dll
 0001:0009b954       __muld                     0019c954 f   coredll:COREDLL.dll
 0001:0009b964       __utod                     0019c964 f   coredll:COREDLL.dll
 0001:0009b974       __addd                     0019c974 f   coredll:COREDLL.dll
 0001:0009b984       __dtou                     0019c984 f   coredll:COREDLL.dll
 0001:0009b994       wcsncmp                    0019c994 f   coredll:COREDLL.dll
 0001:0009b9a4       _itow                      0019c9a4 f   coredll:COREDLL.dll
 0001:0009b9b4       RegCloseKey                0019c9b4 f   coredll:COREDLL.dll
 0001:0009b9c4       wcstok                     0019c9c4 f   coredll:COREDLL.dll
 0001:0009b9d4       RegQueryValueExW           0019c9d4 f   coredll:COREDLL.dll
 0001:0009b9e4       RegOpenKeyExW              0019c9e4 f   coredll:COREDLL.dll
 0001:0009b9f4       RegCreateKeyExW            0019c9f4 f   coredll:COREDLL.dll
 0001:0009ba04       RegSetValueExW             0019ca04 f   coredll:COREDLL.dll
 0001:0009ba14       StringCchPrintfW           0019ca14 f   coredll:COREDLL.dll
 0001:0009ba24       LocalFree                  0019ca24 f   coredll:COREDLL.dll
 0001:0009ba34       LocalAllocTrace            0019ca34 f   coredll:COREDLL.dll
 0001:0009ba44       swscanf                    0019ca44 f   coredll:COREDLL.dll
 0001:0009ba54       TryEnterCriticalSection    0019ca54 f   coredll:COREDLL.dll
 0001:0009ba64       PowerPolicyNotify          0019ca64 f   coredll:COREDLL.dll
 0001:0009ba74       memmove                    0019ca74 f   coredll:COREDLL.dll
 0001:0009ba84       CeSafeCopyMemory           0019ca84 f   coredll:COREDLL.dll
 0001:0009ba94       wcstoul                    0019ca94 f   coredll:COREDLL.dll
 0001:0009baa4       free                       0019caa4 f   coredll:COREDLL.dll
 0001:0009bab4       malloc                     0019cab4 f   coredll:COREDLL.dll
 0001:0009bac4       _byteswap_ushort           0019cac4 f   coredll:COREDLL.dll
 0001:0009bad4       SystemIdleTimerReset       0019cad4 f   coredll:COREDLL.dll
 0001:0009bae4       wcstombs                   0019cae4 f   coredll:COREDLL.dll
 0001:0009baf4       _vsnwprintf                0019caf4 f   coredll:COREDLL.dll
 0001:0009bb04       _vsnprintf                 0019cb04 f   coredll:COREDLL.dll
 0001:0009bb14       rand                       0019cb14 f   coredll:COREDLL.dll
 0001:0009bb24       __divs                     0019cb24 f   coredll:COREDLL.dll
 0001:0009bb34       __itos                     0019cb34 f   coredll:COREDLL.dll
 0001:0009bb44       __muls                     0019cb44 f   coredll:COREDLL.dll
 0001:0009bb54       __stoi                     0019cb54 f   coredll:COREDLL.dll
 0001:0009bb64       LoadStringW                0019cb64 f   coredll:COREDLL.dll
 0001:0009bb74       _wcsnicmp                  0019cb74 f   coredll:COREDLL.dll
 0001:0009bb84       IsBadReadPtr               0019cb84 f   coredll:COREDLL.dll
 0001:0009bb94       IsBadWritePtr              0019cb94 f   coredll:COREDLL.dll
 0001:0009bba4       CreateSemaphoreW           0019cba4 f   coredll:COREDLL.dll
 0001:0009bbb4       ReleaseSemaphore           0019cbb4 f   coredll:COREDLL.dll
 0001:0009bbc4       InterlockedDecrement       0019cbc4 f   coredll:COREDLL.dll
 0001:0009bbd4       InterlockedIncrement       0019cbd4 f   coredll:COREDLL.dll
 0001:0009bbe4       UnmapViewOfFile            0019cbe4 f   coredll:COREDLL.dll
 0001:0009bbf4       MapViewOfFile              0019cbf4 f   coredll:COREDLL.dll
 0001:0009bc04       CreateFileMappingW         0019cc04 f   coredll:COREDLL.dll
 0001:0009bc14       GetFileSize                0019cc14 f   coredll:COREDLL.dll
 0001:0009bc24       LocalReAlloc               0019cc24 f   coredll:COREDLL.dll
 0001:0009bc34       GetSystemTime              0019cc34 f   coredll:COREDLL.dll
 0001:0009bc44       memcmp                     0019cc44 f   coredll:COREDLL.dll
 0001:0009bc54       strcmp                     0019cc54 f   coredll:COREDLL.dll
 0001:0009bc64       StringCchCopyW             0019cc64 f   coredll:COREDLL.dll
 0001:0009bc74       CopyFileW                  0019cc74 f   coredll:COREDLL.dll
 0001:0009bc84       DeleteFileW                0019cc84 f   coredll:COREDLL.dll
 0001:0009bc94       SetFileAttributesW         0019cc94 f   coredll:COREDLL.dll
 0001:0009bca4       MoveFileW                  0019cca4 f   coredll:COREDLL.dll
 0001:0009bcb4       strtoul                    0019ccb4 f   coredll:COREDLL.dll
 0001:0009bcc4       strtok                     0019ccc4 f   coredll:COREDLL.dll
 0001:0009bcd4       RegEnumKeyExW              0019ccd4 f   coredll:COREDLL.dll
 0001:0009bce4       __report_gsfailure         0019cce4 f   coredll:COREDLL.dll
 0001:0009bcf4       LocalAlloc                 0019ccf4 f   coredll:COREDLL.dll
 0001:0009bd04       LocalSize                  0019cd04 f   coredll:COREDLL.dll
 0001:0009bd14       __security_gen_cookie      0019cd14 f   coredll:COREDLL.dll
 0001:0009bd24       ?_Debug_message@std@@YAXPBD0@Z 0019cd24 f   libcpmtd:stdthrow.obj
 0001:0009bde4       ?_Debug_message@std@@YAXPB_W0I@Z 0019cde4 f   libcpmtd:stdthrow.obj
 0001:0009be24       ?_Debug_message@std@@YAXPBG0I@Z 0019ce24 f   libcpmtd:stdthrow.obj
 0001:0009be40       ?_Throw@std@@YAXABVexception@1@@Z 0019ce40 f   libcpmtd:stdthrow.obj
 0001:0009be78       ??0_Init_locks@std@@QAA@XZ 0019ce78 f   libcpmtd:xlock.obj
 0001:0009bed8       ??1_Init_locks@std@@QAA@XZ 0019ced8 f   libcpmtd:xlock.obj
 0001:0009bf30       ?_Init_locks_ctor@_Init_locks@std@@CAXPAV12@@Z 0019cf30 f   libcpmtd:xlock.obj
 0001:0009bf88       ?_Init_locks_dtor@_Init_locks@std@@CAXPAV12@@Z 0019cf88 f   libcpmtd:xlock.obj
 0001:0009bfe0       ??0_Lockit@std@@QAA@XZ     0019cfe0 f   libcpmtd:xlock.obj
 0001:0009c014       ??0_Lockit@std@@QAA@H@Z    0019d014 f   libcpmtd:xlock.obj
 0001:0009c050       ??1_Lockit@std@@QAA@XZ     0019d050 f   libcpmtd:xlock.obj
 0001:0009c080       ?_Lockit_ctor@_Lockit@std@@CAXPAV12@@Z 0019d080 f   libcpmtd:xlock.obj
 0001:0009c0a4       ?_Lockit_ctor@_Lockit@std@@CAXPAV12@H@Z 0019d0a4 f   libcpmtd:xlock.obj
 0001:0009c0dc       ?_Lockit_dtor@_Lockit@std@@CAXPAV12@@Z 0019d0dc f   libcpmtd:xlock.obj
 0001:0009c10c       ??$_Debug_pointer@D@std@@YAXPBDPB_WI@Z 0019d10c f i libcpmtd:string.obj
 0001:0009c134       ??0invalid_argument@std@@QAA@ABV?$basic_string@DU?$char_traits@D@std@@V?$allocator@D@2@@1@@Z 0019d134 f i libcpmtd:string.obj
 0001:0009c164       ??1invalid_argument@std@@UAA@XZ 0019d164 f i libcpmtd:string.obj
 0001:0009c190       ??_Ginvalid_argument@std@@UAAPAXI@Z 0019d190 f i libcpmtd:string.obj
 0001:0009c190       ??_Einvalid_argument@std@@UAAPAXI@Z 0019d190 f i libcpmtd:string.obj
 0001:0009c1dc       ??0out_of_range@std@@QAA@ABV?$basic_string@DU?$char_traits@D@std@@V?$allocator@D@2@@1@@Z 0019d1dc f i libcpmtd:string.obj
 0001:0009c20c       ??1out_of_range@std@@UAA@XZ 0019d20c f i libcpmtd:string.obj
 0001:0009c238       ??_Eout_of_range@std@@UAAPAXI@Z 0019d238 f i libcpmtd:string.obj
 0001:0009c238       ??_Gout_of_range@std@@UAAPAXI@Z 0019d238 f i libcpmtd:string.obj
 0001:0009c28c       ?_Xlen@_String_base@std@@SAXXZ 0019d28c f   libcpmtd:string.obj
 0001:0009c31c       ?_Xran@_String_base@std@@SAXXZ 0019d31c f   libcpmtd:string.obj
 0001:0009c3a4       ??0out_of_range@std@@QAA@ABV01@@Z 0019d3a4 f i libcpmtd:string.obj
 0001:0009c3dc       ?_Xinvarg@_String_base@std@@SAXXZ 0019d3dc f   libcpmtd:string.obj
 0001:0009c464       ??0invalid_argument@std@@QAA@ABV01@@Z 0019d464 f i libcpmtd:string.obj
 0001:0009c494       _Once                      0019d494 f   libcpmtd:xmtx.obj
 0001:0009c520       _Mtxinit                   0019d520 f   libcpmtd:xmtx.obj
 0001:0009c53c       _Mtxdst                    0019d53c f   libcpmtd:xmtx.obj
 0001:0009c558       _Mtxlock                   0019d558 f   libcpmtd:xmtx.obj
 0001:0009c574       _Mtxunlock                 0019d574 f   libcpmtd:xmtx.obj
 0001:0009c590       __InternalCxxFrameHandler  0019d590 f   LIBCMTD:frame_ce.obj
 0001:0009c76c       __CxxFrameHandler3         0019d76c f   LIBCMTD:frame_ce.obj
 0001:0009cf48       __FrameUnwindToState       0019df48 f   LIBCMTD:frame_ce.obj
 0001:0009dcf4       ?_DestructExceptionObject@@YAXPAUEHExceptionRecord@@E@Z 0019ecf4 f   LIBCMTD:frame_ce.obj
 0001:0009de44       ?_OffsetToAddress@@YAPAXHPAKK@Z 0019ee44 f   LIBCMTD:frame_ce.obj
 0001:0009ded0       ?FindFrameInfo@@YAPAU_FrameInfo@@PAK@Z 0019eed0 f   LIBCMTD:frame_ce.obj
 0001:0009df58       ?FindCatchFrameInfo@@YAPAU_FrameInfo@@PAK@Z 0019ef58 f   LIBCMTD:frame_ce.obj
 0001:0009dfdc       ?_GetRangeOfTrysToCheck@@YAPBU_s_TryBlockMapEntry@@PBU_s_FuncInfo@@HHPAI1@Z 0019efdc f   LIBCMTD:frame_ce.obj
 0001:0009e0d4       __GSHandlerCheck_EH        0019f0d4 f   LIBCMTD:gshandlereh.obj
 0001:0009e168       _invalid_parameter         0019f168 f   LIBCMTD:invarginternal.obj
 0001:0009e1b4       _CrtSetReportHookT2        0019f1b4 f   LIBCMTD:dbgrpt.obj
 0001:0009e680       _CrtDbgReportW             0019f680 f   LIBCMTD:dbgrpt.obj
 0001:0009e6f8       _CrtDbgReportTV            0019f6f8 f i LIBCMTD:dbgrpt.obj
 0001:0009e754       __crtMessageWindowW        0019f754 f   LIBCMTD:dbgrpt.obj
 0001:0009ee2c       _invoke_watson_if_error    0019fe2c f i LIBCMTD:dbgrpt.obj
 0001:0009ee80       memcpy_s                   0019fe80 f   LIBCMTD:memcpy_s.obj
 0001:0009f138       memmove_s                  001a0138 f   LIBCMTD:memmove_s.obj
 0001:0009f3ac       __GSHandlerCheckCommon     001a03ac f   LIBCMTD:gshandler.obj
 0001:0009f3f4       __GSHandlerCheck           001a03f4 f   LIBCMTD:gshandler.obj
 0001:0009f424       GetCRTStorage              001a0424 f   LIBCMTD:corecrt.obj
 0001:0009f534       TlsAlloc                   001a0534 f i LIBCMTD:corecrt.obj
 0001:0009f570       TlsFree                    001a0570 f i LIBCMTD:corecrt.obj
 0001:0009f5b4       ?FindFrameForUnwind@@YAPAKPAKPBU_s_FuncInfo@@@Z 001a05b4 f   LIBCMTD:mdframe_arm.obj
 0001:0009f64c       ?FindCatchFrame@@YAPAKPAKK@Z 001a064c f   LIBCMTD:mdframe_arm.obj
 0001:0009f6e4       ?AdjustFrameForCatch@@YAPAKPAKPBU_s_FuncInfo@@@Z 001a06e4 f   LIBCMTD:mdframe_arm.obj
 0001:0009f784       ?GetCurrentState@@YAHPAKPAU_DISPATCHER_CONTEXT@@PBU_s_FuncInfo@@@Z 001a0784 f   LIBCMTD:ehstate_arm_mips.obj
 0001:0009f860       _CallSettingFrame          001a0860     LIBCMTD:handlers_arm.obj
 0001:0009f8a4       _invoke_watson             001a08a4 f   LIBCMTD:invarg.obj
 0001:0009f8d8       _mtinitlocks               001a08d8 f   LIBCMTD:mlock.obj
 0001:0009f9f0       _mtdeletelocks             001a09f0 f   LIBCMTD:mlock.obj
 0001:0009fb74       _mtinitlocknum             001a0b74 f   LIBCMTD:mlock.obj
 0001:0009fcdc       _lock                      001a0cdc f   LIBCMTD:mlock.obj
 0001:0009fdd8       _unlock                    001a0dd8 f   LIBCMTD:mlock.obj
 0001:0009fe18       _lockerr_exit              001a0e18 f   LIBCMTD:mlock.obj
 0001:0009fe40       _CrtDbgBreak               001a0e40 f   LIBCMTD:dbgrptt.obj
 0001:0009fe48       _CrtSetReportMode          001a0e48 f   LIBCMTD:dbgrptt.obj
 0001:000a0070       _CrtSetReportFile          001a1070 f   LIBCMTD:dbgrptt.obj
 0001:000a020c       _CrtSetReportHook          001a120c f   LIBCMTD:dbgrptt.obj
 0001:000a0250       _CrtGetReportHook          001a1250 f   LIBCMTD:dbgrptt.obj
 0001:000a0278       _VCrtDbgReportW            001a1278 f   LIBCMTD:dbgrptt.obj
 0001:000a0e30       __crtMessageBoxW           001a1e30 f   LIBCMTD:crtmbox.obj
 0001:000a1094       wcsncpy_s                  001a2094 f   LIBCMTD:wcsncpy_s.obj
 0001:000a1694       wcscpy_s                   001a2694 f   LIBCMTD:wcscpy_s.obj
 0001:000a1b08       _initp_misc_initcrit       001a2b08 f   LIBCMTD:initcrit.obj
 0001:000a1b34       __crtInitCritSecAndSpinCount 001a2b34 f   LIBCMTD:initcrit.obj
 0001:000a1c64       _amsg_exit                 001a2c64 f   LIBCMTD:crt0dat.obj
 0001:000a1c90       __crtExitProcess           001a2c90 f   LIBCMTD:crt0dat.obj
 0001:000a1cd8       strcpy_s                   001a2cd8 f   LIBCMTD:strcpy_s.obj
 0001:000a212c       wcscat_s                   001a312c f   LIBCMTD:wcscat_s.obj
 0001:000a2710       _itow_s                    001a3710 f   LIBCMTD:xtows.obj
 0001:000a2d9c       _ltow_s                    001a3d9c f   LIBCMTD:xtows.obj
 0001:000a2e1c       _ultow_s                   001a3e1c f   LIBCMTD:xtows.obj
 0001:000a2e70       _encode_pointer            001a3e70 f   LIBCMTD:tidtable.obj
 0001:000a2e98       _encoded_null              001a3e98 f   LIBCMTD:tidtable.obj
 0001:000a2ed0       _decode_pointer            001a3ed0 f   LIBCMTD:tidtable.obj
 0001:000a2ef8       fputs                      001a3ef8 f   coredll:COREDLL.dll
 0001:000a2f08       _getstdfilex               001a3f08 f   coredll:COREDLL.dll
 0001:000a2f18       fflush                     001a3f18 f   coredll:COREDLL.dll
 0001:000a2f28       InterlockedExchange        001a3f28 f   coredll:COREDLL.dll
 0001:000a2f38       ?terminate@std@@YAXXZ      001a3f38 f   coredll:COREDLL.dll
 0001:000a2f48       GetModuleFileNameW         001a3f48 f   coredll:COREDLL.dll
 0001:000a2f58       TlsSetValue                001a3f58 f   coredll:COREDLL.dll
 0001:000a2f68       TlsGetValue                001a3f68 f   coredll:COREDLL.dll
 0001:000a2f78       InterlockedCompareExchange 001a3f78 f   coredll:COREDLL.dll
 0001:000a2f88       TlsCall                    001a3f88 f   coredll:COREDLL.dll
 0001:000a2f98       RaiseException             001a3f98 f   coredll:COREDLL.dll
 0001:000a2fa8       SetLastError               001a3fa8 f   coredll:COREDLL.dll
 0001:000a2fb8       TerminateProcess           001a3fb8 f   coredll:COREDLL.dll
 0002:00006418       ?_EEM_DS@?$deque@PAVCCommand@@V?$allocator@PAVCCommand@@@std@@@std@@2HB 001ab418     atcmd.obj
 0002:0000641c       ??_C@_1CC@JJFJLKM@?$AAR?$AAI?$AAL?$AA?5?$AAH?$AAa?$AAn?$AAd?$AAl?$AAe?$AA?5?$AAN?$AAU?$AAL?$AAL?$AA?$CB?$AA?$AA@ 001ab41c     atcmd.obj
 0002:00006440       ??_C@_1FE@KJJCAGGP@?$AAA?$AAS?$AAS?$AAE?$AAR?$AAT?$AAI?$AAO?$AAN?$AA?5?$AAF?$AAA?$AAI?$AAL?$AAU?$AAR?$AAE?$AA?3?$AA?5?$AA?$DN?$AA?$DN?$AA?$DN?$AA?$DO?$AAF?$AAA?$AAL?$AAS?$AAE?$AA?5?$AA?$CB?$AA?$DN?$AA?5@ 001ab440     atcmd.obj
 0002:00006498       ??_C@_1IK@IKNNEHFL@?$AAc?$AA?3?$AA?2?$AAo?$AAf?$AAf?$AAi?$AAc?$AAa?$AAl?$AA_?$AAb?$AAu?$AAi?$AAl?$AAd?$AA?2?$AAr?$AAi?$AAl?$AAg?$AAo?$AAb?$AAi?$AA?2?$AAs?$AAw?$AA?2?$AAd?$AAl?$AAl?$AAs@ 001ab498     atcmd.obj
 0002:000065e4       ??_C@_1CO@FNIDKHMC@?$AAd?$AAe?$AAq?$AAu?$AAe?$AA?5?$AAe?$AAm?$AAp?$AAt?$AAy?$AA?5?$AAb?$AAe?$AAf?$AAo?$AAr?$AAe?$AA?5?$AAp?$AAo?$AAp?$AA?$AA@ 001ab5e4     atcmd.obj
 0002:00006618       ??_C@_1HO@PJIPAKEN@?$AAC?$AA?3?$AA?2?$AAP?$AAr?$AAo?$AAg?$AAr?$AAa?$AAm?$AA?5?$AAF?$AAi?$AAl?$AAe?$AAs?$AA?2?$AAM?$AAi?$AAc?$AAr?$AAo?$AAs?$AAo?$AAf?$AAt?$AA?5?$AAV?$AAi?$AAs?$AAu?$AAa@ 001ab618     atcmd.obj
 0002:000066d4       ??_C@_1DC@POOIKBAO@?$AAI?$AAT?$AAE?$AAR?$AAA?$AAT?$AAO?$AAR?$AA?5?$AAL?$AAI?$AAS?$AAT?$AA?5?$AAC?$AAO?$AAR?$AAR?$AAU?$AAP?$AAT?$AAE?$AAD?$AA?$CB?$AA?$AA@ 001ab6d4     atcmd.obj
 0002:00006708       ??_C@_1IE@BKKAAKCG@?$AAC?$AA?3?$AA?2?$AAP?$AAr?$AAo?$AAg?$AAr?$AAa?$AAm?$AA?5?$AAF?$AAi?$AAl?$AAe?$AAs?$AA?2?$AAM?$AAi?$AAc?$AAr?$AAo?$AAs?$AAo?$AAf?$AAt?$AA?5?$AAV?$AAi?$AAs?$AAu?$AAa@ 001ab708     atcmd.obj
 0002:0000678c       ??_C@_0BC@KBDMBKEH@deque?$DMT?$DO?5too?5long?$AA@ 001ab78c     atcmd.obj
 0002:0000680c       ?npos@?$basic_string@DU?$char_traits@D@std@@V?$allocator@D@2@@std@@2IB 001ab80c     atcmd.obj
 0002:000069b0       ??_C@_1IC@HKDJIJDA@?$AAC?$AA?3?$AA?2?$AAP?$AAr?$AAo?$AAg?$AAr?$AAa?$AAm?$AA?5?$AAF?$AAi?$AAl?$AAe?$AAs?$AA?2?$AAM?$AAi?$AAc?$AAr?$AAo?$AAs?$AAo?$AAf?$AAt?$AA?5?$AAV?$AAi?$AAs?$AAu?$AAa@ 001ab9b0     atcmd.obj
 0002:00006a34       ??_C@_1CK@EOPGIILJ@?$AAi?$AAn?$AAv?$AAa?$AAl?$AAi?$AAd?$AA?5?$AAn?$AAu?$AAl?$AAl?$AA?5?$AAp?$AAo?$AAi?$AAn?$AAt?$AAe?$AAr?$AA?$AA@ 001aba34     atcmd.obj
 0002:00006a60       ??_C@_1BO@MEPPHOO@?$AA?$CC?$AAo?$AAu?$AAt?$AA?5?$AAo?$AAf?$AA?5?$AAr?$AAa?$AAn?$AAg?$AAe?$AA?$CC?$AA?$AA@ 001aba60     atcmd.obj
 0002:00006a80       ??_C@_1ME@FPINPEIL@?$AAs?$AAt?$AAd?$AA?3?$AA?3?$AA_?$AAD?$AAe?$AAq?$AAu?$AAe?$AA_?$AAc?$AAo?$AAn?$AAs?$AAt?$AA_?$AAi?$AAt?$AAe?$AAr?$AAa?$AAt?$AAo?$AAr?$AA?$DM?$AAc?$AAl?$AAa?$AAs?$AAs@ 001aba80     atcmd.obj
 0002:00006b48       ??_C@_1FG@CMLDHNON@?$AA?$CI?$AA?$CC?$AAS?$AAt?$AAa?$AAn?$AAd?$AAa?$AAr?$AAd?$AA?5?$AAC?$AA?$CL?$AA?$CL?$AA?5?$AAL?$AAi?$AAb?$AAr?$AAa?$AAr?$AAi?$AAe?$AAs?$AA?5?$AAO?$AAu?$AAt?$AA?5?$AAo?$AAf?$AA?5@ 001abb48     atcmd.obj
 0002:00006ba0       ??_C@_1EE@INPCGGNP@?$AAd?$AAe?$AAq?$AAu?$AAe?$AA?5?$AAi?$AAt?$AAe?$AAr?$AAa?$AAt?$AAo?$AAr?$AA?5?$AAn?$AAo?$AAt?$AA?5?$AAd?$AAe?$AAr?$AAe?$AAf?$AAe?$AAr?$AAe?$AAn?$AAc?$AAa?$AAb?$AAl@ 001abba0     atcmd.obj
 0002:00006be4       ??_C@_1CG@JNLFBNGN@?$AA?$CC?$AAi?$AAn?$AAv?$AAa?$AAl?$AAi?$AAd?$AA?5?$AAa?$AAr?$AAg?$AAu?$AAm?$AAe?$AAn?$AAt?$AA?$CC?$AA?$AA@ 001abbe4     atcmd.obj
 0002:00006c10       ??_C@_1NK@DOBEJJKB@?$AAs?$AAt?$AAd?$AA?3?$AA?3?$AA_?$AAD?$AAe?$AAq?$AAu?$AAe?$AA_?$AAc?$AAo?$AAn?$AAs?$AAt?$AA_?$AAi?$AAt?$AAe?$AAr?$AAa?$AAt?$AAo?$AAr?$AA?$DM?$AAc?$AAl?$AAa?$AAs?$AAs@ 001abc10     atcmd.obj
 0002:00006cf0       ??_C@_1BBC@GFBPNMEP@?$AA?$CI?$AA?$CC?$AA_?$AAP?$AAd?$AAe?$AAq?$AAu?$AAe?$AA?5?$AA?$CB?$AA?$DN?$AA?5?$AA0?$AA?5?$AA?$CG?$AA?$CG?$AA?5?$AA?$CI?$AA?$CI?$AA_?$AAM?$AAy?$AAd?$AAe?$AAq?$AAu?$AAe?$AA?5?$AA?$CK?$AA?$CJ?$AA_@ 001abcf0     atcmd.obj
 0002:00006e80       ??_C@_1IA@NDFJEPCJ@?$AAC?$AA?3?$AA?2?$AAP?$AAr?$AAo?$AAg?$AAr?$AAa?$AAm?$AA?5?$AAF?$AAi?$AAl?$AAe?$AAs?$AA?2?$AAM?$AAi?$AAc?$AAr?$AAo?$AAs?$AAo?$AAf?$AAt?$AA?5?$AAV?$AAi?$AAs?$AAu?$AAa@ 001abe80     atcmd.obj
 0002:00006f00       ??_C@_1CO@DGLIKNHI@?$AAi?$AAn?$AAv?$AAa?$AAl?$AAi?$AAd?$AA?5?$AAi?$AAt?$AAe?$AAr?$AAa?$AAt?$AAo?$AAr?$AA?5?$AAr?$AAa?$AAn?$AAg?$AAe?$AA?$AA@ 001abf00     atcmd.obj
 0002:00013c5c       ??_C@_11LOCGONAA@?$AA?$AA@ 001b8c5c     callctrl.obj
 0002:00013c60       ??_C@_1CE@JANOHFNC@?$AAR?$AAa?$AAd?$AAi?$AAo?$AA?5?$AAH?$AAa?$AAn?$AAd?$AAl?$AAe?$AA?5?$AAN?$AAU?$AAL?$AAL?$AA?$AA@ 001b8c60     callctrl.obj
 0002:00013c84       ??_C@_00CNPNBAHC@?$AA@     001b8c84     callctrl.obj
 0002:00013c88       ??_C@_1PI@IPMMDMEC@?$AAs?$AAt?$AAd?$AA?3?$AA?3?$AAl?$AAi?$AAs?$AAt?$AA?$DM?$AAs?$AAt?$AAr?$AAu?$AAc?$AAt?$AA?5?$AAt?$AAa?$AAg?$AAE?$AAM?$AAE?$AAR?$AAG?$AAE?$AAN?$AAC?$AAY?$AA_?$AAN?$AAU@ 001b8c88     callctrl.obj
 0002:00013d80       ??_C@_1EC@HILJLMMC@?$AAl?$AAi?$AAs?$AAt?$AA?5?$AAi?$AAt?$AAe?$AAr?$AAa?$AAt?$AAo?$AAr?$AA?5?$AAn?$AAo?$AAt?$AA?5?$AAd?$AAe?$AAr?$AAe?$AAf?$AAe?$AAr?$AAe?$AAn?$AAc?$AAa?$AAb?$AAl?$AAe@ 001b8d80     callctrl.obj
 0002:00013dc8       ??_C@_1HM@HPOOGGJN@?$AAC?$AA?3?$AA?2?$AAP?$AAr?$AAo?$AAg?$AAr?$AAa?$AAm?$AA?5?$AAF?$AAi?$AAl?$AAe?$AAs?$AA?2?$AAM?$AAi?$AAc?$AAr?$AAo?$AAs?$AAo?$AAf?$AAt?$AA?5?$AAV?$AAi?$AAs?$AAu?$AAa@ 001b8dc8     callctrl.obj
 0002:00013e48       ??_C@_1PK@FBEPCFFG@?$AAs?$AAt?$AAd?$AA?3?$AA?3?$AAl?$AAi?$AAs?$AAt?$AA?$DM?$AAs?$AAt?$AAr?$AAu?$AAc?$AAt?$AA?5?$AAt?$AAa?$AAg?$AAE?$AAM?$AAE?$AAR?$AAG?$AAE?$AAN?$AAC?$AAY?$AA_?$AAN?$AAU@ 001b8e48     callctrl.obj
 0002:00013f48       ??_C@_1EA@DOGAGKDH@?$AAl?$AAi?$AAs?$AAt?$AA?5?$AAi?$AAt?$AAe?$AAr?$AAa?$AAt?$AAo?$AAr?$AA?5?$AAn?$AAo?$AAt?$AA?5?$AAi?$AAn?$AAc?$AAr?$AAe?$AAm?$AAe?$AAn?$AAt?$AAa?$AAb?$AAl?$AAe?$AA?$AA@ 001b8f48     callctrl.obj
 0002:00013fc0       ??_C@_1PC@GOANGADO@?$AAs?$AAt?$AAd?$AA?3?$AA?3?$AAl?$AAi?$AAs?$AAt?$AA?$DM?$AAs?$AAt?$AAr?$AAu?$AAc?$AAt?$AA?5?$AAt?$AAa?$AAg?$AAE?$AAM?$AAE?$AAR?$AAG?$AAE?$AAN?$AAC?$AAY?$AA_?$AAN?$AAU@ 001b8fc0     callctrl.obj
 0002:000140b8       ??_C@_1FO@OCPOOAIA@?$AA?$CI?$AA?$CC?$AAS?$AAt?$AAa?$AAn?$AAd?$AAa?$AAr?$AAd?$AA?5?$AAC?$AA?$CL?$AA?$CL?$AA?5?$AAL?$AAi?$AAb?$AAr?$AAa?$AAr?$AAi?$AAe?$AAs?$AA?5?$AAI?$AAn?$AAv?$AAa?$AAl?$AAi?$AAd@ 001b90b8     callctrl.obj
 0002:00014118       ??_C@_1DI@MDELDGPI@?$AAl?$AAi?$AAs?$AAt?$AA?5?$AAi?$AAt?$AAe?$AAr?$AAa?$AAt?$AAo?$AAr?$AAs?$AA?5?$AAi?$AAn?$AAc?$AAo?$AAm?$AAp?$AAa?$AAt?$AAi?$AAb?$AAl?$AAe?$AA?$AA@ 001b9118     callctrl.obj
 0002:0001a17c       ??_7CChannel@@6B@          001bf17c     channel.obj
 0002:0001a180       ??_C@_1EM@HHCPHIDC@?$AAW?$AAa?$AAi?$AAt?$AAC?$AAo?$AAm?$AAm?$AAE?$AAv?$AAe?$AAn?$AAt?$AA?5?$AAr?$AAe?$AAt?$AAu?$AAr?$AAn?$AAs?$AA?5?$AAw?$AAi?$AAn?$AAE?$AAr?$AAr?$AAo?$AAr?$AA?5?$AA?$DN@ 001bf180     channel.obj
 0002:0001a1d0       ??_C@_1IE@GJFPDDGH@?$AAW?$AAa?$AAi?$AAt?$AAC?$AAo?$AAm?$AAE?$AAv?$AAe?$AAn?$AAt?$AA?5?$AAr?$AAe?$AAt?$AAu?$AAr?$AAn?$AAs?$AA?5?$AAT?$AAR?$AAU?$AAE?$AA?5?$AAw?$AAi?$AAt?$AAh?$AA?5?$AAc@ 001bf1d0     channel.obj
 0002:0001a258       ??_C@_1GA@JNNIHLPG@?$AA?$CF?$AAd?$AA?5?$AAb?$AAy?$AAt?$AAe?$AAs?$AA?5?$AAw?$AAr?$AAi?$AAt?$AAt?$AAe?$AAn?$AA?5?$AAt?$AAo?$AA?5?$AAW?$AAr?$AAi?$AAt?$AAe?$AAR?$AAx?$AAd?$AAD?$AAa?$AAt?$AAa@ 001bf258     channel.obj
 0002:0001a2b8       ??_C@_1EC@DAOPNPPB@?$AAR?$AAe?$AAa?$AAd?$AAF?$AAi?$AAl?$AAe?$AA?5?$AAr?$AAe?$AAt?$AAu?$AAr?$AAn?$AAs?$AA?5?$AAw?$AAi?$AAn?$AAE?$AAr?$AAr?$AAo?$AAr?$AA?5?$AA?$DN?$AA?5?$AA0?$AAx?$AA?$CF?$AAx@ 001bf2b8     channel.obj
 0002:0001a2fc       ??_7ChannelLinker@@6B@     001bf2fc     channel.obj
 0002:00026db8       ??_C@_1HO@LFKIEFJO@?$AAC?$AA?3?$AA?2?$AAP?$AAr?$AAo?$AAg?$AAr?$AAa?$AAm?$AA?5?$AAF?$AAi?$AAl?$AAe?$AAs?$AA?2?$AAM?$AAi?$AAc?$AAr?$AAo?$AAs?$AAo?$AAf?$AAt?$AA?5?$AAV?$AAi?$AAs?$AAu?$AAa@ 001cbdb8     DatERI.obj
 0002:00027028       ??_C@_1EM@MHOKKPFH@?$AAm?$AAa?$AAp?$AA?1?$AAs?$AAe?$AAt?$AA?5?$AAi?$AAn?$AAs?$AAe?$AAr?$AAt?$AA?5?$AAi?$AAt?$AAe?$AAr?$AAa?$AAt?$AAo?$AAr?$AA?5?$AAo?$AAu?$AAt?$AAs?$AAi?$AAd?$AAe?$AA?5@ 001cc028     DatERI.obj
 0002:00027430       ??_C@_1BPM@NPECLHEC@?$AAs?$AAt?$AAd?$AA?3?$AA?3?$AA_?$AAT?$AAr?$AAe?$AAe?$AA?$DM?$AAc?$AAl?$AAa?$AAs?$AAs?$AA?5?$AAs?$AAt?$AAd?$AA?3?$AA?3?$AA_?$AAT?$AAm?$AAa?$AAp?$AA_?$AAt?$AAr?$AAa?$AAi@ 001cc430     DatERI.obj
 0002:0002762c       ??_C@_1DO@CFEEPGGJ@?$AAm?$AAa?$AAp?$AA?1?$AAs?$AAe?$AAt?$AA?5?$AAi?$AAt?$AAe?$AAr?$AAa?$AAt?$AAo?$AAr?$AAs?$AA?5?$AAi?$AAn?$AAc?$AAo?$AAm?$AAp?$AAa?$AAt?$AAi?$AAb?$AAl?$AAe?$AA?$AA@ 001cc62c     DatERI.obj
 0002:00027670       ??_C@_1CAI@LHCAMOFF@?$AAs?$AAt?$AAd?$AA?3?$AA?3?$AA_?$AAT?$AAr?$AAe?$AAe?$AA?$DM?$AAc?$AAl?$AAa?$AAs?$AAs?$AA?5?$AAs?$AAt?$AAd?$AA?3?$AA?3?$AA_?$AAT?$AAm?$AAa?$AAp?$AA_?$AAt?$AAr?$AAa?$AAi@ 001cc670     DatERI.obj
 0002:000279e0       ??_C@_0BE@JONHPENG@map?1set?$DMT?$DO?5too?5long?$AA@ 001cc9e0     DatERI.obj
 0002:00027c18       ??_C@_1BPK@PNLBDCCO@?$AAs?$AAt?$AAd?$AA?3?$AA?3?$AA_?$AAT?$AAr?$AAe?$AAe?$AA?$DM?$AAc?$AAl?$AAa?$AAs?$AAs?$AA?5?$AAs?$AAt?$AAd?$AA?3?$AA?3?$AA_?$AAT?$AAm?$AAa?$AAp?$AA_?$AAt?$AAr?$AAa?$AAi@ 001ccc18     DatERI.obj
 0002:00027e18       ??_C@_1EI@FHEHNNNM@?$AAm?$AAa?$AAp?$AA?1?$AAs?$AAe?$AAt?$AA?5?$AAi?$AAt?$AAe?$AAr?$AAa?$AAt?$AAo?$AAr?$AA?5?$AAn?$AAo?$AAt?$AA?5?$AAd?$AAe?$AAr?$AAe?$AAf?$AAe?$AAr?$AAe?$AAn?$AAc?$AAa@ 001cce18     DatERI.obj
 0002:00027e98       ??_C@_1CAG@OHDPPGBN@?$AAs?$AAt?$AAd?$AA?3?$AA?3?$AA_?$AAT?$AAr?$AAe?$AAe?$AA?$DM?$AAc?$AAl?$AAa?$AAs?$AAs?$AA?5?$AAs?$AAt?$AAd?$AA?3?$AA?3?$AA_?$AAT?$AAm?$AAa?$AAp?$AA_?$AAt?$AAr?$AAa?$AAi@ 001cce98     DatERI.obj
 0002:000280a0       ??_C@_1EK@PPDBPCAN@?$AAm?$AAa?$AAp?$AA?1?$AAs?$AAe?$AAt?$AA?5?$AAe?$AAr?$AAa?$AAs?$AAe?$AA?5?$AAi?$AAt?$AAe?$AAr?$AAa?$AAt?$AAo?$AAr?$AA?5?$AAo?$AAu?$AAt?$AAs?$AAi?$AAd?$AAe?$AA?5?$AAr@ 001cd0a0     DatERI.obj
 0002:00028370       ??_C@_1BOO@IPGPPFFI@?$AAs?$AAt?$AAd?$AA?3?$AA?3?$AA_?$AAT?$AAr?$AAe?$AAe?$AA?$DM?$AAc?$AAl?$AAa?$AAs?$AAs?$AA?5?$AAs?$AAt?$AAd?$AA?3?$AA?3?$AA_?$AAT?$AAm?$AAa?$AAp?$AA_?$AAt?$AAr?$AAa?$AAi@ 001cd370     DatERI.obj
 0002:00028560       ??_C@_1EG@EHJFMBHJ@?$AAm?$AAa?$AAp?$AA?1?$AAs?$AAe?$AAt?$AA?5?$AAi?$AAt?$AAe?$AAr?$AAa?$AAt?$AAo?$AAr?$AA?5?$AAn?$AAo?$AAt?$AA?5?$AAi?$AAn?$AAc?$AAr?$AAe?$AAm?$AAe?$AAn?$AAt?$AAa?$AAb@ 001cd560     DatERI.obj
 0002:000285a8       ??_C@_1BPK@CKAHNOLJ@?$AAs?$AAt?$AAd?$AA?3?$AA?3?$AA_?$AAT?$AAr?$AAe?$AAe?$AA?$DM?$AAc?$AAl?$AAa?$AAs?$AAs?$AA?5?$AAs?$AAt?$AAd?$AA?3?$AA?3?$AA_?$AAT?$AAm?$AAa?$AAp?$AA_?$AAt?$AAr?$AAa?$AAi@ 001cd5a8     DatERI.obj
 0002:000287a8       ??_C@_1BOO@HOKNBAEK@?$AAs?$AAt?$AAd?$AA?3?$AA?3?$AA_?$AAT?$AAr?$AAe?$AAe?$AA?$DM?$AAc?$AAl?$AAa?$AAs?$AAs?$AA?5?$AAs?$AAt?$AAd?$AA?3?$AA?3?$AA_?$AAT?$AAm?$AAa?$AAp?$AA_?$AAt?$AAr?$AAa?$AAi@ 001cd7a8     DatERI.obj
 0002:00028998       ??_C@_1EG@OKCGOALM@?$AAm?$AAa?$AAp?$AA?1?$AAs?$AAe?$AAt?$AA?5?$AAi?$AAt?$AAe?$AAr?$AAa?$AAt?$AAo?$AAr?$AA?5?$AAn?$AAo?$AAt?$AA?5?$AAd?$AAe?$AAc?$AAr?$AAe?$AAm?$AAe?$AAn?$AAt?$AAa?$AAb@ 001cd998     DatERI.obj
 0002:000289e0       ??_C@_1BPK@NLMFDLKL@?$AAs?$AAt?$AAd?$AA?3?$AA?3?$AA_?$AAT?$AAr?$AAe?$AAe?$AA?$DM?$AAc?$AAl?$AAa?$AAs?$AAs?$AA?5?$AAs?$AAt?$AAd?$AA?3?$AA?3?$AA_?$AAT?$AAm?$AAa?$AAp?$AA_?$AAt?$AAr?$AAa?$AAi@ 001cd9e0     DatERI.obj
 0002:00028bdc       ??_C@_1CE@IGJMOCCK@?$AAi?$AAn?$AAv?$AAa?$AAl?$AAi?$AAd?$AA?5?$AAo?$AAp?$AAe?$AAr?$AAa?$AAt?$AAo?$AAr?$AA?$DM?$AA?$AA@ 001cdbdc     DatERI.obj
 0002:00030838       ?_EEM_DS@?$deque@PAUSwiNotifyVariant@@V?$allocator@PAUSwiNotifyVariant@@@std@@@std@@2HB 001d5838     FakeResponse.obj
 0002:0003083c       ??_C@_1DO@PJLLKFHK@?$AAA?$AAS?$AAS?$AAE?$AAR?$AAT?$AA?5?$AAF?$AAA?$AAI?$AAL?$AAU?$AAR?$AAE?$AA?5?$AAa?$AAt?$AA?5?$AA?$CF?$AAs?$AA?5?$AAl?$AAi?$AAn?$AAe?$AA?5?$AA?$CF?$AAd?$AA?$AN?$AA?6?$AA?$AA@ 001d583c     FakeResponse.obj
 0002:00030880       ??_C@_1GC@FIPCILJB@?$AA?4?$AA?4?$AA?2?$AA?4?$AA?4?$AA?2?$AA?4?$AA?4?$AA?2?$AAU?$AAt?$AAi?$AAl?$AAi?$AAt?$AAi?$AAe?$AAs?$AA?2?$AAL?$AAo?$AAg?$AAg?$AAe?$AAr?$AA?2?$AAS?$AAW?$AA_?$AAL?$AAo?$AAg@ 001d5880     FakeResponse.obj
 0002:000308e8       ??_C@_1EG@BPNHNPIG@?$AAl?$AAi?$AAs?$AAt?$AA?5?$AAi?$AAn?$AAs?$AAe?$AAr?$AAt?$AA?5?$AAi?$AAt?$AAe?$AAr?$AAa?$AAt?$AAo?$AAr?$AA?5?$AAo?$AAu?$AAt?$AAs?$AAi?$AAd?$AAe?$AA?5?$AAr?$AAa?$AAn@ 001d58e8     FakeResponse.obj
 0002:000309dc       ??_C@_0BB@MOGOBHAF@list?$DMT?$DO?5too?5long?$AA@ 001d59dc     FakeResponse.obj
 0002:00030aa8       ??_C@_1OI@ECJHJELO@?$AAs?$AAt?$AAd?$AA?3?$AA?3?$AA_?$AAD?$AAe?$AAq?$AAu?$AAe?$AA_?$AAc?$AAo?$AAn?$AAs?$AAt?$AA_?$AAi?$AAt?$AAe?$AAr?$AAa?$AAt?$AAo?$AAr?$AA?$DM?$AAs?$AAt?$AAr?$AAu?$AAc@ 001d5aa8     FakeResponse.obj
 0002:00030b90       ??_C@_1PO@KEGGHOOE@?$AAs?$AAt?$AAd?$AA?3?$AA?3?$AA_?$AAD?$AAe?$AAq?$AAu?$AAe?$AA_?$AAc?$AAo?$AAn?$AAs?$AAt?$AA_?$AAi?$AAt?$AAe?$AAr?$AAa?$AAt?$AAo?$AAr?$AA?$DM?$AAs?$AAt?$AAr?$AAu?$AAc@ 001d5b90     FakeResponse.obj
 0002:00044c78       ??_C@_1EE@BBMFLDOC@?$AAl?$AAi?$AAs?$AAt?$AA?5?$AAe?$AAr?$AAa?$AAs?$AAe?$AA?5?$AAi?$AAt?$AAe?$AAr?$AAa?$AAt?$AAo?$AAr?$AA?5?$AAo?$AAu?$AAt?$AAs?$AAi?$AAd?$AAe?$AA?5?$AAr?$AAa?$AAn?$AAg@ 001e9c78     misc.obj
 0002:00044df0       ??_C@_1EG@NPGGHPOJ@?$AAl?$AAi?$AAs?$AAt?$AA?5?$AAs?$AAp?$AAl?$AAi?$AAc?$AAe?$AA?5?$AAi?$AAt?$AAe?$AAr?$AAa?$AAt?$AAo?$AAr?$AA?5?$AAo?$AAu?$AAt?$AAs?$AAi?$AAd?$AAe?$AA?5?$AAr?$AAa?$AAn@ 001e9df0     misc.obj
 0002:000452bc       ??_C@_1CK@JNHDEEDC@?$AAs?$AAe?$AAq?$AAu?$AAe?$AAn?$AAc?$AAe?$AA?5?$AAn?$AAo?$AAt?$AA?5?$AAo?$AAr?$AAd?$AAe?$AAr?$AAe?$AAd?$AA?$AA@ 001ea2bc     misc.obj
 0002:0004534c       ??_C@_1DM@PIGEIECN@?$AAl?$AAi?$AAs?$AAt?$AA?5?$AAi?$AAn?$AAs?$AAe?$AAr?$AAt?$AAi?$AAo?$AAn?$AA?5?$AAo?$AAv?$AAe?$AAr?$AAl?$AAa?$AAp?$AAs?$AA?5?$AAr?$AAa?$AAn?$AAg?$AAe?$AA?$AA@ 001ea34c     misc.obj
 0002:000454c0       ??_C@_1PK@KCHNJJJH@?$AAs?$AAt?$AAd?$AA?3?$AA?3?$AAl?$AAi?$AAs?$AAt?$AA?$DM?$AAs?$AAt?$AAr?$AAu?$AAc?$AAt?$AA?5?$AAt?$AAa?$AAg?$AAE?$AAM?$AAE?$AAR?$AAG?$AAE?$AAN?$AAC?$AAY?$AA_?$AAN?$AAU@ 001ea4c0     misc.obj
 0002:000455c0       ??_C@_1EA@JDNDELPC@?$AAl?$AAi?$AAs?$AAt?$AA?5?$AAi?$AAt?$AAe?$AAr?$AAa?$AAt?$AAo?$AAr?$AA?5?$AAn?$AAo?$AAt?$AA?5?$AAd?$AAe?$AAc?$AAr?$AAe?$AAm?$AAe?$AAn?$AAt?$AAa?$AAb?$AAl?$AAe?$AA?$AA@ 001ea5c0     misc.obj
 0002:000549dc       ??_7CriticalSection@@6B@   001f99dc     msg.obj
 0002:0006b958       ??_C@_1MI@PAMKCPOP@?$AAs?$AAt?$AAd?$AA?3?$AA?3?$AAl?$AAi?$AAs?$AAt?$AA?$DM?$AAc?$AAl?$AAa?$AAs?$AAs?$AA?5?$AAC?$AAC?$AAo?$AAm?$AAm?$AAa?$AAn?$AAd?$AA?5?$AA?$CK?$AA?0?$AAc?$AAl?$AAa?$AAs?$AAs@ 00210958     Radio.obj
 0002:0006ba20       ??_C@_1MK@MOFINJCK@?$AAs?$AAt?$AAd?$AA?3?$AA?3?$AAl?$AAi?$AAs?$AAt?$AA?$DM?$AAc?$AAl?$AAa?$AAs?$AAs?$AA?5?$AAC?$AAC?$AAo?$AAm?$AAm?$AAa?$AAn?$AAd?$AA?5?$AA?$CK?$AA?0?$AAc?$AAl?$AAa?$AAs?$AAs@ 00210a20     Radio.obj
 0002:0006baf0       ??_C@_1MC@HNICPGGN@?$AAs?$AAt?$AAd?$AA?3?$AA?3?$AAl?$AAi?$AAs?$AAt?$AA?$DM?$AAc?$AAl?$AAa?$AAs?$AAs?$AA?5?$AAC?$AAC?$AAo?$AAm?$AAm?$AAa?$AAn?$AAd?$AA?5?$AA?$CK?$AA?0?$AAc?$AAl?$AAa?$AAs?$AAs@ 00210af0     Radio.obj
 0002:0006bbb8       ??_C@_1BJK@JJMHBPNI@?$AAs?$AAt?$AAd?$AA?3?$AA?3?$AA_?$AAT?$AAr?$AAe?$AAe?$AA?$DM?$AAc?$AAl?$AAa?$AAs?$AAs?$AA?5?$AAs?$AAt?$AAd?$AA?3?$AA?3?$AA_?$AAT?$AAm?$AAa?$AAp?$AA_?$AAt?$AAr?$AAa?$AAi@ 00210bb8     Radio.obj
 0002:0006be08       ??_C@_1BMO@ICFFBCJB@?$AAs?$AAt?$AAd?$AA?3?$AA?3?$AA_?$AAT?$AAr?$AAe?$AAe?$AA?$DM?$AAc?$AAl?$AAa?$AAs?$AAs?$AA?5?$AAs?$AAt?$AAd?$AA?3?$AA?3?$AA_?$AAT?$AAm?$AAa?$AAp?$AA_?$AAt?$AAr?$AAa?$AAi@ 00210e08     Radio.obj
 0002:0006c1c8       ??_C@_1BJI@IIKALLOP@?$AAs?$AAt?$AAd?$AA?3?$AA?3?$AA_?$AAT?$AAr?$AAe?$AAe?$AA?$DM?$AAc?$AAl?$AAa?$AAs?$AAs?$AA?5?$AAs?$AAt?$AAd?$AA?3?$AA?3?$AA_?$AAT?$AAm?$AAa?$AAp?$AA_?$AAt?$AAr?$AAa?$AAi@ 002111c8     Radio.obj
 0002:0006c660       ??_C@_1BMA@JEJMFKGL@?$AAs?$AAt?$AAd?$AA?3?$AA?3?$AA_?$AAT?$AAr?$AAe?$AAe?$AA?$DM?$AAc?$AAl?$AAa?$AAs?$AAs?$AA?5?$AAs?$AAt?$AAd?$AA?3?$AA?3?$AA_?$AAT?$AAm?$AAa?$AAp?$AA_?$AAt?$AAr?$AAa?$AAi@ 00211660     Radio.obj
 0002:0006c820       ??_C@_1BIM@FPJGLLBH@?$AAs?$AAt?$AAd?$AA?3?$AA?3?$AA_?$AAT?$AAr?$AAe?$AAe?$AA?$DM?$AAc?$AAl?$AAa?$AAs?$AAs?$AA?5?$AAs?$AAt?$AAd?$AA?3?$AA?3?$AA_?$AAT?$AAm?$AAa?$AAp?$AA_?$AAt?$AAr?$AAa?$AAi@ 00211820     Radio.obj
 0002:0006c9b0       ??_C@_1BIM@KOFEFOAF@?$AAs?$AAt?$AAd?$AA?3?$AA?3?$AA_?$AAT?$AAr?$AAe?$AAe?$AA?$DM?$AAc?$AAl?$AAa?$AAs?$AAs?$AA?5?$AAs?$AAt?$AAd?$AA?3?$AA?3?$AA_?$AAT?$AAm?$AAa?$AAp?$AA_?$AAt?$AAr?$AAa?$AAi@ 002119b0     Radio.obj
 0002:0007d63c       ?g_tszRegKeyRIL@@3QBGB     0022263c     rilhand.obj
 0002:0007d680       ?g_tszRegKeyAPIInfo@@3QBGB 00222680     rilhand.obj
 0002:00083954       ??_7?$CUnboundedQueue@Urildrvnotification_tag@@@@6B@ 00228954     rilhand.obj
 0002:00083958       ??_7CUniquelyNamedEvent@@6B@ 00228958     rilhand.obj
 0002:0008395c       ??_7CEvent@@6B@            0022895c     rilhand.obj
 0002:000839a0       ??_C@_1IK@IDKOMAEI@?$AAc?$AA?3?$AA?2?$AAo?$AAf?$AAf?$AAi?$AAc?$AAa?$AAl?$AA_?$AAb?$AAu?$AAi?$AAl?$AAd?$AA?2?$AAr?$AAi?$AAl?$AAg?$AAo?$AAb?$AAi?$AA?2?$AAs?$AAw?$AA?2?$AAd?$AAl?$AAl?$AAs@ 002289a0     rilhand.obj
 0002:00083a2c       ??_C@_19GODENFJI@?$AA?$CF?$AAs?$AA?$CF?$AAx?$AA?$AA@ 00228a2c     rilhand.obj
 0002:00083b1c       ??_7Event@@6B@             00228b1c     rilhand.obj
 0002:0008afc8       ??_C@_1BMM@CJGNHDGC@?$AAs?$AAt?$AAd?$AA?3?$AA?3?$AA_?$AAT?$AAr?$AAe?$AAe?$AA?$DM?$AAc?$AAl?$AAa?$AAs?$AAs?$AA?5?$AAs?$AAt?$AAd?$AA?3?$AA?3?$AA_?$AAT?$AAm?$AAa?$AAp?$AA_?$AAt?$AAr?$AAa?$AAi@ 0022ffc8     rilhandndis.obj
 0002:0008b218       ??_C@_1BMA@GFFOLPHJ@?$AAs?$AAt?$AAd?$AA?3?$AA?3?$AA_?$AAT?$AAr?$AAe?$AAe?$AA?$DM?$AAc?$AAl?$AAa?$AAs?$AAs?$AA?5?$AAs?$AAt?$AAd?$AA?3?$AA?3?$AA_?$AAT?$AAm?$AAa?$AAp?$AA_?$AAt?$AAr?$AAa?$AAi@ 00230218     rilhandndis.obj
 0002:000abeec       ??_7StringCollection@@6B@  00250eec     toolbox.obj
 0002:000abefc       ??_7SortedStringCollection@@6B@ 00250efc     toolbox.obj
 0002:000abf10       ??_7?$GrowablePointerCollection@G@@6B@ 00250f10     toolbox.obj
 0002:000abf60       ??_C@_1FK@FNONLNGN@?$AA?$CF?$AAs?$AA?3?$AA?5?$AAD?$AAE?$AAB?$AAU?$AAG?$AAC?$AAH?$AAK?$AA?5?$AAf?$AAa?$AAi?$AAl?$AAe?$AAd?$AA?5?$AAi?$AAn?$AA?5?$AAf?$AAi?$AAl?$AAe?$AA?5?$AA?$CF?$AAs?$AA?5?$AAa@ 00250f60     toolbox.obj
 0002:000abfbc       ??_C@_1BA@LEPJIIOK@?$AAU?$AAn?$AAk?$AAn?$AAo?$AAw?$AAn?$AA?$AA@ 00250fbc     toolbox.obj
 0002:000abfd0       ??_C@_1IK@IBGDELLL@?$AAc?$AA?3?$AA?2?$AAo?$AAf?$AAf?$AAi?$AAc?$AAa?$AAl?$AA_?$AAb?$AAu?$AAi?$AAl?$AAd?$AA?2?$AAr?$AAi?$AAl?$AAg?$AAo?$AAb?$AAi?$AA?2?$AAs?$AAw?$AA?2?$AAd?$AAl?$AAl?$AAs@ 00250fd0     toolbox.obj
 0002:000ac060       ??_7?$GrowableThingCollection@PAG@@6B@ 00251060     toolbox.obj
 0002:000ac0b0       ??_C@_0EF@KGJOBEJL@c?3?2offical_build?2rilgobi?2sw?2dlls@ 002510b0     toolbox.obj
 0002:000ac0f8       ??_7?$GrowableThingCollection@PAX@@6B@ 002510f8     toolbox.obj
 0002:000ac148       ??_7?$GrowableThingCollection@UTaskListTaskData@TaskList@@@@6B@ 00251148     toolbox.obj
 0002:000bc084       ??_C@_0P@GHFPNOJB@bad?5allocation?$AA@ 00261084     libcpmtd:stdthrow.obj
 0002:000bc094       ??_C@_01EEMJAFIK@?6?$AA@   00261094     libcpmtd:stdthrow.obj
 0002:000bc098       ??_C@_07CIFAGBMG@unknown?$AA@ 00261098     libcpmtd:stdthrow.obj
 0002:000bc0a0       ??_C@_0M@LLHBPFNE@exception?3?5?$AA@ 002610a0     libcpmtd:stdthrow.obj
 0002:000bc0ac       ?skipws@?$_Iosb@H@std@@2W4_Fmtflags@12@B 002610ac     libcpmtd:string.obj
 0002:000bc0b0       ?unitbuf@?$_Iosb@H@std@@2W4_Fmtflags@12@B 002610b0     libcpmtd:string.obj
 0002:000bc0b4       ?uppercase@?$_Iosb@H@std@@2W4_Fmtflags@12@B 002610b4     libcpmtd:string.obj
 0002:000bc0b8       ?showbase@?$_Iosb@H@std@@2W4_Fmtflags@12@B 002610b8     libcpmtd:string.obj
 0002:000bc0bc       ?showpoint@?$_Iosb@H@std@@2W4_Fmtflags@12@B 002610bc     libcpmtd:string.obj
 0002:000bc0c0       ?showpos@?$_Iosb@H@std@@2W4_Fmtflags@12@B 002610c0     libcpmtd:string.obj
 0002:000bc0c4       ?left@?$_Iosb@H@std@@2W4_Fmtflags@12@B 002610c4     libcpmtd:string.obj
 0002:000bc0c8       ?right@?$_Iosb@H@std@@2W4_Fmtflags@12@B 002610c8     libcpmtd:string.obj
 0002:000bc0cc       ?internal@?$_Iosb@H@std@@2W4_Fmtflags@12@B 002610cc     libcpmtd:string.obj
 0002:000bc0d0       ?dec@?$_Iosb@H@std@@2W4_Fmtflags@12@B 002610d0     libcpmtd:string.obj
 0002:000bc0d4       ?oct@?$_Iosb@H@std@@2W4_Fmtflags@12@B 002610d4     libcpmtd:string.obj
 0002:000bc0d8       ?hex@?$_Iosb@H@std@@2W4_Fmtflags@12@B 002610d8     libcpmtd:string.obj
 0002:000bc0dc       ?scientific@?$_Iosb@H@std@@2W4_Fmtflags@12@B 002610dc     libcpmtd:string.obj
 0002:000bc0e0       ?fixed@?$_Iosb@H@std@@2W4_Fmtflags@12@B 002610e0     libcpmtd:string.obj
 0002:000bc0e4       ?boolalpha@?$_Iosb@H@std@@2W4_Fmtflags@12@B 002610e4     libcpmtd:string.obj
 0002:000bc0e8       ?_Stdio@?$_Iosb@H@std@@2W4_Fmtflags@12@B 002610e8     libcpmtd:string.obj
 0002:000bc0ec       ?adjustfield@?$_Iosb@H@std@@2W4_Fmtflags@12@B 002610ec     libcpmtd:string.obj
 0002:000bc0f0       ?basefield@?$_Iosb@H@std@@2W4_Fmtflags@12@B 002610f0     libcpmtd:string.obj
 0002:000bc0f4       ?floatfield@?$_Iosb@H@std@@2W4_Fmtflags@12@B 002610f4     libcpmtd:string.obj
 0002:000bc0f8       ?goodbit@?$_Iosb@H@std@@2W4_Iostate@12@B 002610f8     libcpmtd:string.obj
 0002:000bc0fc       ?eofbit@?$_Iosb@H@std@@2W4_Iostate@12@B 002610fc     libcpmtd:string.obj
 0002:000bc100       ?failbit@?$_Iosb@H@std@@2W4_Iostate@12@B 00261100     libcpmtd:string.obj
 0002:000bc104       ?badbit@?$_Iosb@H@std@@2W4_Iostate@12@B 00261104     libcpmtd:string.obj
 0002:000bc108       ?_Hardfail@?$_Iosb@H@std@@2W4_Iostate@12@B 00261108     libcpmtd:string.obj
 0002:000bc10c       ?in@?$_Iosb@H@std@@2W4_Openmode@12@B 0026110c     libcpmtd:string.obj
 0002:000bc110       ?out@?$_Iosb@H@std@@2W4_Openmode@12@B 00261110     libcpmtd:string.obj
 0002:000bc114       ?ate@?$_Iosb@H@std@@2W4_Openmode@12@B 00261114     libcpmtd:string.obj
 0002:000bc118       ?app@?$_Iosb@H@std@@2W4_Openmode@12@B 00261118     libcpmtd:string.obj
 0002:000bc11c       ?trunc@?$_Iosb@H@std@@2W4_Openmode@12@B 0026111c     libcpmtd:string.obj
 0002:000bc120       ?_Nocreate@?$_Iosb@H@std@@2W4_Openmode@12@B 00261120     libcpmtd:string.obj
 0002:000bc124       ?_Noreplace@?$_Iosb@H@std@@2W4_Openmode@12@B 00261124     libcpmtd:string.obj
 0002:000bc128       ?binary@?$_Iosb@H@std@@2W4_Openmode@12@B 00261128     libcpmtd:string.obj
 0002:000bc12c       ?beg@?$_Iosb@H@std@@2W4_Seekdir@12@B 0026112c     libcpmtd:string.obj
 0002:000bc130       ?cur@?$_Iosb@H@std@@2W4_Seekdir@12@B 00261130     libcpmtd:string.obj
 0002:000bc134       ?end@?$_Iosb@H@std@@2W4_Seekdir@12@B 00261134     libcpmtd:string.obj
 0002:000bc13c       ??_7bad_alloc@std@@6B@     0026113c     libcpmtd:string.obj
 0002:000bc148       ??_C@_1FE@OGIJMGPN@?$AAf?$AA?3?$AA?2?$AAs?$AAp?$AA?2?$AAv?$AAc?$AAt?$AAo?$AAo?$AAl?$AAs?$AA?2?$AAc?$AAr?$AAt?$AAc?$AAe?$AA?2?$AAc?$AAr?$AAt?$AAw?$AA3?$AA2?$AA?2?$AAs?$AAt?$AAd?$AAh?$AAp@ 00261148     libcpmtd:string.obj
 0002:000bc1a0       ??_7logic_error@std@@6B@   002611a0     libcpmtd:string.obj
 0002:000bc1ac       ??_7invalid_argument@std@@6B@ 002611ac     libcpmtd:string.obj
 0002:000bc1b8       ??_7length_error@std@@6B@  002611b8     libcpmtd:string.obj
 0002:000bc1c4       ??_7out_of_range@std@@6B@  002611c4     libcpmtd:string.obj
 0002:000bc218       ??_C@_0BA@JFNIOLAK@string?5too?5long?$AA@ 00261218     libcpmtd:string.obj
 0002:000bc274       ??_C@_0BI@CFPLBAOH@invalid?5string?5position?$AA@ 00261274     libcpmtd:string.obj
 0002:000bc2d8       ??_C@_0BI@ILCMCLF@invalid?5string?5argument?$AA@ 002612d8     libcpmtd:string.obj
 0002:000bc2f0       ??_C@_17LGKOMLJ@?$AA?4?$AA?4?$AA?4?$AA?$AA@ 002612f0     LIBCMTD:dbgrpt.obj
 0002:000bc2f8       ??_C@_1CC@CGHMNGDG@?$AAA?$AAs?$AAs?$AAe?$AAr?$AAt?$AAi?$AAo?$AAn?$AA?5?$AAF?$AAa?$AAi?$AAl?$AAe?$AAd?$AA?$AA@ 002612f8     LIBCMTD:dbgrpt.obj
 0002:000bc31c       ??_C@_1M@ILHOPKA@?$AAE?$AAr?$AAr?$AAo?$AAr?$AA?$AA@ 0026131c     LIBCMTD:dbgrpt.obj
 0002:000bc328       ??_C@_1BA@GLMCNLEM@?$AAW?$AAa?$AAr?$AAn?$AAi?$AAn?$AAg?$AA?$AA@ 00261328     LIBCMTD:dbgrpt.obj
 0002:000bc338       ??_C@_1FI@PHIAFFHM@?$AA?$CI?$AA?$CC?$AAT?$AAh?$AAe?$AA?5?$AAh?$AAo?$AAo?$AAk?$AA?5?$AAf?$AAu?$AAn?$AAc?$AAt?$AAi?$AAo?$AAn?$AA?5?$AAi?$AAs?$AA?5?$AAn?$AAo?$AAt?$AA?5?$AAi?$AAn?$AA?5?$AAt?$AAh@ 00261338     LIBCMTD:dbgrpt.obj
 0002:000bc390       ??_C@_1CG@JBJEFOCM@?$AAp?$AAf?$AAn?$AAN?$AAe?$AAw?$AAH?$AAo?$AAo?$AAk?$AA?5?$AA?$CB?$AA?$DN?$AA?5?$AAN?$AAU?$AAL?$AAL?$AA?$AA@ 00261390     LIBCMTD:dbgrpt.obj
 0002:000bc3b8       ??_C@_1CI@OOAHIOG@?$AA_?$AAC?$AAr?$AAt?$AAS?$AAe?$AAt?$AAR?$AAe?$AAp?$AAo?$AAr?$AAt?$AAH?$AAo?$AAo?$AAk?$AAT?$AA2?$AA?$AA@ 002613b8     LIBCMTD:dbgrpt.obj
 0002:000bc3e0       ??_C@_1FC@DDJKODKC@?$AAf?$AA?3?$AA?2?$AAs?$AAp?$AA?2?$AAv?$AAc?$AAt?$AAo?$AAo?$AAl?$AAs?$AA?2?$AAc?$AAr?$AAt?$AAc?$AAe?$AA?2?$AAc?$AAr?$AAt?$AAw?$AA3?$AA2?$AA?2?$AAm?$AAi?$AAs?$AAc?$AA?2@ 002613e0     LIBCMTD:dbgrpt.obj
 0002:000bc438       ??_C@_1HI@OFEHGPPC@?$AAm?$AAo?$AAd?$AAe?$AA?5?$AA?$DN?$AA?$DN?$AA?5?$AA_?$AAC?$AAR?$AAT?$AA_?$AAR?$AAP?$AAT?$AAH?$AAO?$AAO?$AAK?$AA_?$AAI?$AAN?$AAS?$AAT?$AAA?$AAL?$AAL?$AA?5?$AA?$HM?$AA?$HM?$AA?5@ 00261438     LIBCMTD:dbgrpt.obj
 0002:000bc4b0       ??_C@_1EG@PEOEAKBB@?$AAM?$AAi?$AAc?$AAr?$AAo?$AAs?$AAo?$AAf?$AAt?$AA?5?$AAV?$AAi?$AAs?$AAu?$AAa?$AAl?$AA?5?$AAC?$AA?$CL?$AA?$CL?$AA?5?$AAD?$AAe?$AAb?$AAu?$AAg?$AA?5?$AAL?$AAi?$AAb?$AAr?$AAa@ 002614b0     LIBCMTD:dbgrpt.obj
 0002:000bc4f8       ??_C@_1JI@EACPGHID@?$AAw?$AAc?$AAs?$AAc?$AAp?$AAy?$AA_?$AAs?$AA?$CI?$AAs?$AAz?$AAO?$AAu?$AAt?$AAM?$AAe?$AAs?$AAs?$AAa?$AAg?$AAe?$AA?0?$AA?5?$AA4?$AA0?$AA9?$AA6?$AA?0?$AA?5?$AAL?$AA?$CC?$AA_@ 002614f8     LIBCMTD:dbgrpt.obj
 0002:000bc590       ??_C@_1FG@BBOLDHGF@?$AA_?$AAC?$AAr?$AAt?$AAD?$AAb?$AAg?$AAR?$AAe?$AAp?$AAo?$AAr?$AAt?$AA?3?$AA?5?$AAS?$AAt?$AAr?$AAi?$AAn?$AAg?$AA?5?$AAt?$AAo?$AAo?$AA?5?$AAl?$AAo?$AAn?$AAg?$AA?5?$AAo@ 00261590     LIBCMTD:dbgrpt.obj
 0002:000bc5e8       ??_C@_1KG@MFHGLLO@?$AAD?$AAe?$AAb?$AAu?$AAg?$AA?5?$AA?$CF?$AAs?$AA?$CB?$AA?6?$AA?6?$AAP?$AAr?$AAo?$AAg?$AAr?$AAa?$AAm?$AA?3?$AA?5?$AA?$CF?$AAs?$AA?$CF?$AAs?$AA?$CF?$AAs?$AA?$CF?$AAs?$AA?$CF?$AAs?$AA?$CF?$AAs@ 002615e8     LIBCMTD:dbgrpt.obj
 0002:000bc690       ??_C@_1BE@CGCJKGHI@?$AA?6?$AAM?$AAo?$AAd?$AAu?$AAl?$AAe?$AA?3?$AA?5?$AA?$AA@ 00261690     LIBCMTD:dbgrpt.obj
 0002:000bc6a4       ??_C@_1BA@LNHECFIM@?$AA?6?$AAF?$AAi?$AAl?$AAe?$AA?3?$AA?5?$AA?$AA@ 002616a4     LIBCMTD:dbgrpt.obj
 0002:000bc6b4       ??_C@_1BA@GLLGCPCK@?$AA?6?$AAL?$AAi?$AAn?$AAe?$AA?3?$AA?5?$AA?$AA@ 002616b4     LIBCMTD:dbgrpt.obj
 0002:000bc6c4       ??_C@_13LBAGMAIH@?$AA?6?$AA?$AA@ 002616c4     LIBCMTD:dbgrpt.obj
 0002:000bc6c8       ??_C@_1BK@PEDCIPMA@?$AAE?$AAx?$AAp?$AAr?$AAe?$AAs?$AAs?$AAi?$AAo?$AAn?$AA?3?$AA?5?$AA?$AA@ 002616c8     LIBCMTD:dbgrpt.obj
 0002:000bc6e8       ??_C@_1JM@GKDPCMEA@?$AAw?$AAc?$AAs?$AAn?$AAc?$AAp?$AAy?$AA_?$AAs?$AA?$CI?$AAs?$AAz?$AAS?$AAh?$AAo?$AAr?$AAt?$AAP?$AAr?$AAo?$AAg?$AAN?$AAa?$AAm?$AAe?$AA?0?$AA?5?$AA2?$AA6?$AA0?$AA?5?$AA?9@ 002616e8     LIBCMTD:dbgrpt.obj
 0002:000bc788       ??_C@_1GI@DEDNNLCI@?$AAw?$AAc?$AAs?$AAc?$AAp?$AAy?$AA_?$AAs?$AA?$CI?$AAs?$AAz?$AAE?$AAx?$AAe?$AAN?$AAa?$AAm?$AAe?$AA?0?$AA?5?$AA2?$AA6?$AA0?$AA?0?$AA?5?$AAL?$AA?$CC?$AA?$DM?$AAp?$AAr?$AAo?$AAg@ 00261788     LIBCMTD:dbgrpt.obj
 0002:000bc7f0       ??_C@_1CI@PGJIFDEK@?$AA_?$AA_?$AAc?$AAr?$AAt?$AAM?$AAe?$AAs?$AAs?$AAa?$AAg?$AAe?$AAW?$AAi?$AAn?$AAd?$AAo?$AAw?$AAW?$AA?$AA@ 002617f0     LIBCMTD:dbgrpt.obj
 0002:000bc818       ??_C@_1CO@EAEJAADC@?$AA?$DM?$AAp?$AAr?$AAo?$AAg?$AAr?$AAa?$AAm?$AA?5?$AAn?$AAa?$AAm?$AAe?$AA?5?$AAu?$AAn?$AAk?$AAn?$AAo?$AAw?$AAn?$AA?$DO?$AA?$AA@ 00261818     LIBCMTD:dbgrpt.obj
 0002:000bc848       ??_C@_1CK@DDKKOLAN@?$AAs?$AAi?$AAz?$AAe?$AAI?$AAn?$AAB?$AAy?$AAt?$AAe?$AAs?$AA?5?$AA?$DO?$AA?$DN?$AA?5?$AAc?$AAo?$AAu?$AAn?$AAt?$AA?$AA@ 00261848     LIBCMTD:memcpy_s.obj
 0002:000bc874       ??_C@_1BI@DCHLDCPP@?$AAs?$AAr?$AAc?$AA?5?$AA?$CB?$AA?$DN?$AA?5?$AAN?$AAU?$AAL?$AAL?$AA?$AA@ 00261874     LIBCMTD:memcpy_s.obj
 0002:000bc88c       ??_C@_1BC@GKHDJMGB@?$AAm?$AAe?$AAm?$AAc?$AAp?$AAy?$AA_?$AAs?$AA?$AA@ 0026188c     LIBCMTD:memcpy_s.obj
 0002:000bc8a0       ??_C@_1FK@BOBCAACJ@?$AAf?$AA?3?$AA?2?$AAs?$AAp?$AA?2?$AAv?$AAc?$AAt?$AAo?$AAo?$AAl?$AAs?$AA?2?$AAc?$AAr?$AAt?$AAc?$AAe?$AA?2?$AAc?$AAr?$AAt?$AAw?$AA3?$AA2?$AA?2?$AAs?$AAt?$AAr?$AAi?$AAn@ 002618a0     LIBCMTD:memcpy_s.obj
 0002:000bc8fc       ??_C@_1BI@GKKCBDMD@?$AAd?$AAs?$AAt?$AA?5?$AA?$CB?$AA?$DN?$AA?5?$AAN?$AAU?$AAL?$AAL?$AA?$AA@ 002618fc     LIBCMTD:memcpy_s.obj
 0002:000bc914       ??_C@_1BE@NMKKBGPA@?$AAm?$AAe?$AAm?$AAm?$AAo?$AAv?$AAe?$AA_?$AAs?$AA?$AA@ 00261914     LIBCMTD:memmove_s.obj
 0002:000bc928       ??_C@_1FM@JMDLOEFB@?$AAf?$AA?3?$AA?2?$AAs?$AAp?$AA?2?$AAv?$AAc?$AAt?$AAo?$AAo?$AAl?$AAs?$AA?2?$AAc?$AAr?$AAt?$AAc?$AAe?$AA?2?$AAc?$AAr?$AAt?$AAw?$AA3?$AA2?$AA?2?$AAs?$AAt?$AAr?$AAi?$AAn@ 00261928     LIBCMTD:memmove_s.obj
 0002:000bc984       ??_C@_0BJ@IPHDMCNM@fatal?5error?5in?5_lock?5?$CD0?6?$AA@ 00261984     LIBCMTD:mlock.obj
 0002:000bc9a0       ??_C@_1NK@LOFHIHFC@?$AAf?$AAM?$AAo?$AAd?$AAe?$AA?5?$AA?$DN?$AA?$DN?$AA?5?$AA_?$AAC?$AAR?$AAT?$AAD?$AAB?$AAG?$AA_?$AAR?$AAE?$AAP?$AAO?$AAR?$AAT?$AA_?$AAM?$AAO?$AAD?$AAE?$AA?5?$AA?$HM?$AA?$HM?$AA?5@ 002619a0     LIBCMTD:dbgrptt.obj
 0002:000bca7c       ??_C@_1CE@FIHIECNJ@?$AA_?$AAC?$AAr?$AAt?$AAS?$AAe?$AAt?$AAR?$AAe?$AAp?$AAo?$AAr?$AAt?$AAM?$AAo?$AAd?$AAe?$AA?$AA@ 00261a7c     LIBCMTD:dbgrptt.obj
 0002:000bcaa0       ??_C@_1FE@PLIBPAGC@?$AAf?$AA?3?$AA?2?$AAs?$AAp?$AA?2?$AAv?$AAc?$AAt?$AAo?$AAo?$AAl?$AAs?$AA?2?$AAc?$AAr?$AAt?$AAc?$AAe?$AA?2?$AAc?$AAr?$AAt?$AAw?$AA3?$AA2?$AA?2?$AAm?$AAi?$AAs?$AAc?$AA?2@ 00261aa0     LIBCMTD:dbgrptt.obj
 0002:000bcaf8       ??_C@_1FA@IFFFOLDJ@?$AAn?$AAR?$AAp?$AAt?$AAT?$AAy?$AAp?$AAe?$AA?5?$AA?$DO?$AA?$DN?$AA?5?$AA0?$AA?5?$AA?$CG?$AA?$CG?$AA?5?$AAn?$AAR?$AAp?$AAt?$AAT?$AAy?$AAp?$AAe?$AA?5?$AA?$DM?$AA?5?$AA_?$AAC?$AAR?$AAT@ 00261af8     LIBCMTD:dbgrptt.obj
 0002:000bcb48       ??_C@_1CE@IKKEDCME@?$AA_?$AAC?$AAr?$AAt?$AAS?$AAe?$AAt?$AAR?$AAe?$AAp?$AAo?$AAr?$AAt?$AAF?$AAi?$AAl?$AAe?$AA?$AA@ 00261b48     LIBCMTD:dbgrptt.obj
 0002:000bcb70       ??_C@_1MA@LBAMNNOB@?$AAs?$AAt?$AAr?$AAc?$AAp?$AAy?$AA_?$AAs?$AA?$CI?$AAs?$AAz?$AAO?$AAu?$AAt?$AAM?$AAe?$AAs?$AAs?$AAa?$AAg?$AAe?$AA2?$AA?0?$AA?5?$AA4?$AA0?$AA9?$AA6?$AA?0?$AA?5?$AA?$CC?$AA_@ 00261b70     LIBCMTD:dbgrptt.obj
 0002:000bcc30       ??_C@_0DP@GNPEPHJD@_CrtDbgReport?3?5String?5too?5long?5o@ 00261c30     LIBCMTD:dbgrptt.obj
 0002:000bcc70       ??_C@_1FI@DBAIJPJE@?$AAw?$AAc?$AAs?$AAc?$AAp?$AAy?$AA_?$AAs?$AA?$CI?$AAs?$AAz?$AAO?$AAu?$AAt?$AAM?$AAe?$AAs?$AAs?$AAa?$AAg?$AAe?$AA?0?$AA?5?$AA4?$AA0?$AA9?$AA6?$AA?0?$AA?5?$AAs?$AAz?$AAL@ 00261c70     LIBCMTD:dbgrptt.obj
 0002:000bccc8       ??_C@_1BI@JIDBEPIG@?$AA?$CF?$AAs?$AA?$CI?$AA?$CF?$AAd?$AA?$CJ?$AA?5?$AA?3?$AA?5?$AA?$CF?$AAs?$AA?$AA@ 00261cc8     LIBCMTD:dbgrptt.obj
 0002:000bcce0       ??_C@_1EK@PHCBEDKB@?$AAw?$AAc?$AAs?$AAc?$AAa?$AAt?$AA_?$AAs?$AA?$CI?$AAs?$AAz?$AAL?$AAi?$AAn?$AAe?$AAM?$AAe?$AAs?$AAs?$AAa?$AAg?$AAe?$AA?0?$AA?5?$AA4?$AA0?$AA9?$AA6?$AA?0?$AA?5?$AAL?$AA?$CC@ 00261ce0     LIBCMTD:dbgrptt.obj
 0002:000bcd30       ??_C@_1EK@NMDFGHMF@?$AAw?$AAc?$AAs?$AAc?$AAa?$AAt?$AA_?$AAs?$AA?$CI?$AAs?$AAz?$AAL?$AAi?$AAn?$AAe?$AAM?$AAe?$AAs?$AAs?$AAa?$AAg?$AAe?$AA?0?$AA?5?$AA4?$AA0?$AA9?$AA6?$AA?0?$AA?5?$AAL?$AA?$CC@ 00261d30     LIBCMTD:dbgrptt.obj
 0002:000bcd7c       ??_C@_13CMNBPIDO@?$AA?$AN?$AA?$AA@ 00261d7c     LIBCMTD:dbgrptt.obj
 0002:000bcd80       ??_C@_1FK@HPADHBBD@?$AAw?$AAc?$AAs?$AAc?$AAa?$AAt?$AA_?$AAs?$AA?$CI?$AAs?$AAz?$AAL?$AAi?$AAn?$AAe?$AAM?$AAe?$AAs?$AAs?$AAa?$AAg?$AAe?$AA?0?$AA?5?$AA4?$AA0?$AA9?$AA6?$AA?0?$AA?5?$AAs?$AAz@ 00261d80     LIBCMTD:dbgrptt.obj
 0002:000bcde0       ??_C@_1KO@DGAHENCH@?$AAw?$AAc?$AAs?$AAc?$AAp?$AAy?$AA_?$AAs?$AA?$CI?$AAs?$AAz?$AAL?$AAi?$AAn?$AAe?$AAM?$AAe?$AAs?$AAs?$AAa?$AAg?$AAe?$AA?0?$AA?5?$AA4?$AA0?$AA9?$AA6?$AA?0?$AA?5?$AAs?$AAz@ 00261de0     LIBCMTD:dbgrptt.obj
 0002:000bce90       ??_C@_1CE@OJBNHDMO@?$AAA?$AAs?$AAs?$AAe?$AAr?$AAt?$AAi?$AAo?$AAn?$AA?5?$AAf?$AAa?$AAi?$AAl?$AAe?$AAd?$AA?$CB?$AA?$AA@ 00261e90     LIBCMTD:dbgrptt.obj
 0002:000bceb4       ??_C@_1CG@FFFGGODN@?$AAA?$AAs?$AAs?$AAe?$AAr?$AAt?$AAi?$AAo?$AAn?$AA?5?$AAf?$AAa?$AAi?$AAl?$AAe?$AAd?$AA?3?$AA?5?$AA?$AA@ 00261eb4     LIBCMTD:dbgrptt.obj
 0002:000bcee0       ??_C@_1JK@KHFABAEO@?$AAw?$AAc?$AAs?$AAc?$AAp?$AAy?$AA_?$AAs?$AA?$CI?$AAs?$AAz?$AAU?$AAs?$AAe?$AAr?$AAM?$AAe?$AAs?$AAs?$AAa?$AAg?$AAe?$AA?0?$AA?5?$AA4?$AA0?$AA9?$AA6?$AA?0?$AA?5?$AAL?$AA?$CC@ 00261ee0     LIBCMTD:dbgrptt.obj
 0002:000bcf7c       ??_C@_1BA@ELMMDCFC@?$AA?0?$AA?5?$AAL?$AAi?$AAn?$AAe?$AA?5?$AA?$AA@ 00261f7c     LIBCMTD:dbgrptt.obj
 0002:000bcf8c       ??_C@_1BO@OCHMLCAG@?$AA?$DM?$AAf?$AAi?$AAl?$AAe?$AA?5?$AAu?$AAn?$AAk?$AAn?$AAo?$AAw?$AAn?$AA?$DO?$AA?$AA@ 00261f8c     LIBCMTD:dbgrptt.obj
 0002:000bcfb0       ??_C@_1EM@MJFLEDMB@?$AAS?$AAe?$AAc?$AAo?$AAn?$AAd?$AA?5?$AAC?$AAh?$AAa?$AAn?$AAc?$AAe?$AA?5?$AAA?$AAs?$AAs?$AAe?$AAr?$AAt?$AAi?$AAo?$AAn?$AA?5?$AAF?$AAa?$AAi?$AAl?$AAe?$AAd?$AA?3?$AA?5@ 00261fb0     LIBCMTD:dbgrptt.obj
 0002:000bd000       ??_C@_1FA@CNLLOMHI@?$AA_?$AAi?$AAt?$AAo?$AAw?$AA_?$AAs?$AA?$CI?$AAn?$AAL?$AAi?$AAn?$AAe?$AA?0?$AA?5?$AAs?$AAz?$AAL?$AAi?$AAn?$AAe?$AAM?$AAe?$AAs?$AAs?$AAa?$AAg?$AAe?$AA?0?$AA?5?$AA4?$AA0@ 00262000     LIBCMTD:dbgrptt.obj
 0002:000bd050       ??_C@_1CA@HPALHDOD@?$AA_?$AAV?$AAC?$AAr?$AAt?$AAD?$AAb?$AAg?$AAR?$AAe?$AAp?$AAo?$AAr?$AAt?$AAW?$AA?$AA@ 00262050     LIBCMTD:dbgrptt.obj
 0002:000bd070       ??_C@_1CG@MKBKDNCP@?$AAG?$AAe?$AAt?$AAL?$AAa?$AAs?$AAt?$AAA?$AAc?$AAt?$AAi?$AAv?$AAe?$AAP?$AAo?$AAp?$AAu?$AAp?$AA?$AA@ 00262070     LIBCMTD:crtmbox.obj
 0002:000bd098       ??_C@_1CA@HNKPMKAN@?$AAG?$AAe?$AAt?$AAA?$AAc?$AAt?$AAi?$AAv?$AAe?$AAW?$AAi?$AAn?$AAd?$AAo?$AAw?$AA?$AA@ 00262098     LIBCMTD:crtmbox.obj
 0002:000bd0b8       ??_C@_1BI@OGPGOOGK@?$AAM?$AAe?$AAs?$AAs?$AAa?$AAg?$AAe?$AAB?$AAo?$AAx?$AAW?$AA?$AA@ 002620b8     LIBCMTD:crtmbox.obj
 0002:000bd0d0       ??_C@_1BI@IENOMFML@?$AAC?$AAO?$AAR?$AAE?$AAD?$AAL?$AAL?$AA?4?$AAD?$AAL?$AAL?$AA?$AA@ 002620d0     LIBCMTD:crtmbox.obj
 0002:000bd0e8       ??_C@_1DM@MADKGDLO@?$AA?$CI?$AAL?$AA?$CC?$AAB?$AAu?$AAf?$AAf?$AAe?$AAr?$AA?5?$AAi?$AAs?$AA?5?$AAt?$AAo?$AAo?$AA?5?$AAs?$AAm?$AAa?$AAl?$AAl?$AA?$CC?$AA?5?$AA?$CG?$AA?$CG?$AA?5?$AA0?$AA?$CJ?$AA?$AA@ 002620e8     LIBCMTD:wcsncpy_s.obj
 0002:000bd124       ??_C@_1CI@HCPHDDLE@?$AAB?$AAu?$AAf?$AAf?$AAe?$AAr?$AA?5?$AAi?$AAs?$AA?5?$AAt?$AAo?$AAo?$AA?5?$AAs?$AAm?$AAa?$AAl?$AAl?$AA?$AA@ 00262124     LIBCMTD:wcsncpy_s.obj
 0002:000bd14c       ??_C@_1CG@OFBJMIGJ@?$AA?$CI?$AA?$CI?$AA?$CI?$AA_?$AAS?$AAr?$AAc?$AA?$CJ?$AA?$CJ?$AA?$CJ?$AA?5?$AA?$CB?$AA?$DN?$AA?5?$AAN?$AAU?$AAL?$AAL?$AA?$AA@ 0026214c     LIBCMTD:wcsncpy_s.obj
 0002:000bd174       ??_C@_1BE@PMMBFFCC@?$AAw?$AAc?$AAs?$AAn?$AAc?$AAp?$AAy?$AA_?$AAs?$AA?$AA@ 00262174     LIBCMTD:wcsncpy_s.obj
 0002:000bd188       ??_C@_1FG@OHHBDIEA@?$AAf?$AA?3?$AA?2?$AAs?$AAp?$AA?2?$AAv?$AAc?$AAt?$AAo?$AAo?$AAl?$AAs?$AA?2?$AAc?$AAr?$AAt?$AAc?$AAe?$AA?2?$AAc?$AAr?$AAt?$AAw?$AA3?$AA2?$AA?2?$AAh?$AA?2?$AAt?$AAc?$AAs@ 00262188     LIBCMTD:wcsncpy_s.obj
 0002:000bd1e0       ??_C@_1FC@PFMLEHKI@?$AA?$CI?$AA?$CI?$AA_?$AAD?$AAs?$AAt?$AA?$CJ?$AA?$CJ?$AA?5?$AA?$CB?$AA?$DN?$AA?5?$AAN?$AAU?$AAL?$AAL?$AA?5?$AA?$CG?$AA?$CG?$AA?5?$AA?$CI?$AA?$CI?$AA_?$AAS?$AAi?$AAz?$AAe?$AAI?$AAn?$AAW?$AAo?$AAr@ 002621e0     LIBCMTD:wcsncpy_s.obj
 0002:000bd234       ??_C@_1BC@KIONAFPO@?$AAw?$AAc?$AAs?$AAc?$AAp?$AAy?$AA_?$AAs?$AA?$AA@ 00262234     LIBCMTD:wcscpy_s.obj
 0002:000bd248       ??_C@_1FE@IPADLOPJ@?$AAf?$AA?3?$AA?2?$AAs?$AAp?$AA?2?$AAv?$AAc?$AAt?$AAo?$AAo?$AAl?$AAs?$AA?2?$AAc?$AAr?$AAt?$AAc?$AAe?$AA?2?$AAc?$AAr?$AAt?$AAw?$AA3?$AA2?$AA?2?$AAh?$AA?2?$AAt?$AAc?$AAs@ 00262248     LIBCMTD:wcscpy_s.obj
 0002:000bd29c       ??_C@_1BC@CFJEPFGF@?$AAs?$AAt?$AAr?$AAc?$AAp?$AAy?$AA_?$AAs?$AA?$AA@ 0026229c     LIBCMTD:strcpy_s.obj
 0002:000bd2b0       ??_C@_1FC@NCPEPIBI@?$AA?$CI?$AA?$CI?$AA_?$AAD?$AAs?$AAt?$AA?$CJ?$AA?$CJ?$AA?5?$AA?$CB?$AA?$DN?$AA?5?$AAN?$AAU?$AAL?$AAL?$AA?5?$AA?$CG?$AA?$CG?$AA?5?$AA?$CI?$AA?$CI?$AA_?$AAS?$AAi?$AAz?$AAe?$AAI?$AAn?$AAB?$AAy?$AAt@ 002622b0     LIBCMTD:strcpy_s.obj
 0002:000bd308       ??_C@_1FA@MJKDNFFB@?$AA?$CI?$AAL?$AA?$CC?$AAS?$AAt?$AAr?$AAi?$AAn?$AAg?$AA?5?$AAi?$AAs?$AA?5?$AAn?$AAo?$AAt?$AA?5?$AAn?$AAu?$AAl?$AAl?$AA?5?$AAt?$AAe?$AAr?$AAm?$AAi?$AAn?$AAa?$AAt?$AAe?$AAd@ 00262308     LIBCMTD:wcscat_s.obj
 0002:000bd358       ??_C@_1DM@FHLMIEG@?$AAS?$AAt?$AAr?$AAi?$AAn?$AAg?$AA?5?$AAi?$AAs?$AA?5?$AAn?$AAo?$AAt?$AA?5?$AAn?$AAu?$AAl?$AAl?$AA?5?$AAt?$AAe?$AAr?$AAm?$AAi?$AAn?$AAa?$AAt?$AAe?$AAd?$AA?$AA@ 00262358     LIBCMTD:wcscat_s.obj
 0002:000bd394       ??_C@_1BC@PLIEPKPJ@?$AAw?$AAc?$AAs?$AAc?$AAa?$AAt?$AA_?$AAs?$AA?$AA@ 00262394     LIBCMTD:wcscat_s.obj
 0002:000bd3a8       ??_C@_1FE@EHLIBGFJ@?$AAf?$AA?3?$AA?2?$AAs?$AAp?$AA?2?$AAv?$AAc?$AAt?$AAo?$AAo?$AAl?$AAs?$AA?2?$AAc?$AAr?$AAt?$AAc?$AAe?$AA?2?$AAc?$AAr?$AAt?$AAw?$AA3?$AA2?$AA?2?$AAh?$AA?2?$AAt?$AAc?$AAs@ 002623a8     LIBCMTD:wcscat_s.obj
 0002:000bd3fc       ??_C@_1CM@HABGDNLJ@?$AAl?$AAe?$AAn?$AAg?$AAt?$AAh?$AA?5?$AA?$DM?$AA?5?$AAs?$AAi?$AAz?$AAe?$AAI?$AAn?$AAT?$AAC?$AAh?$AAa?$AAr?$AAs?$AA?$AA@ 002623fc     LIBCMTD:xtows.obj
 0002:000bd428       ??_C@_1DE@PCJGDBBD@?$AA2?$AA?5?$AA?$DM?$AA?$DN?$AA?5?$AAr?$AAa?$AAd?$AAi?$AAx?$AA?5?$AA?$CG?$AA?$CG?$AA?5?$AAr?$AAa?$AAd?$AAi?$AAx?$AA?5?$AA?$DM?$AA?$DN?$AA?5?$AA3?$AA6?$AA?$AA@ 00262428     LIBCMTD:xtows.obj
 0002:000bd460       ??_C@_1FA@MKGGAGEI@?$AAs?$AAi?$AAz?$AAe?$AAI?$AAn?$AAT?$AAC?$AAh?$AAa?$AAr?$AAs?$AA?5?$AA?$DO?$AA?5?$AA?$CI?$AAs?$AAi?$AAz?$AAe?$AA_?$AAt?$AA?$CJ?$AA?$CI?$AAi?$AAs?$AA_?$AAn?$AAe?$AAg?$AA?5?$AA?$DP@ 00262460     LIBCMTD:xtows.obj
 0002:000bd4b0       ??_C@_1CC@JNJFIMGE@?$AAs?$AAi?$AAz?$AAe?$AAI?$AAn?$AAT?$AAC?$AAh?$AAa?$AAr?$AAs?$AA?5?$AA?$DO?$AA?5?$AA0?$AA?$AA@ 002624b0     LIBCMTD:xtows.obj
 0002:000bd4d4       ??_C@_1O@NCBFODOE@?$AAx?$AAt?$AAo?$AAw?$AA_?$AAs?$AA?$AA@ 002624d4     LIBCMTD:xtows.obj
 0002:000bd4e8       ??_C@_1FE@LAGNOOBA@?$AAf?$AA?3?$AA?2?$AAs?$AAp?$AA?2?$AAv?$AAc?$AAt?$AAo?$AAo?$AAl?$AAs?$AA?2?$AAc?$AAr?$AAt?$AAc?$AAe?$AA?2?$AAc?$AAr?$AAt?$AAw?$AA3?$AA2?$AA?2?$AAc?$AAo?$AAn?$AAv?$AAe@ 002624e8     LIBCMTD:xtows.obj
 0002:000bd53c       ??_C@_1BI@ICGGMGLK@?$AAb?$AAu?$AAf?$AA?5?$AA?$CB?$AA?$DN?$AA?5?$AAN?$AAU?$AAL?$AAL?$AA?$AA@ 0026253c     LIBCMTD:xtows.obj
 0002:000bd5c8       ??_R4bad_alloc@std@@6B@    002625c8     libcpmtd:string.obj
 0002:000bd5dc       ??_R3bad_alloc@std@@8      002625dc     libcpmtd:string.obj
 0002:000bd5ec       ??_R2bad_alloc@std@@8      002625ec     libcpmtd:string.obj
 0002:000bd5f8       ??_R1A@?0A@EA@bad_alloc@std@@8 002625f8     libcpmtd:string.obj
 0002:000bd614       ??_R1A@?0A@EA@exception@std@@8 00262614     libcpmtd:string.obj
 0002:000bd630       ??_R3exception@std@@8      00262630     libcpmtd:string.obj
 0002:000bd640       ??_R2exception@std@@8      00262640     libcpmtd:string.obj
 0002:000bd648       ??_R4logic_error@std@@6B@  00262648     libcpmtd:string.obj
 0002:000bd65c       ??_R3logic_error@std@@8    0026265c     libcpmtd:string.obj
 0002:000bd66c       ??_R2logic_error@std@@8    0026266c     libcpmtd:string.obj
 0002:000bd678       ??_R1A@?0A@EA@logic_error@std@@8 00262678     libcpmtd:string.obj
 0002:000bd694       ??_R4invalid_argument@std@@6B@ 00262694     libcpmtd:string.obj
 0002:000bd6a8       ??_R3invalid_argument@std@@8 002626a8     libcpmtd:string.obj
 0002:000bd6b8       ??_R2invalid_argument@std@@8 002626b8     libcpmtd:string.obj
 0002:000bd6c8       ??_R1A@?0A@EA@invalid_argument@std@@8 002626c8     libcpmtd:string.obj
 0002:000bd6e4       ??_R4length_error@std@@6B@ 002626e4     libcpmtd:string.obj
 0002:000bd6f8       ??_R3length_error@std@@8   002626f8     libcpmtd:string.obj
 0002:000bd708       ??_R2length_error@std@@8   00262708     libcpmtd:string.obj
 0002:000bd718       ??_R1A@?0A@EA@length_error@std@@8 00262718     libcpmtd:string.obj
 0002:000bd734       ??_R4out_of_range@std@@6B@ 00262734     libcpmtd:string.obj
 0002:000bd748       ??_R3out_of_range@std@@8   00262748     libcpmtd:string.obj
 0002:000bd758       ??_R2out_of_range@std@@8   00262758     libcpmtd:string.obj
 0002:000bd768       ??_R1A@?0A@EA@out_of_range@std@@8 00262768     libcpmtd:string.obj
 0002:000bd9e0       _TI3?AVlength_error@std@@  002629e0     atcmd.obj
 0002:000bd9f0       _CTA3?AVlength_error@std@@ 002629f0     atcmd.obj
 0002:000bda00       _CT??_R0?AVlength_error@std@@@8??0length_error@std@@QAA@ABV01@@Z44 00262a00     atcmd.obj
 0002:000bda1c       _CT??_R0?AVlogic_error@std@@@8??0logic_error@std@@QAA@ABV01@@Z44 00262a1c     atcmd.obj
 0002:000bda38       _CT??_R0?AVexception@std@@@8??0exception@std@@QAA@ABV01@@Z12 00262a38     atcmd.obj
 0002:000bda54       _TI2?AVbad_alloc@std@@     00262a54     atcmd.obj
 0002:000bda64       _CTA2?AVbad_alloc@std@@    00262a64     atcmd.obj
 0002:000bda70       _CT??_R0?AVbad_alloc@std@@@8??0bad_alloc@std@@QAA@ABV01@@Z12 00262a70     atcmd.obj
 0002:000bda8c       _TI3?AVout_of_range@std@@  00262a8c     libcpmtd:string.obj
 0002:000bda9c       _CTA3?AVout_of_range@std@@ 00262a9c     libcpmtd:string.obj
 0002:000bdaac       _CT??_R0?AVout_of_range@std@@@8??0out_of_range@std@@QAA@ABV01@@Z44 00262aac     libcpmtd:string.obj
 0002:000bdac8       _TI3?AVinvalid_argument@std@@ 00262ac8     libcpmtd:string.obj
 0002:000bdad8       _CTA3?AVinvalid_argument@std@@ 00262ad8     libcpmtd:string.obj
 0002:000bdae8       _CT??_R0?AVinvalid_argument@std@@@8??0invalid_argument@std@@QAA@ABV01@@Z44 00262ae8     libcpmtd:string.obj
 0002:000bdb04       __IMPORT_DESCRIPTOR_sw_utilityG 00262b04     sw_utilityG:sw_utilityG.dll
 0002:000bdb18       __IMPORT_DESCRIPTOR_ossvcs 00262b18     ossvcs:ossvcs.dll
 0002:000bdb2c       __IMPORT_DESCRIPTOR_ccoreutl 00262b2c     ccoreutl:ccoreutl.dll
 0002:000bdb40       __IMPORT_DESCRIPTOR_WINSOCK 00262b40     winsock:WINSOCK.dll
 0002:000bdb54       __IMPORT_DESCRIPTOR_iphlpapi 00262b54     Iphlpapi:iphlpapi.dll
 0002:000bdb68       __IMPORT_DESCRIPTOR_SDKRIL 00262b68     sdkril:SDKRIL.dll
 0002:000bdb7c       __IMPORT_DESCRIPTOR_COREDLL 00262b7c     coredll:COREDLL.dll
 0002:000bdb90       __NULL_IMPORT_DESCRIPTOR   00262b90     sw_utilityG:sw_utilityG.dll
 0003:00000000       __imp__wcsicmp             00265000     coredll:COREDLL.dll
 0003:00000004       __imp_SetLastError         00265004     coredll:COREDLL.dll
 0003:00000008       __imp_RaiseException       00265008     coredll:COREDLL.dll
 0003:0000000c       __imp_TlsCall              0026500c     coredll:COREDLL.dll
 0003:00000010       __imp_InterlockedCompareExchange 00265010     coredll:COREDLL.dll
 0003:00000014       __imp_TlsGetValue          00265014     coredll:COREDLL.dll
 0003:00000018       __imp_TlsSetValue          00265018     coredll:COREDLL.dll
 0003:0000001c       __imp_GetModuleFileNameW   0026501c     coredll:COREDLL.dll
 0003:00000020       __imp_?terminate@std@@YAXXZ 00265020     coredll:COREDLL.dll
 0003:00000024       __imp_InterlockedExchange  00265024     coredll:COREDLL.dll
 0003:00000028       __imp_fflush               00265028     coredll:COREDLL.dll
 0003:0000002c       __imp__getstdfilex         0026502c     coredll:COREDLL.dll
 0003:00000030       __imp_fputs                00265030     coredll:COREDLL.dll
 0003:00000034       __imp___security_gen_cookie 00265034     coredll:COREDLL.dll
 0003:00000038       __imp_LocalSize            00265038     coredll:COREDLL.dll
 0003:0000003c       __imp_LocalAlloc           0026503c     coredll:COREDLL.dll
 0003:00000040       __imp___report_gsfailure   00265040     coredll:COREDLL.dll
 0003:00000044       __imp_RegEnumKeyExW        00265044     coredll:COREDLL.dll
 0003:00000048       __imp_strtok               00265048     coredll:COREDLL.dll
 0003:0000004c       __imp_strtoul              0026504c     coredll:COREDLL.dll
 0003:00000050       __imp_MoveFileW            00265050     coredll:COREDLL.dll
 0003:00000054       __imp_SetFileAttributesW   00265054     coredll:COREDLL.dll
 0003:00000058       __imp_DeleteFileW          00265058     coredll:COREDLL.dll
 0003:0000005c       __imp_CopyFileW            0026505c     coredll:COREDLL.dll
 0003:00000060       __imp_StringCchCopyW       00265060     coredll:COREDLL.dll
 0003:00000064       __imp_strcmp               00265064     coredll:COREDLL.dll
 0003:00000068       __imp_memcmp               00265068     coredll:COREDLL.dll
 0003:0000006c       __imp_GetSystemTime        0026506c     coredll:COREDLL.dll
 0003:00000070       __imp_LocalReAlloc         00265070     coredll:COREDLL.dll
 0003:00000074       __imp_GetFileSize          00265074     coredll:COREDLL.dll
 0003:00000078       __imp_CreateFileMappingW   00265078     coredll:COREDLL.dll
 0003:0000007c       __imp_MapViewOfFile        0026507c     coredll:COREDLL.dll
 0003:00000080       __imp_UnmapViewOfFile      00265080     coredll:COREDLL.dll
 0003:00000084       __imp_InterlockedIncrement 00265084     coredll:COREDLL.dll
 0003:00000088       __imp_InterlockedDecrement 00265088     coredll:COREDLL.dll
 0003:0000008c       __imp_ReleaseSemaphore     0026508c     coredll:COREDLL.dll
 0003:00000090       __imp_CreateSemaphoreW     00265090     coredll:COREDLL.dll
 0003:00000094       __imp_IsBadWritePtr        00265094     coredll:COREDLL.dll
 0003:00000098       __imp_IsBadReadPtr         00265098     coredll:COREDLL.dll
 0003:0000009c       __imp__wcsnicmp            0026509c     coredll:COREDLL.dll
 0003:000000a0       __imp_LoadStringW          002650a0     coredll:COREDLL.dll
 0003:000000a4       __imp___stoi               002650a4     coredll:COREDLL.dll
 0003:000000a8       __imp___muls               002650a8     coredll:COREDLL.dll
 0003:000000ac       __imp___itos               002650ac     coredll:COREDLL.dll
 0003:000000b0       __imp___divs               002650b0     coredll:COREDLL.dll
 0003:000000b4       __imp_rand                 002650b4     coredll:COREDLL.dll
 0003:000000b8       __imp__vsnprintf           002650b8     coredll:COREDLL.dll
 0003:000000bc       __imp__vsnwprintf          002650bc     coredll:COREDLL.dll
 0003:000000c0       __imp_wcstombs             002650c0     coredll:COREDLL.dll
 0003:000000c4       __imp_SystemIdleTimerReset 002650c4     coredll:COREDLL.dll
 0003:000000c8       __imp__byteswap_ushort     002650c8     coredll:COREDLL.dll
 0003:000000cc       __imp_malloc               002650cc     coredll:COREDLL.dll
 0003:000000d0       __imp_free                 002650d0     coredll:COREDLL.dll
 0003:000000d4       __imp_wcstoul              002650d4     coredll:COREDLL.dll
 0003:000000d8       __imp_CeSafeCopyMemory     002650d8     coredll:COREDLL.dll
 0003:000000dc       __imp_memmove              002650dc     coredll:COREDLL.dll
 0003:000000e0       __imp_PowerPolicyNotify    002650e0     coredll:COREDLL.dll
 0003:000000e4       __imp_TryEnterCriticalSection 002650e4     coredll:COREDLL.dll
 0003:000000e8       __imp_swscanf              002650e8     coredll:COREDLL.dll
 0003:000000ec       __imp_LocalAllocTrace      002650ec     coredll:COREDLL.dll
 0003:000000f0       __imp_LocalFree            002650f0     coredll:COREDLL.dll
 0003:000000f4       __imp_StringCchPrintfW     002650f4     coredll:COREDLL.dll
 0003:000000f8       __imp_RegSetValueExW       002650f8     coredll:COREDLL.dll
 0003:000000fc       __imp_RegCreateKeyExW      002650fc     coredll:COREDLL.dll
 0003:00000100       __imp_RegOpenKeyExW        00265100     coredll:COREDLL.dll
 0003:00000104       __imp_RegQueryValueExW     00265104     coredll:COREDLL.dll
 0003:00000108       __imp_wcstok               00265108     coredll:COREDLL.dll
 0003:0000010c       __imp_RegCloseKey          0026510c     coredll:COREDLL.dll
 0003:00000110       __imp__itow                00265110     coredll:COREDLL.dll
 0003:00000114       __imp_wcsncmp              00265114     coredll:COREDLL.dll
 0003:00000118       __imp___dtou               00265118     coredll:COREDLL.dll
 0003:0000011c       __imp___addd               0026511c     coredll:COREDLL.dll
 0003:00000120       __imp___utod               00265120     coredll:COREDLL.dll
 0003:00000124       __imp___muld               00265124     coredll:COREDLL.dll
 0003:00000128       __imp_pow                  00265128     coredll:COREDLL.dll
 0003:0000012c       __imp_strstr               0026512c     coredll:COREDLL.dll
 0003:00000130       __imp_SetSystemTime        00265130     coredll:COREDLL.dll
 0003:00000134       __imp_CeSetThreadPriority  00265134     coredll:COREDLL.dll
 0003:00000138       __imp__wcsupr              00265138     coredll:COREDLL.dll
 0003:0000013c       __imp_CreateEventW         0026513c     coredll:COREDLL.dll
 0003:00000140       __imp_FreeLibrary          00265140     coredll:COREDLL.dll
 0003:00000144       __imp_LoadLibraryW         00265144     coredll:COREDLL.dll
 0003:00000148       __imp_GetProcAddressW      00265148     coredll:COREDLL.dll
 0003:0000014c       __imp__itoa                0026514c     coredll:COREDLL.dll
 0003:00000150       __imp_atoi                 00265150     coredll:COREDLL.dll
 0003:00000154       __imp_sprintf              00265154     coredll:COREDLL.dll
 0003:00000158       __imp_DeleteCriticalSection 00265158     coredll:COREDLL.dll
 0003:0000015c       __imp_InitializeCriticalSection 0026515c     coredll:COREDLL.dll
 0003:00000160       __imp_iswctype             00265160     coredll:COREDLL.dll
 0003:00000164       __imp_SystemTimeToFileTime 00265164     coredll:COREDLL.dll
 0003:00000168       __imp_LocalFileTimeToFileTime 00265168     coredll:COREDLL.dll
 0003:0000016c       __imp_FileTimeToSystemTime 0026516c     coredll:COREDLL.dll
 0003:00000170       __imp_KernelIoControl      00265170     coredll:COREDLL.dll
 0003:00000174       __imp_??_L@YAXPAXIHP6AX0@Z1@Z 00265174     coredll:COREDLL.dll
 0003:00000178       __imp_??_M@YAXPAXIHP6AX0@Z@Z 00265178     coredll:COREDLL.dll
 0003:0000017c       __imp_WideCharToMultiByte  0026517c     coredll:COREDLL.dll
 0003:00000180       __imp__wtol                00265180     coredll:COREDLL.dll
 0003:00000184       __imp_wcsncat              00265184     coredll:COREDLL.dll
 0003:00000188       __imp__snprintf            00265188     coredll:COREDLL.dll
 0003:0000018c       __imp_strncpy              0026518c     coredll:COREDLL.dll
 0003:00000190       __imp_strncat              00265190     coredll:COREDLL.dll
 0003:00000194       __imp_wcschr               00265194     coredll:COREDLL.dll
 0003:00000198       __imp_??3@YAXPAX@Z         00265198     coredll:COREDLL.dll
 0003:0000019c       __imp_LeaveCriticalSection 0026519c     coredll:COREDLL.dll
 0003:000001a0       __imp_EnterCriticalSection 002651a0     coredll:COREDLL.dll
 0003:000001a4       __imp_GetTickCount         002651a4     coredll:COREDLL.dll
 0003:000001a8       __imp_??2@YAPAXI@Z         002651a8     coredll:COREDLL.dll
 0003:000001ac       __imp_memset               002651ac     coredll:COREDLL.dll
 0003:000001b0       __imp_SetThreadPriority    002651b0     coredll:COREDLL.dll
 0003:000001b4       __imp_EventModify          002651b4     coredll:COREDLL.dll
 0003:000001b8       __imp___rt_udiv            002651b8     coredll:COREDLL.dll
 0003:000001bc       __imp___CxxThrowException  002651bc     coredll:COREDLL.dll
 0003:000001c0       __imp_??_7type_info@@6B@   002651c0     coredll:COREDLL.dll
 0003:000001c4       __imp_??0exception@std@@QAA@ABV01@@Z 002651c4     coredll:COREDLL.dll
 0003:000001c8       __imp_??1exception@std@@UAA@XZ 002651c8     coredll:COREDLL.dll
 0003:000001cc       __imp_??0exception@std@@QAA@XZ 002651cc     coredll:COREDLL.dll
 0003:000001d0       __imp_strlen               002651d0     coredll:COREDLL.dll
 0003:000001d4       __imp_memcpy               002651d4     coredll:COREDLL.dll
 0003:000001d8       __imp_??0exception@std@@QAA@PBD@Z 002651d8     coredll:COREDLL.dll
 0003:000001dc       __imp_?what@exception@std@@UBAPBDXZ 002651dc     coredll:COREDLL.dll
 0003:000001e0       __imp_wcscmp               002651e0     coredll:COREDLL.dll
 0003:000001e4       __imp_wcslen               002651e4     coredll:COREDLL.dll
 0003:000001e8       __imp_??_V@YAXPAX@Z        002651e8     coredll:COREDLL.dll
 0003:000001ec       __imp__isctype             002651ec     coredll:COREDLL.dll
 0003:000001f0       __imp_??_U@YAPAXI@Z        002651f0     coredll:COREDLL.dll
 0003:000001f4       __imp_Sleep                002651f4     coredll:COREDLL.dll
 0003:000001f8       __imp_wcscpy               002651f8     coredll:COREDLL.dll
 0003:000001fc       __imp_swprintf             002651fc     coredll:COREDLL.dll
 0003:00000200       __imp_strcpy               00265200     coredll:COREDLL.dll
 0003:00000204       __imp_CreateProcessW       00265204     coredll:COREDLL.dll
 0003:00000208       __imp_wcsstr               00265208     coredll:COREDLL.dll
 0003:0000020c       __imp_CreateFileW          0026520c     coredll:COREDLL.dll
 0003:00000210       __imp_CloseHandle          00265210     coredll:COREDLL.dll
 0003:00000214       __imp_EscapeCommFunction   00265214     coredll:COREDLL.dll
 0003:00000218       __imp_strchr               00265218     coredll:COREDLL.dll
 0003:0000021c       __imp_TerminateProcess     0026521c     coredll:COREDLL.dll
 0003:00000220       __imp_NKDbgPrintfW         00265220     coredll:COREDLL.dll
 0003:00000224       __imp_CreateThread         00265224     coredll:COREDLL.dll
 0003:00000228       __imp_WriteFile            00265228     coredll:COREDLL.dll
 0003:0000022c       __imp_strcat               0026522c     coredll:COREDLL.dll
 0003:00000230       __imp_PurgeComm            00265230     coredll:COREDLL.dll
 0003:00000234       __imp_SetCommMask          00265234     coredll:COREDLL.dll
 0003:00000238       __imp_SetCommTimeouts      00265238     coredll:COREDLL.dll
 0003:0000023c       __imp_GetCommModemStatus   0026523c     coredll:COREDLL.dll
 0003:00000240       __imp_SetCommState         00265240     coredll:COREDLL.dll
 0003:00000244       __imp_MessageBoxW          00265244     coredll:COREDLL.dll
 0003:00000248       __imp_ShowWindow           00265248     coredll:COREDLL.dll
 0003:0000024c       __imp_FindWindowW          0026524c     coredll:COREDLL.dll
 0003:00000250       __imp_SetSystemPowerState  00265250     coredll:COREDLL.dll
 0003:00000254       __imp_MultiByteToWideChar  00265254     coredll:COREDLL.dll
 0003:00000258       __imp_GetStoreInformation  00265258     coredll:COREDLL.dll
 0003:0000025c       __imp_CreateMutexW         0026525c     coredll:COREDLL.dll
 0003:00000260       __imp_wcscat               00265260     coredll:COREDLL.dll
 0003:00000264       __imp_GetLastError         00265264     coredll:COREDLL.dll
 0003:00000268       __imp_TerminateThread      00265268     coredll:COREDLL.dll
 0003:0000026c       __imp_WaitForSingleObject  0026526c     coredll:COREDLL.dll
 0003:00000270       __imp_FlushFileBuffers     00265270     coredll:COREDLL.dll
 0003:00000274       __imp_ReadFile             00265274     coredll:COREDLL.dll
 0003:00000278       __imp_WaitCommEvent        00265278     coredll:COREDLL.dll
 0003:0000027c       __imp_DeviceIoControl      0026527c     coredll:COREDLL.dll
 0003:00000280       __imp_OutputDebugStringW   00265280     coredll:COREDLL.dll
 0003:00000284       __imp_wsprintfW            00265284     coredll:COREDLL.dll
 0003:00000288       __imp___C_specific_handler 00265288     coredll:COREDLL.dll
 0003:0000028c       __imp___rt_sdiv            0026528c     coredll:COREDLL.dll
 0003:00000290       __imp_WaitForMultipleObjects 00265290     coredll:COREDLL.dll
 0003:00000294       __imp_wcsncpy              00265294     coredll:COREDLL.dll
 0003:00000298       __imp_abs                  00265298     coredll:COREDLL.dll
 0003:0000029c       __imp__snwprintf           0026529c     coredll:COREDLL.dll
 0003:000002a0       \177COREDLL_NULL_THUNK_DATA 002652a0     coredll:COREDLL.dll
 0003:000002a4       __imp_?PlayAudioTone@CSwiGobiDll@@QAAKPAE@Z 002652a4     sdkril:SDKRIL.dll
 0003:000002a8       __imp_?SwiM2MAV_AudioPlayTone@CSwiGobiDll@@QAAKPAE0PAG@Z 002652a8     sdkril:SDKRIL.dll
 0003:000002ac       __imp_?SwiM2MAV_AudioSetAVEC@CSwiGobiDll@@QAAKPAE0@Z 002652ac     sdkril:SDKRIL.dll
 0003:000002b0       __imp_?SwiM2MAV_AudioSetSTG@CSwiGobiDll@@QAAKPAEPAG@Z 002652b0     sdkril:SDKRIL.dll
 0003:000002b4       __imp_?SwiM2MAV_AudioSetVolume@CSwiGobiDll@@QAAKPAE00@Z 002652b4     sdkril:SDKRIL.dll
 0003:000002b8       __imp_?SwiM2MAV_AudioSetAVNS@CSwiGobiDll@@QAAKPAE0@Z 002652b8     sdkril:SDKRIL.dll
 0003:000002bc       __imp_?SwiM2MAV_AudioSetVolDB@CSwiGobiDll@@QAAKPAE00PAG@Z 002652bc     sdkril:SDKRIL.dll
 0003:000002c0       __imp_?GetAudioProfile@CSwiGobiDll@@QAAKPAE@Z 002652c0     sdkril:SDKRIL.dll
 0003:000002c4       __imp_?SetEchoCancelMode@CSwiGobiDll@@QAAKPAE@Z 002652c4     sdkril:SDKRIL.dll
 0003:000002c8       __imp_?SetNoiseSuppression@CSwiGobiDll@@QAAKPAE@Z 002652c8     sdkril:SDKRIL.dll
 0003:000002cc       __imp_?SetAutoInputGain@CSwiGobiDll@@QAAKPAE@Z 002652cc     sdkril:SDKRIL.dll
 0003:000002d0       __imp_?SetAutoOutputGain@CSwiGobiDll@@QAAKPAE@Z 002652d0     sdkril:SDKRIL.dll
 0003:000002d4       __imp_?SetTXPCMFilter@CSwiGobiDll@@QAAKPAG0PAK0@Z 002652d4     sdkril:SDKRIL.dll
 0003:000002d8       __imp_?SetRXPCMFilter@CSwiGobiDll@@QAAKPAG0PAK0@Z 002652d8     sdkril:SDKRIL.dll
 0003:000002dc       __imp_?SetRXGainLevel@CSwiGobiDll@@QAAKPAEPAG1@Z 002652dc     sdkril:SDKRIL.dll
 0003:000002e0       __imp_?SetAudioProfile@CSwiGobiDll@@QAAKPAE@Z 002652e0     sdkril:SDKRIL.dll
 0003:000002e4       __imp_?SetMICMuteStatus@CSwiGobiDll@@QAAKPAE@Z 002652e4     sdkril:SDKRIL.dll
 0003:000002e8       __imp_?SetSpeakerMuteStatus@CSwiGobiDll@@QAAKPAE@Z 002652e8     sdkril:SDKRIL.dll
 0003:000002ec       __imp_?SetMicVolume@CSwiGobiDll@@QAAKPAG@Z 002652ec     sdkril:SDKRIL.dll
 0003:000002f0       __imp_?SetReceiverVolume@CSwiGobiDll@@QAAKPAE@Z 002652f0     sdkril:SDKRIL.dll
 0003:000002f4       __imp_?SwiM2MAV_AudioGetProfile@CSwiGobiDll@@QAAKPAE000000@Z 002652f4     sdkril:SDKRIL.dll
 0003:000002f8       __imp_?SwiM2MAV_AudioSetTxVolume@CSwiGobiDll@@QAAKPAEPAG@Z 002652f8     sdkril:SDKRIL.dll
 0003:000002fc       __imp_?SwiM2MAV_AudioSetProfile@CSwiGobiDll@@QAAKPAE00000@Z 002652fc     sdkril:SDKRIL.dll
 0003:00000300       __imp_?CancelUSSD@CSwiGobiDll@@QAAKXZ 00265300     sdkril:SDKRIL.dll
 0003:00000304       __imp_?AnswerUSSD@CSwiGobiDll@@QAAKPAUUSSInfo@@@Z 00265304     sdkril:SDKRIL.dll
 0003:00000308       __imp_?OrigUSSD@CSwiGobiDll@@QAAKPAUUSSInfo@@PAGPAUalphaIDInfo@@0PAE3PAUccSUPSType@@@Z 00265308     sdkril:SDKRIL.dll
 0003:0000030c       __imp_?GetCallWaiting@CSwiGobiDll@@QAAKPAE0PAGPAUalphaIDInfo@@00PAUccSUPSType@@@Z 0026530c     sdkril:SDKRIL.dll
 0003:00000310       __imp_?GetCallForwarding@CSwiGobiDll@@QAAKPAE0PAUgetCallFWInfo@@0PAUalphaIDInfo@@00PAUccSUPSType@@PAUgetExtCallFWInfo@@@Z 00265310     sdkril:SDKRIL.dll
 0003:00000314       __imp_?ChangeBarringPwd@CSwiGobiDll@@QAAKPAUcallBarringPwd@@PAGPAUalphaIDInfo@@PAE3PAUccSUPSType@@@Z 00265314     sdkril:SDKRIL.dll
 0003:00000318       __imp_?SetSUPS@CSwiGobiDll@@QAAKPAUvoiceSetSUPSServiceReq@@PAGPAUalphaIDInfo@@PAE3PAUccSUPSType@@@Z 00265318     sdkril:SDKRIL.dll
 0003:0000031c       __imp_?GetCallBarring@CSwiGobiDll@@QAAKPAE00PAGPAUalphaIDInfo@@00PAUccSUPSType@@@Z 0026531c     sdkril:SDKRIL.dll
 0003:00000320       __imp_SwiGetGsmProfileBasic 00265320     sdkril:SDKRIL.dll
 0003:00000324       __imp_SwiSetGsmProfileBasic 00265324     sdkril:SDKRIL.dll
 0003:00000328       __imp_?GetWaitingMessage@CSwiGobiDll@@QAAKPAUwaitingMsgInfo@@@Z 00265328     sdkril:SDKRIL.dll
 0003:0000032c       __imp_??0CSwiGobiDll@@QAA@XZ 0026532c     sdkril:SDKRIL.dll
 0003:00000330       __imp_?Initialize@CSwiGobiDll@@QAA_NXZ 00265330     sdkril:SDKRIL.dll
 0003:00000334       __imp_?GetDormancyState@CSwiGobiDll@@QAAKPAK@Z 00265334     sdkril:SDKRIL.dll
 0003:00000338       __imp_?GetDunCallInfo@CSwiGobiDll@@QAAKPAKPAE101111PA_KPAG221100002221@Z 00265338     sdkril:SDKRIL.dll
 0003:0000033c       __imp_?UIMGetCardStatus@CSwiGobiDll@@QAAKPAHPAUQMI_UIM_GET_CARD_STATUS_RESP@@@Z 0026533c     sdkril:SDKRIL.dll
 0003:00000340       __imp_??1CSwiGobiDll@@QAA@XZ 00265340     sdkril:SDKRIL.dll
 0003:00000344       __imp_?GetRTREConfig@CSwiGobiDll@@QAAKPAE0@Z 00265344     sdkril:SDKRIL.dll
 0003:00000348       __imp_SwiSetPower          00265348     sdkril:SDKRIL.dll
 0003:0000034c       __imp_?DeletePhonebookRecord@CSwiGobiDll@@QAAKPAEPAG1@Z 0026534c     sdkril:SDKRIL.dll
 0003:00000350       __imp_?WritePhonebookRecord@CSwiGobiDll@@QAAKPAEPAG1000000@Z 00265350     sdkril:SDKRIL.dll
 0003:00000354       __imp_?ReadPhonebookRecords@CSwiGobiDll@@QAAKPAEPAG111@Z 00265354     sdkril:SDKRIL.dll
 0003:00000358       __imp_?GetPhonebookCapabilities@CSwiGobiDll@@QAAKPAEPAG1100@Z 00265358     sdkril:SDKRIL.dll
 0003:0000035c       __imp_?ForceXTRADownload@CSwiGobiDll@@QAAKXZ 0026535c     sdkril:SDKRIL.dll
 0003:00000360       __imp_?GetNMEAConfig@CSwiGobiDll@@QAAKPAE00PAG@Z 00265360     sdkril:SDKRIL.dll
 0003:00000364       __imp_?SetNMEAConfig@CSwiGobiDll@@QAAKEEEPAG@Z 00265364     sdkril:SDKRIL.dll
 0003:00000368       __imp_?SetPDSDefaults@CSwiGobiDll@@QAAKKEKK@Z 00265368     sdkril:SDKRIL.dll
 0003:0000036c       __imp_?SetXTRAEmbeddedClient@CSwiGobiDll@@QAAKEE@Z 0026536c     sdkril:SDKRIL.dll
 0003:00000370       __imp_?GetCellLocationInfo@CSwiGobiDll@@QAAKPAUgeranCellInfo@@PAUumtsCellInfo@@PAUcdmaCellInfo@@PAK@Z 00265370     sdkril:SDKRIL.dll
 0003:00000374       __imp_?StartDTMF@CSwiGobiDll@@QAAKPAE00@Z 00265374     sdkril:SDKRIL.dll
 0003:00000378       __imp_?StopDTMF@CSwiGobiDll@@QAAKPAE0@Z 00265378     sdkril:SDKRIL.dll
 0003:0000037c       __imp_?SendFlash@CSwiGobiDll@@QAAKPAEPAD00@Z 0026537c     sdkril:SDKRIL.dll
 0003:00000380       __imp_?ManageCalls@CSwiGobiDll@@QAAKPAE0PAG@Z 00265380     sdkril:SDKRIL.dll
 0003:00000384       __imp_?EndCall@CSwiGobiDll@@QAAKPAE0@Z 00265384     sdkril:SDKRIL.dll
 0003:00000388       __imp_?AnserCall@CSwiGobiDll@@QAAKPAE0@Z 00265388     sdkril:SDKRIL.dll
 0003:0000038c       __imp_SwiPstGetDsMipActiveProf 0026538c     sdkril:SDKRIL.dll
 0003:00000390       __imp_?DialCall@CSwiGobiDll@@QAAKPAUtDialReqParam@@PAEPAUalphaIDInfo@@1PAUccSUPSType@@@Z 00265390     sdkril:SDKRIL.dll
 0003:00000394       \177SDKRIL_NULL_THUNK_DATA 00265394     sdkril:SDKRIL.dll
 0003:00000398       __imp_inet_addr            00265398     winsock:WINSOCK.dll
 0003:0000039c       __imp_ntohs                0026539c     winsock:WINSOCK.dll
 0003:000003a0       __imp_htonl                002653a0     winsock:WINSOCK.dll
 0003:000003a4       \177WINSOCK_NULL_THUNK_DATA 002653a4     winsock:WINSOCK.dll
 0003:000003a8       __imp_PHGetFeatureLevel    002653a8     ccoreutl:ccoreutl.dll
 0003:000003ac       \177ccoreutl_NULL_THUNK_DATA 002653ac     ccoreutl:ccoreutl.dll
 0003:000003b0       __imp_GetAdaptersInfo      002653b0     Iphlpapi:iphlpapi.dll
 0003:000003b4       \177iphlpapi_NULL_THUNK_DATA 002653b4     Iphlpapi:iphlpapi.dll
 0003:000003b8       __imp_GetStatStore         002653b8     ossvcs:ossvcs.dll
 0003:000003bc       __imp_ValidateAPIPermission 002653bc     ossvcs:ossvcs.dll
 0003:000003c0       \177ossvcs_NULL_THUNK_DATA 002653c0     ossvcs:ossvcs.dll
 0003:000003c4       __imp_?ChangeCarrierIndex@@YAJKK@Z 002653c4     sw_utilityG:sw_utilityG.dll
 0003:000003c8       __imp_?InitLog@@YAXPAUHINSTANCE__@@@Z 002653c8     sw_utilityG:sw_utilityG.dll
 0003:000003cc       __imp_?GetVerInfo@@YAPAGPAUHINSTANCE__@@@Z 002653cc     sw_utilityG:sw_utilityG.dll
 0003:000003d0       __imp_?LogV@@YAXPBGZZ      002653d0     sw_utilityG:sw_utilityG.dll
 0003:000003d4       __imp_?SetRegValue@@YAJPAUHKEY__@@PBG11@Z 002653d4     sw_utilityG:sw_utilityG.dll
 0003:000003d8       __imp_?GetRegValue@@YAJPAUHKEY__@@PBG1AAK@Z 002653d8     sw_utilityG:sw_utilityG.dll
 0003:000003dc       __imp_?GetProductFeatures@@YAHAAK@Z 002653dc     sw_utilityG:sw_utilityG.dll
 0003:000003e0       __imp_?SetRegValue@@YAJPAUHKEY__@@PBG1K@Z 002653e0     sw_utilityG:sw_utilityG.dll
 0003:000003e4       __imp_?SWAI_GetRegValue@@YAJPAUHKEY__@@PBG1AAK@Z 002653e4     sw_utilityG:sw_utilityG.dll
 0003:000003e8       __imp_?SWAI_SetRegValue@@YAJPAUHKEY__@@PBG1K@Z 002653e8     sw_utilityG:sw_utilityG.dll
 0003:000003ec       __imp_?SWAI_GetRegValue@@YAJPAUHKEY__@@PBG1PAGPAK@Z 002653ec     sw_utilityG:sw_utilityG.dll
 0003:000003f0       __imp_?DisplayRawData@@YAXIPAEHPBG@Z 002653f0     sw_utilityG:sw_utilityG.dll
 0003:000003f4       __imp_?ConvertPrefMode@@YAH_NH@Z 002653f4     sw_utilityG:sw_utilityG.dll
 0003:000003f8       __imp_?GetRegValue@@YAJPAUHKEY__@@PBG1PAGPAK@Z 002653f8     sw_utilityG:sw_utilityG.dll
 0003:000003fc       __imp_??0CVerInfo@@QAA@PAG@Z 002653fc     sw_utilityG:sw_utilityG.dll
 0003:00000400       __imp_?GetProductVersionStr@CVerInfo@@QAAPAGXZ 00265400     sw_utilityG:sw_utilityG.dll
 0003:00000404       __imp_??1CVerInfo@@QAA@XZ  00265404     sw_utilityG:sw_utilityG.dll
 0003:00000408       __imp_?SW_TtoA@@YAPADPADPAGK@Z 00265408     sw_utilityG:sw_utilityG.dll
 0003:0000040c       __imp_?LocalToUTCTime@@YAHPAU_SYSTEMTIME@@0@Z 0026540c     sw_utilityG:sw_utilityG.dll
 0003:00000410       __imp_?IP2DWORD@@YAKPBG@Z  00265410     sw_utilityG:sw_utilityG.dll
 0003:00000414       __imp_?DWORD2IP@@YAPBGK@Z  00265414     sw_utilityG:sw_utilityG.dll
 0003:00000418       __imp_?GetCarrierIndex@@YAKXZ 00265418     sw_utilityG:sw_utilityG.dll
 0003:0000041c       __imp_?GetDataPortDetails@@YAHPAGAAK@Z 0026541c     sw_utilityG:sw_utilityG.dll
 0003:00000420       __imp_?SW_AtoT@@YAPAGPAGPADK@Z 00265420     sw_utilityG:sw_utilityG.dll
 0003:00000424       __imp_?WriteLog@@YAXKPBGZZ 00265424     sw_utilityG:sw_utilityG.dll
 0003:00000428       __imp_?TBD_Assert@@YA_N_NQBG1H@Z 00265428     sw_utilityG:sw_utilityG.dll
 0003:0000042c       __imp_?LogStoreFileLine@@YAXPAGH@Z 0026542c     sw_utilityG:sw_utilityG.dll
 0003:00000430       __imp_?LogW@@YAXPBGZZ      00265430     sw_utilityG:sw_utilityG.dll
 0003:00000434       __imp_?LogC@@YAXPBGZZ      00265434     sw_utilityG:sw_utilityG.dll
 0003:00000438       __imp_?TBD_Output@@YAXW4TBD_CLASS_TYPE@@W4TBD_OUTPUT_LEVEL@@QBGZZ 00265438     sw_utilityG:sw_utilityG.dll
 0003:0000043c       \177sw_utilityG_NULL_THUNK_DATA 0026543c     sw_utilityG:sw_utilityG.dll
 0003:00000440       __xc_a                     00265440     corelibc:crt0init.obj
 0003:00000458       __xc_z                     00265458     corelibc:crt0init.obj
 0003:0000045c       __xi_a                     0026545c     corelibc:crt0init.obj
 0003:00000460       __xi_z                     00265460     corelibc:crt0init.obj
 0003:00000464       __xp_a                     00265464     corelibc:crt0init.obj
 0003:00000468       __xp_z                     00265468     corelibc:crt0init.obj
 0003:0000046c       __xt_a                     0026546c     corelibc:crt0init.obj
 0003:00000470       __xt_z                     00265470     corelibc:crt0init.obj
 0003:00000b18       ??_R0?AVlength_error@std@@@8 00265b18     atcmd.obj
 0003:00000b38       ??_R0?AVlogic_error@std@@@8 00265b38     atcmd.obj
 0003:00000b58       ??_R0?AVexception@std@@@8  00265b58     atcmd.obj
 0003:00000b74       ??_R0?AVbad_alloc@std@@@8  00265b74     atcmd.obj
 0003:00002cb4       ?g_bRadioOff@@3HA          00267cb4     FakeResponse.obj
 0003:00002cb8       ?bSingleInitThreadProc@@3_NA 00267cb8     FakeResponse.obj
 0003:00004de0       ?Convert2CDMANetworkPref@@3PAW4CDMA_NETWORK_PREF@@A 00269de0     network.obj
 0003:00004dec       ?Convert2UMTSNetworkPref@@3PAW4UMTS_NETWORK_PREF@@A 00269dec     network.obj
 0003:00005498       ?g_IsOSExpectNITZ@@3HA     0026a498     Radio.obj
 0003:0000549c       ?RIL_CALLSTAT_STR@@3PAPAGA 0026a49c     Radio.obj
 0003:00006f38       ?g_IsFirstSend@@3HA        0026bf38     rilhandndis.obj
 0003:00006f40       ?dhcpIpFrameReq@@3PAEA     0026bf40     rilhandndis.obj
 0003:00007728       ?gIsPowerManagedSupported@@3HA 0026c728     rilmain.obj
 0003:00008750       ?smscbsample@@3PADA        0026d750     smscb.obj
 0003:00009b38       __security_cookie_complement 0026eb38     corelibc:seccook.obj
 0003:00009b3c       __security_cookie          0026eb3c     corelibc:seccook.obj
 0003:00009b4c       ??_R0?AVinvalid_argument@std@@@8 0026eb4c     libcpmtd:string.obj
 0003:00009b70       ??_R0?AVout_of_range@std@@@8 0026eb70     libcpmtd:string.obj
 0003:00009cc8       _crtAssertBusy             0026ecc8     LIBCMTD:dbgrptt.obj
 0003:00009ccc       _CrtDbgMode                0026eccc     LIBCMTD:dbgrptt.obj
 0003:00009cd8       _CrtDbgFile                0026ecd8     LIBCMTD:dbgrptt.obj
 0003:00009ce4       _aexit_rtn                 0026ece4     LIBCMTD:crt0dat.obj
 0003:00009ce8       ?g_pCmdQ@@3PAV?$CThreadSafeQueue@PAVCCommand@@@@A 0026ece8     atcmd.obj
 0003:00009cec       ?m_pChannelLinker@ChannelLinker@@2PAV1@A 0026ecec     channel.obj
 0003:00009cf0       ?g_IsCriticalPowerCondition@@3HA 0026ecf0     misc.obj
 0003:00009cf4       ?g_nMsgID@@3KA             0026ecf4     msg.obj
 0003:00009cf8       ?csReceiveSms@@3VCriticalSection@@A 0026ecf8     msg.obj
 0003:00009d10       ?g_dwDelayNITZ@@3KA        0026ed10     Radio.obj
 0003:00009d14       ?theSWINotifCR@@3VCriticalSection@@A 0026ed14     Radio.obj
 0003:00009d2c       ?g_TimeoutAPIDefault@@3KA  0026ed2c     rilhand.obj
 0003:00009d30       ?g_TimeoutCmdInit@@3KA     0026ed30     rilhand.obj
 0003:00009d34       ?g_dwPhoneFeatureLevel@@3KA 0026ed34     rilhand.obj
 0003:00009d38       ?g_dwNetworkType@@3KA      0026ed38     rilhand.obj
 0003:00009d3c       ?g_TimeoutWaitForInit@@3KA 0026ed3c     rilhand.obj
 0003:00009d40       ?g_TimeoutCmdOnline@@3KA   0026ed40     rilhand.obj
 0003:00009d44       ?g_TimeoutCmdNoOp@@3KA     0026ed44     rilhand.obj
 0003:00009d48       ?g_TimeoutDTRDrop@@3KA     0026ed48     rilhand.obj
 0003:00009d4c       ?g_pNotifQ@@3PAV?$CThreadSafeQueue@PAUSwiNotifyVariant@@@@A 0026ed4c     rilhand.obj
 0003:00009d50       ?g_GlobalRILHandle@@3PAVCRilHandle@@A 0026ed50     rilhand.obj
 0003:00009d54       ?g_arrWaitingCommands@@3V?$list@PAVCCommand@@V?$allocator@PAVCCommand@@@std@@@std@@A 0026ed54     rilhand.obj
 0003:00009d70       ?g_tszUserDNS2@@3PAGA      0026ed70     rilhandndis.obj
 0003:00009df0       ?g_tszUserDNS1@@3PAGA      0026edf0     rilhandndis.obj
 0003:00009e70       ?g_pIPChannel@@3PAVCChannel@@A 0026ee70     rilhandndis.obj
 0003:00009e74       ?g_NDISGetFnPtr@@3URILNDISGETFNPTR@@A 0026ee74     rilhandndis.obj
 0003:00009e7c       ?g_hSWUSBNDISEvent@@3PAXA  0026ee7c     rilhandndis.obj
 0003:00009e80       ?g_csClosing@@3UCRITICAL_SECTION@@A 0026ee80     rilmain.obj
 0003:00009e94       ?g_hCriticalErrorEvent@@3PAXA 0026ee94     rilmain.obj
 0003:00009e98       ?g_hDriverPresentEvent@@3PAXA 0026ee98     rilmain.obj
 0003:00009e9c       ?g_dwReadyState@@3KA       0026ee9c     rilmain.obj
 0003:00009ea0       ?g_dwLastError@@3KA        0026eea0     rilmain.obj
 0003:00009ea4       ?g_hinstDll@@3PAXA         0026eea4     rilmain.obj
 0003:00009ea8       ?g_SignalCriticalErrorEventId@@3KA 0026eea8     rilmain.obj
 0003:00009eac       ?g_hDeviceJustResumedEvent@@3PAXA 0026eeac     rilmain.obj
 0003:00009eb0       ?g_CriticalLogging@@3HA    0026eeb0     rilmain.obj
 0003:00009eb4       ?gLastDeviceDx@@3W4_CEDEVICE_POWER_STATE@@A 0026eeb4     rilmain.obj
 0003:0000a058       __onexitend                0026f058     <common>
 0003:0000a05c       __onexitbegin              0026f05c     <common>
 0003:0000a060       _exitflag                  0026f060     <common>
 0003:0000a064       _pRawDllMain               0026f064     <common>
 0003:0000a068       _pfnReportHook             0026f068     <common>
 0003:0000a06c       _pReportHookListW          0026f06c     <common>
 0003:0000a070       _pReportHookList           0026f070     <common>

 entry point at        0001:0009ab14

 Static symbols

 0001:fffff030       __unwind$91603             00100030 f   Radio.obj
 0001:fffff038       __unwind$88119             00100038 f   FakeResponse.obj
 0001:fffff038       __unwind$41054             00100038 f   DatERI.obj
 0001:fffff038       __unwind$92966             00100038 f   Radio.obj
 0001:fffff038       __unwind$86624             00100038 f   rilhandndis.obj
 0001:fffff038       __unwind$89910             00100038 f   misc.obj
 0001:fffff044       __unwind$89334             00100044 f   misc.obj
 0001:fffff044       __unwind$86275             00100044 f   callctrl.obj
 0001:fffff044       __unwind$87923             00100044 f   FakeResponse.obj
 0001:fffff044       __unwind$87329             00100044 f   rilmain.obj
 0001:fffff044       __unwind$89599             00100044 f   rilhand.obj
 0001:fffff044       __unwind$86050             00100044 f   rilhandndis.obj
 0001:fffff044       __unwind$39240             00100044 f   DatERI.obj
 0001:fffff044       __unwind$90874             00100044 f   Radio.obj
 0001:fffff058       __unwind$18609             00100058 f   libcpmtd:string.obj
 0001:fffff058       __unwind$87637             00100058 f   rilmain.obj
 0001:fffff058       __unwind$18984             00100058 f   libcpmtd:string.obj
 0001:fffff058       __unwind$90741             00100058 f   rilhand.obj
 0001:fffff058       __unwind$90269             00100058 f   misc.obj
 0001:fffff058       __unwind$87111             00100058 f   rilhandndis.obj
 0001:fffff058       __unwind$93758             00100058 f   Radio.obj
 0001:fffff058       __unwind$93732             00100058 f   Radio.obj
 0001:fffff05c       __unwind$86539             0010005c f   rilhandndis.obj
 0001:fffff05c       __unwind$92881             0010005c f   Radio.obj
 0001:fffff05c       __unwind$89825             0010005c f   misc.obj
 0001:fffff05c       __unwind$40969             0010005c f   DatERI.obj
 0001:fffff05c       __unwind$88034             0010005c f   FakeResponse.obj
 0001:fffff060       __unwind$19542             00100060 f   libcpmtd:string.obj
 0001:fffff064       __unwind$93871             00100064 f   Radio.obj
 0001:fffff064       __unwind$41683             00100064 f   DatERI.obj
 0001:fffff064       __unwind$89018             00100064 f   FakeResponse.obj
 0001:fffff064       __unwind$88325             00100064 f   FakeResponse.obj
 0001:fffff064       __unwind$90142             00100064 f   misc.obj
 0001:fffff064       __unwind$86891             00100064 f   rilhandndis.obj
 0001:fffff068       __unwind$18537             00100068 f   libcpmtd:string.obj
 0001:fffff070       __unwind$88348             00100070 f   FakeResponse.obj
 0001:fffff070       __unwind$41732             00100070 f   DatERI.obj
 0001:fffff070       __unwind$93894             00100070 f   Radio.obj
 0001:fffff070       __unwind$90165             00100070 f   misc.obj
 0001:fffff070       __unwind$86914             00100070 f   rilhandndis.obj
 0001:fffff074       __unwind$87551             00100074 f   rilmain.obj
 0001:fffff074       __unwind$90508             00100074 f   rilhand.obj
 0001:fffff078       __unwind$86095             00100078 f   rilhandndis.obj
 0001:fffff078       __unwind$89635             00100078 f   rilhand.obj
 0001:fffff078       __unwind$39956             00100078 f   DatERI.obj
 0001:fffff078       __unwind$90910             00100078 f   Radio.obj
 0001:fffff078       __unwind$87374             00100078 f   rilmain.obj
 0001:fffff078       __unwind$90816             00100078 f   misc.obj
 0001:fffff080       __unwind$91585             00100080 f   Radio.obj
 0001:fffff084       __unwind$92946             00100084 f   Radio.obj
 0001:fffff084       __unwind$86604             00100084 f   rilhandndis.obj
 0001:fffff084       __unwind$41034             00100084 f   DatERI.obj
 0001:fffff084       __unwind$89890             00100084 f   misc.obj
 0001:fffff084       __unwind$88099             00100084 f   FakeResponse.obj
 0001:fffff08c       __unwind$87552             0010008c f   rilmain.obj
 0001:fffff08c       __unwind$90509             0010008c f   rilhand.obj
 0001:fffff0a0       __unwind$86330             001000a0 f   callctrl.obj
 0001:fffff0a0       __unwind$89654             001000a0 f   rilhand.obj
 0001:fffff0a0       __unwind$86114             001000a0 f   rilhandndis.obj
 0001:fffff0a0       __unwind$90287             001000a0 f   misc.obj
 0001:fffff0a0       __unwind$88490             001000a0 f   FakeResponse.obj
 0001:fffff0a0       __unwind$87393             001000a0 f   rilmain.obj
 0001:fffff0a0       __unwind$90929             001000a0 f   Radio.obj
 0001:fffff0a0       __unwind$39975             001000a0 f   DatERI.obj
 0001:fffff0ac       __catch$92155              001000ac f   Radio.obj
 0001:fffff0b4       __unwind$92846             001000b4 f   Radio.obj
 0001:fffff0d8       __catch$92819              001000d8 f   Radio.obj
 0001:fffff0e4       __unwind$92132             001000e4 f   Radio.obj
 0001:fffff0f4       __unwind$90450             001000f4 f   rilhand.obj
 0001:fffff0f4       __unwind$87238             001000f4 f   rilmain.obj
 0001:fffff108       __catch$18380              00100108 f   libcpmtd:string.obj
 0001:fffff10c       __unwind$87239             0010010c f   rilmain.obj
 0001:fffff10c       __unwind$90451             0010010c f   rilhand.obj
 0001:fffff124       __unwind$90453             00100124 f   rilhand.obj
 0001:fffff124       __unwind$87241             00100124 f   rilmain.obj
 0001:fffff144       __catch$18378              00100144 f   libcpmtd:string.obj
 0001:fffff16c       __unwind$84057             0010016c f   command.obj
 0001:fffff1b0       __unwind$87442             001001b0 f   rilmain.obj
 0001:fffff1b0       __unwind$90588             001001b0 f   rilhand.obj
 0001:fffff1b8       __catch$90196              001001b8 f   misc.obj
 0001:fffff1b8       __catch$86945              001001b8 f   rilhandndis.obj
 0001:fffff1b8       __catch$88379              001001b8 f   FakeResponse.obj
 0001:fffff1b8       __catch$93925              001001b8 f   Radio.obj
 0001:fffff1b8       __catch$41763              001001b8 f   DatERI.obj
 0001:fffff1c8       __unwind$90589             001001c8 f   rilhand.obj
 0001:fffff1c8       __unwind$87443             001001c8 f   rilmain.obj
 0001:fffff1e0       __unwind$90590             001001e0 f   rilhand.obj
 0001:fffff1e0       __unwind$87444             001001e0 f   rilmain.obj
 0001:fffff1f0       __catch$86943              001001f0 f   rilhandndis.obj
 0001:fffff1f0       __catch$88377              001001f0 f   FakeResponse.obj
 0001:fffff1f0       __catch$41761              001001f0 f   DatERI.obj
 0001:fffff1f0       __catch$93923              001001f0 f   Radio.obj
 0001:fffff1f0       __catch$90194              001001f0 f   misc.obj
 0001:00000498       __unwind$85333             00101498 f   atcmd.obj
 0001:000004b8       __unwind$85334             001014b8 f   atcmd.obj
 0001:000011f8       __unwind$85599             001021f8 f i atcmd.obj
 0001:000013e0       __unwind$85641             001023e0 f i atcmd.obj
 0001:00001874       __unwind$85805             00102874 f i atcmd.obj
 0001:00001d04       __unwind$85883             00102d04 f i atcmd.obj
 0001:00002474       __unwind$85991             00103474 f i atcmd.obj
 0001:00002530       __unwind$86028             00103530 f i atcmd.obj
 0001:000026e0       __unwind$86093             001036e0 f i atcmd.obj
 0001:00002734       __unwind$86113             00103734 f i atcmd.obj
 0001:00002e8c       __unwind$86294             00103e8c f i atcmd.obj
 0001:00002f18       __unwind$86317             00103f18 f i atcmd.obj
 0001:00003148       __catch$86348              00104148 f i atcmd.obj
 0001:00003180       __catch$86346              00104180 f i atcmd.obj
 0001:00003a20       __unwind$86583             00104a20 f i atcmd.obj
 0001:00003af0       __unwind$86608             00104af0 f i atcmd.obj
 0001:000047c0       __unwind$86175             001057c0 f   callctrl.obj
 0001:000047d8       __unwind$86176             001057d8 f   callctrl.obj
 0001:000047f0       __unwind$86177             001057f0 f   callctrl.obj
 0001:00004808       __unwind$86178             00105808 f   callctrl.obj
 0001:00004a44       __unwind$86351             00105a44 f   callctrl.obj
 0001:00004a5c       __unwind$86352             00105a5c f   callctrl.obj
 0001:00004a74       __unwind$86353             00105a74 f   callctrl.obj
 0001:00004a8c       __unwind$86354             00105a8c f   callctrl.obj
 0001:00005030       __unwind$86403             00106030 f   callctrl.obj
 0001:0000569c       __unwind$86538             0010669c f   callctrl.obj
 0001:00006258       __unwind$86674             00107258 f   callctrl.obj
 0001:00007938       __unwind$86928             00108938 f   callctrl.obj
 0001:00007fd4       __unwind$86972             00108fd4 f   callctrl.obj
 0001:00008550       __unwind$87060             00109550 f   callctrl.obj
 0001:00008968       __unwind$87105             00109968 f   callctrl.obj
 0001:00009350       __unwind$87132             0010a350 f   callctrl.obj
 0001:000095f4       __unwind$87205             0010a5f4 f   callctrl.obj
 0001:000098f8       __unwind$87251             0010a8f8 f   callctrl.obj
 0001:0000a2d4       __unwind$87314             0010b2d4 f   callctrl.obj
 0001:0000a5f8       __unwind$87353             0010b5f8 f   callctrl.obj
 0001:0000a738       __unwind$87380             0010b738 f   callctrl.obj
 0001:0000a91c       __unwind$87414             0010b91c f   callctrl.obj
 0001:0000adac       __unwind$87468             0010bdac f   callctrl.obj
 0001:0000afb0       __unwind$87487             0010bfb0 f   callctrl.obj
 0001:0000b13c       __unwind$87513             0010c13c f   callctrl.obj
 0001:0000b850       __unwind$87580             0010c850 f   callctrl.obj
 0001:0000b9f4       __unwind$87623             0010c9f4 f   callctrl.obj
 0001:0000bb38       __unwind$87656             0010cb38 f   callctrl.obj
 0001:0000bc7c       __unwind$87679             0010cc7c f   callctrl.obj
 0001:0000bd9c       __unwind$87700             0010cd9c f   callctrl.obj
 0001:0000c034       __unwind$87720             0010d034 f   callctrl.obj
 0001:0000c2f0       __unwind$87769             0010d2f0 f   callctrl.obj
 0001:0001019c       __unwind$88187             0011119c f   callctrl.obj
 0001:000101b4       __unwind$88188             001111b4 f   callctrl.obj
 0001:00010544       __unwind$88242             00111544 f   callctrl.obj
 0001:00010938       __unwind$88270             00111938 f   callctrl.obj
 0001:00010aec       __unwind$86311             00111aec f i callctrl.obj
 0001:00011450       __unwind$88452             00112450 f i callctrl.obj
 0001:00012c54       __unwind$31996             00113c54 f   channel.obj
 0001:00012c6c       __unwind$31997             00113c6c f   channel.obj
 0001:00013a78       __unwind$83767             00114a78 f   command.obj
 0001:00013a90       __unwind$83768             00114a90 f   command.obj
 0001:00016314       __unwind$39103             00117314 f   DatERI.obj
 0001:00016330       __unwind$39104             00117330 f   DatERI.obj
 0001:0001638c       __unwind$39139             0011738c f   DatERI.obj
 0001:000163a8       __unwind$39140             001173a8 f   DatERI.obj
 0001:0001660c       __unwind$39166             0011760c f   DatERI.obj
 0001:00016624       __unwind$39168             00117624 f   DatERI.obj
 0001:0001663c       __unwind$39169             0011763c f   DatERI.obj
 0001:00016654       __unwind$39171             00117654 f   DatERI.obj
 0001:00017870       __unwind$39356             00118870 f   DatERI.obj
 0001:00017890       __unwind$39358             00118890 f   DatERI.obj
 0001:000178b0       __unwind$39359             001188b0 f   DatERI.obj
 0001:000178d0       __unwind$39361             001188d0 f   DatERI.obj
 0001:00018070       __unwind$39424             00119070 f   DatERI.obj
 0001:00018088       __unwind$39425             00119088 f   DatERI.obj
 0001:00018170       __unwind$39452             00119170 f   DatERI.obj
 0001:00018188       __unwind$39453             00119188 f   DatERI.obj
 0001:000185c4       __unwind$39502             001195c4 f i DatERI.obj
 0001:000185dc       __unwind$39504             001195dc f i DatERI.obj
 0001:00018610       __unwind$39508             00119610 f i DatERI.obj
 0001:00018658       __unwind$39539             00119658 f i DatERI.obj
 0001:00018964       __unwind$39591             00119964 f i DatERI.obj
 0001:00018984       __unwind$39593             00119984 f i DatERI.obj
 0001:000189c0       __unwind$39595             001199c0 f i DatERI.obj
 0001:000189fc       __unwind$39597             001199fc f i DatERI.obj
 0001:00018c28       __unwind$39659             00119c28 f i DatERI.obj
 0001:00018c40       __unwind$39661             00119c40 f i DatERI.obj
 0001:00018c74       __unwind$39665             00119c74 f i DatERI.obj
 0001:00018cbc       __unwind$39696             00119cbc f i DatERI.obj
 0001:00018f08       __unwind$39759             00119f08 f i DatERI.obj
 0001:00018f20       __unwind$39760             00119f20 f i DatERI.obj
 0001:00019050       __unwind$39803             0011a050 f i DatERI.obj
 0001:00019068       __unwind$39804             0011a068 f i DatERI.obj
 0001:00019558       __unwind$40075             0011a558 f i DatERI.obj
 0001:0001a2f8       __unwind$40112             0011b2f8 f i DatERI.obj
 0001:0001a318       __unwind$40113             0011b318 f i DatERI.obj
 0001:0001a338       __unwind$40114             0011b338 f i DatERI.obj
 0001:0001a374       __unwind$40117             0011b374 f i DatERI.obj
 0001:0001a394       __unwind$40118             0011b394 f i DatERI.obj
 0001:0001a3b4       __unwind$40119             0011b3b4 f i DatERI.obj
 0001:0001a3f0       __unwind$40122             0011b3f0 f i DatERI.obj
 0001:0001a410       __unwind$40123             0011b410 f i DatERI.obj
 0001:0001a430       __unwind$40124             0011b430 f i DatERI.obj
 0001:0001a46c       __unwind$40127             0011b46c f i DatERI.obj
 0001:0001a83c       __unwind$40296             0011b83c f i DatERI.obj
 0001:0001a970       __unwind$40344             0011b970 f i DatERI.obj
 0001:0001b710       __unwind$40381             0011c710 f i DatERI.obj
 0001:0001b730       __unwind$40382             0011c730 f i DatERI.obj
 0001:0001b750       __unwind$40383             0011c750 f i DatERI.obj
 0001:0001b78c       __unwind$40386             0011c78c f i DatERI.obj
 0001:0001b7ac       __unwind$40387             0011c7ac f i DatERI.obj
 0001:0001b7cc       __unwind$40388             0011c7cc f i DatERI.obj
 0001:0001b808       __unwind$40391             0011c808 f i DatERI.obj
 0001:0001b828       __unwind$40392             0011c828 f i DatERI.obj
 0001:0001b848       __unwind$40393             0011c848 f i DatERI.obj
 0001:0001b884       __unwind$40396             0011c884 f i DatERI.obj
 0001:0001bc54       __unwind$40565             0011cc54 f i DatERI.obj
 0001:0001c538       __unwind$40788             0011d538 f i DatERI.obj
 0001:0001c558       __unwind$40789             0011d558 f i DatERI.obj
 0001:0001c594       __unwind$40792             0011d594 f i DatERI.obj
 0001:0001c5b4       __unwind$40793             0011d5b4 f i DatERI.obj
 0001:0001c5d4       __unwind$40794             0011d5d4 f i DatERI.obj
 0001:0001c5f4       __unwind$40795             0011d5f4 f i DatERI.obj
 0001:0001c828       __unwind$40859             0011d828 f i DatERI.obj
 0001:0001c840       __unwind$40860             0011d840 f i DatERI.obj
 0001:0001c858       __unwind$40862             0011d858 f i DatERI.obj
 0001:0001c88c       __unwind$40864             0011d88c f i DatERI.obj
 0001:0001c8c0       __unwind$40868             0011d8c0 f i DatERI.obj
 0001:0001d050       __unwind$40925             0011e050 f i DatERI.obj
 0001:0001d6b0       __unwind$41327             0011e6b0 f i DatERI.obj
 0001:0001d6d0       __unwind$41328             0011e6d0 f i DatERI.obj
 0001:0001d70c       __unwind$41331             0011e70c f i DatERI.obj
 0001:0001d72c       __unwind$41332             0011e72c f i DatERI.obj
 0001:0001d74c       __unwind$41333             0011e74c f i DatERI.obj
 0001:0001d76c       __unwind$41334             0011e76c f i DatERI.obj
 0001:0001d9a0       __unwind$41398             0011e9a0 f i DatERI.obj
 0001:0001d9b8       __unwind$41399             0011e9b8 f i DatERI.obj
 0001:0001d9d0       __unwind$41401             0011e9d0 f i DatERI.obj
 0001:0001da04       __unwind$41403             0011ea04 f i DatERI.obj
 0001:0001da38       __unwind$41407             0011ea38 f i DatERI.obj
 0001:0001e1c8       __unwind$41463             0011f1c8 f i DatERI.obj
 0001:0001e490       __unwind$41569             0011f490 f i DatERI.obj
 0001:0001e664       __unwind$41629             0011f664 f i DatERI.obj
 0001:0001f360       __unwind$41824             00120360 f i DatERI.obj
 0001:0001f378       __unwind$41825             00120378 f i DatERI.obj
 0001:0001f85c       __catch$41871              0012085c f i DatERI.obj
 0001:0001f9a4       __catch$41903              001209a4 f i DatERI.obj
 0001:0001f9e0       __unwind$41904             001209e0 f i DatERI.obj
 0001:000205f4       __unwind$41983             001215f4 f i DatERI.obj
 0001:0002060c       __unwind$41984             0012160c f i DatERI.obj
 0001:00020af0       __catch$42030              00121af0 f i DatERI.obj
 0001:00020c38       __catch$42062              00121c38 f i DatERI.obj
 0001:00020c74       __unwind$42063             00121c74 f i DatERI.obj
 0001:00023958       __unwind$87446             00124958 f   FakeResponse.obj
 0001:00024194       __unwind$87586             00125194 f   FakeResponse.obj
 0001:00024a14       __unwind$87821             00125a14 f   FakeResponse.obj
 0001:000250ac       __unwind$87878             001260ac f i FakeResponse.obj
 0001:00025238       __catch$87969              00126238 f i FakeResponse.obj
 0001:00025374       __unwind$87996             00126374 f i FakeResponse.obj
 0001:00025530       __unwind$88472             00126530 f i FakeResponse.obj
 0001:00025910       __unwind$88890             00126910 f i FakeResponse.obj
 0001:00025fa8       __unwind$89085             00126fa8 f i FakeResponse.obj
 0001:0002763c       __unwind$84828             0012863c f   gprs.obj
 0001:00027654       __unwind$84829             00128654 f   gprs.obj
 0001:0002b678       __unwind$87990             0012c678 f   misc.obj
 0001:00033bec       __unwind$88375             00134bec f   misc.obj
 0001:00033c20       __unwind$88376             00134c20 f   misc.obj
 0001:00033c54       __unwind$88377             00134c54 f   misc.obj
 0001:00033c88       __unwind$88378             00134c88 f   misc.obj
 0001:00033cbc       __unwind$88379             00134cbc f   misc.obj
 0001:00033cf0       __unwind$88380             00134cf0 f   misc.obj
 0001:00033d24       __unwind$88381             00134d24 f   misc.obj
 0001:00033d58       __unwind$88382             00134d58 f   misc.obj
 0001:00035ad4       __unwind$89184             00136ad4 f   misc.obj
 0001:0003620c       __unwind$89273             0013720c f   misc.obj
 0001:0003622c       __unwind$89274             0013722c f   misc.obj
 0001:0003624c       __unwind$89275             0013724c f   misc.obj
 0001:00037328       __unwind$89511             00138328 f i misc.obj
 0001:00037370       __unwind$89529             00138370 f i misc.obj
 0001:00037630       __unwind$89639             00138630 f i misc.obj
 0001:000376fc       __catch$89662              001386fc f i misc.obj
 0001:00037a4c       __catch$89763              00138a4c f i misc.obj
 0001:00037b88       __unwind$89790             00138b88 f i misc.obj
 0001:000380a8       __unwind$90395             001390a8 f i misc.obj
 0001:000380c8       __unwind$90396             001390c8 f i misc.obj
 0001:000380f4       __unwind$90397             001390f4 f i misc.obj
 0001:00038114       __unwind$90398             00139114 f i misc.obj
 0001:00038134       __unwind$90399             00139134 f i misc.obj
 0001:000384a8       __unwind$90469             001394a8 f i misc.obj
 0001:000384c8       __unwind$90470             001394c8 f i misc.obj
 0001:000384e8       __unwind$90471             001394e8 f i misc.obj
 0001:00038508       __unwind$90472             00139508 f i misc.obj
 0001:00038528       __unwind$90473             00139528 f i misc.obj
 0001:00038548       __unwind$90475             00139548 f i misc.obj
 0001:00038568       __unwind$90477             00139568 f i misc.obj
 0001:00038588       __unwind$90478             00139588 f i misc.obj
 0001:000385a8       __unwind$90479             001395a8 f i misc.obj
 0001:000385c8       __unwind$90481             001395c8 f i misc.obj
 0001:000385e8       __unwind$90482             001395e8 f i misc.obj
 0001:00038784       __unwind$90576             00139784 f i misc.obj
 0001:0003879c       __unwind$90577             0013979c f i misc.obj
 0001:000387b4       __unwind$90578             001397b4 f i misc.obj
 0001:000387cc       __unwind$90580             001397cc f i misc.obj
 0001:000387e4       __unwind$90581             001397e4 f i misc.obj
 0001:00038afc       __unwind$90845             00139afc f i misc.obj
 0001:00038d14       __unwind$90885             00139d14 f i misc.obj
 0001:00038d2c       __unwind$90886             00139d2c f i misc.obj
 0001:00038d44       __unwind$90887             00139d44 f i misc.obj
 0001:00038ec4       __unwind$90929             00139ec4 f i misc.obj
 0001:00038ee4       __unwind$90931             00139ee4 f i misc.obj
 0001:00038f04       __unwind$90932             00139f04 f i misc.obj
 0001:000390fc       __unwind$90977             0013a0fc f i misc.obj
 0001:0003911c       __unwind$90978             0013a11c f i misc.obj
 0001:0003913c       __unwind$90979             0013a13c f i misc.obj
 0001:00039510       __unwind$91024             0013a510 f i misc.obj
 0001:00039528       __unwind$91025             0013a528 f i misc.obj
 0001:00039540       __unwind$91026             0013a540 f i misc.obj
 0001:00039558       __unwind$91027             0013a558 f i misc.obj
 0001:00039570       __unwind$91028             0013a570 f i misc.obj
 0001:00039588       __unwind$91029             0013a588 f i misc.obj
 0001:000395a0       __unwind$91030             0013a5a0 f i misc.obj
 0001:000395b8       __unwind$91032             0013a5b8 f i misc.obj
 0001:0003964c       __unwind$91110             0013a64c f i misc.obj
 0001:00039664       __unwind$91111             0013a664 f i misc.obj
 0001:000398b8       __unwind$91154             0013a8b8 f i misc.obj
 0001:000398d0       __unwind$91155             0013a8d0 f i misc.obj
 0001:000398e8       __unwind$91157             0013a8e8 f i misc.obj
 0001:0003991c       __unwind$91159             0013a91c f i misc.obj
 0001:00039950       __unwind$91163             0013a950 f i misc.obj
 0001:00039984       __unwind$91166             0013a984 f i misc.obj
 0001:00039c28       __unwind$91232             0013ac28 f i misc.obj
 0001:00039c48       __unwind$91233             0013ac48 f i misc.obj
 0001:00039c68       __unwind$91234             0013ac68 f i misc.obj
 0001:00039c88       __unwind$91236             0013ac88 f i misc.obj
 0001:00039cc4       __unwind$91238             0013acc4 f i misc.obj
 0001:00039d00       __unwind$91242             0013ad00 f i misc.obj
 0001:00039d20       __unwind$91244             0013ad20 f i misc.obj
 0001:00039d40       __unwind$91245             0013ad40 f i misc.obj
 0001:00039e70       __unwind$91376             0013ae70 f i misc.obj
 0001:00039e90       __unwind$91377             0013ae90 f i misc.obj
 0001:00039eb0       __unwind$91378             0013aeb0 f i misc.obj
 0001:00039ed0       __unwind$91380             0013aed0 f i misc.obj
 0001:0003a0f0       __unwind$91498             0013b0f0 f i misc.obj
 0001:0003a110       __unwind$91499             0013b110 f i misc.obj
 0001:0003a130       __unwind$91500             0013b130 f i misc.obj
 0001:0003a150       __unwind$91501             0013b150 f i misc.obj
 0001:0003a170       __unwind$91502             0013b170 f i misc.obj
 0001:0003a234       __unwind$91547             0013b234 f i misc.obj
 0001:0003a24c       __unwind$91548             0013b24c f i misc.obj
 0001:0003a264       __unwind$91549             0013b264 f i misc.obj
 0001:0003a320       __unwind$91585             0013b320 f i misc.obj
 0001:0003a340       __unwind$91586             0013b340 f i misc.obj
 0001:0003a360       __unwind$91587             0013b360 f i misc.obj
 0001:0003a4cc       __unwind$91634             0013b4cc f i misc.obj
 0001:0003a4ec       __unwind$91635             0013b4ec f i misc.obj
 0001:0003a50c       __unwind$91636             0013b50c f i misc.obj
 0001:0003a684       __catch$91679              0013b684 f i misc.obj
 0001:0003a730       __unwind$91680             0013b730 f i misc.obj
 0001:0003a748       __unwind$91681             0013b748 f i misc.obj
 0001:0003a760       __unwind$91682             0013b760 f i misc.obj
 0001:0003a778       __unwind$91683             0013b778 f i misc.obj
 0001:0003a790       __unwind$91685             0013b790 f i misc.obj
 0001:0003a7a8       __unwind$91687             0013b7a8 f i misc.obj
 0001:0003a840       __unwind$91749             0013b840 f i misc.obj
 0001:0003a858       __unwind$91750             0013b858 f i misc.obj
 0001:0003a9c8       __unwind$91798             0013b9c8 f i misc.obj
 0001:0003b1bc       __unwind$83758             0013c1bc f   monitor.obj
 0001:0003c914       __unwind$85739             0013d914 f   msg.obj
 0001:0003d194       __unwind$85867             0013e194 f   msg.obj
 0001:0003e8a4       __unwind$86006             0013f8a4 f   msg.obj
 0001:0003f994       __unwind$86155             00140994 f   msg.obj
 0001:00041ae0       __unwind$86255             00142ae0 f   msg.obj
 0001:00044304       __unwind$86584             00145304 f   msg.obj
 0001:00044324       __unwind$86585             00145324 f   msg.obj
 0001:00046038       __unwind$85141             00147038 f   network.obj
 0001:00047720       __unwind$85318             00148720 f   network.obj
 0001:00048194       __unwind$85352             00149194 f   network.obj
 0001:000496fc       __unwind$85619             0014a6fc f   network.obj
 0001:0004a0f8       __unwind$89650             0014b0f8 f   Radio.obj
 0001:0004a110       __unwind$89651             0014b110 f   Radio.obj
 0001:0004a138       __unwind$89652             0014b138 f   Radio.obj
 0001:0004a158       __unwind$89653             0014b158 f   Radio.obj
 0001:0004a174       __unwind$89654             0014b174 f   Radio.obj
 0001:0004a194       __unwind$89655             0014b194 f   Radio.obj
 0001:0004a32c       __unwind$89720             0014b32c f   Radio.obj
 0001:0004a344       __unwind$89721             0014b344 f   Radio.obj
 0001:0004a36c       __unwind$89722             0014b36c f   Radio.obj
 0001:0004a38c       __unwind$89723             0014b38c f   Radio.obj
 0001:0004a3a8       __unwind$89724             0014b3a8 f   Radio.obj
 0001:0004a3c8       __unwind$89725             0014b3c8 f   Radio.obj
 0001:0004b2c8       __unwind$89850             0014c2c8 f   Radio.obj
 0001:0004b2e0       __unwind$89851             0014c2e0 f   Radio.obj
 0001:0004d998       __unwind$90251             0014e998 f   Radio.obj
 0001:000516e4       __unwind$90362             001526e4 f   Radio.obj
 0001:0005170c       __unwind$90363             0015270c f   Radio.obj
 0001:00051734       __unwind$90364             00152734 f   Radio.obj
 0001:0005175c       __unwind$90365             0015275c f   Radio.obj
 0001:0005177c       __unwind$90366             0015277c f   Radio.obj
 0001:000517a4       __unwind$90367             001527a4 f   Radio.obj
 0001:000517cc       __unwind$90368             001527cc f   Radio.obj
 0001:000517ec       __unwind$90369             001527ec f   Radio.obj
 0001:0005180c       __unwind$90370             0015280c f   Radio.obj
 0001:0005182c       __unwind$90371             0015282c f   Radio.obj
 0001:0005184c       __unwind$90372             0015284c f   Radio.obj
 0001:0005186c       __unwind$90373             0015286c f   Radio.obj
 0001:0005188c       __unwind$90374             0015288c f   Radio.obj
 0001:000518ac       __unwind$90375             001528ac f   Radio.obj
 0001:000518cc       __unwind$90376             001528cc f   Radio.obj
 0001:000518ec       __unwind$90377             001528ec f   Radio.obj
 0001:0005190c       __unwind$90378             0015290c f   Radio.obj
 0001:0005192c       __unwind$90379             0015292c f   Radio.obj
 0001:0005194c       __unwind$90380             0015294c f   Radio.obj
 0001:0005196c       __unwind$90381             0015296c f   Radio.obj
 0001:00051a34       ?BSCompareOperatorNames@@YAHPBX0@Z 00152a34 f   Radio.obj
 0001:00051cd0       __unwind$90799             00152cd0 f   Radio.obj
 0001:00051ce8       __unwind$90800             00152ce8 f   Radio.obj
 0001:00051d00       __unwind$90801             00152d00 f   Radio.obj
 0001:00051d18       __unwind$90802             00152d18 f   Radio.obj
 0001:0005270c       __unwind$90961             0015370c f   Radio.obj
 0001:0005272c       __unwind$90962             0015372c f   Radio.obj
 0001:0005274c       __unwind$90963             0015374c f   Radio.obj
 0001:0005276c       __unwind$90964             0015376c f   Radio.obj
 0001:0005278c       __unwind$90965             0015378c f   Radio.obj
 0001:000527ac       __unwind$90966             001537ac f   Radio.obj
 0001:000527cc       __unwind$90967             001537cc f   Radio.obj
 0001:000527ec       __unwind$90968             001537ec f   Radio.obj
 0001:0005280c       __unwind$90969             0015380c f   Radio.obj
 0001:00055a9c       __unwind$91371             00156a9c f   Radio.obj
 0001:00055abc       __unwind$91372             00156abc f   Radio.obj
 0001:00055ae4       __unwind$91373             00156ae4 f   Radio.obj
 0001:00056060       __unwind$91474             00157060 f   Radio.obj
 0001:00056080       __unwind$91475             00157080 f   Radio.obj
 0001:000560a0       __unwind$91476             001570a0 f   Radio.obj
 0001:000562ac       __unwind$91556             001572ac f   Radio.obj
 0001:000564f8       __unwind$91671             001574f8 f i Radio.obj
 0001:000566fc       __unwind$91710             001576fc f i Radio.obj
 0001:00056714       __unwind$91712             00157714 f i Radio.obj
 0001:00056748       __unwind$91716             00157748 f i Radio.obj
 0001:00056790       __unwind$91747             00157790 f i Radio.obj
 0001:00056900       __unwind$91790             00157900 f i Radio.obj
 0001:00056918       __unwind$91791             00157918 f i Radio.obj
 0001:00056930       __unwind$91793             00157930 f i Radio.obj
 0001:00056e10       __unwind$92231             00157e10 f i Radio.obj
 0001:00056f54       __unwind$92254             00157f54 f i Radio.obj
 0001:00057120       __unwind$92337             00158120 f i Radio.obj
 0001:00057f14       __unwind$92385             00158f14 f i Radio.obj
 0001:00057f34       __unwind$92386             00158f34 f i Radio.obj
 0001:00057f54       __unwind$92387             00158f54 f i Radio.obj
 0001:00057f90       __unwind$92390             00158f90 f i Radio.obj
 0001:00057fb0       __unwind$92391             00158fb0 f i Radio.obj
 0001:00057fd0       __unwind$92392             00158fd0 f i Radio.obj
 0001:0005800c       __unwind$92395             0015900c f i Radio.obj
 0001:0005802c       __unwind$92396             0015902c f i Radio.obj
 0001:0005804c       __unwind$92397             0015904c f i Radio.obj
 0001:00058088       __unwind$92400             00159088 f i Radio.obj
 0001:00058238       __unwind$92530             00159238 f i Radio.obj
 0001:00058424       __unwind$92567             00159424 f i Radio.obj
 0001:0005843c       __unwind$92568             0015943c f i Radio.obj
 0001:00058454       __unwind$92569             00159454 f i Radio.obj
 0001:00058bec       __unwind$93213             00159bec f i Radio.obj
 0001:00058c04       __unwind$93214             00159c04 f i Radio.obj
 0001:00058c1c       __unwind$93216             00159c1c f i Radio.obj
 0001:00058c50       __unwind$93218             00159c50 f i Radio.obj
 0001:00058c84       __unwind$93222             00159c84 f i Radio.obj
 0001:00059510       __unwind$93442             0015a510 f i Radio.obj
 0001:00059530       __unwind$93443             0015a530 f i Radio.obj
 0001:0005956c       __unwind$93446             0015a56c f i Radio.obj
 0001:0005958c       __unwind$93447             0015a58c f i Radio.obj
 0001:000595ac       __unwind$93448             0015a5ac f i Radio.obj
 0001:000595cc       __unwind$93449             0015a5cc f i Radio.obj
 0001:00059800       __unwind$93513             0015a800 f i Radio.obj
 0001:00059818       __unwind$93514             0015a818 f i Radio.obj
 0001:00059830       __unwind$93516             0015a830 f i Radio.obj
 0001:00059864       __unwind$93518             0015a864 f i Radio.obj
 0001:00059898       __unwind$93522             0015a898 f i Radio.obj
 0001:0005a028       __unwind$93578             0015b028 f i Radio.obj
 0001:0005a3bc       __unwind$93706             0015b3bc f i Radio.obj
 0001:0005a3d4       __unwind$93707             0015b3d4 f i Radio.obj
 0001:0005b0fc       __unwind$93993             0015c0fc f i Radio.obj
 0001:0005b114       __unwind$93994             0015c114 f i Radio.obj
 0001:0005b79c       __catch$94087              0015c79c f i Radio.obj
 0001:0005c400       __unwind$94145             0015d400 f i Radio.obj
 0001:0005c418       __unwind$94146             0015d418 f i Radio.obj
 0001:0005ca20       __catch$94215              0015da20 f i Radio.obj
 0001:0005cb68       __catch$94247              0015db68 f i Radio.obj
 0001:0005cba4       __unwind$94248             0015dba4 f i Radio.obj
 0001:0005cca0       __unwind$94307             0015dca0 f i Radio.obj
 0001:0005ccb8       __unwind$94308             0015dcb8 f i Radio.obj
 0001:0005cd44       __unwind$94333             0015dd44 f i Radio.obj
 0001:0005ce54       __unwind$94369             0015de54 f i Radio.obj
 0001:0005ce6c       __unwind$94370             0015de6c f i Radio.obj
 0001:0005cf38       __unwind$94404             0015df38 f i Radio.obj
 0001:0005e8bc       __unwind$95151             0015f8bc f i Radio.obj
 0001:00060a2c       __unwind$88560             00161a2c f   rilhand.obj
 0001:00060a54       __unwind$88561             00161a54 f   rilhand.obj
 0001:00060a74       __unwind$88562             00161a74 f   rilhand.obj
 0001:000610c8       __unwind$88650             001620c8 f   rilhand.obj
 0001:000610f0       __unwind$88651             001620f0 f   rilhand.obj
 0001:00061110       __unwind$88652             00162110 f   rilhand.obj
 0001:00061130       __unwind$88653             00162130 f   rilhand.obj
 0001:00061a88       __unwind$88786             00162a88 f   rilhand.obj
 0001:00061aa8       __unwind$88787             00162aa8 f   rilhand.obj
 0001:00061ac8       __unwind$88788             00162ac8 f   rilhand.obj
 0001:0006271c       __unwind$89008             0016371c f   rilhand.obj
 0001:0006273c       __unwind$89009             0016373c f   rilhand.obj
 0001:0006275c       __unwind$89010             0016375c f   rilhand.obj
 0001:00063130       __unwind$89209             00164130 f   rilhand.obj
 0001:000632ac       __unwind$89258             001642ac f   rilhand.obj
 0001:00063460       __unwind$89286             00164460 f   rilhand.obj
 0001:00063804       __unwind$89314             00164804 f   rilhand.obj
 0001:000646ac       __unwind$89382             001656ac f   rilhand.obj
 0001:000646cc       __unwind$89383             001656cc f   rilhand.obj
 0001:000646ec       __unwind$89384             001656ec f   rilhand.obj
 0001:0006470c       __unwind$89385             0016570c f   rilhand.obj
 0001:0006472c       __unwind$89386             0016572c f   rilhand.obj
 0001:0006474c       __unwind$89387             0016574c f   rilhand.obj
 0001:0006476c       __unwind$89388             0016576c f   rilhand.obj
 0001:0006478c       __unwind$89389             0016578c f   rilhand.obj
 0001:000647ac       __unwind$89390             001657ac f   rilhand.obj
 0001:0006496c       __unwind$89672             0016596c f   rilhand.obj
 0001:00064984       __unwind$89673             00165984 f   rilhand.obj
 0001:00064ad4       __unwind$89716             00165ad4 f   rilhand.obj
 0001:00064aec       __unwind$89717             00165aec f   rilhand.obj
 0001:00064c28       __unwind$89759             00165c28 f   rilhand.obj
 0001:00068bc0       ?ReadStrValue@@YAJPAUHKEY__@@PBG1QAGK@Z 00169bc0 f   rilhand.obj
 0001:00069a24       __unwind$90320             0016aa24 f   rilhand.obj
 0001:00069a44       __unwind$90321             0016aa44 f   rilhand.obj
 0001:00069a64       __unwind$90322             0016aa64 f   rilhand.obj
 0001:00069a84       __unwind$90324             0016aa84 f   rilhand.obj
 0001:0006a1ec       __unwind$90799             0016b1ec f i rilhand.obj
 0001:0006a370       __unwind$90841             0016b370 f i rilhand.obj
 0001:0006a42c       __unwind$90868             0016b42c f i rilhand.obj
 0001:0006a7a0       __unwind$90952             0016b7a0 f i rilhand.obj
 0001:0006ac1c       __unwind$91021             0016bc1c f i rilhand.obj
 0001:0006aee8       __unwind$91071             0016bee8 f i rilhand.obj
 0001:0006aff8       __unwind$91112             0016bff8 f i rilhand.obj
 0001:0006b018       __unwind$91113             0016c018 f i rilhand.obj
 0001:0006b154       __unwind$91192             0016c154 f i rilhand.obj
 0001:0006b16c       __unwind$91193             0016c16c f i rilhand.obj
 0001:0006b188       __unwind$91194             0016c188 f i rilhand.obj
 0001:0006b268       __unwind$91246             0016c268 f i rilhand.obj
 0001:0006b288       __unwind$91247             0016c288 f i rilhand.obj
 0001:0006b2f8       __unwind$91272             0016c2f8 f i rilhand.obj
 0001:0006b310       __unwind$91273             0016c310 f i rilhand.obj
 0001:0006b32c       __unwind$91274             0016c32c f i rilhand.obj
 0001:0006b418       __unwind$91342             0016c418 f i rilhand.obj
 0001:0006b490       __unwind$91369             0016c490 f i rilhand.obj
 0001:0006bff4       __unwind$91753             0016cff4 f i rilhand.obj
 0001:0006c100       __catch$91797              0016d100 f i rilhand.obj
 0001:0006c2d0       __unwind$91977             0016d2d0 f i rilhand.obj
 0001:0006f2bc       __unwind$85423             001702bc f   rilhandndis.obj
 0001:00072574       __unwind$85955             00173574 f i rilhandndis.obj
 0001:0007258c       __unwind$85957             0017358c f i rilhandndis.obj
 0001:000725c0       __unwind$85961             001735c0 f i rilhandndis.obj
 0001:00073444       __unwind$86178             00174444 f i rilhandndis.obj
 0001:00073464       __unwind$86179             00174464 f i rilhandndis.obj
 0001:00073484       __unwind$86180             00174484 f i rilhandndis.obj
 0001:000734c0       __unwind$86183             001744c0 f i rilhandndis.obj
 0001:000734e0       __unwind$86184             001744e0 f i rilhandndis.obj
 0001:00073500       __unwind$86185             00174500 f i rilhandndis.obj
 0001:0007353c       __unwind$86188             0017453c f i rilhandndis.obj
 0001:0007355c       __unwind$86189             0017455c f i rilhandndis.obj
 0001:0007357c       __unwind$86190             0017457c f i rilhandndis.obj
 0001:000735b8       __unwind$86193             001745b8 f i rilhandndis.obj
 0001:00073aa8       __unwind$86433             00174aa8 f i rilhandndis.obj
 0001:00073ac8       __unwind$86434             00174ac8 f i rilhandndis.obj
 0001:00073b04       __unwind$86437             00174b04 f i rilhandndis.obj
 0001:00073b24       __unwind$86438             00174b24 f i rilhandndis.obj
 0001:00073b44       __unwind$86439             00174b44 f i rilhandndis.obj
 0001:00073b64       __unwind$86440             00174b64 f i rilhandndis.obj
 0001:00074220       __unwind$86498             00175220 f i rilhandndis.obj
 0001:00074594       __catch$87053              00175594 f i rilhandndis.obj
 0001:000745d0       __unwind$87054             001755d0 f i rilhandndis.obj
 0001:000754d8       __unwind$86525             001764d8 f   rilmain.obj
 0001:00075980       __unwind$86645             00176980 f   rilmain.obj
 0001:00075998       __unwind$86646             00176998 f   rilmain.obj
 0001:00075c0c       __unwind$86716             00176c0c f   rilmain.obj
 0001:0007d0f4       __unwind$87688             0017e0f4 f i rilmain.obj
 0001:00083b50       ?ParseCellBroadcastHeader@@YAHQBEIAAUrilmessage_tag@@AAI@Z 00184b50 f   smscb.obj
 0001:00083d34       ?ParseCellBroadcastDCS@@YAHEAAUrilmsgdcs_tag@@AAI@Z 00184d34 f   smscb.obj
 0001:000842c4       ?SetDCSLanguageType@@YAXAAUrilmsgdcs_tag@@KK@Z 001852c4 f   smscb.obj
 0001:0008af08       __unwind$30780             0018bf08 f   toolbox.obj
 0001:0008ccc4       __unwind$31119             0018dcc4 f   toolbox.obj
 0001:0008d39c       __unwind$31316             0018e39c f   toolbox.obj
 0001:0008d3b8       __unwind$31317             0018e3b8 f   toolbox.obj
 0001:0008d3d4       __unwind$31318             0018e3d4 f   toolbox.obj
 0001:0008d544       __unwind$31341             0018e544 f   toolbox.obj
 0001:0008d560       __unwind$31342             0018e560 f   toolbox.obj
 0001:0008d57c       __unwind$31343             0018e57c f   toolbox.obj
 0001:0008d598       __unwind$31344             0018e598 f   toolbox.obj
 0001:0008d878       __unwind$31372             0018e878 f   toolbox.obj
 0001:0008db74       __unwind$31392             0018eb74 f   toolbox.obj
 0001:0008dc80       __unwind$31407             0018ec80 f   toolbox.obj
 0001:0008e08c       __unwind$31435             0018f08c f   toolbox.obj
 0001:00093284       ?BSCompareListValues@@YAHPBX0@Z 00194284 f   util.obj
 0001:00093394       ?BSCompareListStrings@@YAHPBX0@Z 00194394 f   util.obj
 0001:00094318       __unwind$84702             00195318 f   util.obj
 0001:000973d8       __unwind$84703             001983d8 f   voice.obj
 0001:0009acd8       _initterm                  0019bcd8 f   corelibc:crt0dat.obj
 0001:0009ad78       doexit                     0019bd78 f   corelibc:crt0dat.obj
 0001:0009c2e0       __unwind$18810             0019d2e0 f   libcpmtd:string.obj
 0001:0009c370       __unwind$19010             0019d370 f   libcpmtd:string.obj
 0001:0009c430       __unwind$19588             0019d430 f   libcpmtd:string.obj
 0001:0009c7e8       ?FindHandler@@YAEPAUEHExceptionRecord@@PAKPAU_CONTEXT@@PAU_DISPATCHER_CONTEXT@@PBU_s_FuncInfo@@H@Z 0019d7e8 f   LIBCMTD:frame_ce.obj
 0001:0009cddc       ?TypeMatch@@YAHPBU_s_HandlerType@@PBU_s_CatchableType@@PBU_s_ThrowInfo@@@Z 0019dddc f   LIBCMTD:frame_ce.obj
 0001:0009d1a0       ?FrameUnwindFilter@@YAHPAU_EXCEPTION_POINTERS@@@Z 0019e1a0 f   LIBCMTD:frame_ce.obj
 0001:0009d22c       ?CallCatchBlock@@YAPAXPAUEHExceptionRecord@@PAKPAU_CONTEXT@@PBU_s_FuncInfo@@PAXHK@Z 0019e22c f   LIBCMTD:frame_ce.obj
 0001:0009d7c8       ?CanThisExceptionObjectBeDestructed@@YAEPAUEHExceptionRecord@@E@Z 0019e7c8 f   LIBCMTD:frame_ce.obj
 0001:0009da54       ?BuildCatchObject@@YAXPAUEHExceptionRecord@@PAKPBU_s_HandlerType@@PBU_s_CatchableType@@@Z 0019ea54 f   LIBCMTD:frame_ce.obj
 0001:0009dda4       ?AdjustPointer@@YAPAXPAXABUPMD@@@Z 0019eda4 f   LIBCMTD:frame_ce.obj
 0001:000a1c28       __crtInitCritSecNoSpinCount 001a2c28 f   LIBCMTD:initcrit.obj
 0001:000a27c0       xtow_s                     001a37c0 f   LIBCMTD:xtows.obj
 0001:000a2fc8       ??__EcsReceiveSms@@YAXXZ   001a3fc8 f   msg.obj
 0001:000a2fe8       ??__EtheSWINotifCR@@YAXXZ  001a3fe8 f   Radio.obj
 0001:000a3008       ??__Eg_arrWaitingCommands@@YAXXZ 001a4008 f   rilhand.obj
 0001:000a3028       ??__Einitlocks@std@@YAXXZ  001a4028 f   libcpmtd:xlock.obj
 0001:000a3064       ??__FcsReceiveSms@@YAXXZ   001a4064 f   msg.obj
 0001:000a3078       ??__FtheSWINotifCR@@YAXXZ  001a4078 f   Radio.obj
 0001:000a308c       ??__Fg_arrWaitingCommands@@YAXXZ 001a408c f   rilhand.obj
 0001:000a30a0       ??__Finitlocks@std@@YAXXZ  001a40a0 f   libcpmtd:xlock.obj
